 CryMovie

 Timestamp is 5036d351 (Fri Aug 24 03:05:21 2012)

 Preferred load address is 34000000

 Start         Length     Name                   Class
 0001:00000000 00058adaH .text                   CODE
 0001:00058ae0 00000324H .text$yc                CODE
 0001:00058e10 00000553H .text$yd                CODE
 0002:00000000 0000014cH .idata$5                DATA
 0002:0000014c 00000004H .CRT$XCA                DATA
 0002:00000150 00000050H .CRT$XCU                DATA
 0002:000001a0 00000004H .CRT$XCZ                DATA
 0002:000001a4 00000004H .CRT$XIA                DATA
 0002:000001a8 00000004H .CRT$XIAA               DATA
 0002:000001ac 00000004H .CRT$XIC                DATA
 0002:000001b0 00000004H .CRT$XIZ                DATA
 0002:000001c0 00005cc0H .rdata                  DATA
 0002:00005e80 0000005dH .rdata$debug            DATA
 0002:00005ee0 00000004H .rdata$sxdata           DATA
 0002:00005ee4 00000004H .rtc$IAA                DATA
 0002:00005ee8 00000004H .rtc$IZZ                DATA
 0002:00005eec 00000004H .rtc$TAA                DATA
 0002:00005ef0 00000004H .rtc$TZZ                DATA
 0002:00005ef8 00000064H .xdata$x                DATA
 0002:00005f5c 0000003cH .idata$2                DATA
 0002:00005f98 00000014H .idata$3                DATA
 0002:00005fac 0000014cH .idata$4                DATA
 0002:000060f8 00000568H .idata$6                DATA
 0002:00006660 00000072H .edata                  DATA
 0003:00000000 00000220H .data                   DATA
 0003:00000220 00002a1cH .bss                    DATA
 0004:00000000 00000004H .tls$                   DATA
 0005:00000000 00000058H .rsrc$01                DATA
 0005:00000060 00000248H .rsrc$02                DATA

  Address         Publics by Value              Rva+Base       Lib:Object

 0000:00000000       __except_list              00000000     <absolute>
 0000:00000001       ___safe_se_handler_count   00000001     <absolute>
 0000:00009876       __ldused                   00009876     <absolute>
 0000:00009876       __fltused                  00009876     <absolute>
 0000:00000000       ___ImageBase               34000000     <linker-defined>
 0001:00000000       ?Release@CAnimNode@@UAEXXZ 34001000 f i AnimLightNode.obj
 0001:00000030       ?GetUser@CMovieSystem@@UAEPAUIMovieUser@@XZ 34001030 f i Movie.obj
 0001:00000030       ?GetSpline@?$TAnimSplineTrack@U?$Quat_tpl@M@@@@UBEPAUISplineInterpolator@@XZ 34001030 f i Movie.obj
 0001:00000030       ?GetValueType@CCompoundSplineTrack@@UAE?AW4EAnimValue@@XZ 34001030 f i CompoundSplineTrack.obj
 0001:00000030       ?GetSpline@?$TAnimSplineTrack@M@@UBEPAUISplineInterpolator@@XZ 34001030 f i Movie.obj
 0001:00000030       ?GetSpline@?$TAnimSplineTrack@U?$Vec3_tpl@M@@@@UBEPAUISplineInterpolator@@XZ 34001030 f i Movie.obj
 0001:00000030       ?GetName@CAnimSequenceGroup@@UBEPBDXZ 34001030 f i AnimSequenceGroup.obj
 0001:00000030       ?GetSpline@?$TAnimSplineTrack@U?$Vec2_tpl@M@@@@UBEPAUISplineInterpolator@@XZ 34001030 f i CompoundSplineTrack.obj
 0001:00000030       ?GetId@CAnimNode@@UBEHXZ   34001030 f i AnimLightNode.obj
 0001:00000040       ?GetMovieSystem@CAnimNode@@UAEPAUIMovieSystem@@XZ 34001040 f i AnimLightNode.obj
 0001:00000050       ?SetNodeAnimator@CAnimNode@@UAEXPAUIAnimNodeAnimator@@@Z 34001050 f i AnimLightNode.obj
 0001:00000060       ?SetParent@CAnimNode@@UAEXPAUIAnimNode@@@Z 34001060 f i AnimLightNode.obj
 0001:00000070       ?NeedToRender@CAnimNode@@MBE_NXZ 34001070 f i AnimLightNode.obj
 0001:00000070       ?IsBoneLinkTransformEnabled@CAnimNode@@UBE_NXZ 34001070 f i AnimSequence.obj
 0001:00000080       ?GetEntityGuid@CAnimEntityNode@@UAEPA_KXZ 34001080 f i AnimLightNode.obj
 0001:00000090       ?GetPos@CAnimEntityNode@@UAE?AU?$Vec3_tpl@M@@XZ 34001090 f i AnimLightNode.obj
 0001:000000b0       ?GetScale@CAnimEntityNode@@UAE?AU?$Vec3_tpl@M@@XZ 340010b0 f i AnimLightNode.obj
 0001:000000e0       ?GetType@CAnimLightNode@@UBE?AW4EAnimNodeType@@XZ 340010e0 f i AnimLightNode.obj
 0001:000000f0       ?GetMemoryUsage@CAnimLightNode@@UBEXPAVICrySizer@@@Z 340010f0 f i AnimLightNode.obj
 0001:00000110       ?Activate@CAnimLightNode@@UAEX_N@Z 34001110 f   AnimLightNode.obj
 0001:00000130       ?GetParamCount@CAnimLightNode@@UBEHXZ 34001130 f   AnimLightNode.obj
 0001:00000140       ??_ECAnimLightNode@@$4PPPPPPPM@A@AEPAXI@Z 34001140 f i AnimLightNode.obj
 0001:00000150       ?Release@CAnimNode@@$4PPPPPPPM@BJI@AEXXZ 34001150 f i AnimLightNode.obj
 0001:00000160       ??1ScriptAnyValue@@QAE@XZ  34001160 f i AnimLightNode.obj
 0001:000001b0       ??8AnimParamType@@QBE_NABV0@@Z 340011b0 f i AnimLightNode.obj
 0001:000001e0       ??1AnimParamType@@QAE@XZ   340011e0 f i AnimLightNode.obj
 0001:00000210       ?CryFatalError@@YAXPBDZZ   34001210 f i AnimLightNode.obj
 0001:00000280       ?AddRef@?$_i_reference_target@H@@UAEXXZ 34001280 f i AnimLightNode.obj
 0001:00000290       ?Release@?$_i_reference_target@H@@UAEXXZ 34001290 f i AnimLightNode.obj
 0001:000002c0       ??_G?$_i_reference_target@H@@UAEPAXI@Z 340012c0 f i AnimLightNode.obj
 0001:000002c0       ??_E?$_i_reference_target@H@@UAEPAXI@Z 340012c0 f i AnimLightNode.obj
 0001:000002f0       ?GetRotate@CAnimEntityNode@@UAE?AU?$Quat_tpl@M@@XZ 340012f0 f i AnimLightNode.obj
 0001:00000320       ??0CAnimLightNode@@QAE@XZ  34001320 f   AnimLightNode.obj
 0001:000003f0       ?GetValueFromTrack@CAnimLightNode@@ABE_NVAnimParamType@@MAAM@Z 340013f0 f   AnimLightNode.obj
 0001:00000470       ?GetValueFromTrack@CAnimLightNode@@ABE_NVAnimParamType@@MAAU?$Vec3_tpl@M@@@Z 34001470 f   AnimLightNode.obj
 0001:000004f0       ?CreateTrack@CAnimLightNode@@UAEPAUIAnimTrack@@ABVAnimParamType@@@Z 340014f0 f   AnimLightNode.obj
 0001:00000590       ?Serialize@CAnimLightNode@@UAEXAAVXmlNodeRef@@_N1@Z 34001590 f   AnimLightNode.obj
 0001:000006e0       ?SetParamValue@CAnimLightNode@@UAE_NMVAnimParamType@@M@Z 340016e0 f   AnimLightNode.obj
 0001:000007b0       ??4AnimParamType@@QAEAAV0@ABV0@@Z 340017b0 f i AnimLightNode.obj
 0001:00000800       ??$SetValue@M@IScriptTable@@QAEXPBDABM@Z 34001800 f i AnimLightNode.obj
 0001:00000870       ??$SetValue@U?$Vec3_tpl@M@@@IScriptTable@@QAEXPBDABU?$Vec3_tpl@M@@@Z 34001870 f i AnimLightNode.obj
 0001:000008f0       ?_Free@?$CryStringT@D@@IAEXXZ 340018f0 f i AnimLightNode.obj
 0001:00000930       ??_GCAnimLightNode@@UAEPAXI@Z 34001930 f i AnimLightNode.obj
 0001:00000930       ??_ECAnimLightNode@@UAEPAXI@Z 34001930 f i AnimLightNode.obj
 0001:00000990       ?Animate@CAnimLightNode@@UAEXAAUSAnimContext@@@Z 34001990 f   AnimLightNode.obj
 0001:00000cb0       ?CreateDefaultTracks@CAnimLightNode@@UAEXXZ 34001cb0 f   AnimLightNode.obj
 0001:00000df0       ?SetParamValue@CAnimLightNode@@UAE_NMVAnimParamType@@ABU?$Vec3_tpl@M@@@Z 34001df0 f   AnimLightNode.obj
 0001:00000e70       ??4SParamInfo@IAnimNode@@QAEAAU01@ABU01@@Z 34001e70 f i AnimLightNode.obj
 0001:00000ed0       ?GetParamInfoFromId@CAnimLightNode@@UBE_NABVAnimParamType@@AAUSParamInfo@IAnimNode@@@Z 34001ed0 f   AnimLightNode.obj
 0001:00000f80       ?_AllocData@?$CryStringT@D@@IAEXI@Z 34001f80 f i AnimLightNode.obj
 0001:00000fd0       ?_Assign@?$CryStringT@D@@IAEXPBDI@Z 34001fd0 f i AnimLightNode.obj
 0001:00001080       ?GetParamInfo@CAnimLightNode@@UBE_NHAAUSParamInfo@IAnimNode@@@Z 34002080 f   AnimLightNode.obj
 0001:000010b0       ??4?$CryStringT@D@@QAEAAV0@PBD@Z 340020b0 f i AnimLightNode.obj
 0001:000010f0       ?SetName@CAnimNode@@UAEXPBD@Z 340020f0 f i AnimLightNode.obj
 0001:00001130       ?GetGroup@CAnimSequence@@UBEPAUIAnimSequenceGroup@@XZ 34002130 f   AnimSequence.obj
 0001:00001140       ?SetGroup@CAnimSequence@@UAEXPAUIAnimSequenceGroup@@@Z 34002140 f   AnimSequence.obj
 0001:000011c0       ?SetFlags@CAnimSequence@@UAEXH@Z 340021c0 f   AnimSequence.obj
 0001:000011d0       ?GetFlags@CAnimSequence@@UBEHXZ 340021d0 f   AnimSequence.obj
 0001:000011e0       ?GetCutSceneFlags@CAnimSequence@@UBEH_N@Z 340021e0 f   AnimSequence.obj
 0001:00001220       ?SetParentSequence@CAnimSequence@@UAEXPAUIAnimSequence@@@Z 34002220 f   AnimSequence.obj
 0001:00001230       ?GetParentSequence@CAnimSequence@@UBEPBUIAnimSequence@@XZ 34002230 f   AnimSequence.obj
 0001:00001240       ?__stl_throw_length_error@stlpmtx_std@@YAXPBD@Z 34002240 f i AnimSequence.obj
 0001:00001260       ?SetActiveDirector@CAnimSequence@@UAEXPAUIAnimNode@@@Z 34002260 f   AnimSequence.obj
 0001:00001290       ?GetActiveDirector@CAnimSequence@@UBEPAUIAnimNode@@XZ 34002290 f   AnimSequence.obj
 0001:00001290       ?GetSequenceStopBehavior@CMovieSystem@@UAE?AW4ESequenceStopBehavior@IMovieSystem@@XZ 34002290 f   Movie.obj
 0001:000012a0       ??$__copy_backward@PAV?$_smart_ptr@UIAnimNode@@@@PAV1@H@priv@stlpmtx_std@@YAPAV?$_smart_ptr@UIAnimNode@@@@PAV2@00ABUrandom_access_iterator_tag@1@PAH@Z 340022a0 f i AnimSequence.obj
 0001:00001310       ??$__fill@PAV?$_smart_ptr@UIAnimNode@@@@V1@H@priv@stlpmtx_std@@YAXPAV?$_smart_ptr@UIAnimNode@@@@0ABV2@ABUrandom_access_iterator_tag@1@PAH@Z 34002310 f i AnimSequence.obj
 0001:00001370       ?_Rotate_left@?$_Rb_global@_N@priv@stlpmtx_std@@SAXPAU_Rb_tree_node_base@23@AAPAU423@@Z 34002370 f i AnimSequence.obj
 0001:000013c0       ?_Rotate_right@?$_Rb_global@_N@priv@stlpmtx_std@@SAXPAU_Rb_tree_node_base@23@AAPAU423@@Z 340023c0 f i AnimSequence.obj
 0001:00001410       ??0CAnimNodeGroup@@QAE@XZ  34002410 f i AnimSequence.obj
 0001:00001480       ?ResetHard@CAnimNode@@UAEXXZ 34002480 f i AnimSequence.obj
 0001:00001480       ?Resume@CAnimScriptVarNode@@UAEXXZ 34002480 f i ScriptVarNode.obj
 0001:00001480       ?Resume@CAnimCVarNode@@UAEXXZ 34002480 f i CVarNode.obj
 0001:00001490       ?GetTime@CAnimNode@@UAEMXZ 34002490 f i AnimSequence.obj
 0001:000014a0       ?AddFrameStart@CDummyMemReplay@@UAEXXZ 340024a0 f i AnimSequence.obj
 0001:000014a0       ?DumpSymbols@CDummyMemReplay@@UAEXXZ 340024a0 f i AnimSequence.obj
 0001:000014a0       ?ExitScope@CDummyMemReplay@@UAEXXZ 340024a0 f i AnimSequence.obj
 0001:000014a0       ?StillUpdate@CAnimNode@@UAEXXZ 340024a0 f i AnimSequence.obj
 0001:000014a0       ?AddScreenshot@CDummyMemReplay@@UAEXXZ 340024a0 f i AnimSequence.obj
 0001:000014a0       ?Reset@CCommentNode@@UAEXXZ 340024a0 f i CommentNode.obj
 0001:000014a0       ?Resume@CAnimNode@@UAEXXZ  340024a0 f i AnimLightNode.obj
 0001:000014a0       ?UpdateDynamicParams@CAnimNode@@UAEXXZ 340024a0 f i AnimSequence.obj
 0001:000014a0       ?Render@CAnimNode@@UAEXXZ  340024a0 f i AnimLightNode.obj
 0001:000014a0       ?Pause@CAnimNode@@UAEXXZ   340024a0 f i AnimSequence.obj
 0001:000014a0       ?CreateDefaultTracks@CAnimNode@@UAEXXZ 340024a0 f i AnimSequence.obj
 0001:000014a0       ?DumpStats@CDummyMemReplay@@UAEXXZ 340024a0 f i AnimSequence.obj
 0001:000014a0       ?RemoveContext@CDummyMemReplay@@UAEXXZ 340024a0 f i AnimSequence.obj
 0001:000014a0       ?sp_enable_shared_from_this@detail@boost@@YAXZZ 340024a0 f i CryMovie.obj
 0001:000014a0       ?Stop@CDummyMemReplay@@UAEXXZ 340024a0 f i AnimSequence.obj
 0001:000014a0       ?Flush@CDummyMemReplay@@UAEXXZ 340024a0 f i AnimSequence.obj
 0001:000014a0       ?SortKeys@CCompoundSplineTrack@@UAEXXZ 340024a0 f i CompoundSplineTrack.obj
 0001:000014a0       ?AddLabelFmt@CDummyMemReplay@@UAAXPBDZZ 340024a0 f i AnimSequence.obj
 0001:000014a0       ?Reset@CAnimNode@@UAEXXZ   340024a0 f i AnimSequence.obj
 0001:000014b0       ?GetType@CAnimNodeGroup@@UBE?AW4EAnimNodeType@@XZ 340024b0 f i AnimSequence.obj
 0001:000014c0       ?GetParamInfo@CAnimNodeGroup@@UBE_NHAAUSParamInfo@IAnimNode@@@Z 340024c0 f i AnimSequence.obj
 0001:000014c0       ?GetParamInfoFromId@CAnimNodeGroup@@UBE_NABVAnimParamType@@AAUSParamInfo@IAnimNode@@@Z 340024c0 f i AnimSequence.obj
 0001:000014d0       ?Release@CAnimNode@@$4PPPPPPPM@A@AEXXZ 340024d0 f i AnimSequence.obj
 0001:000014e0       ?GetRotate@CAnimNode@@UAE?AU?$Quat_tpl@M@@XZ 340024e0 f i AnimSequence.obj
 0001:00001500       ?GetPos@CAnimNode@@UAE?AU?$Vec3_tpl@M@@XZ 34002500 f i AnimSequence.obj
 0001:00001500       ?GetScale@CAnimNode@@UAE?AU?$Vec3_tpl@M@@XZ 34002500 f i AnimSequence.obj
 0001:00001520       ?EnterScope@CDummyMemReplay@@UAE_NW4Class@EMemReplayAllocClass@@GH@Z 34002520 f i AnimSequence.obj
 0001:00001530       ?MarkBucket@CDummyMemReplay@@UAEXHIPAXI@Z 34002530 f i AnimSequence.obj
 0001:00001530       ?ExitScope_Realloc@CDummyMemReplay@@UAEXIIII@Z 34002530 f i AnimSequence.obj
 0001:00001530       ?AddContextV@CDummyMemReplay@@UAEXHIPBDPAD@Z 34002530 f i AnimSequence.obj
 0001:00001540       ?MarkPool@CDummyMemReplay@@UAEXHIPAXIPBD@Z 34002540 f i AnimSequence.obj
 0001:00001550       ?AddTexturePoolContext@CDummyMemReplay@@UAEXPAXHHHPBDI@Z 34002550 f i AnimSequence.obj
 0001:00001560       ??_ECDummyMemReplay@@UAEPAXI@Z 34002560 f i AnimSequence.obj
 0001:00001560       ??_GCDummyMemReplay@@UAEPAXI@Z 34002560 f i AnimSequence.obj
 0001:00001560       ??_EIMemReplay@@UAEPAXI@Z  34002560 f i AnimSequence.obj
 0001:00001560       ??_GIMemReplay@@UAEPAXI@Z  34002560 f i AnimSequence.obj
 0001:00001590       ?CreateNodeInternal@CAnimSequence@@AAEPAUIAnimNode@@W4EAnimNodeType@@I@Z 34002590 f   AnimSequence.obj
 0001:000017b0       ?CreateNode@CAnimSequence@@UAEPAUIAnimNode@@W4EAnimNodeType@@@Z 340027b0 f   AnimSequence.obj
 0001:000017d0       ?CopyNodeChildren@CAnimSequence@@AAEXAAVXmlNodeRef@@PAUIAnimNode@@@Z 340027d0 f   AnimSequence.obj
 0001:000018a0       ?CopyNodes@CAnimSequence@@UAEXAAVXmlNodeRef@@PAPAUIAnimNode@@I@Z 340028a0 f   AnimSequence.obj
 0001:00001930       ??$SetGlobalValue@PBD@IScriptSystem@@QAEXPBDABQBD@Z 34002930 f i AnimSequence.obj
 0001:000019a0       ??$?8D@@YA_NABV?$CryStringT@D@@PBD@Z 340029a0 f i AnimSequence.obj
 0001:000019f0       ??$__copy@PAV?$_smart_ptr@UIAnimNode@@@@PAV1@H@priv@stlpmtx_std@@YAPAV?$_smart_ptr@UIAnimNode@@@@PAV2@00ABUrandom_access_iterator_tag@1@PAH@Z 340029f0 f i AnimSequence.obj
 0001:00001a60       ??$__find@PAV?$CryStringT@D@@PBD@priv@stlpmtx_std@@YAPAV?$CryStringT@D@@PAV2@0ABQBDABUrandom_access_iterator_tag@1@@Z 34002a60 f i AnimSequence.obj
 0001:00001c30       ?_Rebalance@?$_Rb_global@_N@priv@stlpmtx_std@@SAXPAU_Rb_tree_node_base@23@AAPAU423@@Z 34002c30 f i AnimSequence.obj
 0001:00001df0       ?_AllocData@?$CryStackStringT@D$0CAA@@@QAEXI@Z 34002df0 f i AnimSequence.obj
 0001:00001e60       ?_Concatenate@?$CryStackStringT@D$0CAA@@@QAEXPBDI0I@Z 34002e60 f i AnimSequence.obj
 0001:00001ed0       ?CryGetIMemReplay@@YAPAUIMemReplay@@XZ 34002ed0 f i AnimSequence.obj
 0001:00001f30       ?GetNodeCount@CAnimSequence@@UBEHXZ 34002f30 f   AnimSequence.obj
 0001:00001f40       ?GetNode@CAnimSequence@@UBEPAUIAnimNode@@H@Z 34002f40 f   AnimSequence.obj
 0001:00001f50       ?Reset@CAnimSequence@@UAEX_N@Z 34002f50 f   AnimSequence.obj
 0001:00002030       ?ResetHard@CAnimSequence@@UAEXXZ 34003030 f   AnimSequence.obj
 0001:000020e0       ?Pause@CAnimSequence@@UAEXXZ 340030e0 f   AnimSequence.obj
 0001:00002120       ?Resume@CAnimSequence@@UAEXXZ 34003120 f   AnimSequence.obj
 0001:00002160       ?StillUpdate@CAnimSequence@@UAEXXZ 34003160 f   AnimSequence.obj
 0001:000021a0       ?Animate@CAnimSequence@@UAEXAAUSAnimContext@@@Z 340031a0 f   AnimSequence.obj
 0001:00002280       ?Render@CAnimSequence@@UAEXXZ 34003280 f   AnimSequence.obj
 0001:000022b0       ?Activate@CAnimSequence@@UAEXXZ 340032b0 f   AnimSequence.obj
 0001:00002300       ?SetTimeRange@CAnimSequence@@UAEXV?$TRange@M@@@Z 34003300 f   AnimSequence.obj
 0001:00002360       ?AdjustKeysToTimeRange@CAnimSequence@@UAEXABV?$TRange@M@@@Z 34003360 f   AnimSequence.obj
 0001:00002460       ?GetTrackEventsCount@CAnimSequence@@UBEHXZ 34003460 f   AnimSequence.obj
 0001:00002470       ?GetTrackEvent@CAnimSequence@@UBEPBDH@Z 34003470 f   AnimSequence.obj
 0001:000024b0       ?FindNodeById@CAnimSequence@@QAEPAUIAnimNode@@H@Z 340034b0 f   AnimSequence.obj
 0001:000024e0       ?FindNodeByName@CAnimSequence@@UAEPAUIAnimNode@@PBDPBU2@@Z 340034e0 f   AnimSequence.obj
 0001:00002540       ?IsAncestorOf@CAnimSequence@@UBE_NPBUIAnimSequence@@@Z 34003540 f   AnimSequence.obj
 0001:000026a0       ?_M_erase@?$_Rb_tree@HU?$less@H@stlpmtx_std@@U?$pair@$$CBHPAUIAnimNode@@@2@U?$_Select1st@U?$pair@$$CBHPAUIAnimNode@@@stlpmtx_std@@@priv@2@U?$_MapTraitsT@U?$pair@$$CBHPAUIAnimNode@@@stlpmtx_std@@@52@V?$allocator@U?$pair@$$CBHPAUIAnimNode@@@stlpmtx_std@@@2@@priv@stlpmtx_std@@AAEXPAU_Rb_tree_node_base@23@@Z 340036a0 f i AnimSequence.obj
 0001:000026a0       ?_M_erase@?$_Rb_tree@PAUIEntity@@U?$less@PAUIEntity@@@stlpmtx_std@@U?$pair@QAUIEntity@@PAUIAnimNode@@@3@U?$_Select1st@U?$pair@QAUIEntity@@PAUIAnimNode@@@stlpmtx_std@@@priv@3@U?$_MapTraitsT@U?$pair@QAUIEntity@@PAUIAnimNode@@@stlpmtx_std@@@63@V?$allocator@U?$pair@QAUIEntity@@PAUIAnimNode@@@stlpmtx_std@@@3@@priv@stlpmtx_std@@AAEXPAU_Rb_tree_node_base@23@@Z 340036a0 f i Movie.obj
 0001:000026e0       ??$__ucopy@PAV?$_smart_ptr@UIAnimNode@@@@PAV1@H@priv@stlpmtx_std@@YAPAV?$_smart_ptr@UIAnimNode@@@@PAV2@00ABUrandom_access_iterator_tag@1@PAH@Z 340036e0 f i AnimSequence.obj
 0001:00002730       ??0?$CryStackStringT@D$0CAA@@@QAE@PBD@Z 34003730 f i AnimSequence.obj
 0001:000027a0       ?_ConcatenateInPlace@?$CryStackStringT@D$0CAA@@@QAEXPBDI@Z 340037a0 f i AnimSequence.obj
 0001:00002810       ?_Concatenate@?$CryStringT@D@@IAEXPBDI0I@Z 34003810 f i AnimSequence.obj
 0001:000028b0       ?NotifyTrackEvent@CAnimSequence@@AAEXW4EReason@ITrackEventListener@@PBD1@Z 340038b0 f   AnimSequence.obj
 0001:000028f0       ?TriggerTrackEvent@CAnimSequence@@UAEXPBD0@Z 340038f0 f   AnimSequence.obj
 0001:00002930       ??$swap@V?$CryStringT@D@@@stlpmtx_std@@YAXAAV?$CryStringT@D@@0@Z 34003930 f i AnimSequence.obj
 0001:000029e0       ??$__uninitialized_fill_n@PAV?$_smart_ptr@UIAnimNode@@@@IV1@@priv@stlpmtx_std@@YAPAV?$_smart_ptr@UIAnimNode@@@@PAV2@IABV2@@Z 340039e0 f i AnimSequence.obj
 0001:00002a40       ??$__copy@PAV?$CryStringT@D@@PAV1@H@priv@stlpmtx_std@@YAPAV?$CryStringT@D@@PAV2@00ABUrandom_access_iterator_tag@1@PAH@Z 34003a40 f i AnimSequence.obj
 0001:00002b10       ??$__destroy_range_aux@V?$reverse_iterator@PAV?$_smart_ptr@UIAnimNode@@@@@stlpmtx_std@@V?$_smart_ptr@UIAnimNode@@@@@stlpmtx_std@@YAXV?$reverse_iterator@PAV?$_smart_ptr@UIAnimNode@@@@@0@0PAV?$_smart_ptr@UIAnimNode@@@@ABU__false_type@0@@Z 34003b10 f i AnimSequence.obj
 0001:00002b50       ??0?$CryStringT@D@@QAE@PBD@Z 34003b50 f i AnimSequence.obj
 0001:00002bc0       ??0?$CryStringT@D@@QAE@PBDI@Z 34003bc0 f i AnimSequence.obj
 0001:00002c20       ?_ConcatenateInPlace@?$CryStringT@D@@IAEXPBDI@Z 34003c20 f i AnimSequence.obj
 0001:00002cb0       ??$__ucopy@PAV?$CryStringT@D@@PAV1@H@priv@stlpmtx_std@@YAPAV?$CryStringT@D@@PAV2@00ABUrandom_access_iterator_tag@1@PAH@Z 34003cb0 f i AnimSequence.obj
 0001:00002d00       ?SetName@CAnimSequence@@UAEXPBD@Z 34003d00 f   AnimSequence.obj
 0001:00002d90       ?SetGroupAndName@CAnimSequence@@UAEXPAUIAnimSequenceGroup@@PBD@Z 34003d90 f   AnimSequence.obj
 0001:00002e40       ?Deactivate@CAnimSequence@@UAEXXZ 34003e40 f   AnimSequence.obj
 0001:00003020       ?PrecacheData@CAnimSequence@@UAEXM@Z 34004020 f   AnimSequence.obj
 0001:00003170       ?RenameTrackEvent@CAnimSequence@@UAE_NPBD0@Z 34004170 f   AnimSequence.obj
 0001:00003240       ?MoveUpTrackEvent@CAnimSequence@@UAE_NPBD@Z 34004240 f   AnimSequence.obj
 0001:00003300       ?MoveDownTrackEvent@CAnimSequence@@UAE_NPBD@Z 34004300 f   AnimSequence.obj
 0001:000033c0       ?RemoveTrackEventListener@CAnimSequence@@UAEXPAUITrackEventListener@@@Z 340043c0 f   AnimSequence.obj
 0001:00003410       ?erase@?$_Impl_vector@V?$_smart_ptr@UIAnimNode@@@@V?$allocator@V?$_smart_ptr@UIAnimNode@@@@@stlpmtx_std@@@priv@stlpmtx_std@@QAEPAV?$_smart_ptr@UIAnimNode@@@@PAV4@@Z 34004410 f i AnimSequence.obj
 0001:00003480       ?Right@?$CryStringT@D@@QBE?AV1@I@Z 34004480 f i AnimSequence.obj
 0001:000034d0       ??$AddObject@UTrackDesc@CAnimNode@@V?$allocator@UTrackDesc@CAnimNode@@@stlpmtx_std@@@ICrySizer@@QAEXABV?$vector@UTrackDesc@CAnimNode@@V?$allocator@UTrackDesc@CAnimNode@@@stlpmtx_std@@@stlpmtx_std@@@Z 340044d0 f i AnimSequence.obj
 0001:00003550       ?Enable@CLogIndenter@@QAAX_NPBDZZ 34004550 f i AnimSequence.obj
 0001:000035f0       ?_M_fill_insert_aux@?$_Impl_vector@V?$_smart_ptr@UIAnimNode@@@@V?$allocator@V?$_smart_ptr@UIAnimNode@@@@@stlpmtx_std@@@priv@stlpmtx_std@@AAEXPAV?$_smart_ptr@UIAnimNode@@@@IABV4@ABU__false_type@3@@Z 340045f0 f i AnimSequence.obj
 0001:00003730       ?_M_insert@?$_Rb_tree@HU?$less@H@stlpmtx_std@@U?$pair@$$CBHPAUIAnimNode@@@2@U?$_Select1st@U?$pair@$$CBHPAUIAnimNode@@@stlpmtx_std@@@priv@2@U?$_MapTraitsT@U?$pair@$$CBHPAUIAnimNode@@@stlpmtx_std@@@52@V?$allocator@U?$pair@$$CBHPAUIAnimNode@@@stlpmtx_std@@@2@@priv@stlpmtx_std@@AAE?AU?$_Rb_tree_iterator@U?$pair@$$CBHPAUIAnimNode@@@stlpmtx_std@@U?$_MapTraitsT@U?$pair@$$CBHPAUIAnimNode@@@stlpmtx_std@@@priv@2@@23@PAU_Rb_tree_node_base@23@ABU?$pair@$$CBHPAUIAnimNode@@@3@00@Z 34004730 f i AnimSequence.obj
 0001:000037f0       ?insert_unique@?$_Rb_tree@HU?$less@H@stlpmtx_std@@U?$pair@$$CBHPAUIAnimNode@@@2@U?$_Select1st@U?$pair@$$CBHPAUIAnimNode@@@stlpmtx_std@@@priv@2@U?$_MapTraitsT@U?$pair@$$CBHPAUIAnimNode@@@stlpmtx_std@@@52@V?$allocator@U?$pair@$$CBHPAUIAnimNode@@@stlpmtx_std@@@2@@priv@stlpmtx_std@@QAE?AU?$pair@U?$_Rb_tree_iterator@U?$pair@$$CBHPAUIAnimNode@@@stlpmtx_std@@U?$_MapTraitsT@U?$pair@$$CBHPAUIAnimNode@@@stlpmtx_std@@@priv@2@@priv@stlpmtx_std@@_N@3@ABU?$pair@$$CBHPAUIAnimNode@@@3@@Z 340047f0 f i AnimSequence.obj
 0001:000038b0       ??$__destroy_range_aux@PAV?$CryStringT@D@@V1@@stlpmtx_std@@YAXPAV?$CryStringT@D@@00ABU__false_type@0@@Z 340048b0 f i AnimSequence.obj
 0001:00003900       ??Y?$CryStringT@D@@QAEAAV0@PBD@Z 34004900 f i AnimSequence.obj
 0001:00003940       ??$__uninitialized_fill_n@PAV?$CryStringT@D@@IV1@@priv@stlpmtx_std@@YAPAV?$CryStringT@D@@PAV2@IABV2@@Z 34004940 f i AnimSequence.obj
 0001:00003990       ??$__destroy_range_aux@V?$reverse_iterator@PAV?$CryStringT@D@@@stlpmtx_std@@V?$CryStringT@D@@@stlpmtx_std@@YAXV?$reverse_iterator@PAV?$CryStringT@D@@@0@0PAV?$CryStringT@D@@ABU__false_type@0@@Z 34004990 f i AnimSequence.obj
 0001:000039e0       ?GetMemoryUsage@CAnimNode@@UBEXPAVICrySizer@@@Z 340049e0 f i AnimSequence.obj
 0001:00003a10       ?GetMemoryUsage@CAnimNodeGroup@@UBEXPAVICrySizer@@@Z 34004a10 f i AnimSequence.obj
 0001:00003a50       ?_M_erase@?$_Impl_vector@V?$CryStringT@D@@V?$allocator@V?$CryStringT@D@@@stlpmtx_std@@@priv@stlpmtx_std@@AAEPAV?$CryStringT@D@@PAV4@ABU__false_type@3@@Z 34004a50 f i AnimSequence.obj
 0001:00003ad0       ?insert_unique@?$_Rb_tree@HU?$less@H@stlpmtx_std@@U?$pair@$$CBHPAUIAnimNode@@@2@U?$_Select1st@U?$pair@$$CBHPAUIAnimNode@@@stlpmtx_std@@@priv@2@U?$_MapTraitsT@U?$pair@$$CBHPAUIAnimNode@@@stlpmtx_std@@@52@V?$allocator@U?$pair@$$CBHPAUIAnimNode@@@stlpmtx_std@@@2@@priv@stlpmtx_std@@QAE?AU?$_Rb_tree_iterator@U?$pair@$$CBHPAUIAnimNode@@@stlpmtx_std@@U?$_MapTraitsT@U?$pair@$$CBHPAUIAnimNode@@@stlpmtx_std@@@priv@2@@23@U423@ABU?$pair@$$CBHPAUIAnimNode@@@3@@Z 34004ad0 f i AnimSequence.obj
 0001:00003cc0       ??$?HD@@YA?AV?$CryStringT@D@@ABV0@PBD@Z 34004cc0 f i AnimSequence.obj
 0001:00003d20       ?GetFullName@CAnimSequence@@UBEPBDXZ 34004d20 f   AnimSequence.obj
 0001:00003fc0       ?_M_insert_overflow_aux@?$_Impl_vector@V?$_smart_ptr@UIAnimNode@@@@V?$allocator@V?$_smart_ptr@UIAnimNode@@@@@stlpmtx_std@@@priv@stlpmtx_std@@AAEXPAV?$_smart_ptr@UIAnimNode@@@@ABV4@ABU__false_type@3@I_N@Z 34004fc0 f i AnimSequence.obj
 0001:00004150       ?RemoveNode@CAnimSequence@@UAEXPAUIAnimNode@@@Z 34005150 f   AnimSequence.obj
 0001:00004330       ?AddTrackEventListener@CAnimSequence@@UAEXPAUITrackEventListener@@@Z 34005330 f   AnimSequence.obj
 0001:00004380       ??$?AH@?$map@HPAUIAnimNode@@U?$less@H@stlpmtx_std@@V?$allocator@U?$pair@$$CBHPAUIAnimNode@@@stlpmtx_std@@@3@@stlpmtx_std@@QAEAAPAUIAnimNode@@ABH@Z 34005380 f i AnimSequence.obj
 0001:00004400       ?_M_insert_overflow_aux@?$_Impl_vector@V?$CryStringT@D@@V?$allocator@V?$CryStringT@D@@@stlpmtx_std@@@priv@stlpmtx_std@@AAEXPAV?$CryStringT@D@@ABV4@ABU__false_type@3@I_N@Z 34005400 f i AnimSequence.obj
 0001:00004590       ?PasteNodes@CAnimSequence@@UAEXABVXmlNodeRef@@PAUIAnimNode@@@Z 34005590 f   AnimSequence.obj
 0001:000047d0       ?push_back@?$_Impl_vector@V?$_smart_ptr@UIAnimNode@@@@V?$allocator@V?$_smart_ptr@UIAnimNode@@@@@stlpmtx_std@@@priv@stlpmtx_std@@QAEXABV?$_smart_ptr@UIAnimNode@@@@@Z 340057d0 f i AnimSequence.obj
 0001:00004840       ??$reconstruct@V?$vector@V?$_smart_ptr@UIAnimNode@@@@V?$allocator@V?$_smart_ptr@UIAnimNode@@@@@stlpmtx_std@@@stlpmtx_std@@@stl@@YAXAAV?$vector@V?$_smart_ptr@UIAnimNode@@@@V?$allocator@V?$_smart_ptr@UIAnimNode@@@@@stlpmtx_std@@@stlpmtx_std@@@Z 34005840 f i AnimSequence.obj
 0001:000048c0       ??0CAnimSequence@@QAE@PAUIMovieSystem@@I@Z 340058c0 f   AnimSequence.obj
 0001:000049a0       ?GetId@CAnimSequence@@UBEIXZ 340059a0 f i AnimSequence.obj
 0001:000049a0       ?GetFlags@CCompoundSplineTrack@@UAEHXZ 340059a0 f i CompoundSplineTrack.obj
 0001:000049b0       ?GetTime@CAnimEntityNode@@UAEMXZ 340059b0 f i AnimLightNode.obj
 0001:000049b0       ?GetFixedTimeStep@CAnimSequence@@UBEMXZ 340059b0 f i AnimSequence.obj
 0001:000049c0       ?SetFixedTimeStep@CAnimSequence@@UAEXM@Z 340059c0 f i AnimSequence.obj
 0001:000049e0       ?SetOwner@CAnimSequence@@UAEXPAUIAnimSequenceOwner@@@Z 340059e0 f i AnimSequence.obj
 0001:000049f0       ?GetOwner@CAnimSequence@@UBEPAUIAnimSequenceOwner@@XZ 340059f0 f i AnimSequence.obj
 0001:00004a00       ?GetTimeRange@CAnimSequence@@UAE?AV?$TRange@M@@XZ 34005a00 f i AnimSequence.obj
 0001:00004a20       ??$AddObject@V?$_smart_ptr@UIAnimNode@@@@V?$allocator@V?$_smart_ptr@UIAnimNode@@@@@stlpmtx_std@@@ICrySizer@@QAEXABV?$vector@V?$_smart_ptr@UIAnimNode@@@@V?$allocator@V?$_smart_ptr@UIAnimNode@@@@@stlpmtx_std@@@stlpmtx_std@@@Z 34005a20 f i AnimSequence.obj
 0001:00004aa0       ??$AddObject@PAUITrackEventListener@@V?$allocator@PAUITrackEventListener@@@stlpmtx_std@@@ICrySizer@@QAEXABV?$list@PAUITrackEventListener@@V?$allocator@PAUITrackEventListener@@@stlpmtx_std@@@stlpmtx_std@@@Z 34005aa0 f i AnimSequence.obj
 0001:00004af0       ?GetMemoryUsage@CAnimSequence@@UBEXPAVICrySizer@@@Z 34005af0 f i AnimSequence.obj
 0001:00004b40       ??1CAnimSequence@@UAE@XZ   34005b40 f   AnimSequence.obj
 0001:00004ca0       ?RemoveTrackEvent@CAnimSequence@@UAE_NPBD@Z 34005ca0 f   AnimSequence.obj
 0001:00004d00       ?insert@?$vector@V?$_smart_ptr@UIAnimNode@@@@V?$allocator@V?$_smart_ptr@UIAnimNode@@@@@stlpmtx_std@@@stlpmtx_std@@QAEPAV?$_smart_ptr@UIAnimNode@@@@PAV3@ABV3@@Z 34005d00 f i AnimSequence.obj
 0001:00004d60       ?push_back@?$_Impl_vector@V?$CryStringT@D@@V?$allocator@V?$CryStringT@D@@@stlpmtx_std@@@priv@stlpmtx_std@@QAEXABV?$CryStringT@D@@@Z 34005d60 f i AnimSequence.obj
 0001:00004dd0       ??_ECAnimSequence@@UAEPAXI@Z 34005dd0 f i AnimSequence.obj
 0001:00004dd0       ??_GCAnimSequence@@UAEPAXI@Z 34005dd0 f i AnimSequence.obj
 0001:00004e00       ?ReorderNode@CAnimSequence@@UAEXPAUIAnimNode@@0_N@Z 34005e00 f   AnimSequence.obj
 0001:00004f80       ??$reconstruct@V?$vector@V?$CryStringT@D@@V?$allocator@V?$CryStringT@D@@@stlpmtx_std@@@stlpmtx_std@@@stl@@YAXAAV?$vector@V?$CryStringT@D@@V?$allocator@V?$CryStringT@D@@@stlpmtx_std@@@stlpmtx_std@@@Z 34005f80 f i AnimSequence.obj
 0001:00005000       ?AddNode@CAnimSequence@@UAE_NPAUIAnimNode@@@Z 34006000 f   AnimSequence.obj
 0001:000051d0       ?Serialize@CAnimSequence@@UAEXAAVXmlNodeRef@@_N1I1@Z 340061d0 f   AnimSequence.obj
 0001:000059d0       ?ClearTrackEvents@CAnimSequence@@UAEXXZ 340069d0 f   AnimSequence.obj
 0001:00005a30       ??$push_back_unique@V?$vector@V?$CryStringT@D@@V?$allocator@V?$CryStringT@D@@@stlpmtx_std@@@stlpmtx_std@@PBD@stl@@YA_NAAV?$vector@V?$CryStringT@D@@V?$allocator@V?$CryStringT@D@@@stlpmtx_std@@@stlpmtx_std@@ABQBD@Z 34006a30 f i AnimSequence.obj
 0001:00005ab0       ?RemoveAll@CAnimSequence@@UAEXXZ 34006ab0 f   AnimSequence.obj
 0001:00005ae0       ?AddTrackEvent@CAnimSequence@@UAE_NPBD@Z 34006ae0 f   AnimSequence.obj
 0001:00005b20       ?GetParent@CAnimSequenceGroup@@UBEPAUIAnimSequenceGroup@@XZ 34006b20 f   AnimSequenceGroup.obj
 0001:00005b30       ??$__copy_backward@PAV?$_smart_ptr@UIAnimSequenceGroup@@@@PAV1@H@priv@stlpmtx_std@@YAPAV?$_smart_ptr@UIAnimSequenceGroup@@@@PAV2@00ABUrandom_access_iterator_tag@1@PAH@Z 34006b30 f i AnimSequenceGroup.obj
 0001:00005b30       ??$__copy_backward@PAV?$_smart_ptr@UIAnimSequence@@@@PAV1@H@priv@stlpmtx_std@@YAPAV?$_smart_ptr@UIAnimSequence@@@@PAV2@00ABUrandom_access_iterator_tag@1@PAH@Z 34006b30 f i AnimSequenceGroup.obj
 0001:00005b90       ??$__find@PAV?$_smart_ptr@UIAnimNode@@@@PAUIAnimNode@@@priv@stlpmtx_std@@YAPAV?$_smart_ptr@UIAnimNode@@@@PAV2@0ABQAUIAnimNode@@ABUrandom_access_iterator_tag@1@@Z 34006b90 f i AnimSequence.obj
 0001:00005b90       ??$__find@PAV?$_smart_ptr@UIAnimSequenceGroup@@@@PAUIAnimSequenceGroup@@@priv@stlpmtx_std@@YAPAV?$_smart_ptr@UIAnimSequenceGroup@@@@PAV2@0ABQAUIAnimSequenceGroup@@ABUrandom_access_iterator_tag@1@@Z 34006b90 f i AnimSequenceGroup.obj
 0001:00005b90       ??$__find@PAPAUIMovieListener@@PAU1@@priv@stlpmtx_std@@YAPAPAUIMovieListener@@PAPAU2@0ABQAU2@ABUrandom_access_iterator_tag@1@@Z 34006b90 f i Movie.obj
 0001:00005b90       ??$__find@PAV?$_smart_ptr@UIAnimSequence@@@@PAUIAnimSequence@@@priv@stlpmtx_std@@YAPAV?$_smart_ptr@UIAnimSequence@@@@PAV2@0ABQAUIAnimSequence@@ABUrandom_access_iterator_tag@1@@Z 34006b90 f i AnimSequenceGroup.obj
 0001:00005c00       ??$__copy@PAV?$_smart_ptr@UIAnimSequence@@@@PAV1@H@priv@stlpmtx_std@@YAPAV?$_smart_ptr@UIAnimSequence@@@@PAV2@00ABUrandom_access_iterator_tag@1@PAH@Z 34006c00 f i AnimSequenceGroup.obj
 0001:00005c00       ??$__copy@PAV?$_smart_ptr@UIAnimSequenceGroup@@@@PAV1@H@priv@stlpmtx_std@@YAPAV?$_smart_ptr@UIAnimSequenceGroup@@@@PAV2@00ABUrandom_access_iterator_tag@1@PAH@Z 34006c00 f i AnimSequenceGroup.obj
 0001:00005c60       ?GetChildSequencesCount@CAnimSequenceGroup@@UBEIXZ 34006c60 f   AnimSequenceGroup.obj
 0001:00005c70       ?GetChildGroupsCount@CAnimSequenceGroup@@UBEIXZ 34006c70 f   AnimSequenceGroup.obj
 0001:00005c80       ?GetChildSequence@CAnimSequenceGroup@@UBEPAUIAnimSequence@@I@Z 34006c80 f   AnimSequenceGroup.obj
 0001:00005cb0       ?GetChildGroup@CAnimSequenceGroup@@UBEPAUIAnimSequenceGroup@@I@Z 34006cb0 f   AnimSequenceGroup.obj
 0001:00005ce0       ??4?$CryStringT@D@@QAEAAV0@ABV0@@Z 34006ce0 f i AnimSequence.obj
 0001:00005ce0       ??4XmlString@@QAEAAV0@ABV0@@Z 34006ce0 f i AnimSequenceGroup.obj
 0001:00005d40       ??$__uninitialized_fill_n@PAV?$_smart_ptr@UIAnimSequence@@@@IV1@@priv@stlpmtx_std@@YAPAV?$_smart_ptr@UIAnimSequence@@@@PAV2@IABV2@@Z 34006d40 f i AnimSequenceGroup.obj
 0001:00005d40       ??$__uninitialized_fill_n@PAV?$_smart_ptr@VCControlParamBase@CFXNodeDescription@@@@IV1@@priv@stlpmtx_std@@YAPAV?$_smart_ptr@VCControlParamBase@CFXNodeDescription@@@@PAV2@IABV2@@Z 34006d40 f i AnimPostFXNode.obj
 0001:00005d40       ??$__uninitialized_fill_n@PAV?$_smart_ptr@UIAnimSequenceGroup@@@@IV1@@priv@stlpmtx_std@@YAPAV?$_smart_ptr@UIAnimSequenceGroup@@@@PAV2@IABV2@@Z 34006d40 f i AnimSequenceGroup.obj
 0001:00005d90       ??1XmlString@@QAE@XZ       34006d90 f i AnimSequenceGroup.obj
 0001:00005d90       ??1?$CryStringT@D@@QAE@XZ  34006d90 f i AnimSequence.obj
 0001:00005dc0       ?SetName@CAnimSequenceGroup@@UAEXPBD@Z 34006dc0 f   AnimSequenceGroup.obj
 0001:00005e40       ?SetParent@CAnimSequenceGroup@@UAEXPAUIAnimSequenceGroup@@@Z 34006e40 f   AnimSequenceGroup.obj
 0001:00005ec0       ?SetParentAndName@CAnimSequenceGroup@@UAEXPAUIAnimSequenceGroup@@PBD@Z 34006ec0 f   AnimSequenceGroup.obj
 0001:00005f60       ??R?$LexicoCompare@UIAnimSequenceGroup@@@@QBE_NV?$_smart_ptr@UIAnimSequenceGroup@@@@0@Z 34006f60 f i AnimSequenceGroup.obj
 0001:00006020       ??R?$LexicoCompare@UIAnimSequence@@@@QBE_NV?$_smart_ptr@UIAnimSequence@@@@0@Z 34007020 f i AnimSequenceGroup.obj
 0001:000060e0       ??$__unguarded_linear_insert@PAV?$_smart_ptr@UIAnimSequenceGroup@@@@V1@U?$LexicoCompare@UIAnimSequenceGroup@@@@@priv@stlpmtx_std@@YAXPAV?$_smart_ptr@UIAnimSequenceGroup@@@@V2@U?$LexicoCompare@UIAnimSequenceGroup@@@@@Z 340070e0 f i AnimSequenceGroup.obj
 0001:00006180       ??$__unguarded_linear_insert@PAV?$_smart_ptr@UIAnimSequence@@@@V1@U?$LexicoCompare@UIAnimSequence@@@@@priv@stlpmtx_std@@YAXPAV?$_smart_ptr@UIAnimSequence@@@@V2@U?$LexicoCompare@UIAnimSequence@@@@@Z 34007180 f i AnimSequenceGroup.obj
 0001:00006220       ??$__push_heap@PAV?$_smart_ptr@UIAnimSequenceGroup@@@@HV1@U?$LexicoCompare@UIAnimSequenceGroup@@@@@stlpmtx_std@@YAXPAV?$_smart_ptr@UIAnimSequenceGroup@@@@HHV1@U?$LexicoCompare@UIAnimSequenceGroup@@@@@Z 34007220 f i AnimSequenceGroup.obj
 0001:000062f0       ??$__push_heap@PAV?$_smart_ptr@UIAnimSequence@@@@HV1@U?$LexicoCompare@UIAnimSequence@@@@@stlpmtx_std@@YAXPAV?$_smart_ptr@UIAnimSequence@@@@HHV1@U?$LexicoCompare@UIAnimSequence@@@@@Z 340072f0 f i AnimSequenceGroup.obj
 0001:000063c0       ?OnRenamed@CAnimSequenceGroup@@UBEXPBD@Z 340073c0 f   AnimSequenceGroup.obj
 0001:00006860       ?erase@?$vector@V?$_smart_ptr@UIAnimSequence@@@@V?$allocator@V?$_smart_ptr@UIAnimSequence@@@@@stlpmtx_std@@@stlpmtx_std@@QAEPAV?$_smart_ptr@UIAnimSequence@@@@PAV3@@Z 34007860 f i AnimSequenceGroup.obj
 0001:00006860       ?erase@?$vector@V?$_smart_ptr@UIAnimSequenceGroup@@@@V?$allocator@V?$_smart_ptr@UIAnimSequenceGroup@@@@@stlpmtx_std@@@stlpmtx_std@@QAEPAV?$_smart_ptr@UIAnimSequenceGroup@@@@PAV3@@Z 34007860 f i AnimSequenceGroup.obj
 0001:000068c0       ??$__median@V?$_smart_ptr@UIAnimSequenceGroup@@@@U?$LexicoCompare@UIAnimSequenceGroup@@@@@priv@stlpmtx_std@@YAABV?$_smart_ptr@UIAnimSequenceGroup@@@@ABV2@00U?$LexicoCompare@UIAnimSequenceGroup@@@@@Z 340078c0 f i AnimSequenceGroup.obj
 0001:000069e0       ??$__unguarded_partition@PAV?$_smart_ptr@UIAnimSequenceGroup@@@@V1@U?$LexicoCompare@UIAnimSequenceGroup@@@@@priv@stlpmtx_std@@YAPAV?$_smart_ptr@UIAnimSequenceGroup@@@@PAV2@0V2@U?$LexicoCompare@UIAnimSequenceGroup@@@@@Z 340079e0 f i AnimSequenceGroup.obj
 0001:00006a90       ??$__median@V?$_smart_ptr@UIAnimSequence@@@@U?$LexicoCompare@UIAnimSequence@@@@@priv@stlpmtx_std@@YAABV?$_smart_ptr@UIAnimSequence@@@@ABV2@00U?$LexicoCompare@UIAnimSequence@@@@@Z 34007a90 f i AnimSequenceGroup.obj
 0001:00006bb0       ??$__unguarded_partition@PAV?$_smart_ptr@UIAnimSequence@@@@V1@U?$LexicoCompare@UIAnimSequence@@@@@priv@stlpmtx_std@@YAPAV?$_smart_ptr@UIAnimSequence@@@@PAV2@0V2@U?$LexicoCompare@UIAnimSequence@@@@@Z 34007bb0 f i AnimSequenceGroup.obj
 0001:00006c60       ??$__linear_insert@PAV?$_smart_ptr@UIAnimSequenceGroup@@@@V1@U?$LexicoCompare@UIAnimSequenceGroup@@@@@priv@stlpmtx_std@@YAXPAV?$_smart_ptr@UIAnimSequenceGroup@@@@0V2@U?$LexicoCompare@UIAnimSequenceGroup@@@@@Z 34007c60 f i AnimSequenceGroup.obj
 0001:00006d20       ??$__linear_insert@PAV?$_smart_ptr@UIAnimSequence@@@@V1@U?$LexicoCompare@UIAnimSequence@@@@@priv@stlpmtx_std@@YAXPAV?$_smart_ptr@UIAnimSequence@@@@0V2@U?$LexicoCompare@UIAnimSequence@@@@@Z 34007d20 f i AnimSequenceGroup.obj
 0001:00006de0       ??$__adjust_heap@PAV?$_smart_ptr@UIAnimSequenceGroup@@@@HV1@U?$LexicoCompare@UIAnimSequenceGroup@@@@@stlpmtx_std@@YAXPAV?$_smart_ptr@UIAnimSequenceGroup@@@@HHV1@U?$LexicoCompare@UIAnimSequenceGroup@@@@@Z 34007de0 f i AnimSequenceGroup.obj
 0001:00006ed0       ??$__adjust_heap@PAV?$_smart_ptr@UIAnimSequence@@@@HV1@U?$LexicoCompare@UIAnimSequence@@@@@stlpmtx_std@@YAXPAV?$_smart_ptr@UIAnimSequence@@@@HHV1@U?$LexicoCompare@UIAnimSequence@@@@@Z 34007ed0 f i AnimSequenceGroup.obj
 0001:00006fc0       ?GetFullName@CAnimSequenceGroup@@UBEPBDXZ 34007fc0 f   AnimSequenceGroup.obj
 0001:00007200       ?Serialize@CAnimSequenceGroup@@UAEXAAVXmlNodeRef@@_N@Z 34008200 f   AnimSequenceGroup.obj
 0001:000078e0       ??1?$_Impl_vector@V?$_smart_ptr@UIAnimSequence@@@@V?$allocator@V?$_smart_ptr@UIAnimSequence@@@@@stlpmtx_std@@@priv@stlpmtx_std@@QAE@XZ 340088e0 f i AnimSequenceGroup.obj
 0001:000078e0       ??1?$_Impl_vector@V?$_smart_ptr@VCControlParamBase@CFXNodeDescription@@@@V?$allocator@V?$_smart_ptr@VCControlParamBase@CFXNodeDescription@@@@@stlpmtx_std@@@priv@stlpmtx_std@@QAE@XZ 340088e0 f i AnimPostFXNode.obj
 0001:000078e0       ??1?$_Impl_vector@V?$_smart_ptr@UIAnimSequenceGroup@@@@V?$allocator@V?$_smart_ptr@UIAnimSequenceGroup@@@@@stlpmtx_std@@@priv@stlpmtx_std@@QAE@XZ 340088e0 f i AnimSequenceGroup.obj
 0001:00007930       ??$__insertion_sort@PAV?$_smart_ptr@UIAnimSequenceGroup@@@@V1@U?$LexicoCompare@UIAnimSequenceGroup@@@@@priv@stlpmtx_std@@YAXPAV?$_smart_ptr@UIAnimSequenceGroup@@@@00U?$LexicoCompare@UIAnimSequenceGroup@@@@@Z 34008930 f i AnimSequenceGroup.obj
 0001:00007980       ??$__unguarded_insertion_sort@PAV?$_smart_ptr@UIAnimSequenceGroup@@@@U?$LexicoCompare@UIAnimSequenceGroup@@@@@priv@stlpmtx_std@@YAXPAV?$_smart_ptr@UIAnimSequenceGroup@@@@0U?$LexicoCompare@UIAnimSequenceGroup@@@@@Z 34008980 f i AnimSequenceGroup.obj
 0001:000079d0       ??$__insertion_sort@PAV?$_smart_ptr@UIAnimSequence@@@@V1@U?$LexicoCompare@UIAnimSequence@@@@@priv@stlpmtx_std@@YAXPAV?$_smart_ptr@UIAnimSequence@@@@00U?$LexicoCompare@UIAnimSequence@@@@@Z 340089d0 f i AnimSequenceGroup.obj
 0001:00007a20       ??$__unguarded_insertion_sort@PAV?$_smart_ptr@UIAnimSequence@@@@U?$LexicoCompare@UIAnimSequence@@@@@priv@stlpmtx_std@@YAXPAV?$_smart_ptr@UIAnimSequence@@@@0U?$LexicoCompare@UIAnimSequence@@@@@Z 34008a20 f i AnimSequenceGroup.obj
 0001:00007a70       ??$__make_heap@PAV?$_smart_ptr@UIAnimSequenceGroup@@@@U?$LexicoCompare@UIAnimSequenceGroup@@@@V1@H@stlpmtx_std@@YAXPAV?$_smart_ptr@UIAnimSequenceGroup@@@@0U?$LexicoCompare@UIAnimSequenceGroup@@@@0PAH@Z 34008a70 f i AnimSequenceGroup.obj
 0001:00007ac0       ??$__make_heap@PAV?$_smart_ptr@UIAnimSequence@@@@U?$LexicoCompare@UIAnimSequence@@@@V1@H@stlpmtx_std@@YAXPAV?$_smart_ptr@UIAnimSequence@@@@0U?$LexicoCompare@UIAnimSequence@@@@0PAH@Z 34008ac0 f i AnimSequenceGroup.obj
 0001:00007b10       ?RemoveChildSequence@CAnimSequenceGroup@@UAE_NPAUIAnimSequence@@@Z 34008b10 f   AnimSequenceGroup.obj
 0001:00007b50       ?RemoveChildGroup@CAnimSequenceGroup@@UAE_NPAUIAnimSequenceGroup@@@Z 34008b50 f   AnimSequenceGroup.obj
 0001:00007b90       ??0CAnimSequenceGroup@@QAE@PAUIMovieSystem@@@Z 34008b90 f   AnimSequenceGroup.obj
 0001:00007c00       ??$AddObject@V?$_smart_ptr@UIAnimSequenceGroup@@@@V?$allocator@V?$_smart_ptr@UIAnimSequenceGroup@@@@@stlpmtx_std@@@ICrySizer@@QAEXABV?$vector@V?$_smart_ptr@UIAnimSequenceGroup@@@@V?$allocator@V?$_smart_ptr@UIAnimSequenceGroup@@@@@stlpmtx_std@@@stlpmtx_std@@@Z 34008c00 f i AnimSequenceGroup.obj
 0001:00007c70       ??$AddObject@V?$_smart_ptr@UIAnimSequence@@@@V?$allocator@V?$_smart_ptr@UIAnimSequence@@@@@stlpmtx_std@@@ICrySizer@@QAEXABV?$vector@V?$_smart_ptr@UIAnimSequence@@@@V?$allocator@V?$_smart_ptr@UIAnimSequence@@@@@stlpmtx_std@@@stlpmtx_std@@@Z 34008c70 f i AnimSequenceGroup.obj
 0001:00007cf0       ?GetMemoryUsage@CAnimSequenceGroup@@UBEXPAVICrySizer@@@Z 34008cf0 f i AnimSequenceGroup.obj
 0001:00007d40       ??1CAnimSequenceGroup@@UAE@XZ 34008d40 f i AnimSequenceGroup.obj
 0001:00007dc0       ??_ECAnimSequenceGroup@@UAEPAXI@Z 34008dc0 f i AnimSequenceGroup.obj
 0001:00007dc0       ??_GCAnimSequenceGroup@@UAEPAXI@Z 34008dc0 f i AnimSequenceGroup.obj
 0001:00007df0       ??$sort_heap@PAV?$_smart_ptr@UIAnimSequenceGroup@@@@U?$LexicoCompare@UIAnimSequenceGroup@@@@@stlpmtx_std@@YAXPAV?$_smart_ptr@UIAnimSequenceGroup@@@@0U?$LexicoCompare@UIAnimSequenceGroup@@@@@Z 34008df0 f i AnimSequenceGroup.obj
 0001:00007ea0       ??$sort_heap@PAV?$_smart_ptr@UIAnimSequence@@@@U?$LexicoCompare@UIAnimSequence@@@@@stlpmtx_std@@YAXPAV?$_smart_ptr@UIAnimSequence@@@@0U?$LexicoCompare@UIAnimSequence@@@@@Z 34008ea0 f i AnimSequenceGroup.obj
 0001:00007f50       ??$__partial_sort@PAV?$_smart_ptr@UIAnimSequenceGroup@@@@V1@U?$LexicoCompare@UIAnimSequenceGroup@@@@@priv@stlpmtx_std@@YAXPAV?$_smart_ptr@UIAnimSequenceGroup@@@@000U?$LexicoCompare@UIAnimSequenceGroup@@@@@Z 34008f50 f i AnimSequenceGroup.obj
 0001:00008040       ??$__partial_sort@PAV?$_smart_ptr@UIAnimSequence@@@@V1@U?$LexicoCompare@UIAnimSequence@@@@@priv@stlpmtx_std@@YAXPAV?$_smart_ptr@UIAnimSequence@@@@000U?$LexicoCompare@UIAnimSequence@@@@@Z 34009040 f i AnimSequenceGroup.obj
 0001:00008130       ?Clear@CAnimSequenceGroup@@UAEXXZ 34009130 f   AnimSequenceGroup.obj
 0001:000081a0       ??$push_back_unique@V?$vector@V?$_smart_ptr@UIAnimSequence@@@@V?$allocator@V?$_smart_ptr@UIAnimSequence@@@@@stlpmtx_std@@@stlpmtx_std@@PAUIAnimSequence@@@stl@@YA_NAAV?$vector@V?$_smart_ptr@UIAnimSequence@@@@V?$allocator@V?$_smart_ptr@UIAnimSequence@@@@@stlpmtx_std@@@stlpmtx_std@@ABQAUIAnimSequence@@@Z 340091a0 f i AnimSequenceGroup.obj
 0001:000081a0       ??$push_back_unique@V?$vector@V?$_smart_ptr@UIAnimSequenceGroup@@@@V?$allocator@V?$_smart_ptr@UIAnimSequenceGroup@@@@@stlpmtx_std@@@stlpmtx_std@@PAUIAnimSequenceGroup@@@stl@@YA_NAAV?$vector@V?$_smart_ptr@UIAnimSequenceGroup@@@@V?$allocator@V?$_smart_ptr@UIAnimSequenceGroup@@@@@stlpmtx_std@@@stlpmtx_std@@ABQAUIAnimSequenceGroup@@@Z 340091a0 f i AnimSequenceGroup.obj
 0001:00008240       ?AddChildSequence@CAnimSequenceGroup@@UAE_NPAUIAnimSequence@@@Z 34009240 f   AnimSequenceGroup.obj
 0001:00008260       ?AddChildGroup@CAnimSequenceGroup@@UAE_NPAUIAnimSequenceGroup@@@Z 34009260 f   AnimSequenceGroup.obj
 0001:00008280       ??$__introsort_loop@PAV?$_smart_ptr@UIAnimSequenceGroup@@@@V1@HU?$LexicoCompare@UIAnimSequenceGroup@@@@@priv@stlpmtx_std@@YAXPAV?$_smart_ptr@UIAnimSequenceGroup@@@@00HU?$LexicoCompare@UIAnimSequenceGroup@@@@@Z 34009280 f i AnimSequenceGroup.obj
 0001:00008320       ??$__introsort_loop@PAV?$_smart_ptr@UIAnimSequence@@@@V1@HU?$LexicoCompare@UIAnimSequence@@@@@priv@stlpmtx_std@@YAXPAV?$_smart_ptr@UIAnimSequence@@@@00HU?$LexicoCompare@UIAnimSequence@@@@@Z 34009320 f i AnimSequenceGroup.obj
 0001:000083c0       ??$sort@PAV?$_smart_ptr@UIAnimSequenceGroup@@@@U?$LexicoCompare@UIAnimSequenceGroup@@@@@stlpmtx_std@@YAXPAV?$_smart_ptr@UIAnimSequenceGroup@@@@0U?$LexicoCompare@UIAnimSequenceGroup@@@@@Z 340093c0 f i AnimSequenceGroup.obj
 0001:00008440       ??$sort@PAV?$_smart_ptr@UIAnimSequence@@@@U?$LexicoCompare@UIAnimSequence@@@@@stlpmtx_std@@YAXPAV?$_smart_ptr@UIAnimSequence@@@@0U?$LexicoCompare@UIAnimSequence@@@@@Z 34009440 f i AnimSequenceGroup.obj
 0001:000084c0       ?Sort@CAnimSequenceGroup@@UAEXXZ 340094c0 f   AnimSequenceGroup.obj
 0001:00008530       ?Init@_CryMemoryManagerPoolHelper@@SAXXZ 34009530 f i CryMovie.obj
 0001:000086b0       ?CryGetIMemoryManager@@YAPAUIMemoryManager@@XZ 340096b0 f   CryMovie.obj
 0001:000086f0       ?CryInterlockedDecrement@@YAJPCH@Z 340096f0 f   CryMovie.obj
 0001:00008700       ?CryCreateCriticalSectionInplace@@YAXPAX@Z 34009700 f   CryMovie.obj
 0001:00008710       ?CryGetCurrentThreadId@@YAIXZ 34009710 f   CryMovie.obj
 0001:00008720       ?CryPureCallHandler@@YAXXZ 34009720 f   CryMovie.obj
 0001:00008730       ?CryInvalidParameterHandler@@YAXPB_W00II@Z 34009730 f   CryMovie.obj
 0001:00008740       _ModuleInitISystem         34009740 f   CryMovie.obj
 0001:000087f0       _CryModuleGetMemoryInfo    340097f0 f   CryMovie.obj
 0001:00008840       ?CryDeleteCriticalSectionInplace@@YAXPAX@Z 34009840 f   CryMovie.obj
 0001:00008870       ?OnSystemEvent@CSystemEventListner_Movie@@UAEXW4ESystemEvent@@II@Z 34009870 f i CryMovie.obj
 0001:00008890       ??$?8D@@YA_NABV?$CryStringT@D@@0@Z 34009890 f i CryMovie.obj
 0001:000088e0       _CryModuleMalloc           340098e0 f   CryMovie.obj
 0001:00008970       _CryModuleFree             34009970 f   CryMovie.obj
 0001:000089d0       _CryModuleMemalign         340099d0 f   CryMovie.obj
 0001:00008a60       ??2@YAPAXI@Z               34009a60 f   CryMovie.obj
 0001:00008ab0       ??3@YAXPAX@Z               34009ab0 f   CryMovie.obj
 0001:00008b30       ??_EICryFactory@@MAEPAXI@Z 34009b30 f i CryMovie.obj
 0001:00008b30       ??_GICryFactory@@MAEPAXI@Z 34009b30 f i CryMovie.obj
 0001:00008b60       ??_GCSystemEventListner_Movie@@UAEPAXI@Z 34009b60 f i CryMovie.obj
 0001:00008b60       ??_GISystemEventListener@@UAEPAXI@Z 34009b60 f i CryMovie.obj
 0001:00008b60       ??_EISystemEventListener@@UAEPAXI@Z 34009b60 f i CryMovie.obj
 0001:00008b60       ??_ECSystemEventListner_Movie@@UAEPAXI@Z 34009b60 f i CryMovie.obj
 0001:00008b90       ?GetFactory@CEngineModule_CryMovie@@UBEPAUICryFactory@@XZ 34009b90 f i CryMovie.obj
 0001:00008ba0       ?GetName@CEngineModule_CryMovie@@MAEPBDXZ 34009ba0 f i CryMovie.obj
 0001:00008bb0       ?GetCategory@CEngineModule_CryMovie@@MAEPBDXZ 34009bb0 f i CryMovie.obj
 0001:00008bc0       ?Initialize@CEngineModule_CryMovie@@MAE_NAAUSSystemGlobalEnvironment@@ABUSSystemInitParams@@@Z 34009bc0 f i CryMovie.obj
 0001:00008c60       ??_GCEngineModule_CryMovie@@MAEPAXI@Z 34009c60 f i CryMovie.obj
 0001:00008c60       ??_EICryUnknown@@MAEPAXI@Z 34009c60 f i CryMovie.obj
 0001:00008c60       ??_GICryUnknown@@MAEPAXI@Z 34009c60 f i CryMovie.obj
 0001:00008c60       ??_ECEngineModule_CryMovie@@MAEPAXI@Z 34009c60 f i CryMovie.obj
 0001:00008c90       ?_MakeUnique@?$CryStringT@D@@IAEXXZ 34009c90 f i CryMovie.obj
 0001:00008d30       ??0CFactory@CEngineModule_CryMovie@@AAE@XZ 34009d30 f i CryMovie.obj
 0001:00008de0       ?GetClassNameA@CFactory@CEngineModule_CryMovie@@UBEPBDXZ 34009de0 f i CryMovie.obj
 0001:00008df0       ?GetClassID@CFactory@CEngineModule_CryMovie@@UBEABUCryGUID@@XZ 34009df0 f i CryMovie.obj
 0001:00008e00       ?ClassSupports@CFactory@CEngineModule_CryMovie@@UBEXAAPBUCryGUID@@AAI@Z 34009e00 f i CryMovie.obj
 0001:00008e20       ?destroy@sp_counted_base@detail@boost@@UAEXXZ 34009e20 f i CryMovie.obj
 0001:00008e20       ?Release@CMovieSystem@@UAEXXZ 34009e20 f i Movie.obj
 0001:00008e30       ??$throw_exception@Vbad_alloc@std@@@boost@@YAXABVbad_alloc@std@@@Z 34009e30 f i CryMovie.obj
 0001:00008e60       ?ClassSupports@CFactory@CEngineModule_CryMovie@@UBE_NABUCryGUID@@@Z 34009e60 f i CryMovie.obj
 0001:00008eb0       ?dispose@?$sp_counted_impl_p@VCEngineModule_CryMovie@@@detail@boost@@UAEXXZ 34009eb0 f i CryMovie.obj
 0001:00008ec0       ??_GCFactory@CEngineModule_CryMovie@@UAEPAXI@Z 34009ec0 f i CryMovie.obj
 0001:00008ec0       ??_ECFactory@CEngineModule_CryMovie@@UAEPAXI@Z 34009ec0 f i CryMovie.obj
 0001:00008ef0       ??_E?$sp_counted_impl_p@VCEngineModule_CryMovie@@@detail@boost@@UAEPAXI@Z 34009ef0 f i CryMovie.obj
 0001:00008ef0       ??_Gsp_counted_base@detail@boost@@UAEPAXI@Z 34009ef0 f i CryMovie.obj
 0001:00008ef0       ??_G?$sp_counted_impl_p@VCEngineModule_CryMovie@@@detail@boost@@UAEPAXI@Z 34009ef0 f i CryMovie.obj
 0001:00008ef0       ??_Esp_counted_base@detail@boost@@UAEPAXI@Z 34009ef0 f i CryMovie.obj
 0001:00008f20       ??$?0VCEngineModule_CryMovie@@@shared_count@detail@boost@@QAE@PAVCEngineModule_CryMovie@@@Z 34009f20 f i CryMovie.obj
 0001:00008fd0       ??_Gbad_alloc@std@@UAEPAXI@Z 34009fd0 f i CryMovie.obj
 0001:00008fd0       ??_Ebad_alloc@std@@UAEPAXI@Z 34009fd0 f i CryMovie.obj
 0001:00009000       ?QueryInterface@CEngineModule_CryMovie@@MBEPAXABUCryGUID@@@Z 3400a000 f i CryMovie.obj
 0001:00009060       ?append@?$CryStringT@D@@QAEAAV1@ID@Z 3400a060 f i CryMovie.obj
 0001:00009110       ?CreateClassInstance@CFactory@CEngineModule_CryMovie@@UBE?AV?$shared_ptr@UICryUnknown@@@boost@@XZ 3400a110 f i CryMovie.obj
 0001:000091e0       ??_EISplineInterpolator@@UAEPAXI@Z 3400a1e0 f i Movie.obj
 0001:000091e0       ??_GISplineInterpolator@@UAEPAXI@Z 3400a1e0 f i Movie.obj
 0001:00009210       ??4XmlNodeRef@@QAEAAV0@ABV0@@Z 3400a210 f i Movie.obj
 0001:00009240       ?CryLogAlways@@YAXPBDZZ    3400a240 f i Movie.obj
 0001:00009270       ?DeleteSequenceGroup@CMovieSystem@@UAEXPAUIAnimSequenceGroup@@@Z 3400a270 f   Movie.obj
 0001:000092b0       ?PlaySequence@CMovieSystem@@UAEXPBDPAUIAnimSequence@@_N2MM@Z 3400a2b0 f   Movie.obj
 0001:00009320       ?StopSequence@CMovieSystem@@UAE_NPBD@Z 3400a320 f   Movie.obj
 0001:00009350       ?Callback@CMovieSystem@@QAEXW4ECallbackReason@IMovieCallback@@PAUIAnimNode@@@Z 3400a350 f   Movie.obj
 0001:00009370       ?SetCameraParams@CMovieSystem@@UAEXABUSCameraParams@@@Z 3400a370 f   Movie.obj
 0001:000093c0       ?SendGlobalEvent@CMovieSystem@@UAEXPBD@Z 3400a3c0 f   Movie.obj
 0001:000093e0       ?Pause@CMovieSystem@@UAEXXZ 3400a3e0 f   Movie.obj
 0001:000093f0       ?Resume@CMovieSystem@@UAEXXZ 3400a3f0 f   Movie.obj
 0001:00009400       ?OnPlaySound@CMovieSystem@@QAEXPAUIAnimSequence@@PAUISound@@@Z 3400a400 f   Movie.obj
 0001:00009440       ?SetSequenceStopBehavior@CMovieSystem@@UAEXW4ESequenceStopBehavior@IMovieSystem@@@Z 3400a440 f   Movie.obj
 0001:00009450       ?GoToFrameCmd@CMovieSystem@@KAXPAUIConsoleCmdArgs@@@Z 3400a450 f   Movie.obj
 0001:000094c0       ?ListSequencesCmd@CMovieSystem@@KAXPAUIConsoleCmdArgs@@@Z 3400a4c0 f   Movie.obj
 0001:00009520       ?PlaySequencesCmd@CMovieSystem@@KAXPAUIConsoleCmdArgs@@@Z 3400a520 f   Movie.obj
 0001:00009560       ?StartCapture@CMovieSystem@@UAEXABUICaptureKey@@@Z 3400a560 f   Movie.obj
 0001:00009580       ?EndCapture@CMovieSystem@@UAEXXZ 3400a580 f   Movie.obj
 0001:00009590       ?SerializeSequenceGroups@CMovieSystem@@UAEXAAVXmlNodeRef@@_N@Z 3400a590 f   Movie.obj
 0001:00009630       ?GetEntityNodeParamCount@CMovieSystem@@UBEHXZ 3400a630 f   Movie.obj
 0001:00009640       ?GetEntityNodeParamInfo@CMovieSystem@@UBE_NHAAUSParamInfo@IAnimNode@@@Z 3400a640 f   Movie.obj
 0001:00009660       ??E?$_Rb_tree_iterator@U?$pair@$$CBHPAUIAnimNode@@@stlpmtx_std@@U?$_MapTraitsT@U?$pair@$$CBHPAUIAnimNode@@@stlpmtx_std@@@priv@2@@priv@stlpmtx_std@@QAEAAU012@XZ 3400a660 f i AnimSequence.obj
 0001:00009660       ??E?$_Rb_tree_iterator@U?$pair@$$CBW4EAnimNodeType@@V?$_smart_ptr@VCFXNodeDescription@@@@@stlpmtx_std@@U?$_MapTraitsT@U?$pair@$$CBW4EAnimNodeType@@V?$_smart_ptr@VCFXNodeDescription@@@@@stlpmtx_std@@@priv@2@@priv@stlpmtx_std@@QAEAAU012@XZ 3400a660 f i AnimPostFXNode.obj
 0001:00009660       ??E?$_Rb_tree_iterator@U?$pair@QAUIEntity@@PAUIAnimNode@@@stlpmtx_std@@U?$_MapTraitsT@U?$pair@QAUIEntity@@PAUIAnimNode@@@stlpmtx_std@@@priv@2@@priv@stlpmtx_std@@QAEAAU012@XZ 3400a660 f i Movie.obj
 0001:00009660       ??E?$_Rb_tree_iterator@U?$pair@QAUIAnimSequence@@V?$vector@PAUIMovieListener@@V?$allocator@PAUIMovieListener@@@stlpmtx_std@@@stlpmtx_std@@@stlpmtx_std@@U?$_MapTraitsT@U?$pair@QAUIAnimSequence@@V?$vector@PAUIMovieListener@@V?$allocator@PAUIMovieListener@@@stlpmtx_std@@@stlpmtx_std@@@stlpmtx_std@@@priv@2@@priv@stlpmtx_std@@QAEAAU012@XZ 3400a660 f i Movie.obj
 0001:000096a0       ??_GIMovieSystem@@UAEPAXI@Z 3400a6a0 f i Movie.obj
 0001:000096a0       ??_EIMovieSystem@@UAEPAXI@Z 3400a6a0 f i Movie.obj
 0001:000096d0       ?SaveToColladaInFixedFPS@IAnimTrack@@UAEXABUSColladaExporterSaveProperties@@VXmlNodeRef@@PBD2@Z 3400a6d0 f i Movie.obj
 0001:000096f0       ?NextKeyByTime@IAnimTrack@@UBEHH@Z 3400a6f0 f i Movie.obj
 0001:00009720       ?GetCount@SMovieSequenceAutoComplete@@UBEHXZ 3400a720 f i Movie.obj
 0001:00009730       ?GetValue@SMovieSequenceAutoComplete@@UBEPBDH@Z 3400a730 f i Movie.obj
 0001:00009760       ??_EIConsoleArgumentAutoComplete@@UAEPAXI@Z 3400a760 f i Movie.obj
 0001:00009760       ??_GIConsoleArgumentAutoComplete@@UAEPAXI@Z 3400a760 f i Movie.obj
 0001:00009760       ??_GSMovieSequenceAutoComplete@@UAEPAXI@Z 3400a760 f i Movie.obj
 0001:00009760       ??_ESMovieSequenceAutoComplete@@UAEPAXI@Z 3400a760 f i Movie.obj
 0001:00009790       ?CreateSequenceGroup@CMovieSystem@@UAEPAUIAnimSequenceGroup@@PBDPAU2@@Z 3400a790 f   Movie.obj
 0001:000097f0       ?ControlCapture@CMovieSystem@@UAEXXZ 3400a7f0 f   Movie.obj
 0001:00009a00       ?GetRootGroup@CMovieSystem@@UBEPAUIAnimSequenceGroup@@XZ 3400aa00 f   Movie.obj
 0001:00009a00       ?GetFlags@CAnimNode@@UBEHXZ 3400aa00 f   AnimNode.obj
 0001:00009a00       ?GetName@CAnimSequence@@UBEPBDXZ 3400aa00 f   AnimSequence.obj
 0001:00009a10       ?GetLightAnimSet@CLightAnimWrapper@@SAPAUIAnimSequence@@XZ 3400aa10 f   Movie.obj
 0001:00009a20       ?SetLightAnimSet@CLightAnimWrapper@@SAXPAUIAnimSequence@@@Z 3400aa20 f   Movie.obj
 0001:00009a50       ??0ICaptureKey@@QAE@XZ     3400aa50 f i Movie.obj
 0001:00009b50       ?Draw2dLabel@IRenderer@@QAAXMMMPBM_NPBDZZ 3400ab50 f i Movie.obj
 0001:00009c20       ?_Rebalance_for_erase@?$_Rb_global@_N@priv@stlpmtx_std@@SAPAU_Rb_tree_node_base@23@PAU423@AAPAU423@11@Z 3400ac20 f i Movie.obj
 0001:00009f10       ?FindSequence@CMovieSystem@@UBEPAUIAnimSequence@@PBD@Z 3400af10 f   Movie.obj
 0001:00009f70       ?FindSequenceById@CMovieSystem@@UBEPAUIAnimSequence@@I@Z 3400af70 f   Movie.obj
 0001:00009fd0       ?GetSequence@CMovieSystem@@UBEPAUIAnimSequence@@H@Z 3400afd0 f   Movie.obj
 0001:0000a000       ?GetNumSequences@CMovieSystem@@UBEHXZ 3400b000 f   Movie.obj
 0001:0000a010       ?GetPlayingSequence@CMovieSystem@@UBEPAUIAnimSequence@@H@Z 3400b010 f   Movie.obj
 0001:0000a040       ?GetNumPlayingSequences@CMovieSystem@@UBEHXZ 3400b040 f   Movie.obj
 0001:0000a060       ?OnSequenceRenamed@CMovieSystem@@UAEHPBD0@Z 3400b060 f   Movie.obj
 0001:0000a210       ?OnCameraRenamed@CMovieSystem@@UAEHPBD0@Z 3400b210 f   Movie.obj
 0001:0000a3f0       ?IsPlaying@CMovieSystem@@UBE_NPAUIAnimSequence@@@Z 3400b3f0 f   Movie.obj
 0001:0000a420       ?PlayOnLoadSequences@CMovieSystem@@UAEXXZ 3400b420 f   Movie.obj
 0001:0000a4c0       ?StillUpdate@CMovieSystem@@UAEXXZ 3400b4c0 f   Movie.obj
 0001:0000a500       ?Render@CMovieSystem@@UAEXXZ 3400b500 f   Movie.obj
 0001:0000a530       ?PauseCutScenes@CMovieSystem@@UAEXXZ 3400b530 f   Movie.obj
 0001:0000a590       ?ResumeCutScenes@CMovieSystem@@UAEXXZ 3400b590 f   Movie.obj
 0001:0000a600       ?GetPlayingTime@CMovieSystem@@UAEMPAUIAnimSequence@@@Z 3400b600 f   Movie.obj
 0001:0000a650       ?GetPlayingSpeed@CMovieSystem@@UAEMPAUIAnimSequence@@@Z 3400b650 f   Movie.obj
 0001:0000a6a0       ?SetPlayingTime@CMovieSystem@@UAE_NPAUIAnimSequence@@M@Z 3400b6a0 f   Movie.obj
 0001:0000a700       ?SetPlayingSpeed@CMovieSystem@@UAE_NPAUIAnimSequence@@M@Z 3400b700 f   Movie.obj
 0001:0000a760       ?GetStartEndTime@CMovieSystem@@UAE_NPAUIAnimSequence@@AAM1@Z 3400b760 f   Movie.obj
 0001:0000a7d0       ?SetStartEndTime@CMovieSystem@@UAE_NPAUIAnimSequence@@MM@Z 3400b7d0 f   Movie.obj
 0001:0000a830       ?Resolve@CLightAnimWrapper@@UAE_NXZ 3400b830 f   Movie.obj
 0001:0000a870       ??R?$less@V?$CryStringT@D@@@stlpmtx_std@@QBE_NABV?$CryStringT@D@@0@Z 3400b870 f i Movie.obj
 0001:0000a8c0       ?allocate@?$_STLP_alloc_proxy@PAUSkelAnimUpdateCMD@CMovieSystem@@U12@V?$allocator@USkelAnimUpdateCMD@CMovieSystem@@@stlpmtx_std@@@priv@stlpmtx_std@@QAEPAUSkelAnimUpdateCMD@CMovieSystem@@IAAI@Z 3400b8c0 f i Movie.obj
 0001:0000a920       ??$_M_find@V?$CryStringT@D@@@?$_Rb_tree@V?$CryStringT@D@@U?$less@V?$CryStringT@D@@@stlpmtx_std@@U?$pair@$$CBV?$CryStringT@D@@PAVCLightAnimWrapper@@@3@U?$_Select1st@U?$pair@$$CBV?$CryStringT@D@@PAVCLightAnimWrapper@@@stlpmtx_std@@@priv@3@U?$_MapTraitsT@U?$pair@$$CBV?$CryStringT@D@@PAVCLightAnimWrapper@@@stlpmtx_std@@@63@V?$allocator@U?$pair@$$CBV?$CryStringT@D@@PAVCLightAnimWrapper@@@stlpmtx_std@@@3@@priv@stlpmtx_std@@ABEPAU_Rb_tree_node_base@12@ABV?$CryStringT@D@@@Z 3400b920 f i Movie.obj
 0001:0000a9c0       ??$__copy@PAUPlayingSequence@@PAU1@H@priv@stlpmtx_std@@YAPAUPlayingSequence@@PAU2@00ABUrandom_access_iterator_tag@1@PAH@Z 3400b9c0 f i Movie.obj
 0001:0000aa50       ??_EILightAnimWrapper@@MAEPAXI@Z 3400ba50 f i Movie.obj
 0001:0000aa50       ??_GILightAnimWrapper@@MAEPAXI@Z 3400ba50 f i Movie.obj
 0001:0000aab0       ?_M_insert_overflow@?$_Impl_vector@IV?$allocator@I@stlpmtx_std@@@priv@stlpmtx_std@@AAEXPAIABIABU__true_type@3@I_N@Z 3400bab0 f i EntityNode.obj
 0001:0000aab0       ?_M_insert_overflow@?$_Impl_vector@PBXV?$allocator@PBX@stlpmtx_std@@@priv@stlpmtx_std@@AAEXPAPBXABQBXABU__true_type@3@I_N@Z 3400bab0 f i Movie.obj
 0001:0000aab0       ?_M_insert_overflow@?$_Impl_vector@PAXV?$allocator@PAX@stlpmtx_std@@@priv@stlpmtx_std@@AAEXPAPAXABQAXABU__true_type@3@I_N@Z 3400bab0 f i Movie.obj
 0001:0000ac00       ??0SkelAnimUpdateCMD@CMovieSystem@@QAE@ABU01@@Z 3400bc00 f i Movie.obj
 0001:0000ac70       ??$__ufill@PAUPlayingSequence@@U1@H@priv@stlpmtx_std@@YAXPAUPlayingSequence@@0ABU2@ABUrandom_access_iterator_tag@1@PAH@Z 3400bc70 f i Movie.obj
 0001:0000acf0       ??$__ucopy@PAUPlayingSequence@@PAU1@H@priv@stlpmtx_std@@YAPAUPlayingSequence@@PAU2@00ABUrandom_access_iterator_tag@1@PAH@Z 3400bcf0 f i Movie.obj
 0001:0000ad70       ?Load@CMovieSystem@@UAE_NPBD0@Z 3400bd70 f   Movie.obj
 0001:0000b1b0       ?Serialize@CMovieSystem@@UAEXAAVXmlNodeRef@@_N11@Z 3400c1b0 f   Movie.obj
 0001:0000b3f0       ??0?$_Vector_base@PAXV?$allocator@PAX@stlpmtx_std@@@priv@stlpmtx_std@@QAE@IABV?$allocator@PAX@2@@Z 3400c3f0 f i Movie.obj
 0001:0000b4a0       ??$__copy@PAUSkelAnimUpdateCMD@CMovieSystem@@PAU12@H@priv@stlpmtx_std@@YAPAUSkelAnimUpdateCMD@CMovieSystem@@PAU23@00ABUrandom_access_iterator_tag@1@PAH@Z 3400c4a0 f i Movie.obj
 0001:0000b5d0       ?substr@?$CryStringT@D@@QBE?AV1@II@Z 3400c5d0 f i Movie.obj
 0001:0000b620       ?Format@?$CryStringT@D@@QAAAAV1@PBDZZ 3400c620 f i Movie.obj
 0001:0000b690       ?GoToFrame@CMovieSystem@@UAEXPBDM@Z 3400c690 f   Movie.obj
 0001:0000b7a0       ?FindLightAnim@CLightAnimWrapper@@CAPAV1@PBD@Z 3400c7a0 f   Movie.obj
 0001:0000b810       ?Tokenize@?$CryStringT@D@@QBE?AV1@PBDAAH@Z 3400c810 f i Movie.obj
 0001:0000b8d0       ??$find_and_erase@V?$vector@PAUIMovieListener@@V?$allocator@PAUIMovieListener@@@stlpmtx_std@@@stlpmtx_std@@PAUIMovieListener@@@stl@@YA_NAAV?$vector@PAUIMovieListener@@V?$allocator@PAUIMovieListener@@@stlpmtx_std@@@stlpmtx_std@@ABQAUIMovieListener@@@Z 3400c8d0 f i Movie.obj
 0001:0000b940       ??$__ufill@PAUSkelAnimUpdateCMD@CMovieSystem@@U12@H@priv@stlpmtx_std@@YAXPAUSkelAnimUpdateCMD@CMovieSystem@@0ABU23@ABUrandom_access_iterator_tag@1@PAH@Z 3400c940 f i Movie.obj
 0001:0000b9e0       ??$__destroy_range_aux@V?$reverse_iterator@PAUSkelAnimUpdateCMD@CMovieSystem@@@stlpmtx_std@@USkelAnimUpdateCMD@CMovieSystem@@@stlpmtx_std@@YAXV?$reverse_iterator@PAUSkelAnimUpdateCMD@CMovieSystem@@@0@0PAUSkelAnimUpdateCMD@CMovieSystem@@ABU__false_type@0@@Z 3400c9e0 f i Movie.obj
 0001:0000ba40       ??$__destroy_range_aux@PAUSkelAnimUpdateCMD@CMovieSystem@@U12@@stlpmtx_std@@YAXPAUSkelAnimUpdateCMD@CMovieSystem@@00ABU__false_type@0@@Z 3400ca40 f i Movie.obj
 0001:0000baa0       ??$__ucopy@PAUSkelAnimUpdateCMD@CMovieSystem@@PAU12@H@priv@stlpmtx_std@@YAPAUSkelAnimUpdateCMD@CMovieSystem@@PAU23@00ABUrandom_access_iterator_tag@1@PAH@Z 3400caa0 f i Movie.obj
 0001:0000bb40       ?FindSequenceGroup@CMovieSystem@@UBEPAUIAnimSequenceGroup@@PBD@Z 3400cb40 f   Movie.obj
 0001:0000bdd0       ?ShowPlayedSequencesDebug@CMovieSystem@@AAEXXZ 3400cdd0 f   Movie.obj
 0001:0000c120       ?erase@?$vector@UPlayingSequence@@V?$allocator@UPlayingSequence@@@stlpmtx_std@@@stlpmtx_std@@QAEPAUPlayingSequence@@PAU3@@Z 3400d120 f i Movie.obj
 0001:0000c180       ??1?$_Impl_vector@UPlayingSequence@@V?$allocator@UPlayingSequence@@@stlpmtx_std@@@priv@stlpmtx_std@@QAE@XZ 3400d180 f i Movie.obj
 0001:0000c1d0       ??$AddContainer@U?$DynArray@U?$TCBSplineKey@U?$Quat_tpl@M@@@spline@@HU?$SmallDynStorage@U?$TCBSplineKey@U?$Quat_tpl@M@@@spline@@HUStandardAlloc@NAlloc@@@NArray@@@@@ICrySizer@@QAE_NABU?$DynArray@U?$TCBSplineKey@U?$Quat_tpl@M@@@spline@@HU?$SmallDynStorage@U?$TCBSplineKey@U?$Quat_tpl@M@@@spline@@HUStandardAlloc@NAlloc@@@NArray@@@@@Z 3400d1d0 f i Movie.obj
 0001:0000c260       ?GetMemoryUsage@?$TSpline@U?$TCBSplineKey@U?$Quat_tpl@M@@@spline@@VHermitBasis@2@@spline@@UBEXPAVICrySizer@@_N@Z 3400d260 f i Movie.obj
 0001:0000c2a0       ??$AddContainer@U?$DynArray@U?$TCBSplineKeyEx@M@spline@@HU?$SmallDynStorage@U?$TCBSplineKeyEx@M@spline@@HUStandardAlloc@NAlloc@@@NArray@@@@@ICrySizer@@QAE_NABU?$DynArray@U?$TCBSplineKeyEx@M@spline@@HU?$SmallDynStorage@U?$TCBSplineKeyEx@M@spline@@HUStandardAlloc@NAlloc@@@NArray@@@@@Z 3400d2a0 f i Movie.obj
 0001:0000c330       ?GetMemoryUsage@?$TSpline@U?$TCBSplineKeyEx@M@spline@@VHermitBasis@2@@spline@@UBEXPAVICrySizer@@_N@Z 3400d330 f i Movie.obj
 0001:0000c370       ??$AddContainer@U?$DynArray@U?$TCBSplineKeyEx@U?$Vec3_tpl@M@@@spline@@HU?$SmallDynStorage@U?$TCBSplineKeyEx@U?$Vec3_tpl@M@@@spline@@HUStandardAlloc@NAlloc@@@NArray@@@@@ICrySizer@@QAE_NABU?$DynArray@U?$TCBSplineKeyEx@U?$Vec3_tpl@M@@@spline@@HU?$SmallDynStorage@U?$TCBSplineKeyEx@U?$Vec3_tpl@M@@@spline@@HUStandardAlloc@NAlloc@@@NArray@@@@@Z 3400d370 f i Movie.obj
 0001:0000c3f0       ?GetMemoryUsage@?$TSpline@U?$TCBSplineKeyEx@U?$Vec3_tpl@M@@@spline@@VHermitBasis@2@@spline@@UBEXPAVICrySizer@@_N@Z 3400d3f0 f i Movie.obj
 0001:0000c430       ??0?$vector@PAUIMovieListener@@V?$allocator@PAUIMovieListener@@@stlpmtx_std@@@stlpmtx_std@@QAE@ABV01@@Z 3400d430 f i Movie.obj
 0001:0000c490       ?push_back@?$vector@PAUIAnimSequence@@V?$allocator@PAUIAnimSequence@@@stlpmtx_std@@@stlpmtx_std@@QAEXABQAUIAnimSequence@@@Z 3400d490 f i Movie.obj
 0001:0000c4e0       ??_GTCBQuatSpline@spline@@UAEPAXI@Z 3400d4e0 f i Movie.obj
 0001:0000c4e0       ??_ETCBQuatSpline@spline@@UAEPAXI@Z 3400d4e0 f i Movie.obj
 0001:0000c4e0       ??_E?$TSpline@U?$TCBSplineKey@U?$Quat_tpl@M@@@spline@@VHermitBasis@2@@spline@@UAEPAXI@Z 3400d4e0 f i Movie.obj
 0001:0000c4e0       ??_G?$TSpline@U?$TCBSplineKey@U?$Quat_tpl@M@@@spline@@VHermitBasis@2@@spline@@UAEPAXI@Z 3400d4e0 f i Movie.obj
 0001:0000c530       ??_E?$TCBSpline@MU?$TCBSplineKeyEx@M@spline@@@spline@@UAEPAXI@Z 3400d530 f i Movie.obj
 0001:0000c530       ??_G?$TSpline@U?$TCBSplineKeyEx@M@spline@@VHermitBasis@2@@spline@@UAEPAXI@Z 3400d530 f i Movie.obj
 0001:0000c530       ??_G?$TCBSpline@MU?$TCBSplineKeyEx@M@spline@@@spline@@UAEPAXI@Z 3400d530 f i Movie.obj
 0001:0000c530       ??_E?$TSpline@U?$TCBSplineKeyEx@M@spline@@VHermitBasis@2@@spline@@UAEPAXI@Z 3400d530 f i Movie.obj
 0001:0000c580       ?_M_erase@?$_Rb_tree@V?$CryStringT@D@@U?$less@V?$CryStringT@D@@@stlpmtx_std@@U?$pair@$$CBV?$CryStringT@D@@PAVCLightAnimWrapper@@@3@U?$_Select1st@U?$pair@$$CBV?$CryStringT@D@@PAVCLightAnimWrapper@@@stlpmtx_std@@@priv@3@U?$_MapTraitsT@U?$pair@$$CBV?$CryStringT@D@@PAVCLightAnimWrapper@@@stlpmtx_std@@@63@V?$allocator@U?$pair@$$CBV?$CryStringT@D@@PAVCLightAnimWrapper@@@stlpmtx_std@@@3@@priv@stlpmtx_std@@AAEXPAU_Rb_tree_node_base@23@@Z 3400d580 f i Movie.obj
 0001:0000c580       ?_M_erase@?$_Rb_tree@V?$CryStringT@D@@U?$less@V?$CryStringT@D@@@stlpmtx_std@@V1@U?$_Identity@V?$CryStringT@D@@@priv@3@U?$_SetTraitsT@V?$CryStringT@D@@@53@V?$allocator@V?$CryStringT@D@@@3@@priv@stlpmtx_std@@AAEXPAU_Rb_tree_node_base@23@@Z 3400d580 f i EntityNode.obj
 0001:0000c5e0       ?_M_insert_overflow_aux@?$_Impl_vector@UPlayingSequence@@V?$allocator@UPlayingSequence@@@stlpmtx_std@@@priv@stlpmtx_std@@AAEXPAUPlayingSequence@@ABU4@ABU__false_type@3@I_N@Z 3400d5e0 f i Movie.obj
 0001:0000c7c0       ??$push_back_unique@V?$vector@PAUIMovieListener@@V?$allocator@PAUIMovieListener@@@stlpmtx_std@@@stlpmtx_std@@PAUIMovieListener@@@stl@@YA_NAAV?$vector@PAUIMovieListener@@V?$allocator@PAUIMovieListener@@@stlpmtx_std@@@stlpmtx_std@@ABQAUIMovieListener@@@Z 3400d7c0 f i Movie.obj
 0001:0000c830       ?_M_create_node@?$_Rb_tree@V?$CryStringT@D@@U?$less@V?$CryStringT@D@@@stlpmtx_std@@U?$pair@$$CBV?$CryStringT@D@@PAVCLightAnimWrapper@@@3@U?$_Select1st@U?$pair@$$CBV?$CryStringT@D@@PAVCLightAnimWrapper@@@stlpmtx_std@@@priv@3@U?$_MapTraitsT@U?$pair@$$CBV?$CryStringT@D@@PAVCLightAnimWrapper@@@stlpmtx_std@@@63@V?$allocator@U?$pair@$$CBV?$CryStringT@D@@PAVCLightAnimWrapper@@@stlpmtx_std@@@3@@priv@stlpmtx_std@@IAEPAU_Rb_tree_node_base@23@ABU?$pair@$$CBV?$CryStringT@D@@PAVCLightAnimWrapper@@@3@@Z 3400d830 f i Movie.obj
 0001:0000c8a0       ?NotifyListeners@CMovieSystem@@IAEXPAUIAnimSequence@@W4EMovieEvent@IMovieListener@@@Z 3400d8a0 f   Movie.obj
 0001:0000c9b0       ?InternalStopSequence@CMovieSystem@@IAE_NPAUIAnimSequence@@_N@Z 3400d9b0 f   Movie.obj
 0001:0000cba0       ?AbortSequence@CMovieSystem@@UAE_NPAUIAnimSequence@@_N@Z 3400dba0 f   Movie.obj
 0001:0000cc20       ?Reset@CMovieSystem@@UAEX_N0@Z 3400dc20 f   Movie.obj
 0001:0000cd10       ?Update@CMovieSystem@@UAEXM@Z 3400dd10 f   Movie.obj
 0001:0000cfd0       ??0?$TSpline@U?$TCBSplineKey@U?$Quat_tpl@M@@@spline@@VHermitBasis@2@@spline@@QAE@XZ 3400dfd0 f i Movie.obj
 0001:0000d030       ??0?$TSpline@U?$TCBSplineKeyEx@M@spline@@VHermitBasis@2@@spline@@QAE@XZ 3400e030 f i Movie.obj
 0001:0000d090       ??0?$TSpline@U?$TCBSplineKeyEx@U?$Vec3_tpl@M@@@spline@@VHermitBasis@2@@spline@@QAE@XZ 3400e090 f i Movie.obj
 0001:0000d0f0       ?erase@?$_Rb_tree@PAUIAnimSequence@@U?$less@PAUIAnimSequence@@@stlpmtx_std@@U?$pair@QAUIAnimSequence@@V?$vector@PAUIMovieListener@@V?$allocator@PAUIMovieListener@@@stlpmtx_std@@@stlpmtx_std@@@3@U?$_Select1st@U?$pair@QAUIAnimSequence@@V?$vector@PAUIMovieListener@@V?$allocator@PAUIMovieListener@@@stlpmtx_std@@@stlpmtx_std@@@stlpmtx_std@@@priv@3@U?$_MapTraitsT@U?$pair@QAUIAnimSequence@@V?$vector@PAUIMovieListener@@V?$allocator@PAUIMovieListener@@@stlpmtx_std@@@stlpmtx_std@@@stlpmtx_std@@@63@V?$allocator@U?$pair@QAUIAnimSequence@@V?$vector@PAUIMovieListener@@V?$allocator@PAUIMovieListener@@@stlpmtx_std@@@stlpmtx_std@@@stlpmtx_std@@@3@@priv@stlpmtx_std@@QAEXU?$_Rb_tree_iterator@U?$pair@QAUIAnimSequence@@V?$vector@PAUIMovieListener@@V?$allocator@PAUIMovieListener@@@stlpmtx_std@@@stlpmtx_std@@@stlpmtx_std@@U?$_MapTraitsT@U?$pair@QAUIAnimSequence@@V?$vector@PAUIMovieListener@@V?$allocator@PAUIMovieListener@@@stlpmtx_std@@@stlpmtx_std@@@stlpmtx_std@@@priv@2@@23@@Z 3400e0f0 f i Movie.obj
 0001:0000d150       ?_M_erase@?$_Rb_tree@PAUIAnimSequence@@U?$less@PAUIAnimSequence@@@stlpmtx_std@@U?$pair@QAUIAnimSequence@@V?$vector@PAUIMovieListener@@V?$allocator@PAUIMovieListener@@@stlpmtx_std@@@stlpmtx_std@@@3@U?$_Select1st@U?$pair@QAUIAnimSequence@@V?$vector@PAUIMovieListener@@V?$allocator@PAUIMovieListener@@@stlpmtx_std@@@stlpmtx_std@@@stlpmtx_std@@@priv@3@U?$_MapTraitsT@U?$pair@QAUIAnimSequence@@V?$vector@PAUIMovieListener@@V?$allocator@PAUIMovieListener@@@stlpmtx_std@@@stlpmtx_std@@@stlpmtx_std@@@63@V?$allocator@U?$pair@QAUIAnimSequence@@V?$vector@PAUIMovieListener@@V?$allocator@PAUIMovieListener@@@stlpmtx_std@@@stlpmtx_std@@@stlpmtx_std@@@3@@priv@stlpmtx_std@@AAEXPAU_Rb_tree_node_base@23@@Z 3400e150 f i Movie.obj
 0001:0000d210       ?_M_insert@?$_Rb_tree@V?$CryStringT@D@@U?$less@V?$CryStringT@D@@@stlpmtx_std@@U?$pair@$$CBV?$CryStringT@D@@PAVCLightAnimWrapper@@@3@U?$_Select1st@U?$pair@$$CBV?$CryStringT@D@@PAVCLightAnimWrapper@@@stlpmtx_std@@@priv@3@U?$_MapTraitsT@U?$pair@$$CBV?$CryStringT@D@@PAVCLightAnimWrapper@@@stlpmtx_std@@@63@V?$allocator@U?$pair@$$CBV?$CryStringT@D@@PAVCLightAnimWrapper@@@stlpmtx_std@@@3@@priv@stlpmtx_std@@AAE?AU?$_Rb_tree_iterator@U?$pair@$$CBV?$CryStringT@D@@PAVCLightAnimWrapper@@@stlpmtx_std@@U?$_MapTraitsT@U?$pair@$$CBV?$CryStringT@D@@PAVCLightAnimWrapper@@@stlpmtx_std@@@priv@2@@23@PAU_Rb_tree_node_base@23@ABU?$pair@$$CBV?$CryStringT@D@@PAVCLightAnimWrapper@@@3@00@Z 3400e210 f i Movie.obj
 0001:0000d2b0       ??$_Copy_Construct_aux@U?$pair@QAUIAnimSequence@@V?$vector@PAUIMovieListener@@V?$allocator@PAUIMovieListener@@@stlpmtx_std@@@stlpmtx_std@@@stlpmtx_std@@@stlpmtx_std@@YAXPAU?$pair@QAUIAnimSequence@@V?$vector@PAUIMovieListener@@V?$allocator@PAUIMovieListener@@@stlpmtx_std@@@stlpmtx_std@@@0@ABU10@ABU__false_type@0@@Z 3400e2b0 f i Movie.obj
 0001:0000d320       ?StopSequence@CMovieSystem@@UAE_NPAUIAnimSequence@@@Z 3400e320 f   Movie.obj
 0001:0000d340       ?compMiddleDeriv@?$TCBSpline@MU?$TCBSplineKeyEx@M@spline@@@spline@@AAEXH@Z 3400e340 f i Movie.obj
 0001:0000d620       ?comp2KeyDeriv@?$TCBSpline@MU?$TCBSplineKeyEx@M@spline@@@spline@@AAEXXZ 3400e620 f i Movie.obj
 0001:0000d690       ?comp_deriv@?$TCBSpline@MU?$TCBSplineKeyEx@M@spline@@@spline@@UAEXXZ 3400e690 f i Movie.obj
 0001:0000d7f0       ?interp_keys@?$TCBSpline@MU?$TCBSplineKeyEx@M@spline@@@spline@@MAEXHHMAAM@Z 3400e7f0 f i Movie.obj
 0001:0000d900       ?calc_ease@?$TCBSpline@U?$Vec3_tpl@M@@U?$TCBSplineKeyEx@U?$Vec3_tpl@M@@@spline@@@spline@@IAEMMMM@Z 3400e900 f i Movie.obj
 0001:0000d900       ?calc_ease@?$TCBSpline@MU?$TCBSplineKeyEx@M@spline@@@spline@@IAEMMMM@Z 3400e900 f i Movie.obj
 0001:0000d900       ?calc_ease@?$TCBSpline@U?$Quat_tpl@M@@U?$TCBSplineKey@U?$Quat_tpl@M@@@spline@@@spline@@IAEMMMM@Z 3400e900 f i Movie.obj
 0001:0000d9e0       ?compMiddleDeriv@?$TCBSpline@U?$Vec3_tpl@M@@U?$TCBSplineKeyEx@U?$Vec3_tpl@M@@@spline@@@spline@@AAEXH@Z 3400e9e0 f i Movie.obj
 0001:0000deb0       ?compFirstDeriv@?$TCBSpline@U?$Vec3_tpl@M@@U?$TCBSplineKeyEx@U?$Vec3_tpl@M@@@spline@@@spline@@AAEXXZ 3400eeb0 f i Movie.obj
 0001:0000df90       ?compLastDeriv@?$TCBSpline@U?$Vec3_tpl@M@@U?$TCBSplineKeyEx@U?$Vec3_tpl@M@@@spline@@@spline@@AAEXXZ 3400ef90 f i Movie.obj
 0001:0000e0a0       ?comp2KeyDeriv@?$TCBSpline@U?$Vec3_tpl@M@@U?$TCBSplineKeyEx@U?$Vec3_tpl@M@@@spline@@@spline@@AAEXXZ 3400f0a0 f i Movie.obj
 0001:0000e1c0       ?comp_deriv@?$TCBSpline@U?$Vec3_tpl@M@@U?$TCBSplineKeyEx@U?$Vec3_tpl@M@@@spline@@@spline@@UAEXXZ 3400f1c0 f i Movie.obj
 0001:0000e260       ?interp_keys@?$TCBSpline@U?$Vec3_tpl@M@@U?$TCBSplineKeyEx@U?$Vec3_tpl@M@@@spline@@@spline@@MAEXHHMAAU?$Vec3_tpl@M@@@Z 3400f260 f i Movie.obj
 0001:0000e440       ??_E?$TSpline@U?$TCBSplineKeyEx@U?$Vec3_tpl@M@@@spline@@VHermitBasis@2@@spline@@UAEPAXI@Z 3400f440 f i Movie.obj
 0001:0000e440       ??_E?$TCBSpline@U?$Vec3_tpl@M@@U?$TCBSplineKeyEx@U?$Vec3_tpl@M@@@spline@@@spline@@UAEPAXI@Z 3400f440 f i Movie.obj
 0001:0000e440       ??_G?$TCBSpline@U?$Vec3_tpl@M@@U?$TCBSplineKeyEx@U?$Vec3_tpl@M@@@spline@@@spline@@UAEPAXI@Z 3400f440 f i Movie.obj
 0001:0000e440       ??_G?$TSpline@U?$TCBSplineKeyEx@U?$Vec3_tpl@M@@@spline@@VHermitBasis@2@@spline@@UAEPAXI@Z 3400f440 f i Movie.obj
 0001:0000e490       ?push_back@?$_Impl_vector@UPlayingSequence@@V?$allocator@UPlayingSequence@@@stlpmtx_std@@@priv@stlpmtx_std@@QAEXABUPlayingSequence@@@Z 3400f490 f i Movie.obj
 0001:0000e520       ?insert_unique@?$_Rb_tree@V?$CryStringT@D@@U?$less@V?$CryStringT@D@@@stlpmtx_std@@U?$pair@$$CBV?$CryStringT@D@@PAVCLightAnimWrapper@@@3@U?$_Select1st@U?$pair@$$CBV?$CryStringT@D@@PAVCLightAnimWrapper@@@stlpmtx_std@@@priv@3@U?$_MapTraitsT@U?$pair@$$CBV?$CryStringT@D@@PAVCLightAnimWrapper@@@stlpmtx_std@@@63@V?$allocator@U?$pair@$$CBV?$CryStringT@D@@PAVCLightAnimWrapper@@@stlpmtx_std@@@3@@priv@stlpmtx_std@@QAE?AU?$pair@U?$_Rb_tree_iterator@U?$pair@$$CBV?$CryStringT@D@@PAVCLightAnimWrapper@@@stlpmtx_std@@U?$_MapTraitsT@U?$pair@$$CBV?$CryStringT@D@@PAVCLightAnimWrapper@@@stlpmtx_std@@@priv@2@@priv@stlpmtx_std@@_N@3@ABU?$pair@$$CBV?$CryStringT@D@@PAVCLightAnimWrapper@@@3@@Z 3400f520 f i Movie.obj
 0001:0000e6a0       ?_M_insert_overflow_aux@?$_Impl_vector@USkelAnimUpdateCMD@CMovieSystem@@V?$allocator@USkelAnimUpdateCMD@CMovieSystem@@@stlpmtx_std@@@priv@stlpmtx_std@@AAEXPAUSkelAnimUpdateCMD@CMovieSystem@@ABU45@ABU__false_type@3@I_N@Z 3400f6a0 f i Movie.obj
 0001:0000e840       ??$_M_allocate_and_copy@PAUSkelAnimUpdateCMD@CMovieSystem@@@?$_Impl_vector@USkelAnimUpdateCMD@CMovieSystem@@V?$allocator@USkelAnimUpdateCMD@CMovieSystem@@@stlpmtx_std@@@priv@stlpmtx_std@@AAEPAUSkelAnimUpdateCMD@CMovieSystem@@AAIPAU34@1@Z 3400f840 f i Movie.obj
 0001:0000e8b0       ?RemoveCachedLightAnim@CLightAnimWrapper@@CAXPBD@Z 3400f8b0 f   Movie.obj
 0001:0000e920       ??_EISplineBackup@@UAEPAXI@Z 3400f920 f i Movie.obj
 0001:0000e920       ??_GISplineBackup@@UAEPAXI@Z 3400f920 f i Movie.obj
 0001:0000e950       ?alloc@StandardAlloc@NAlloc@@SAPAXAAI_NH@Z 3400f950 f i Movie.obj
 0001:0000e9d0       ??$move_init@U?$TCBSplineKeyEx@M@spline@@@NArray@@YAXPAU?$TCBSplineKeyEx@M@spline@@0I@Z 3400f9d0 f i Movie.obj
 0001:0000ea10       ?seek_key@?$TSpline@U?$TCBSplineKeyEx@M@spline@@VHermitBasis@2@@spline@@IAEHM@Z 3400fa10 f i Movie.obj
 0001:0000ea90       ?init@?$DynArray@U?$TCBSplineKeyEx@M@spline@@HU?$SmallDynStorage@U?$TCBSplineKeyEx@M@spline@@HUStandardAlloc@NAlloc@@@NArray@@@@KAPAU?$TCBSplineKeyEx@M@spline@@U?$Array@U?$TCBSplineKeyEx@M@spline@@HU?$ArrayStorage@U?$TCBSplineKeyEx@M@spline@@H@NArray@@@@PBU23@@Z 3400fa90 f i Movie.obj
 0001:0000eae0       ?assign@?$Array@U?$TCBSplineKeyEx@M@spline@@HU?$SmallDynStorage@U?$TCBSplineKeyEx@M@spline@@HUStandardAlloc@NAlloc@@@NArray@@@@QAEXU?$Array@$$CBU?$TCBSplineKeyEx@M@spline@@HU?$ArrayStorage@$$CBU?$TCBSplineKeyEx@M@spline@@H@NArray@@@@@Z 3400fae0 f i Movie.obj
 0001:0000eb70       ??$__unguarded_linear_insert@PAU?$TCBSplineKeyEx@M@spline@@U12@U?$less@U?$TCBSplineKeyEx@M@spline@@@stlpmtx_std@@@priv@stlpmtx_std@@YAXPAU?$TCBSplineKeyEx@M@spline@@U23@U?$less@U?$TCBSplineKeyEx@M@spline@@@1@@Z 3400fb70 f i Movie.obj
 0001:0000ec40       ??$__push_heap@PAU?$TCBSplineKeyEx@M@spline@@HU12@U?$less@U?$TCBSplineKeyEx@M@spline@@@stlpmtx_std@@@stlpmtx_std@@YAXPAU?$TCBSplineKeyEx@M@spline@@HHU12@U?$less@U?$TCBSplineKeyEx@M@spline@@@0@@Z 3400fc40 f i Movie.obj
 0001:0000ed40       ??$__copy_backward@PAU?$TCBSplineKeyEx@M@spline@@PAU12@H@priv@stlpmtx_std@@YAPAU?$TCBSplineKeyEx@M@spline@@PAU23@00ABUrandom_access_iterator_tag@1@PAH@Z 3400fd40 f i Movie.obj
 0001:0000ef60       ?FindKeysInRange@?$CBaseSplineInterpolator@MV?$TCBSpline@MU?$TCBSplineKeyEx@M@spline@@@spline@@@spline@@UAEXMMAAH0@Z 3400ff60 f i Movie.obj
 0001:0000f090       ?GetKeyTime@?$CBaseSplineInterpolator@MV?$TCBSpline@MU?$TCBSplineKeyEx@M@spline@@@spline@@@spline@@UAEMH@Z 34010090 f i Movie.obj
 0001:0000f0c0       ?GetKeyValue@?$CBaseSplineInterpolator@MV?$TCBSpline@MU?$TCBSplineKeyEx@M@spline@@@spline@@@spline@@UAE_NHAAY03M@Z 340100c0 f i Movie.obj
 0001:0000f100       ?SetKeyValue@?$CBaseSplineInterpolator@MV?$TCBSpline@MU?$TCBSplineKeyEx@M@spline@@@spline@@@spline@@UAEXHQAM@Z 34010100 f i Movie.obj
 0001:0000f140       ?SetKeyTime@?$CBaseSplineInterpolator@MV?$TCBSpline@MU?$TCBSplineKeyEx@M@spline@@@spline@@@spline@@UAEXHM@Z 34010140 f i Movie.obj
 0001:0000f180       ?SetKeyTangents@?$CBaseSplineInterpolator@MV?$TCBSpline@MU?$TCBSplineKeyEx@M@spline@@@spline@@@spline@@UAEXHQAM0@Z 34010180 f i Movie.obj
 0001:0000f1d0       ?GetKeyTangents@?$CBaseSplineInterpolator@MV?$TCBSpline@MU?$TCBSplineKeyEx@M@spline@@@spline@@@spline@@UAE_NHAAY03M0@Z 340101d0 f i Movie.obj
 0001:0000f210       ?GetKeyFlags@?$CBaseSplineInterpolator@MV?$TCBSpline@MU?$TCBSplineKeyEx@M@spline@@@spline@@@spline@@UAEHH@Z 34010210 f i Movie.obj
 0001:0000f240       ?set_size@?$SmallDynStorage@U?$TCBSplineKeyEx@M@spline@@HUStandardAlloc@NAlloc@@@NArray@@QAEXH@Z 34010240 f i Movie.obj
 0001:0000f2d0       ?resize_raw@?$SmallDynStorage@U?$TCBSplineKeyEx@M@spline@@HUStandardAlloc@NAlloc@@@NArray@@QAEXHH_N@Z 340102d0 f i Movie.obj
 0001:0000f430       ?expand_raw@?$DynArray@U?$TCBSplineKeyEx@M@spline@@HU?$SmallDynStorage@U?$TCBSplineKeyEx@M@spline@@HUStandardAlloc@NAlloc@@@NArray@@@@IAEPAU?$TCBSplineKeyEx@M@spline@@PAU23@H@Z 34010430 f i Movie.obj
 0001:0000f4c0       ??$__unguarded_insertion_sort_aux@PAU?$TCBSplineKeyEx@M@spline@@U12@U?$less@U?$TCBSplineKeyEx@M@spline@@@stlpmtx_std@@@priv@stlpmtx_std@@YAXPAU?$TCBSplineKeyEx@M@spline@@00U?$less@U?$TCBSplineKeyEx@M@spline@@@1@@Z 340104c0 f i Movie.obj
 0001:0000f5d0       ??$__adjust_heap@PAU?$TCBSplineKeyEx@M@spline@@HU12@U?$less@U?$TCBSplineKeyEx@M@spline@@@stlpmtx_std@@@stlpmtx_std@@YAXPAU?$TCBSplineKeyEx@M@spline@@HHU12@U?$less@U?$TCBSplineKeyEx@M@spline@@@0@@Z 340105d0 f i Movie.obj
 0001:0000f6f0       ?insert_raw@?$DynArray@U?$TCBSplineKeyEx@M@spline@@HU?$SmallDynStorage@U?$TCBSplineKeyEx@M@spline@@HUStandardAlloc@NAlloc@@@NArray@@@@QAE?AU?$Array@U?$TCBSplineKeyEx@M@spline@@HU?$ArrayStorage@U?$TCBSplineKeyEx@M@spline@@H@NArray@@@@PAU?$TCBSplineKeyEx@M@spline@@H@Z 340106f0 f i Movie.obj
 0001:0000f7e0       ??$__make_heap@PAU?$TCBSplineKeyEx@M@spline@@U?$less@U?$TCBSplineKeyEx@M@spline@@@stlpmtx_std@@U12@H@stlpmtx_std@@YAXPAU?$TCBSplineKeyEx@M@spline@@0U?$less@U?$TCBSplineKeyEx@M@spline@@@0@0PAH@Z 340107e0 f i Movie.obj
 0001:0000f970       ??$__pop_heap_aux@PAU?$TCBSplineKeyEx@M@spline@@U12@U?$less@U?$TCBSplineKeyEx@M@spline@@@stlpmtx_std@@@stlpmtx_std@@YAXPAU?$TCBSplineKeyEx@M@spline@@00U?$less@U?$TCBSplineKeyEx@M@spline@@@0@@Z 34010970 f i Movie.obj
 0001:0000fa10       ?erase@?$DynArray@U?$TCBSplineKeyEx@M@spline@@HU?$SmallDynStorage@U?$TCBSplineKeyEx@M@spline@@HUStandardAlloc@NAlloc@@@NArray@@@@QAEPAU?$TCBSplineKeyEx@M@spline@@PAU23@0@Z 34010a10 f i Movie.obj
 0001:0000fc40       ??$__unguarded_partition@PAU?$TCBSplineKeyEx@M@spline@@U12@U?$less@U?$TCBSplineKeyEx@M@spline@@@stlpmtx_std@@@priv@stlpmtx_std@@YAPAU?$TCBSplineKeyEx@M@spline@@PAU23@0U23@U?$less@U?$TCBSplineKeyEx@M@spline@@@1@@Z 34010c40 f i Movie.obj
 0001:0000fd30       ??4?$DynArray@U?$TCBSplineKeyEx@M@spline@@HU?$SmallDynStorage@U?$TCBSplineKeyEx@M@spline@@HUStandardAlloc@NAlloc@@@NArray@@@@QAEAAU0@U?$Array@$$CBU?$TCBSplineKeyEx@M@spline@@HU?$ArrayStorage@$$CBU?$TCBSplineKeyEx@M@spline@@H@NArray@@@@@Z 34010d30 f i Movie.obj
 0001:0000fde0       ??0?$DynArray@U?$TCBSplineKeyEx@M@spline@@HU?$SmallDynStorage@U?$TCBSplineKeyEx@M@spline@@HUStandardAlloc@NAlloc@@@NArray@@@@QAE@ABU0@@Z 34010de0 f i Movie.obj
 0001:0000fe90       ?RemoveKey@?$CBaseSplineInterpolator@MV?$TCBSpline@MU?$TCBSplineKeyEx@M@spline@@@spline@@@spline@@UAEXH@Z 34010e90 f i Movie.obj
 0001:0000fee0       ?RemoveKeysInRange@?$CBaseSplineInterpolator@MV?$TCBSpline@MU?$TCBSplineKeyEx@M@spline@@@spline@@@spline@@UAEXMM@Z 34010ee0 f i Movie.obj
 0001:00010010       ??$__insertion_sort@PAU?$TCBSplineKeyEx@M@spline@@U12@U?$less@U?$TCBSplineKeyEx@M@spline@@@stlpmtx_std@@@priv@stlpmtx_std@@YAXPAU?$TCBSplineKeyEx@M@spline@@00U?$less@U?$TCBSplineKeyEx@M@spline@@@1@@Z 34011010 f i Movie.obj
 0001:00010110       ??$__partial_sort@PAU?$TCBSplineKeyEx@M@spline@@U12@U?$less@U?$TCBSplineKeyEx@M@spline@@@stlpmtx_std@@@priv@stlpmtx_std@@YAXPAU?$TCBSplineKeyEx@M@spline@@000U?$less@U?$TCBSplineKeyEx@M@spline@@@1@@Z 34011110 f i Movie.obj
 0001:00010260       ?InsertKey@?$CBaseSplineInterpolator@MV?$TCBSpline@MU?$TCBSplineKeyEx@M@spline@@@spline@@@spline@@UAEHMQAM@Z 34011260 f i Movie.obj
 0001:000103c0       ??$__final_insertion_sort@PAU?$TCBSplineKeyEx@M@spline@@U?$less@U?$TCBSplineKeyEx@M@spline@@@stlpmtx_std@@@priv@stlpmtx_std@@YAXPAU?$TCBSplineKeyEx@M@spline@@0U?$less@U?$TCBSplineKeyEx@M@spline@@@1@@Z 340113c0 f i Movie.obj
 0001:00010430       ?GetValueType@CBoolTrack@@UAE?AW4EAnimValue@@XZ 34011430 f i AnimNode.obj
 0001:00010430       ?GetCurveType@?$TAnimSplineTrack@U?$Quat_tpl@M@@@@UAE?AW4EAnimCurveType@@XZ 34011430 f i Movie.obj
 0001:00010430       ?GetNumDimensions@?$CBaseSplineInterpolator@U?$Vec3_tpl@M@@V?$TCBSpline@U?$Vec3_tpl@M@@U?$TCBSplineKeyEx@U?$Vec3_tpl@M@@@spline@@@spline@@@spline@@UAEHXZ 34011430 f i Movie.obj
 0001:00010430       ?GetType@CAnimCameraNode@@UBE?AW4EAnimNodeType@@XZ 34011430 f i AnimCameraNode.obj
 0001:00010440       ??$move_init@U?$TCBSplineKeyEx@U?$Vec3_tpl@M@@@spline@@@NArray@@YAXPAU?$TCBSplineKeyEx@U?$Vec3_tpl@M@@@spline@@0I@Z 34011440 f i Movie.obj
 0001:00010480       ?seek_key@?$TSpline@U?$TCBSplineKeyEx@U?$Vec3_tpl@M@@@spline@@VHermitBasis@2@@spline@@IAEHM@Z 34011480 f i Movie.obj
 0001:000104f0       ?init@?$DynArray@U?$TCBSplineKeyEx@U?$Vec3_tpl@M@@@spline@@HU?$SmallDynStorage@U?$TCBSplineKeyEx@U?$Vec3_tpl@M@@@spline@@HUStandardAlloc@NAlloc@@@NArray@@@@KAPAU?$TCBSplineKeyEx@U?$Vec3_tpl@M@@@spline@@U?$Array@U?$TCBSplineKeyEx@U?$Vec3_tpl@M@@@spline@@HU?$ArrayStorage@U?$TCBSplineKeyEx@U?$Vec3_tpl@M@@@spline@@H@NArray@@@@PBU23@@Z 340114f0 f i Movie.obj
 0001:00010540       ?assign@?$Array@U?$TCBSplineKeyEx@U?$Vec3_tpl@M@@@spline@@HU?$SmallDynStorage@U?$TCBSplineKeyEx@U?$Vec3_tpl@M@@@spline@@HUStandardAlloc@NAlloc@@@NArray@@@@QAEXU?$Array@$$CBU?$TCBSplineKeyEx@U?$Vec3_tpl@M@@@spline@@HU?$ArrayStorage@$$CBU?$TCBSplineKeyEx@U?$Vec3_tpl@M@@@spline@@H@NArray@@@@@Z 34011540 f i Movie.obj
 0001:000105c0       ??$__unguarded_linear_insert@PAU?$TCBSplineKeyEx@U?$Vec3_tpl@M@@@spline@@U12@U?$less@U?$TCBSplineKeyEx@U?$Vec3_tpl@M@@@spline@@@stlpmtx_std@@@priv@stlpmtx_std@@YAXPAU?$TCBSplineKeyEx@U?$Vec3_tpl@M@@@spline@@U23@U?$less@U?$TCBSplineKeyEx@U?$Vec3_tpl@M@@@spline@@@1@@Z 340115c0 f i Movie.obj
 0001:00010670       ??$__push_heap@PAU?$TCBSplineKeyEx@U?$Vec3_tpl@M@@@spline@@HU12@U?$less@U?$TCBSplineKeyEx@U?$Vec3_tpl@M@@@spline@@@stlpmtx_std@@@stlpmtx_std@@YAXPAU?$TCBSplineKeyEx@U?$Vec3_tpl@M@@@spline@@HHU12@U?$less@U?$TCBSplineKeyEx@U?$Vec3_tpl@M@@@spline@@@0@@Z 34011670 f i Movie.obj
 0001:00010750       ??$__copy_backward@PAU?$TCBSplineKeyEx@U?$Vec3_tpl@M@@@spline@@PAU12@H@priv@stlpmtx_std@@YAPAU?$TCBSplineKeyEx@U?$Vec3_tpl@M@@@spline@@PAU23@00ABUrandom_access_iterator_tag@1@PAH@Z 34011750 f i Movie.obj
 0001:00010940       ?FindKeysInRange@?$CBaseSplineInterpolator@U?$Vec3_tpl@M@@V?$TCBSpline@U?$Vec3_tpl@M@@U?$TCBSplineKeyEx@U?$Vec3_tpl@M@@@spline@@@spline@@@spline@@UAEXMMAAH0@Z 34011940 f i Movie.obj
 0001:00010a70       ?GetKeyTime@?$CBaseSplineInterpolator@U?$Vec3_tpl@M@@V?$TCBSpline@U?$Vec3_tpl@M@@U?$TCBSplineKeyEx@U?$Vec3_tpl@M@@@spline@@@spline@@@spline@@UAEMH@Z 34011a70 f i Movie.obj
 0001:00010aa0       ?GetKeyValue@?$CBaseSplineInterpolator@U?$Vec3_tpl@M@@V?$TCBSpline@U?$Vec3_tpl@M@@U?$TCBSplineKeyEx@U?$Vec3_tpl@M@@@spline@@@spline@@@spline@@UAE_NHAAY03M@Z 34011aa0 f i Movie.obj
 0001:00010af0       ?SetKeyValue@?$CBaseSplineInterpolator@U?$Vec3_tpl@M@@V?$TCBSpline@U?$Vec3_tpl@M@@U?$TCBSplineKeyEx@U?$Vec3_tpl@M@@@spline@@@spline@@@spline@@UAEXHQAM@Z 34011af0 f i Movie.obj
 0001:00010b40       ?SetKeyTime@?$CBaseSplineInterpolator@U?$Vec3_tpl@M@@V?$TCBSpline@U?$Vec3_tpl@M@@U?$TCBSplineKeyEx@U?$Vec3_tpl@M@@@spline@@@spline@@@spline@@UAEXHM@Z 34011b40 f i Movie.obj
 0001:00010b80       ?SetKeyTangents@?$CBaseSplineInterpolator@U?$Vec3_tpl@M@@V?$TCBSpline@U?$Vec3_tpl@M@@U?$TCBSplineKeyEx@U?$Vec3_tpl@M@@@spline@@@spline@@@spline@@UAEXHQAM0@Z 34011b80 f i Movie.obj
 0001:00010bf0       ?GetKeyTangents@?$CBaseSplineInterpolator@U?$Vec3_tpl@M@@V?$TCBSpline@U?$Vec3_tpl@M@@U?$TCBSplineKeyEx@U?$Vec3_tpl@M@@@spline@@@spline@@@spline@@UAE_NHAAY03M0@Z 34011bf0 f i Movie.obj
 0001:00010c60       ?GetKeyFlags@?$CBaseSplineInterpolator@U?$Vec3_tpl@M@@V?$TCBSpline@U?$Vec3_tpl@M@@U?$TCBSplineKeyEx@U?$Vec3_tpl@M@@@spline@@@spline@@@spline@@UAEHH@Z 34011c60 f i Movie.obj
 0001:00010c90       ?set_size@?$SmallDynStorage@U?$TCBSplineKeyEx@U?$Vec3_tpl@M@@@spline@@HUStandardAlloc@NAlloc@@@NArray@@QAEXH@Z 34011c90 f i Movie.obj
 0001:00010d20       ?resize_raw@?$SmallDynStorage@U?$TCBSplineKeyEx@U?$Vec3_tpl@M@@@spline@@HUStandardAlloc@NAlloc@@@NArray@@QAEXHH_N@Z 34011d20 f i Movie.obj
 0001:00010e80       ?expand_raw@?$DynArray@U?$TCBSplineKeyEx@U?$Vec3_tpl@M@@@spline@@HU?$SmallDynStorage@U?$TCBSplineKeyEx@U?$Vec3_tpl@M@@@spline@@HUStandardAlloc@NAlloc@@@NArray@@@@IAEPAU?$TCBSplineKeyEx@U?$Vec3_tpl@M@@@spline@@PAU23@H@Z 34011e80 f i Movie.obj
 0001:00010f10       ??$__unguarded_insertion_sort_aux@PAU?$TCBSplineKeyEx@U?$Vec3_tpl@M@@@spline@@U12@U?$less@U?$TCBSplineKeyEx@U?$Vec3_tpl@M@@@spline@@@stlpmtx_std@@@priv@stlpmtx_std@@YAXPAU?$TCBSplineKeyEx@U?$Vec3_tpl@M@@@spline@@00U?$less@U?$TCBSplineKeyEx@U?$Vec3_tpl@M@@@spline@@@1@@Z 34011f10 f i Movie.obj
 0001:00010ff0       ??$__adjust_heap@PAU?$TCBSplineKeyEx@U?$Vec3_tpl@M@@@spline@@HU12@U?$less@U?$TCBSplineKeyEx@U?$Vec3_tpl@M@@@spline@@@stlpmtx_std@@@stlpmtx_std@@YAXPAU?$TCBSplineKeyEx@U?$Vec3_tpl@M@@@spline@@HHU12@U?$less@U?$TCBSplineKeyEx@U?$Vec3_tpl@M@@@spline@@@0@@Z 34011ff0 f i Movie.obj
 0001:000110f0       ?insert_raw@?$DynArray@U?$TCBSplineKeyEx@U?$Vec3_tpl@M@@@spline@@HU?$SmallDynStorage@U?$TCBSplineKeyEx@U?$Vec3_tpl@M@@@spline@@HUStandardAlloc@NAlloc@@@NArray@@@@QAE?AU?$Array@U?$TCBSplineKeyEx@U?$Vec3_tpl@M@@@spline@@HU?$ArrayStorage@U?$TCBSplineKeyEx@U?$Vec3_tpl@M@@@spline@@H@NArray@@@@PAU?$TCBSplineKeyEx@U?$Vec3_tpl@M@@@spline@@H@Z 340120f0 f i Movie.obj
 0001:000111d0       ??$__make_heap@PAU?$TCBSplineKeyEx@U?$Vec3_tpl@M@@@spline@@U?$less@U?$TCBSplineKeyEx@U?$Vec3_tpl@M@@@spline@@@stlpmtx_std@@U12@H@stlpmtx_std@@YAXPAU?$TCBSplineKeyEx@U?$Vec3_tpl@M@@@spline@@0U?$less@U?$TCBSplineKeyEx@U?$Vec3_tpl@M@@@spline@@@0@0PAH@Z 340121d0 f i Movie.obj
 0001:00011330       ?erase@?$DynArray@U?$TCBSplineKeyEx@U?$Vec3_tpl@M@@@spline@@HU?$SmallDynStorage@U?$TCBSplineKeyEx@U?$Vec3_tpl@M@@@spline@@HUStandardAlloc@NAlloc@@@NArray@@@@QAEPAU?$TCBSplineKeyEx@U?$Vec3_tpl@M@@@spline@@PAU23@0@Z 34012330 f i Movie.obj
 0001:00011550       ??$__unguarded_partition@PAU?$TCBSplineKeyEx@U?$Vec3_tpl@M@@@spline@@U12@U?$less@U?$TCBSplineKeyEx@U?$Vec3_tpl@M@@@spline@@@stlpmtx_std@@@priv@stlpmtx_std@@YAPAU?$TCBSplineKeyEx@U?$Vec3_tpl@M@@@spline@@PAU23@0U23@U?$less@U?$TCBSplineKeyEx@U?$Vec3_tpl@M@@@spline@@@1@@Z 34012550 f i Movie.obj
 0001:00011620       ??4?$DynArray@U?$TCBSplineKeyEx@U?$Vec3_tpl@M@@@spline@@HU?$SmallDynStorage@U?$TCBSplineKeyEx@U?$Vec3_tpl@M@@@spline@@HUStandardAlloc@NAlloc@@@NArray@@@@QAEAAU0@U?$Array@$$CBU?$TCBSplineKeyEx@U?$Vec3_tpl@M@@@spline@@HU?$ArrayStorage@$$CBU?$TCBSplineKeyEx@U?$Vec3_tpl@M@@@spline@@H@NArray@@@@@Z 34012620 f i Movie.obj
 0001:000116c0       ??0?$DynArray@U?$TCBSplineKeyEx@U?$Vec3_tpl@M@@@spline@@HU?$SmallDynStorage@U?$TCBSplineKeyEx@U?$Vec3_tpl@M@@@spline@@HUStandardAlloc@NAlloc@@@NArray@@@@QAE@ABU0@@Z 340126c0 f i Movie.obj
 0001:00011770       ??$sort_heap@PAU?$TCBSplineKeyEx@U?$Vec3_tpl@M@@@spline@@U?$less@U?$TCBSplineKeyEx@U?$Vec3_tpl@M@@@spline@@@stlpmtx_std@@@stlpmtx_std@@YAXPAU?$TCBSplineKeyEx@U?$Vec3_tpl@M@@@spline@@0U?$less@U?$TCBSplineKeyEx@U?$Vec3_tpl@M@@@spline@@@0@@Z 34012770 f i Movie.obj
 0001:00011860       ?RemoveKey@?$CBaseSplineInterpolator@U?$Vec3_tpl@M@@V?$TCBSpline@U?$Vec3_tpl@M@@U?$TCBSplineKeyEx@U?$Vec3_tpl@M@@@spline@@@spline@@@spline@@UAEXH@Z 34012860 f i Movie.obj
 0001:000118b0       ?RemoveKeysInRange@?$CBaseSplineInterpolator@U?$Vec3_tpl@M@@V?$TCBSpline@U?$Vec3_tpl@M@@U?$TCBSplineKeyEx@U?$Vec3_tpl@M@@@spline@@@spline@@@spline@@UAEXMM@Z 340128b0 f i Movie.obj
 0001:000119f0       ??$__insertion_sort@PAU?$TCBSplineKeyEx@U?$Vec3_tpl@M@@@spline@@U12@U?$less@U?$TCBSplineKeyEx@U?$Vec3_tpl@M@@@spline@@@stlpmtx_std@@@priv@stlpmtx_std@@YAXPAU?$TCBSplineKeyEx@U?$Vec3_tpl@M@@@spline@@00U?$less@U?$TCBSplineKeyEx@U?$Vec3_tpl@M@@@spline@@@1@@Z 340129f0 f i Movie.obj
 0001:00011ae0       ??$__partial_sort@PAU?$TCBSplineKeyEx@U?$Vec3_tpl@M@@@spline@@U12@U?$less@U?$TCBSplineKeyEx@U?$Vec3_tpl@M@@@spline@@@stlpmtx_std@@@priv@stlpmtx_std@@YAXPAU?$TCBSplineKeyEx@U?$Vec3_tpl@M@@@spline@@000U?$less@U?$TCBSplineKeyEx@U?$Vec3_tpl@M@@@spline@@@1@@Z 34012ae0 f i Movie.obj
 0001:00011bd0       ?InsertKey@?$CBaseSplineInterpolator@U?$Vec3_tpl@M@@V?$TCBSpline@U?$Vec3_tpl@M@@U?$TCBSplineKeyEx@U?$Vec3_tpl@M@@@spline@@@spline@@@spline@@UAEHMQAM@Z 34012bd0 f i Movie.obj
 0001:00011d60       ??$__final_insertion_sort@PAU?$TCBSplineKeyEx@U?$Vec3_tpl@M@@@spline@@U?$less@U?$TCBSplineKeyEx@U?$Vec3_tpl@M@@@spline@@@stlpmtx_std@@@priv@stlpmtx_std@@YAXPAU?$TCBSplineKeyEx@U?$Vec3_tpl@M@@@spline@@0U?$less@U?$TCBSplineKeyEx@U?$Vec3_tpl@M@@@spline@@@1@@Z 34012d60 f i Movie.obj
 0001:00011dd0       ?compKeyDeriv@TCBQuatSpline@spline@@AAEXH@Z 34012dd0 f i Movie.obj
 0001:00012b00       ?interp_keys@TCBQuatSpline@spline@@MAEXHHMAAU?$Quat_tpl@M@@@Z 34013b00 f i Movie.obj
 0001:000134e0       ?comp_deriv@TCBQuatSpline@spline@@UAEXXZ 340144e0 f i Movie.obj
 0001:00013530       ??0?$SSplineBackup@V?$TCBSpline@MU?$TCBSplineKeyEx@M@spline@@@spline@@@spline@@QAE@ABV?$TCBSpline@MU?$TCBSplineKeyEx@M@spline@@@1@@Z 34014530 f i Movie.obj
 0001:000135a0       ??_E?$SSplineBackup@V?$TCBSpline@MU?$TCBSplineKeyEx@M@spline@@@spline@@@spline@@W3AEPAXI@Z 340145a0 f i Movie.obj
 0001:000135b0       ??_G?$SSplineBackup@V?$TCBSpline@MU?$TCBSplineKeyEx@M@spline@@@spline@@@spline@@UAEPAXI@Z 340145b0 f i Movie.obj
 0001:000135b0       ??_E?$SSplineBackup@V?$TCBSpline@MU?$TCBSplineKeyEx@M@spline@@@spline@@@spline@@UAEPAXI@Z 340145b0 f i Movie.obj
 0001:00013610       ??0?$SSplineBackup@V?$TCBSpline@U?$Vec3_tpl@M@@U?$TCBSplineKeyEx@U?$Vec3_tpl@M@@@spline@@@spline@@@spline@@QAE@ABV?$TCBSpline@U?$Vec3_tpl@M@@U?$TCBSplineKeyEx@U?$Vec3_tpl@M@@@spline@@@1@@Z 34014610 f i Movie.obj
 0001:00013680       ?Release@?$SSplineBackup@V?$BezierSpline@U?$Vec2_tpl@M@@U?$SplineKeyEx@U?$Vec2_tpl@M@@@spline@@@spline@@@spline@@UAEXXZ 34014680 f i CompoundSplineTrack.obj
 0001:00013680       ?Release@?$SSplineBackup@VTCBQuatSpline@spline@@@spline@@UAEXXZ 34014680 f i Movie.obj
 0001:00013680       ?Release@?$SSplineBackup@V?$TCBSpline@MU?$TCBSplineKeyEx@M@spline@@@spline@@@spline@@UAEXXZ 34014680 f i Movie.obj
 0001:00013680       ?Release@?$SSplineBackup@V?$TCBSpline@U?$Vec3_tpl@M@@U?$TCBSplineKeyEx@U?$Vec3_tpl@M@@@spline@@@spline@@@spline@@UAEXXZ 34014680 f i Movie.obj
 0001:000136a0       ??_E?$SSplineBackup@V?$TCBSpline@U?$Vec3_tpl@M@@U?$TCBSplineKeyEx@U?$Vec3_tpl@M@@@spline@@@spline@@@spline@@W3AEPAXI@Z 340146a0 f i Movie.obj
 0001:000136b0       ??_G?$SSplineBackup@V?$TCBSpline@U?$Vec3_tpl@M@@U?$TCBSplineKeyEx@U?$Vec3_tpl@M@@@spline@@@spline@@@spline@@UAEPAXI@Z 340146b0 f i Movie.obj
 0001:000136b0       ??_E?$SSplineBackup@V?$TCBSpline@U?$Vec3_tpl@M@@U?$TCBSplineKeyEx@U?$Vec3_tpl@M@@@spline@@@spline@@@spline@@UAEPAXI@Z 340146b0 f i Movie.obj
 0001:00013710       ?reserve@?$_Impl_vector@USkelAnimUpdateCMD@CMovieSystem@@V?$allocator@USkelAnimUpdateCMD@CMovieSystem@@@stlpmtx_std@@@priv@stlpmtx_std@@QAEXI@Z 34014710 f i Movie.obj
 0001:000137e0       ??$__introsort_loop@PAU?$TCBSplineKeyEx@M@spline@@U12@HU?$less@U?$TCBSplineKeyEx@M@spline@@@stlpmtx_std@@@priv@stlpmtx_std@@YAXPAU?$TCBSplineKeyEx@M@spline@@00HU?$less@U?$TCBSplineKeyEx@M@spline@@@1@@Z 340147e0 f i Movie.obj
 0001:000138e0       ??$__introsort_loop@PAU?$TCBSplineKeyEx@U?$Vec3_tpl@M@@@spline@@U12@HU?$less@U?$TCBSplineKeyEx@U?$Vec3_tpl@M@@@spline@@@stlpmtx_std@@@priv@stlpmtx_std@@YAXPAU?$TCBSplineKeyEx@U?$Vec3_tpl@M@@@spline@@00HU?$less@U?$TCBSplineKeyEx@U?$Vec3_tpl@M@@@spline@@@1@@Z 340148e0 f i Movie.obj
 0001:000139e0       ??1CMovieSystem@@UAE@XZ    340149e0 f   Movie.obj
 0001:00013aa0       ?SetUser@CMovieSystem@@UAEXPAUIMovieUser@@@Z 34014aa0 f i Movie.obj
 0001:00013ab0       ?GetSystem@CMovieSystem@@UAEPAUISystem@@XZ 34014ab0 f i Movie.obj
 0001:00013ac0       ?GrabNextSequenceId@CMovieSystem@@UAEIXZ 34014ac0 f i Movie.obj
 0001:00013ad0       ?SetRecording@CMovieSystem@@UAEX_N@Z 34014ad0 f i Movie.obj
 0001:00013ae0       ?IsRecording@CMovieSystem@@UBE_NXZ 34014ae0 f i Movie.obj
 0001:00013af0       ?EnableCameraShake@CMovieSystem@@UAEX_N@Z 34014af0 f i Movie.obj
 0001:00013b00       ?IsCameraShakeEnabled@CMovieSystem@@UBE_NXZ 34014b00 f i Movie.obj
 0001:00013b10       ?SetCallback@CMovieSystem@@UAEXPAUIMovieCallback@@@Z 34014b10 f i Movie.obj
 0001:00013b20       ?GetSubTrackCount@CCompoundSplineTrack@@UBEHXZ 34014b20 f i CompoundSplineTrack.obj
 0001:00013b20       ?GetCallback@CMovieSystem@@UAEPAUIMovieCallback@@XZ 34014b20 f i Movie.obj
 0001:00013b20       ?GetName@CAnimNode@@UAEPBDXZ 34014b20 f i AnimLightNode.obj
 0001:00013b30       ?GetCameraParams@CMovieSystem@@UBEABUSCameraParams@@XZ 34014b30 f i Movie.obj
 0001:00013b40       ?GetOverrideCamName@CMovieSystem@@UBEPBDXZ 34014b40 f i Movie.obj
 0001:00013b50       ?IsPhysicsEventsEnabled@CMovieSystem@@UBE_NXZ 34014b50 f i Movie.obj
 0001:00013b60       ?EnablePhysicsEvents@CMovieSystem@@UAEX_N@Z 34014b60 f i Movie.obj
 0001:00013b70       ?EnableBatchRenderMode@CMovieSystem@@UAEX_N@Z 34014b70 f i Movie.obj
 0001:00013b80       ?IsInBatchRenderMode@CMovieSystem@@UBE_NXZ 34014b80 f i Movie.obj
 0001:00013b90       ??$AddObject@UPlayingSequence@@V?$allocator@UPlayingSequence@@@stlpmtx_std@@@ICrySizer@@QAEXABV?$vector@UPlayingSequence@@V?$allocator@UPlayingSequence@@@stlpmtx_std@@@stlpmtx_std@@@Z 34014b90 f i Movie.obj
 0001:00013c10       ??$AddObject@PAUIAnimSequence@@V?$vector@PAUIMovieListener@@V?$allocator@PAUIMovieListener@@@stlpmtx_std@@@stlpmtx_std@@U?$less@PAUIAnimSequence@@@3@V?$allocator@U?$pair@QAUIAnimSequence@@V?$vector@PAUIMovieListener@@V?$allocator@PAUIMovieListener@@@stlpmtx_std@@@stlpmtx_std@@@stlpmtx_std@@@3@@ICrySizer@@QAEXABV?$map@PAUIAnimSequence@@V?$vector@PAUIMovieListener@@V?$allocator@PAUIMovieListener@@@stlpmtx_std@@@stlpmtx_std@@U?$less@PAUIAnimSequence@@@3@V?$allocator@U?$pair@QAUIAnimSequence@@V?$vector@PAUIMovieListener@@V?$allocator@PAUIMovieListener@@@stlpmtx_std@@@stlpmtx_std@@@stlpmtx_std@@@3@@stlpmtx_std@@@Z 34014c10 f i Movie.obj
 0001:00013ce0       ?GetMemoryUsage@CMovieSystem@@UBEXPAVICrySizer@@@Z 34014ce0 f i Movie.obj
 0001:00013d30       ?CreateSequence@CMovieSystem@@UAEPAUIAnimSequence@@PBDPAUIAnimSequenceGroup@@_NI@Z 34014d30 f   Movie.obj
 0001:00013e10       ?LoadSequence@CMovieSystem@@UAEPAUIAnimSequence@@AAVXmlNodeRef@@_N@Z 34014e10 f   Movie.obj
 0001:00013ef0       ?RemoveSequence@CMovieSystem@@UAEXPAUIAnimSequence@@@Z 34014ef0 f   Movie.obj
 0001:00013ff0       ?PlaySequence@CMovieSystem@@UAEXPAUIAnimSequence@@0_N1MM@Z 34014ff0 f   Movie.obj
 0001:00014200       ?StopAllSequences@CMovieSystem@@UAEXXZ 34015200 f   Movie.obj
 0001:00014270       ?StopAllCutScenes@CMovieSystem@@UAEXXZ 34015270 f   Movie.obj
 0001:000143e0       ?CacheLightAnim@CLightAnimWrapper@@CAXPBDPAV1@@Z 340153e0 f   Movie.obj
 0001:00014480       ?Backup@?$CBaseSplineInterpolator@MV?$TCBSpline@MU?$TCBSplineKeyEx@M@spline@@@spline@@@spline@@UAEPAUISplineBackup@@XZ 34015480 f i Movie.obj
 0001:000144c0       ?Restore@?$CBaseSplineInterpolator@MV?$TCBSpline@MU?$TCBSplineKeyEx@M@spline@@@spline@@@spline@@UAEXPAUISplineBackup@@@Z 340154c0 f i Movie.obj
 0001:00014520       ?Backup@?$CBaseSplineInterpolator@U?$Vec3_tpl@M@@V?$TCBSpline@U?$Vec3_tpl@M@@U?$TCBSplineKeyEx@U?$Vec3_tpl@M@@@spline@@@spline@@@spline@@UAEPAUISplineBackup@@XZ 34015520 f i Movie.obj
 0001:00014560       ?Restore@?$CBaseSplineInterpolator@U?$Vec3_tpl@M@@V?$TCBSpline@U?$Vec3_tpl@M@@U?$TCBSplineKeyEx@U?$Vec3_tpl@M@@@spline@@@spline@@@spline@@UAEXPAUISplineBackup@@@Z 34015560 f i Movie.obj
 0001:000145c0       ??_E?$TrackSplineInterpolator@M@spline@@W3AEPAXI@Z 340155c0 f i Movie.obj
 0001:000145d0       ?SetKeyInTangent@?$TrackSplineInterpolator@M@spline@@UAEXHQAM@Z 340155d0 f i Movie.obj
 0001:00014670       ?SetKeyOutTangent@?$TrackSplineInterpolator@M@spline@@UAEXHQAM@Z 34015670 f i Movie.obj
 0001:00014710       ?SetKeyFlags@?$TrackSplineInterpolator@M@spline@@UAEXHH@Z 34015710 f i Movie.obj
 0001:000147c0       ??_G?$TrackSplineInterpolator@M@spline@@UAEPAXI@Z 340157c0 f i Movie.obj
 0001:000147c0       ??_E?$TrackSplineInterpolator@M@spline@@UAEPAXI@Z 340157c0 f i Movie.obj
 0001:00014820       ??_E?$TrackSplineInterpolator@U?$Vec3_tpl@M@@@spline@@W3AEPAXI@Z 34015820 f i Movie.obj
 0001:00014830       ?SetKeyInTangent@?$TrackSplineInterpolator@U?$Vec3_tpl@M@@@spline@@UAEXHQAM@Z 34015830 f i Movie.obj
 0001:00014880       ?SetKeyOutTangent@?$TrackSplineInterpolator@U?$Vec3_tpl@M@@@spline@@UAEXHQAM@Z 34015880 f i Movie.obj
 0001:000148d0       ?SetKeyFlags@?$TrackSplineInterpolator@U?$Vec3_tpl@M@@@spline@@UAEXHH@Z 340158d0 f i Movie.obj
 0001:00014910       ??_E?$TrackSplineInterpolator@U?$Vec3_tpl@M@@@spline@@UAEPAXI@Z 34015910 f i Movie.obj
 0001:00014910       ??_G?$TrackSplineInterpolator@U?$Vec3_tpl@M@@@spline@@UAEPAXI@Z 34015910 f i Movie.obj
 0001:00014970       ?GetCurveType@?$TAnimSplineTrack@U?$Vec2_tpl@M@@@@UAE?AW4EAnimCurveType@@XZ 34015970 f i CompoundSplineTrack.obj
 0001:00014970       ?GetNumDimensions@?$CBaseSplineInterpolator@U?$Quat_tpl@M@@VTCBQuatSpline@spline@@@spline@@UAEHXZ 34015970 f i Movie.obj
 0001:00014970       ?GetType@CAnimCVarNode@@UBE?AW4EAnimNodeType@@XZ 34015970 f i CVarNode.obj
 0001:00014970       ?GetCurveType@CCompoundSplineTrack@@UAE?AW4EAnimCurveType@@XZ 34015970 f i CompoundSplineTrack.obj
 0001:00014980       ?assign@?$Array@U?$TCBSplineKey@U?$Quat_tpl@M@@@spline@@HU?$SmallDynStorage@U?$TCBSplineKey@U?$Quat_tpl@M@@@spline@@HUStandardAlloc@NAlloc@@@NArray@@@@QAEXU?$Array@$$CBU?$TCBSplineKey@U?$Quat_tpl@M@@@spline@@HU?$ArrayStorage@$$CBU?$TCBSplineKey@U?$Quat_tpl@M@@@spline@@H@NArray@@@@@Z 34015980 f i Movie.obj
 0001:00014a00       ??$__unguarded_linear_insert@PAU?$TCBSplineKey@U?$Quat_tpl@M@@@spline@@U12@U?$less@U?$TCBSplineKey@U?$Quat_tpl@M@@@spline@@@stlpmtx_std@@@priv@stlpmtx_std@@YAXPAU?$TCBSplineKey@U?$Quat_tpl@M@@@spline@@U23@U?$less@U?$TCBSplineKey@U?$Quat_tpl@M@@@spline@@@1@@Z 34015a00 f i Movie.obj
 0001:00014a90       ??$__push_heap@PAU?$TCBSplineKey@U?$Quat_tpl@M@@@spline@@HU12@U?$less@U?$TCBSplineKey@U?$Quat_tpl@M@@@spline@@@stlpmtx_std@@@stlpmtx_std@@YAXPAU?$TCBSplineKey@U?$Quat_tpl@M@@@spline@@HHU12@U?$less@U?$TCBSplineKey@U?$Quat_tpl@M@@@spline@@@0@@Z 34015a90 f i Movie.obj
 0001:00014b50       ??$__copy_backward@PAU?$TCBSplineKey@U?$Quat_tpl@M@@@spline@@PAU12@H@priv@stlpmtx_std@@YAPAU?$TCBSplineKey@U?$Quat_tpl@M@@@spline@@PAU23@00ABUrandom_access_iterator_tag@1@PAH@Z 34015b50 f i Movie.obj
 0001:00014cf0       ?GetKeyTime@?$CBaseSplineInterpolator@U?$Quat_tpl@M@@VTCBQuatSpline@spline@@@spline@@UAEMH@Z 34015cf0 f i Movie.obj
 0001:00014d20       ?GetKeyValue@?$CBaseSplineInterpolator@U?$Quat_tpl@M@@VTCBQuatSpline@spline@@@spline@@UAE_NHAAY03M@Z 34015d20 f i Movie.obj
 0001:00014d70       ?SetKeyValue@?$CBaseSplineInterpolator@U?$Quat_tpl@M@@VTCBQuatSpline@spline@@@spline@@UAEXHQAM@Z 34015d70 f i Movie.obj
 0001:00014dc0       ?SetKeyTime@?$CBaseSplineInterpolator@U?$Quat_tpl@M@@VTCBQuatSpline@spline@@@spline@@UAEXHM@Z 34015dc0 f i Movie.obj
 0001:00014e00       ?SetKeyInTangent@?$CBaseSplineInterpolator@U?$Quat_tpl@M@@VTCBQuatSpline@spline@@@spline@@UAEXHQAM@Z 34015e00 f i Movie.obj
 0001:00014e50       ?SetKeyOutTangent@?$CBaseSplineInterpolator@U?$Quat_tpl@M@@VTCBQuatSpline@spline@@@spline@@UAEXHQAM@Z 34015e50 f i Movie.obj
 0001:00014ea0       ?SetKeyTangents@?$CBaseSplineInterpolator@U?$Quat_tpl@M@@VTCBQuatSpline@spline@@@spline@@UAEXHQAM0@Z 34015ea0 f i Movie.obj
 0001:00014f10       ?GetKeyTangents@?$CBaseSplineInterpolator@U?$Quat_tpl@M@@VTCBQuatSpline@spline@@@spline@@UAE_NHAAY03M0@Z 34015f10 f i Movie.obj
 0001:00014f80       ?SetKeyFlags@?$CBaseSplineInterpolator@U?$Quat_tpl@M@@VTCBQuatSpline@spline@@@spline@@UAEXHH@Z 34015f80 f i Movie.obj
 0001:00014fc0       ?GetKeyFlags@?$CBaseSplineInterpolator@U?$Quat_tpl@M@@VTCBQuatSpline@spline@@@spline@@UAEHH@Z 34015fc0 f i Movie.obj
 0001:00014ff0       ?seek_key@?$TSpline@U?$TCBSplineKey@U?$Quat_tpl@M@@@spline@@VHermitBasis@2@@spline@@IAEHM@Z 34015ff0 f i Movie.obj
 0001:00015070       ??0?$TCBSplineKey@U?$Quat_tpl@M@@@spline@@QAE@ABU01@@Z 34016070 f i Movie.obj
 0001:000150f0       ?init@?$DynArray@U?$TCBSplineKey@U?$Quat_tpl@M@@@spline@@HU?$SmallDynStorage@U?$TCBSplineKey@U?$Quat_tpl@M@@@spline@@HUStandardAlloc@NAlloc@@@NArray@@@@KAPAU?$TCBSplineKey@U?$Quat_tpl@M@@@spline@@U?$Array@U?$TCBSplineKey@U?$Quat_tpl@M@@@spline@@HU?$ArrayStorage@U?$TCBSplineKey@U?$Quat_tpl@M@@@spline@@H@NArray@@@@ABU23@@Z 340160f0 f i Movie.obj
 0001:000151a0       ??$__unguarded_insertion_sort_aux@PAU?$TCBSplineKey@U?$Quat_tpl@M@@@spline@@U12@U?$less@U?$TCBSplineKey@U?$Quat_tpl@M@@@spline@@@stlpmtx_std@@@priv@stlpmtx_std@@YAXPAU?$TCBSplineKey@U?$Quat_tpl@M@@@spline@@00U?$less@U?$TCBSplineKey@U?$Quat_tpl@M@@@spline@@@1@@Z 340161a0 f i Movie.obj
 0001:00015250       ??$__adjust_heap@PAU?$TCBSplineKey@U?$Quat_tpl@M@@@spline@@HU12@U?$less@U?$TCBSplineKey@U?$Quat_tpl@M@@@spline@@@stlpmtx_std@@@stlpmtx_std@@YAXPAU?$TCBSplineKey@U?$Quat_tpl@M@@@spline@@HHU12@U?$less@U?$TCBSplineKey@U?$Quat_tpl@M@@@spline@@@0@@Z 34016250 f i Movie.obj
 0001:00015330       ?FindKeysInRange@?$CBaseSplineInterpolator@U?$Quat_tpl@M@@VTCBQuatSpline@spline@@@spline@@UAEXMMAAH0@Z 34016330 f i Movie.obj
 0001:00015460       ?init@?$DynArray@U?$TCBSplineKey@U?$Quat_tpl@M@@@spline@@HU?$SmallDynStorage@U?$TCBSplineKey@U?$Quat_tpl@M@@@spline@@HUStandardAlloc@NAlloc@@@NArray@@@@KAPAU?$TCBSplineKey@U?$Quat_tpl@M@@@spline@@U?$Array@U?$TCBSplineKey@U?$Quat_tpl@M@@@spline@@HU?$ArrayStorage@U?$TCBSplineKey@U?$Quat_tpl@M@@@spline@@H@NArray@@@@PBU23@@Z 34016460 f i Movie.obj
 0001:00015510       ?set_size@?$SmallDynStorage@U?$TCBSplineKey@U?$Quat_tpl@M@@@spline@@HUStandardAlloc@NAlloc@@@NArray@@QAEXH@Z 34016510 f i Movie.obj
 0001:000155a0       ??$move_init@U?$TCBSplineKey@U?$Quat_tpl@M@@@spline@@@NArray@@YAXPAU?$TCBSplineKey@U?$Quat_tpl@M@@@spline@@0I@Z 340165a0 f i Movie.obj
 0001:000155e0       ??$__make_heap@PAU?$TCBSplineKey@U?$Quat_tpl@M@@@spline@@U?$less@U?$TCBSplineKey@U?$Quat_tpl@M@@@spline@@@stlpmtx_std@@U12@H@stlpmtx_std@@YAXPAU?$TCBSplineKey@U?$Quat_tpl@M@@@spline@@0U?$less@U?$TCBSplineKey@U?$Quat_tpl@M@@@spline@@@0@0PAH@Z 340165e0 f i Movie.obj
 0001:000156c0       ?resize_raw@?$SmallDynStorage@U?$TCBSplineKey@U?$Quat_tpl@M@@@spline@@HUStandardAlloc@NAlloc@@@NArray@@QAEXHH_N@Z 340166c0 f i Movie.obj
 0001:00015820       ?expand_raw@?$DynArray@U?$TCBSplineKey@U?$Quat_tpl@M@@@spline@@HU?$SmallDynStorage@U?$TCBSplineKey@U?$Quat_tpl@M@@@spline@@HUStandardAlloc@NAlloc@@@NArray@@@@IAEPAU?$TCBSplineKey@U?$Quat_tpl@M@@@spline@@PAU23@H@Z 34016820 f i Movie.obj
 0001:000158b0       ?erase@?$DynArray@U?$TCBSplineKey@U?$Quat_tpl@M@@@spline@@HU?$SmallDynStorage@U?$TCBSplineKey@U?$Quat_tpl@M@@@spline@@HUStandardAlloc@NAlloc@@@NArray@@@@QAEPAU?$TCBSplineKey@U?$Quat_tpl@M@@@spline@@PAU23@0@Z 340168b0 f i Movie.obj
 0001:00015a90       ?insert_raw@?$DynArray@U?$TCBSplineKey@U?$Quat_tpl@M@@@spline@@HU?$SmallDynStorage@U?$TCBSplineKey@U?$Quat_tpl@M@@@spline@@HUStandardAlloc@NAlloc@@@NArray@@@@QAE?AU?$Array@U?$TCBSplineKey@U?$Quat_tpl@M@@@spline@@HU?$ArrayStorage@U?$TCBSplineKey@U?$Quat_tpl@M@@@spline@@H@NArray@@@@PAU?$TCBSplineKey@U?$Quat_tpl@M@@@spline@@H@Z 34016a90 f i Movie.obj
 0001:00015bd0       ??$__unguarded_partition@PAU?$TCBSplineKey@U?$Quat_tpl@M@@@spline@@U12@U?$less@U?$TCBSplineKey@U?$Quat_tpl@M@@@spline@@@stlpmtx_std@@@priv@stlpmtx_std@@YAPAU?$TCBSplineKey@U?$Quat_tpl@M@@@spline@@PAU23@0U23@U?$less@U?$TCBSplineKey@U?$Quat_tpl@M@@@spline@@@1@@Z 34016bd0 f i Movie.obj
 0001:00015d20       ??$sort_heap@PAU?$TCBSplineKey@U?$Quat_tpl@M@@@spline@@U?$less@U?$TCBSplineKey@U?$Quat_tpl@M@@@spline@@@stlpmtx_std@@@stlpmtx_std@@YAXPAU?$TCBSplineKey@U?$Quat_tpl@M@@@spline@@0U?$less@U?$TCBSplineKey@U?$Quat_tpl@M@@@spline@@@0@@Z 34016d20 f i Movie.obj
 0001:00015f00       ??4?$DynArray@U?$TCBSplineKey@U?$Quat_tpl@M@@@spline@@HU?$SmallDynStorage@U?$TCBSplineKey@U?$Quat_tpl@M@@@spline@@HUStandardAlloc@NAlloc@@@NArray@@@@QAEAAU0@U?$Array@$$CBU?$TCBSplineKey@U?$Quat_tpl@M@@@spline@@HU?$ArrayStorage@$$CBU?$TCBSplineKey@U?$Quat_tpl@M@@@spline@@H@NArray@@@@@Z 34016f00 f i Movie.obj
 0001:00015fb0       ??$__insertion_sort@PAU?$TCBSplineKey@U?$Quat_tpl@M@@@spline@@U12@U?$less@U?$TCBSplineKey@U?$Quat_tpl@M@@@spline@@@stlpmtx_std@@@priv@stlpmtx_std@@YAXPAU?$TCBSplineKey@U?$Quat_tpl@M@@@spline@@00U?$less@U?$TCBSplineKey@U?$Quat_tpl@M@@@spline@@@1@@Z 34016fb0 f i Movie.obj
 0001:00016080       ??$__partial_sort@PAU?$TCBSplineKey@U?$Quat_tpl@M@@@spline@@U12@U?$less@U?$TCBSplineKey@U?$Quat_tpl@M@@@spline@@@stlpmtx_std@@@priv@stlpmtx_std@@YAXPAU?$TCBSplineKey@U?$Quat_tpl@M@@@spline@@000U?$less@U?$TCBSplineKey@U?$Quat_tpl@M@@@spline@@@1@@Z 34017080 f i Movie.obj
 0001:00016220       ?RemoveKey@?$CBaseSplineInterpolator@U?$Quat_tpl@M@@VTCBQuatSpline@spline@@@spline@@UAEXH@Z 34017220 f i Movie.obj
 0001:00016260       ?RemoveKeysInRange@?$CBaseSplineInterpolator@U?$Quat_tpl@M@@VTCBQuatSpline@spline@@@spline@@UAEXMM@Z 34017260 f i Movie.obj
 0001:000163a0       ??0?$DynArray@U?$TCBSplineKey@U?$Quat_tpl@M@@@spline@@HU?$SmallDynStorage@U?$TCBSplineKey@U?$Quat_tpl@M@@@spline@@HUStandardAlloc@NAlloc@@@NArray@@@@QAE@ABU0@@Z 340173a0 f i Movie.obj
 0001:00016420       ??$__final_insertion_sort@PAU?$TCBSplineKey@U?$Quat_tpl@M@@@spline@@U?$less@U?$TCBSplineKey@U?$Quat_tpl@M@@@spline@@@stlpmtx_std@@@priv@stlpmtx_std@@YAXPAU?$TCBSplineKey@U?$Quat_tpl@M@@@spline@@0U?$less@U?$TCBSplineKey@U?$Quat_tpl@M@@@spline@@@1@@Z 34017420 f i Movie.obj
 0001:00016490       ??$__introsort_loop@PAU?$TCBSplineKey@U?$Quat_tpl@M@@@spline@@U12@HU?$less@U?$TCBSplineKey@U?$Quat_tpl@M@@@spline@@@stlpmtx_std@@@priv@stlpmtx_std@@YAXPAU?$TCBSplineKey@U?$Quat_tpl@M@@@spline@@00HU?$less@U?$TCBSplineKey@U?$Quat_tpl@M@@@spline@@@1@@Z 34017490 f i Movie.obj
 0001:000165f0       ?InsertKey@?$CBaseSplineInterpolator@U?$Quat_tpl@M@@VTCBQuatSpline@spline@@@spline@@UAEHMQAM@Z 340175f0 f i Movie.obj
 0001:00016760       ??$sort@PAU?$TCBSplineKey@U?$Quat_tpl@M@@@spline@@@stlpmtx_std@@YAXPAU?$TCBSplineKey@U?$Quat_tpl@M@@@spline@@0@Z 34017760 f i Movie.obj
 0001:000167c0       ??$reconstruct@V?$map@V?$CryStringT@D@@PAVCLightAnimWrapper@@U?$less@V?$CryStringT@D@@@stlpmtx_std@@V?$allocator@U?$pair@$$CBV?$CryStringT@D@@PAVCLightAnimWrapper@@@stlpmtx_std@@@4@@stlpmtx_std@@@stl@@YAXAAV?$map@V?$CryStringT@D@@PAVCLightAnimWrapper@@U?$less@V?$CryStringT@D@@@stlpmtx_std@@V?$allocator@U?$pair@$$CBV?$CryStringT@D@@PAVCLightAnimWrapper@@@stlpmtx_std@@@4@@stlpmtx_std@@@Z 340177c0 f i Movie.obj
 0001:00016830       ??$sort@PAU?$TCBSplineKeyEx@M@spline@@@stlpmtx_std@@YAXPAU?$TCBSplineKeyEx@M@spline@@0@Z 34017830 f i Movie.obj
 0001:00016890       ??$sort@PAU?$TCBSplineKeyEx@U?$Vec3_tpl@M@@@spline@@@stlpmtx_std@@YAXPAU?$TCBSplineKeyEx@U?$Vec3_tpl@M@@@spline@@0@Z 34017890 f i Movie.obj
 0001:000168f0       ?_M_insert@?$_Rb_tree@PAUIAnimSequence@@U?$less@PAUIAnimSequence@@@stlpmtx_std@@U?$pair@QAUIAnimSequence@@V?$vector@PAUIMovieListener@@V?$allocator@PAUIMovieListener@@@stlpmtx_std@@@stlpmtx_std@@@3@U?$_Select1st@U?$pair@QAUIAnimSequence@@V?$vector@PAUIMovieListener@@V?$allocator@PAUIMovieListener@@@stlpmtx_std@@@stlpmtx_std@@@stlpmtx_std@@@priv@3@U?$_MapTraitsT@U?$pair@QAUIAnimSequence@@V?$vector@PAUIMovieListener@@V?$allocator@PAUIMovieListener@@@stlpmtx_std@@@stlpmtx_std@@@stlpmtx_std@@@63@V?$allocator@U?$pair@QAUIAnimSequence@@V?$vector@PAUIMovieListener@@V?$allocator@PAUIMovieListener@@@stlpmtx_std@@@stlpmtx_std@@@stlpmtx_std@@@3@@priv@stlpmtx_std@@AAE?AU?$_Rb_tree_iterator@U?$pair@QAUIAnimSequence@@V?$vector@PAUIMovieListener@@V?$allocator@PAUIMovieListener@@@stlpmtx_std@@@stlpmtx_std@@@stlpmtx_std@@U?$_MapTraitsT@U?$pair@QAUIAnimSequence@@V?$vector@PAUIMovieListener@@V?$allocator@PAUIMovieListener@@@stlpmtx_std@@@stlpmtx_std@@@stlpmtx_std@@@priv@2@@23@PAU_Rb_tree_node_base@23@ABU?$pair@QAUIAnimSequence@@V?$vector@PAUIMovieListener@@V?$allocator@PAUIMovieListener@@@stlpmtx_std@@@stlpmtx_std@@@3@00@Z 340178f0 f i Movie.obj
 0001:00016a10       ?insert_unique@?$_Rb_tree@PAUIAnimSequence@@U?$less@PAUIAnimSequence@@@stlpmtx_std@@U?$pair@QAUIAnimSequence@@V?$vector@PAUIMovieListener@@V?$allocator@PAUIMovieListener@@@stlpmtx_std@@@stlpmtx_std@@@3@U?$_Select1st@U?$pair@QAUIAnimSequence@@V?$vector@PAUIMovieListener@@V?$allocator@PAUIMovieListener@@@stlpmtx_std@@@stlpmtx_std@@@stlpmtx_std@@@priv@3@U?$_MapTraitsT@U?$pair@QAUIAnimSequence@@V?$vector@PAUIMovieListener@@V?$allocator@PAUIMovieListener@@@stlpmtx_std@@@stlpmtx_std@@@stlpmtx_std@@@63@V?$allocator@U?$pair@QAUIAnimSequence@@V?$vector@PAUIMovieListener@@V?$allocator@PAUIMovieListener@@@stlpmtx_std@@@stlpmtx_std@@@stlpmtx_std@@@3@@priv@stlpmtx_std@@QAE?AU?$pair@U?$_Rb_tree_iterator@U?$pair@QAUIAnimSequence@@V?$vector@PAUIMovieListener@@V?$allocator@PAUIMovieListener@@@stlpmtx_std@@@stlpmtx_std@@@stlpmtx_std@@U?$_MapTraitsT@U?$pair@QAUIAnimSequence@@V?$vector@PAUIMovieListener@@V?$allocator@PAUIMovieListener@@@stlpmtx_std@@@stlpmtx_std@@@stlpmtx_std@@@priv@2@@priv@stlpmtx_std@@_N@3@ABU?$pair@QAUIAnimSequence@@V?$vector@PAUIMovieListener@@V?$allocator@PAUIMovieListener@@@stlpmtx_std@@@stlpmtx_std@@@3@@Z 34017a10 f i Movie.obj
 0001:00016ad0       ??0CMovieSystem@@QAE@PAUISystem@@@Z 34017ad0 f   Movie.obj
 0001:00016e10       ??_ECMovieSystem@@UAEPAXI@Z 34017e10 f i Movie.obj
 0001:00016e10       ??_GCMovieSystem@@UAEPAXI@Z 34017e10 f i Movie.obj
 0001:00016e40       ??_ECLightAnimWrapper@@EAEPAXI@Z 34017e40 f i Movie.obj
 0001:00016e40       ??_GCLightAnimWrapper@@EAEPAXI@Z 34017e40 f i Movie.obj
 0001:00016eb0       ?Create@CLightAnimWrapper@@SAPAV1@PBD@Z 34017eb0 f   Movie.obj
 0001:00016f40       ?ReconstructCache@CLightAnimWrapper@@SAXXZ 34017f40 f   Movie.obj
 0001:00016f80       ?interpolate@?$TSpline@U?$TCBSplineKey@U?$Quat_tpl@M@@@spline@@VHermitBasis@2@@spline@@QAE_NMAAU?$Quat_tpl@M@@@Z 34017f80 f i Movie.obj
 0001:000170d0       ?Interpolate@?$CBaseSplineInterpolator@U?$Quat_tpl@M@@VTCBQuatSpline@spline@@@spline@@UAEXMAAY03M@Z 340180d0 f i Movie.obj
 0001:00017120       ?Restore@?$CBaseSplineInterpolator@U?$Quat_tpl@M@@VTCBQuatSpline@spline@@@spline@@UAEXPAUISplineBackup@@@Z 34018120 f i Movie.obj
 0001:00017180       ??_E?$TrackSplineInterpolator@U?$Quat_tpl@M@@@spline@@W3AEPAXI@Z 34018180 f i Movie.obj
 0001:00017190       ??_E?$TrackSplineInterpolator@U?$Quat_tpl@M@@@spline@@UAEPAXI@Z 34018190 f i Movie.obj
 0001:00017190       ??_G?$TrackSplineInterpolator@U?$Quat_tpl@M@@@spline@@UAEPAXI@Z 34018190 f i Movie.obj
 0001:000171f0       ??0?$SSplineBackup@VTCBQuatSpline@spline@@@spline@@QAE@ABVTCBQuatSpline@1@@Z 340181f0 f i Movie.obj
 0001:00017260       ??_E?$SSplineBackup@VTCBQuatSpline@spline@@@spline@@W3AEPAXI@Z 34018260 f i Movie.obj
 0001:00017270       ??_G?$SSplineBackup@VTCBQuatSpline@spline@@@spline@@UAEPAXI@Z 34018270 f i Movie.obj
 0001:00017270       ??_E?$SSplineBackup@VTCBQuatSpline@spline@@@spline@@UAEPAXI@Z 34018270 f i Movie.obj
 0001:000172d0       ?insert_unique@?$_Rb_tree@PAUIAnimSequence@@U?$less@PAUIAnimSequence@@@stlpmtx_std@@U?$pair@QAUIAnimSequence@@V?$vector@PAUIMovieListener@@V?$allocator@PAUIMovieListener@@@stlpmtx_std@@@stlpmtx_std@@@3@U?$_Select1st@U?$pair@QAUIAnimSequence@@V?$vector@PAUIMovieListener@@V?$allocator@PAUIMovieListener@@@stlpmtx_std@@@stlpmtx_std@@@stlpmtx_std@@@priv@3@U?$_MapTraitsT@U?$pair@QAUIAnimSequence@@V?$vector@PAUIMovieListener@@V?$allocator@PAUIMovieListener@@@stlpmtx_std@@@stlpmtx_std@@@stlpmtx_std@@@63@V?$allocator@U?$pair@QAUIAnimSequence@@V?$vector@PAUIMovieListener@@V?$allocator@PAUIMovieListener@@@stlpmtx_std@@@stlpmtx_std@@@stlpmtx_std@@@3@@priv@stlpmtx_std@@QAE?AU?$_Rb_tree_iterator@U?$pair@QAUIAnimSequence@@V?$vector@PAUIMovieListener@@V?$allocator@PAUIMovieListener@@@stlpmtx_std@@@stlpmtx_std@@@stlpmtx_std@@U?$_MapTraitsT@U?$pair@QAUIAnimSequence@@V?$vector@PAUIMovieListener@@V?$allocator@PAUIMovieListener@@@stlpmtx_std@@@stlpmtx_std@@@stlpmtx_std@@@priv@2@@23@U423@ABU?$pair@QAUIAnimSequence@@V?$vector@PAUIMovieListener@@V?$allocator@PAUIMovieListener@@@stlpmtx_std@@@stlpmtx_std@@@3@@Z 340182d0 f i Movie.obj
 0001:000174c0       ??$reconstruct@V?$map@PAUIAnimSequence@@V?$vector@PAUIMovieListener@@V?$allocator@PAUIMovieListener@@@stlpmtx_std@@@stlpmtx_std@@U?$less@PAUIAnimSequence@@@3@V?$allocator@U?$pair@QAUIAnimSequence@@V?$vector@PAUIMovieListener@@V?$allocator@PAUIMovieListener@@@stlpmtx_std@@@stlpmtx_std@@@stlpmtx_std@@@3@@stlpmtx_std@@@stl@@YAXAAV?$map@PAUIAnimSequence@@V?$vector@PAUIMovieListener@@V?$allocator@PAUIMovieListener@@@stlpmtx_std@@@stlpmtx_std@@U?$less@PAUIAnimSequence@@@3@V?$allocator@U?$pair@QAUIAnimSequence@@V?$vector@PAUIMovieListener@@V?$allocator@PAUIMovieListener@@@stlpmtx_std@@@stlpmtx_std@@@stlpmtx_std@@@3@@stlpmtx_std@@@Z 340184c0 f i Movie.obj
 0001:00017530       ??0?$TAnimSplineTrack@M@@QAE@XZ 34018530 f i Movie.obj
 0001:000175b0       ?SelectKeyAllDimensions@ISplineInterpolator@@QAEXH_N@Z 340185b0 f i Movie.obj
 0001:00017620       ?GetKeyValueRange@?$TAnimSplineTrack@M@@UBEXAAM0@Z 34018620 f i Movie.obj
 0001:00017640       ?SetKeyValueRange@?$TAnimSplineTrack@M@@UAEXMM@Z 34018640 f i Movie.obj
 0001:00017660       ?SetSelected@?$TAnimSplineTrack@M@@UAEX_N@Z 34018660 f i Movie.obj
 0001:00017680       ?GetFlags@?$TAnimSplineTrack@M@@UAEHXZ 34018680 f i Movie.obj
 0001:00017680       ?GetSequence@CAnimNode@@UAEPAUIAnimSequence@@XZ 34018680 f i AnimLightNode.obj
 0001:00017690       ?SetDefaultValue@?$TAnimSplineTrack@M@@UAEXABM@Z 34018690 f i Movie.obj
 0001:000176a0       ?GetCustomColor@?$TAnimSplineTrack@M@@UBE?AU?$Color_tpl@E@@XZ 340186a0 f i Movie.obj
 0001:000176b0       ?HasCustomColor@?$TAnimSplineTrack@M@@UBE_NXZ 340186b0 f i Movie.obj
 0001:000176c0       ?ClearCustomColor@?$TAnimSplineTrack@M@@UAEXXZ 340186c0 f i Movie.obj
 0001:000176d0       ??$sprintf_s@$0EA@@@YAHAAY0EA@DPBDZZ 340186d0 f i Movie.obj
 0001:000176f0       ?GetParameterType@?$TAnimSplineTrack@M@@UBE?AVAnimParamType@@XZ 340186f0 f i Movie.obj
 0001:00017710       ?SetFlags@?$TAnimSplineTrack@M@@UAEXH@Z 34018710 f i Movie.obj
 0001:00017750       ?SetTimeRange@?$TAnimSplineTrack@U?$Vec2_tpl@M@@@@UAEXABV?$TRange@M@@@Z 34018750 f i CompoundSplineTrack.obj
 0001:00017750       ?SetTimeRange@?$TAnimSplineTrack@U?$Quat_tpl@M@@@@UAEXABV?$TRange@M@@@Z 34018750 f i Movie.obj
 0001:00017750       ?SetTimeRange@?$TAnimSplineTrack@M@@UAEXABV?$TRange@M@@@Z 34018750 f i Movie.obj
 0001:00017750       ?SetTimeRange@?$TAnimSplineTrack@U?$Vec3_tpl@M@@@@UAEXABV?$TRange@M@@@Z 34018750 f i Movie.obj
 0001:00017770       ?CreateKey@?$TAnimSplineTrack@M@@UAEHM@Z 34018770 f i Movie.obj
 0001:000177d0       ?SetCustomColor@?$TAnimSplineTrack@M@@UAEXU?$Color_tpl@E@@@Z 340187d0 f i Movie.obj
 0001:00017800       ??$?0M@?$Ang3_tpl@M@@QAE@ABU?$Quat_tpl@M@@@Z 34018800 f i Movie.obj
 0001:00017950       ?SetParameterType@?$TAnimSplineTrack@M@@UAEXVAnimParamType@@@Z 34018950 f i Movie.obj
 0001:000179c0       ?GetMemoryUsage@?$TAnimSplineTrack@M@@UBEXPAVICrySizer@@@Z 340189c0 f i Movie.obj
 0001:00017a00       ?init@?$DynArray@U?$TCBSplineKeyEx@M@spline@@HU?$SmallDynStorage@U?$TCBSplineKeyEx@M@spline@@HUStandardAlloc@NAlloc@@@NArray@@@@KAPAU?$TCBSplineKeyEx@M@spline@@U?$Array@U?$TCBSplineKeyEx@M@spline@@HU?$ArrayStorage@U?$TCBSplineKeyEx@M@spline@@H@NArray@@@@@Z 34018a00 f i Movie.obj
 0001:00017a80       ?Serialize@?$TAnimSplineTrack@M@@UAE_NAAVXmlNodeRef@@_N1@Z 34018a80 f i Movie.obj
 0001:00017f50       ?SerializeSelection@?$TAnimSplineTrack@M@@UAE_NAAVXmlNodeRef@@_N1M@Z 34018f50 f i Movie.obj
 0001:000183a0       ?GetKeyInfo@?$TAnimSplineTrack@M@@UAEXHAAPBDAAM@Z 340193a0 f i Movie.obj
 0001:000183f0       ??_G?$TAnimSplineTrack@M@@UAEPAXI@Z 340193f0 f i Movie.obj
 0001:000183f0       ??_E?$TAnimSplineTrack@M@@UAEPAXI@Z 340193f0 f i Movie.obj
 0001:00018450       ?GetNumKeys@?$TAnimSplineTrack@U?$Quat_tpl@M@@@@UBEHXZ 34019450 f i Movie.obj
 0001:00018450       ?GetNumKeys@?$TAnimSplineTrack@U?$Vec3_tpl@M@@@@UBEHXZ 34019450 f i Movie.obj
 0001:00018450       ?GetNumKeys@?$TAnimSplineTrack@U?$Vec2_tpl@M@@@@UBEHXZ 34019450 f i CompoundSplineTrack.obj
 0001:00018450       ?GetNumKeys@?$TAnimSplineTrack@M@@UBEHXZ 34019450 f i Movie.obj
 0001:00018460       ?GetKey@?$TAnimSplineTrack@M@@UBEXHPAUIKey@@@Z 34019460 f i Movie.obj
 0001:000184b0       ?SetKey@?$TAnimSplineTrack@M@@UAEXHPAUIKey@@@Z 340194b0 f i Movie.obj
 0001:00018500       ?GetKeyTime@?$TAnimSplineTrack@M@@UBEMH@Z 34019500 f i Movie.obj
 0001:00018520       ?GetKeyFlags@?$TAnimSplineTrack@M@@UAEHH@Z 34019520 f i Movie.obj
 0001:00018540       ?SetKeyFlags@?$TAnimSplineTrack@M@@UAEXHH@Z 34019540 f i Movie.obj
 0001:00018560       ?FindKey@?$TAnimSplineTrack@M@@UAEHM@Z 34019560 f i Movie.obj
 0001:000185b0       ?SetKeyAtTime@?$TAnimSplineTrack@M@@QAEXMPAUIKey@@@Z 340195b0 f i Movie.obj
 0001:00018650       ??1SColladaExportData@?$TAnimSplineTrack@U?$Vec3_tpl@M@@@@QAE@XZ 34019650 f i Movie.obj
 0001:00018650       ??1SColladaExportData@?$TAnimSplineTrack@U?$Quat_tpl@M@@@@QAE@XZ 34019650 f i Movie.obj
 0001:00018650       ??1SColladaExportData@?$TAnimSplineTrack@M@@QAE@XZ 34019650 f i Movie.obj
 0001:00018650       ??1SColladaExportData@?$TAnimSplineTrack@U?$Vec2_tpl@M@@@@QAE@XZ 34019650 f i CompoundSplineTrack.obj
 0001:000186e0       ?_M_create_node@?$_Rb_tree@HU?$less@H@stlpmtx_std@@U?$pair@$$CBHPAUIAnimNode@@@2@U?$_Select1st@U?$pair@$$CBHPAUIAnimNode@@@stlpmtx_std@@@priv@2@U?$_MapTraitsT@U?$pair@$$CBHPAUIAnimNode@@@stlpmtx_std@@@52@V?$allocator@U?$pair@$$CBHPAUIAnimNode@@@stlpmtx_std@@@2@@priv@stlpmtx_std@@IAEPAU_Rb_tree_node_base@23@ABU?$pair@$$CBHPAUIAnimNode@@@3@@Z 340196e0 f i AnimSequence.obj
 0001:000186e0       ?_M_create_node@?$_Rb_tree@PAUIEntity@@U?$less@PAUIEntity@@@stlpmtx_std@@U?$pair@QAUIEntity@@PAUIAnimNode@@@3@U?$_Select1st@U?$pair@QAUIEntity@@PAUIAnimNode@@@stlpmtx_std@@@priv@3@U?$_MapTraitsT@U?$pair@QAUIEntity@@PAUIAnimNode@@@stlpmtx_std@@@63@V?$allocator@U?$pair@QAUIEntity@@PAUIAnimNode@@@stlpmtx_std@@@3@@priv@stlpmtx_std@@IAEPAU_Rb_tree_node_base@23@ABU?$pair@QAUIEntity@@PAUIAnimNode@@@3@@Z 340196e0 f i Movie.obj
 0001:00018730       ?SetValue@?$TAnimSplineTrack@M@@UAEXMABM_N@Z 34019730 f i Movie.obj
 0001:000187a0       ?_M_insert@?$_Rb_tree@PAUIEntity@@U?$less@PAUIEntity@@@stlpmtx_std@@U?$pair@QAUIEntity@@PAUIAnimNode@@@3@U?$_Select1st@U?$pair@QAUIEntity@@PAUIAnimNode@@@stlpmtx_std@@@priv@3@U?$_MapTraitsT@U?$pair@QAUIEntity@@PAUIAnimNode@@@stlpmtx_std@@@63@V?$allocator@U?$pair@QAUIEntity@@PAUIAnimNode@@@stlpmtx_std@@@3@@priv@stlpmtx_std@@AAE?AU?$_Rb_tree_iterator@U?$pair@QAUIEntity@@PAUIAnimNode@@@stlpmtx_std@@U?$_MapTraitsT@U?$pair@QAUIEntity@@PAUIAnimNode@@@stlpmtx_std@@@priv@2@@23@PAU_Rb_tree_node_base@23@ABU?$pair@QAUIEntity@@PAUIAnimNode@@@3@00@Z 340197a0 f i Movie.obj
 0001:00018860       ?insert_unique@?$_Rb_tree@PAUIEntity@@U?$less@PAUIEntity@@@stlpmtx_std@@U?$pair@QAUIEntity@@PAUIAnimNode@@@3@U?$_Select1st@U?$pair@QAUIEntity@@PAUIAnimNode@@@stlpmtx_std@@@priv@3@U?$_MapTraitsT@U?$pair@QAUIEntity@@PAUIAnimNode@@@stlpmtx_std@@@63@V?$allocator@U?$pair@QAUIEntity@@PAUIAnimNode@@@stlpmtx_std@@@3@@priv@stlpmtx_std@@QAE?AU?$pair@U?$_Rb_tree_iterator@U?$pair@QAUIEntity@@PAUIAnimNode@@@stlpmtx_std@@U?$_MapTraitsT@U?$pair@QAUIEntity@@PAUIAnimNode@@@stlpmtx_std@@@priv@2@@priv@stlpmtx_std@@_N@3@ABU?$pair@QAUIEntity@@PAUIAnimNode@@@3@@Z 34019860 f i Movie.obj
 0001:00018920       ?WriteToColladaFile@?$TAnimSplineTrack@U?$Quat_tpl@M@@@@QAEXVXmlNodeRef@@PBD1ABUSColladaExportData@1@@Z 34019920 f i Movie.obj
 0001:00018920       ?WriteToColladaFile@?$TAnimSplineTrack@M@@QAEXVXmlNodeRef@@PBD1ABUSColladaExportData@1@@Z 34019920 f i Movie.obj
 0001:00018920       ?WriteToColladaFile@?$TAnimSplineTrack@U?$Vec3_tpl@M@@@@QAEXVXmlNodeRef@@PBD1ABUSColladaExportData@1@@Z 34019920 f i Movie.obj
 0001:00018920       ?WriteToColladaFile@?$TAnimSplineTrack@U?$Vec2_tpl@M@@@@QAEXVXmlNodeRef@@PBD1ABUSColladaExportData@1@@Z 34019920 f i CompoundSplineTrack.obj
 0001:00019440       ?insert_unique@?$_Rb_tree@PAUIEntity@@U?$less@PAUIEntity@@@stlpmtx_std@@U?$pair@QAUIEntity@@PAUIAnimNode@@@3@U?$_Select1st@U?$pair@QAUIEntity@@PAUIAnimNode@@@stlpmtx_std@@@priv@3@U?$_MapTraitsT@U?$pair@QAUIEntity@@PAUIAnimNode@@@stlpmtx_std@@@63@V?$allocator@U?$pair@QAUIEntity@@PAUIAnimNode@@@stlpmtx_std@@@3@@priv@stlpmtx_std@@QAE?AU?$_Rb_tree_iterator@U?$pair@QAUIEntity@@PAUIAnimNode@@@stlpmtx_std@@U?$_MapTraitsT@U?$pair@QAUIEntity@@PAUIAnimNode@@@stlpmtx_std@@@priv@2@@23@U423@ABU?$pair@QAUIEntity@@PAUIAnimNode@@@3@@Z 3401a440 f i Movie.obj
 0001:00019630       ?RemoveKey@?$TAnimSplineTrack@M@@UAEXH@Z 3401a630 f i Movie.obj
 0001:00019680       ??$?APAUIEntity@@@?$map@PAUIEntity@@PAUIAnimNode@@U?$less@PAUIEntity@@@stlpmtx_std@@V?$allocator@U?$pair@QAUIEntity@@PAUIAnimNode@@@stlpmtx_std@@@4@@stlpmtx_std@@QAEAAPAUIAnimNode@@ABQAUIEntity@@@Z 3401a680 f i Movie.obj
 0001:00019700       ?SetNumKeys@?$TAnimSplineTrack@M@@UAEXH@Z 3401a700 f i Movie.obj
 0001:00019770       ?SaveToColladaInFixedFPS@?$TAnimSplineTrack@U?$Vec2_tpl@M@@@@UAEXABUSColladaExporterSaveProperties@@VXmlNodeRef@@PBD2@Z 3401a770 f i CompoundSplineTrack.obj
 0001:00019770       ?SaveToColladaInFixedFPS@?$TAnimSplineTrack@U?$Vec3_tpl@M@@@@UAEXABUSColladaExporterSaveProperties@@VXmlNodeRef@@PBD2@Z 3401a770 f i Movie.obj
 0001:00019770       ?SaveToColladaInFixedFPS@?$TAnimSplineTrack@M@@UAEXABUSColladaExporterSaveProperties@@VXmlNodeRef@@PBD2@Z 3401a770 f i Movie.obj
 0001:00019770       ?SaveToColladaInFixedFPS@?$TAnimSplineTrack@U?$Quat_tpl@M@@@@UAEXABUSColladaExporterSaveProperties@@VXmlNodeRef@@PBD2@Z 3401a770 f i Movie.obj
 0001:0001ab10       ??0?$TAnimSplineTrack@U?$Vec3_tpl@M@@@@QAE@XZ 3401bb10 f i Movie.obj
 0001:0001abb0       ?GetParamCount@CAnimCVarNode@@UBEHXZ 3401bbb0 f i CVarNode.obj
 0001:0001abb0       ?GetSplineType@?$CBaseSplineInterpolator@U?$Quat_tpl@M@@VTCBQuatSpline@spline@@@spline@@UAE?AW4ESplineType@@XZ 3401bbb0 f i Movie.obj
 0001:0001abb0       ?GetSplineType@?$CBaseSplineInterpolator@U?$Vec2_tpl@M@@V?$BezierSpline@U?$Vec2_tpl@M@@U?$SplineKeyEx@U?$Vec2_tpl@M@@@spline@@@spline@@@spline@@UAE?AW4ESplineType@@XZ 3401bbb0 f i CompoundSplineTrack.obj
 0001:0001abb0       ?GetType@CAnimEntityNode@@UBE?AW4EAnimNodeType@@XZ 3401bbb0 f i EntityNode.obj
 0001:0001abb0       ?GetValueType@?$TAnimSplineTrack@U?$Vec3_tpl@M@@@@UAE?AW4EAnimValue@@XZ 3401bbb0 f i Movie.obj
 0001:0001abb0       ?GetSplineType@?$CBaseSplineInterpolator@U?$Vec3_tpl@M@@V?$TCBSpline@U?$Vec3_tpl@M@@U?$TCBSplineKeyEx@U?$Vec3_tpl@M@@@spline@@@spline@@@spline@@UAE?AW4ESplineType@@XZ 3401bbb0 f i Movie.obj
 0001:0001abb0       ?GetParamCount@CAnimScriptVarNode@@UBEHXZ 3401bbb0 f i ScriptVarNode.obj
 0001:0001abb0       ?GetSplineType@?$CBaseSplineInterpolator@MV?$TCBSpline@MU?$TCBSplineKeyEx@M@spline@@@spline@@@spline@@UAE?AW4ESplineType@@XZ 3401bbb0 f i Movie.obj
 0001:0001abb0       ?GetNumDimensions@?$TrackSplineInterpolator@U?$Vec2_tpl@M@@@spline@@UAEHXZ 3401bbb0 f i CompoundSplineTrack.obj
 0001:0001abb0       ?GetParamCount@CAnimEventNode@@UBEHXZ 3401bbb0 f i EventNode.obj
 0001:0001abb0       ?GetNumDimensions@?$CBaseSplineInterpolator@MV?$TCBSpline@MU?$TCBSplineKeyEx@M@spline@@@spline@@@spline@@UAEHXZ 3401bbb0 f i Movie.obj
 0001:0001abb0       ?GetCurveType@?$TAnimSplineTrack@M@@UAE?AW4EAnimCurveType@@XZ 3401bbb0 f i Movie.obj
 0001:0001abc0       ?GetKeyValueRange@?$TAnimSplineTrack@U?$Vec3_tpl@M@@@@UBEXAAM0@Z 3401bbc0 f i Movie.obj
 0001:0001abe0       ?SetKeyValueRange@?$TAnimSplineTrack@U?$Vec3_tpl@M@@@@UAEXMM@Z 3401bbe0 f i Movie.obj
 0001:0001ac00       ?LoadFromCollada@?$TAnimSplineTrack@M@@UAE_NVXmlNodeRef@@@Z 3401bc00 f i Movie.obj
 0001:0001ac00       ?LoadFromCollada@IAnimTrack@@UAE_NVXmlNodeRef@@@Z 3401bc00 f i Movie.obj
 0001:0001ac00       ?LoadFromCollada@?$TAnimSplineTrack@U?$Quat_tpl@M@@@@UAE_NVXmlNodeRef@@@Z 3401bc00 f i Movie.obj
 0001:0001ac00       ?LoadFromCollada@?$TAnimSplineTrack@U?$Vec3_tpl@M@@@@UAE_NVXmlNodeRef@@@Z 3401bc00 f i Movie.obj
 0001:0001ac20       ?SetSelected@?$TAnimSplineTrack@U?$Vec3_tpl@M@@@@UAEX_N@Z 3401bc20 f i Movie.obj
 0001:0001ac40       ?GetFlags@?$TAnimSplineTrack@U?$Vec3_tpl@M@@@@UAEHXZ 3401bc40 f i Movie.obj
 0001:0001ac50       ?SetDefaultValue@?$TAnimSplineTrack@U?$Vec3_tpl@M@@@@UAEXABU?$Vec3_tpl@M@@@Z 3401bc50 f i Movie.obj
 0001:0001ac70       ?GetCustomColor@?$TAnimSplineTrack@U?$Vec3_tpl@M@@@@UBE?AU?$Color_tpl@E@@XZ 3401bc70 f i Movie.obj
 0001:0001ac80       ?HasCustomColor@?$TAnimSplineTrack@U?$Vec3_tpl@M@@@@UBE_NXZ 3401bc80 f i Movie.obj
 0001:0001ac90       ?ClearCustomColor@?$TAnimSplineTrack@U?$Vec3_tpl@M@@@@UAEXXZ 3401bc90 f i Movie.obj
 0001:0001aca0       ?SetFlags@?$TAnimSplineTrack@U?$Vec3_tpl@M@@@@UAEXH@Z 3401bca0 f i Movie.obj
 0001:0001ace0       ?CreateKey@?$TAnimSplineTrack@U?$Vec3_tpl@M@@@@UAEHM@Z 3401bce0 f i Movie.obj
 0001:0001ad50       ?CopyKey@?$TAnimSplineTrack@M@@UAEHPAUIAnimTrack@@H@Z 3401bd50 f i Movie.obj
 0001:0001ad50       ?CopyKey@?$TAnimSplineTrack@U?$Vec3_tpl@M@@@@UAEHPAUIAnimTrack@@H@Z 3401bd50 f i Movie.obj
 0001:0001ad50       ?CopyKey@?$TAnimSplineTrack@U?$Quat_tpl@M@@@@UAEHPAUIAnimTrack@@H@Z 3401bd50 f i Movie.obj
 0001:0001ade0       ?SetCustomColor@?$TAnimSplineTrack@U?$Vec3_tpl@M@@@@UAEXU?$Color_tpl@E@@@Z 3401bde0 f i Movie.obj
 0001:0001ae10       ?OffsetKeyPosition@?$TAnimSplineTrack@U?$Vec3_tpl@M@@@@UAEXABU?$Vec3_tpl@M@@@Z 3401be10 f i Movie.obj
 0001:0001aed0       ?GetMemoryUsage@?$TAnimSplineTrack@U?$Vec3_tpl@M@@@@UBEXPAVICrySizer@@@Z 3401bed0 f i Movie.obj
 0001:0001af10       ?Serialize@?$TAnimSplineTrack@U?$Vec3_tpl@M@@@@UAE_NAAVXmlNodeRef@@_N1@Z 3401bf10 f i Movie.obj
 0001:0001b410       ?SerializeSelection@?$TAnimSplineTrack@U?$Vec3_tpl@M@@@@UAE_NAAVXmlNodeRef@@_N1M@Z 3401c410 f i Movie.obj
 0001:0001b8a0       ?GetKeyInfo@?$TAnimSplineTrack@U?$Vec3_tpl@M@@@@UAEXHAAPBDAAM@Z 3401c8a0 f i Movie.obj
 0001:0001b900       ??_G?$TAnimSplineTrack@U?$Vec3_tpl@M@@@@UAEPAXI@Z 3401c900 f i Movie.obj
 0001:0001b900       ??_E?$TAnimSplineTrack@U?$Vec3_tpl@M@@@@UAEPAXI@Z 3401c900 f i Movie.obj
 0001:0001b960       ?GetKey@?$TAnimSplineTrack@U?$Vec3_tpl@M@@@@UBEXHPAUIKey@@@Z 3401c960 f i Movie.obj
 0001:0001b9c0       ?SetKey@?$TAnimSplineTrack@U?$Vec3_tpl@M@@@@UAEXHPAUIKey@@@Z 3401c9c0 f i Movie.obj
 0001:0001ba40       ?GetKeyTime@?$TAnimSplineTrack@U?$Vec3_tpl@M@@@@UBEMH@Z 3401ca40 f i Movie.obj
 0001:0001ba60       ?GetKeyFlags@?$TAnimSplineTrack@U?$Vec3_tpl@M@@@@UAEHH@Z 3401ca60 f i Movie.obj
 0001:0001ba80       ?SetKeyFlags@?$TAnimSplineTrack@U?$Vec3_tpl@M@@@@UAEXHH@Z 3401ca80 f i Movie.obj
 0001:0001baa0       ?FindKey@?$TAnimSplineTrack@U?$Vec3_tpl@M@@@@UAEHM@Z 3401caa0 f i Movie.obj
 0001:0001baf0       ?SetKeyAtTime@?$TAnimSplineTrack@U?$Vec3_tpl@M@@@@QAEXMPAUIKey@@@Z 3401caf0 f i Movie.obj
 0001:0001bb90       ?init@?$DynArray@U?$TCBSplineKeyEx@U?$Vec3_tpl@M@@@spline@@HU?$SmallDynStorage@U?$TCBSplineKeyEx@U?$Vec3_tpl@M@@@spline@@HUStandardAlloc@NAlloc@@@NArray@@@@KAPAU?$TCBSplineKeyEx@U?$Vec3_tpl@M@@@spline@@U?$Array@U?$TCBSplineKeyEx@U?$Vec3_tpl@M@@@spline@@HU?$ArrayStorage@U?$TCBSplineKeyEx@U?$Vec3_tpl@M@@@spline@@H@NArray@@@@@Z 3401cb90 f i Movie.obj
 0001:0001bc10       ?SetValue@?$TAnimSplineTrack@U?$Vec3_tpl@M@@@@UAEXMABU?$Vec3_tpl@M@@_N@Z 3401cc10 f i Movie.obj
 0001:0001bca0       ?RemoveKey@?$TAnimSplineTrack@U?$Vec3_tpl@M@@@@UAEXH@Z 3401cca0 f i Movie.obj
 0001:0001bcf0       ?SetNumKeys@?$TAnimSplineTrack@U?$Vec3_tpl@M@@@@UAEXH@Z 3401ccf0 f i Movie.obj
 0001:0001bd60       ?QueueStopAnimationsAllLayers@CMovieSystem@@QAEXPAUICharacterInstance@@@Z 3401cd60 f   Movie.obj
 0001:0001be50       ?QueueStartAnimation@CMovieSystem@@QAEXPAUICharacterInstance@@PBDABUCryCharAnimationParams@@@Z 3401ce50 f   Movie.obj
 0001:0001bf80       ?QueueManualSeekAnimationInFIFO@CMovieSystem@@QAEXPAUICharacterInstance@@IIM_N@Z 3401cf80 f   Movie.obj
 0001:0001c080       ?QueueSetLayerTime@CMovieSystem@@QAEXPAUICharacterInstance@@IM@Z 3401d080 f   Movie.obj
 0001:0001c180       ?QueueSetTrackViewMixingWeight@CMovieSystem@@QAEXPAUICharacterInstance@@IM@Z 3401d180 f   Movie.obj
 0001:0001c280       ?ApplyQueuedSkelAnimCmds@CMovieSystem@@UAEXXZ 3401d280 f   Movie.obj
 0001:0001c4d0       ?CreateLightAnimWrapper@CMovieSystem@@UBEPAUILightAnimWrapper@@PBD@Z 3401d4d0 f   Movie.obj
 0001:0001c4f0       ?Backup@?$CBaseSplineInterpolator@U?$Quat_tpl@M@@VTCBQuatSpline@spline@@@spline@@UAEPAUISplineBackup@@XZ 3401d4f0 f i Movie.obj
 0001:0001c530       ?SortKeys@?$TAnimSplineTrack@M@@UAEXXZ 3401d530 f i Movie.obj
 0001:0001c560       ?interpolate@?$TSpline@U?$TCBSplineKeyEx@M@spline@@VHermitBasis@2@@spline@@QAE_NMAAM@Z 3401d560 f i Movie.obj
 0001:0001c690       ?SortKeys@?$TAnimSplineTrack@U?$Vec3_tpl@M@@@@UAEXXZ 3401d690 f i Movie.obj
 0001:0001c6c0       ?interpolate@?$TSpline@U?$TCBSplineKeyEx@U?$Vec3_tpl@M@@@spline@@VHermitBasis@2@@spline@@QAE_NMAAU?$Vec3_tpl@M@@@Z 3401d6c0 f i Movie.obj
 0001:0001c800       ?GetValue@?$TAnimSplineTrack@M@@UAEXMAAM@Z 3401d800 f i Movie.obj
 0001:0001c840       ?GetValue@?$TAnimSplineTrack@U?$Vec3_tpl@M@@@@UAEXMAAU?$Vec3_tpl@M@@@Z 3401d840 f i Movie.obj
 0001:0001c890       ??0?$TAnimSplineTrack@U?$Quat_tpl@M@@@@QAE@XZ 3401d890 f i Movie.obj
 0001:0001c920       ?GetCurveType@?$TAnimSplineTrack@U?$Vec3_tpl@M@@@@UAE?AW4EAnimCurveType@@XZ 3401d920 f i Movie.obj
 0001:0001c920       ?GetValueType@?$TAnimSplineTrack@U?$Quat_tpl@M@@@@UAE?AW4EAnimValue@@XZ 3401d920 f i Movie.obj
 0001:0001c920       ?GetType@CAnimSceneNode@@UBE?AW4EAnimNodeType@@XZ 3401d920 f i SceneNode.obj
 0001:0001c930       ?GetKeyValueRange@?$TAnimSplineTrack@U?$Quat_tpl@M@@@@UBEXAAM0@Z 3401d930 f i Movie.obj
 0001:0001c950       ?SetKeyValueRange@?$TAnimSplineTrack@U?$Quat_tpl@M@@@@UAEXMM@Z 3401d950 f i Movie.obj
 0001:0001c970       ?SetSelected@?$TAnimSplineTrack@U?$Quat_tpl@M@@@@UAEX_N@Z 3401d970 f i Movie.obj
 0001:0001c990       ?GetFlags@?$TAnimSplineTrack@U?$Quat_tpl@M@@@@UAEHXZ 3401d990 f i Movie.obj
 0001:0001c990       ?GetParent@CAnimNode@@UBEPAUIAnimNode@@XZ 3401d990 f i AnimLightNode.obj
 0001:0001c9a0       ?CloneKey@?$TAnimSplineTrack@M@@UAEHH@Z 3401d9a0 f i Movie.obj
 0001:0001c9a0       ?CloneKey@?$TAnimSplineTrack@U?$Quat_tpl@M@@@@UAEHH@Z 3401d9a0 f i Movie.obj
 0001:0001c9a0       ?CloneKey@?$TAnimSplineTrack@U?$Vec2_tpl@M@@@@UAEHH@Z 3401d9a0 f i CompoundSplineTrack.obj
 0001:0001c9a0       ?CloneKey@?$TAnimSplineTrack@U?$Vec3_tpl@M@@@@UAEHH@Z 3401d9a0 f i Movie.obj
 0001:0001c9c0       ?GetCustomColor@?$TAnimSplineTrack@U?$Quat_tpl@M@@@@UBE?AU?$Color_tpl@E@@XZ 3401d9c0 f i Movie.obj
 0001:0001c9d0       ?HasCustomColor@?$TAnimSplineTrack@U?$Quat_tpl@M@@@@UBE_NXZ 3401d9d0 f i Movie.obj
 0001:0001c9e0       ?ClearCustomColor@?$TAnimSplineTrack@U?$Quat_tpl@M@@@@UAEXXZ 3401d9e0 f i Movie.obj
 0001:0001c9f0       ?GetParameterType@?$TAnimSplineTrack@U?$Quat_tpl@M@@@@UBE?AVAnimParamType@@XZ 3401d9f0 f i Movie.obj
 0001:0001ca10       ?SetFlags@?$TAnimSplineTrack@U?$Quat_tpl@M@@@@UAEXH@Z 3401da10 f i Movie.obj
 0001:0001ca50       ?SetDefaultValue@?$TAnimSplineTrack@U?$Quat_tpl@M@@@@UAEXABU?$Quat_tpl@M@@@Z 3401da50 f i Movie.obj
 0001:0001ca80       ?SetCustomColor@?$TAnimSplineTrack@U?$Quat_tpl@M@@@@UAEXU?$Color_tpl@E@@@Z 3401da80 f i Movie.obj
 0001:0001cab0       ??$?0M@?$Ang3_tpl@M@@QAE@ABU?$Matrix33_tpl@M@@@Z 3401dab0 f i Movie.obj
 0001:0001cb80       ?SetParameterType@?$TAnimSplineTrack@U?$Quat_tpl@M@@@@UAEXVAnimParamType@@@Z 3401db80 f i Movie.obj
 0001:0001cbf0       ?GetKey@?$TAnimSplineTrack@U?$Quat_tpl@M@@@@UBEXHPAUIKey@@@Z 3401dbf0 f i Movie.obj
 0001:0001cc50       ?SetKey@?$TAnimSplineTrack@U?$Quat_tpl@M@@@@UAEXHPAUIKey@@@Z 3401dc50 f i Movie.obj
 0001:0001ccc0       ?GetKeyTime@?$TAnimSplineTrack@U?$Quat_tpl@M@@@@UBEMH@Z 3401dcc0 f i Movie.obj
 0001:0001cce0       ?GetKeyFlags@?$TAnimSplineTrack@U?$Quat_tpl@M@@@@UAEHH@Z 3401dce0 f i Movie.obj
 0001:0001cd00       ?SetKeyFlags@?$TAnimSplineTrack@U?$Quat_tpl@M@@@@UAEXHH@Z 3401dd00 f i Movie.obj
 0001:0001cd20       ?FindKey@?$TAnimSplineTrack@U?$Quat_tpl@M@@@@UAEHM@Z 3401dd20 f i Movie.obj
 0001:0001cd70       ?CreateKey@?$TAnimSplineTrack@U?$Quat_tpl@M@@@@UAEHM@Z 3401dd70 f i Movie.obj
 0001:0001ce10       ?SetKeyAtTime@?$TAnimSplineTrack@U?$Quat_tpl@M@@@@QAEXMPAUIKey@@@Z 3401de10 f i Movie.obj
 0001:0001ceb0       ?GetMemoryUsage@?$TAnimSplineTrack@U?$Quat_tpl@M@@@@UBEXPAVICrySizer@@@Z 3401deb0 f i Movie.obj
 0001:0001cef0       ?init@?$DynArray@U?$TCBSplineKey@U?$Quat_tpl@M@@@spline@@HU?$SmallDynStorage@U?$TCBSplineKey@U?$Quat_tpl@M@@@spline@@HUStandardAlloc@NAlloc@@@NArray@@@@KAPAU?$TCBSplineKey@U?$Quat_tpl@M@@@spline@@U?$Array@U?$TCBSplineKey@U?$Quat_tpl@M@@@spline@@HU?$ArrayStorage@U?$TCBSplineKey@U?$Quat_tpl@M@@@spline@@H@NArray@@@@@Z 3401def0 f i Movie.obj
 0001:0001cf50       ?Serialize@?$TAnimSplineTrack@U?$Quat_tpl@M@@@@UAE_NAAVXmlNodeRef@@_N1@Z 3401df50 f i Movie.obj
 0001:0001d450       ?SerializeSelection@?$TAnimSplineTrack@U?$Quat_tpl@M@@@@UAE_NAAVXmlNodeRef@@_N1M@Z 3401e450 f i Movie.obj
 0001:0001d8e0       ?SetValue@?$TAnimSplineTrack@U?$Quat_tpl@M@@@@UAEXMABU?$Quat_tpl@M@@_N@Z 3401e8e0 f i Movie.obj
 0001:0001d980       ?GetKeyInfo@?$TAnimSplineTrack@U?$Quat_tpl@M@@@@UAEXHAAPBDAAM@Z 3401e980 f i Movie.obj
 0001:0001daf0       ??_G?$TAnimSplineTrack@U?$Quat_tpl@M@@@@UAEPAXI@Z 3401eaf0 f i Movie.obj
 0001:0001daf0       ??_E?$TAnimSplineTrack@U?$Quat_tpl@M@@@@UAEPAXI@Z 3401eaf0 f i Movie.obj
 0001:0001db50       ?RemoveKey@?$TAnimSplineTrack@U?$Quat_tpl@M@@@@UAEXH@Z 3401eb50 f i Movie.obj
 0001:0001db90       ?SetNumKeys@?$TAnimSplineTrack@U?$Quat_tpl@M@@@@UAEXH@Z 3401eb90 f i Movie.obj
 0001:0001dc00       ?SortKeys@?$TAnimSplineTrack@U?$Quat_tpl@M@@@@UAEXXZ 3401ec00 f i Movie.obj
 0001:0001dc30       ?GetValue@?$TAnimSplineTrack@U?$Quat_tpl@M@@@@UAEXMAAU?$Quat_tpl@M@@@Z 3401ec30 f i Movie.obj
 0001:0001dc80       ?CreateTrack@CMovieSystem@@UAEPAUIAnimTrack@@W4EAnimCurveType@@@Z 3401ec80 f   Movie.obj
 0001:0001dce0       ?RemoveAllSequences@CMovieSystem@@UAEXXZ 3401ece0 f   Movie.obj
 0001:0001dd80       ?Interpolate@?$CBaseSplineInterpolator@MV?$TCBSpline@MU?$TCBSplineKeyEx@M@spline@@@spline@@@spline@@UAEXMAAY03M@Z 3401ed80 f i Movie.obj
 0001:0001ddb0       ?Interpolate@?$CBaseSplineInterpolator@U?$Vec3_tpl@M@@V?$TCBSpline@U?$Vec3_tpl@M@@U?$TCBSplineKeyEx@U?$Vec3_tpl@M@@@spline@@@spline@@@spline@@UAEXMAAY03M@Z 3401edb0 f i Movie.obj
 0001:0001ddf0       ??$?APAUIAnimSequence@@@?$map@PAUIAnimSequence@@V?$vector@PAUIMovieListener@@V?$allocator@PAUIMovieListener@@@stlpmtx_std@@@stlpmtx_std@@U?$less@PAUIAnimSequence@@@3@V?$allocator@U?$pair@QAUIAnimSequence@@V?$vector@PAUIMovieListener@@V?$allocator@PAUIMovieListener@@@stlpmtx_std@@@stlpmtx_std@@@stlpmtx_std@@@3@@stlpmtx_std@@QAEAAV?$vector@PAUIMovieListener@@V?$allocator@PAUIMovieListener@@@stlpmtx_std@@@1@ABQAUIAnimSequence@@@Z 3401edf0 f i Movie.obj
 0001:0001df30       ?AddMovieListener@CMovieSystem@@UAE_NPAUIAnimSequence@@PAUIMovieListener@@@Z 3401ef30 f   Movie.obj
 0001:0001dfa0       ?RemoveMovieListener@CMovieSystem@@UAE_NPAUIAnimSequence@@PAUIMovieListener@@@Z 3401efa0 f   Movie.obj
 0001:0001e010       ?DeInitialize@?$Node_Alloc_Lock@$00$00@@SAXXZ 3401f010 f i StdAfx.obj
 0001:0001e060       ?GetKeyInfo@CBoolTrack@@UAEXHAAPBDAAM@Z 3401f060 f   BoolTrack.obj
 0001:0001e080       ?SetValue@CBoolTrack@@UAEXMAB_N_N@Z 3401f080 f   BoolTrack.obj
 0001:0001e090       ?GetValue@CBoolTrack@@UAEXMAA_N@Z 3401f090 f   BoolTrack.obj
 0001:0001e0e0       ??$sprintf_s@$0BAA@@@YAHAAY0BAA@DPBDZZ 3401f0e0 f i CaptureTrack.obj
 0001:0001e100       ?SerializeKey@CCaptureTrack@@UAEXAAUICaptureKey@@AAVXmlNodeRef@@_N@Z 3401f100 f   CaptureTrack.obj
 0001:0001e380       ?GetKeyInfo@CCaptureTrack@@UAEXHAAPBDAAM@Z 3401f380 f   CaptureTrack.obj
 0001:0001e4a0       ?SerializeKey@CCharacterTrack@@UAEXAAUICharacterKey@@AAVXmlNodeRef@@_N@Z 3401f4a0 f   CharacterTrack.obj
 0001:0001e700       ?Serialize@?$TAnimTrack@UICharacterKey@@@@UAE_NAAVXmlNodeRef@@_N1@Z 3401f700 f i CharacterTrack.obj
 0001:0001e9b0       ?Serialize@CCharacterTrack@@UAE_NAAVXmlNodeRef@@_N1@Z 3401f9b0 f   CharacterTrack.obj
 0001:0001ea10       ?GetKeyInfo@CCharacterTrack@@UAEXHAAPBDAAM@Z 3401fa10 f   CharacterTrack.obj
 0001:0001eb20       ?GetKeyDuration@CCharacterTrack@@QBEMH@Z 3401fb20 f   CharacterTrack.obj
 0001:0001ec30       ?GetKeyInfo@CCommentTrack@@UAEXHAAPBDAAM@Z 3401fc30 f   CommentTrack.obj
 0001:0001ec90       ?SerializeKey@CCommentTrack@@UAEXAAUICommentKey@@AAVXmlNodeRef@@_N@Z 3401fc90 f   CommentTrack.obj
 0001:0001ee20       ??$__destroy_range_aux@V?$reverse_iterator@PAUICommentKey@@@stlpmtx_std@@UICommentKey@@@stlpmtx_std@@YAXV?$reverse_iterator@PAUICommentKey@@@0@0PAUICommentKey@@ABU__false_type@0@@Z 3401fe20 f i CommentTrack.obj
 0001:0001ee70       ?GetValueType@?$TAnimTrack@UIBoolKey@@@@UAE?AW4EAnimValue@@XZ 3401fe70 f i AnimNode.obj
 0001:0001ee70       ?GetValueType@?$TAnimTrack@UIExprKey@@@@UAE?AW4EAnimValue@@XZ 3401fe70 f i AnimNode.obj
 0001:0001ee70       ?GetCurveType@?$TAnimTrack@UIDiscreteFloatKey@@@@UAE?AW4EAnimCurveType@@XZ 3401fe70 f i GotoTrack.obj
 0001:0001ee70       ?GetValueType@?$TAnimTrack@UIScreenFaderKey@@@@UAE?AW4EAnimValue@@XZ 3401fe70 f i ScreenFaderTrack.obj
 0001:0001ee70       ?GetValueType@?$TAnimTrack@UIConsoleKey@@@@UAE?AW4EAnimValue@@XZ 3401fe70 f i AnimNode.obj
 0001:0001ee70       ?GetValueType@?$TAnimTrack@UICharacterKey@@@@UAE?AW4EAnimValue@@XZ 3401fe70 f i AnimNode.obj
 0001:0001ee70       ?GetValueType@?$TAnimTrack@UISequenceKey@@@@UAE?AW4EAnimValue@@XZ 3401fe70 f i AnimNode.obj
 0001:0001ee70       ?GetCurveType@?$TAnimTrack@UIEventKey@@@@UAE?AW4EAnimCurveType@@XZ 3401fe70 f i AnimNode.obj
 0001:0001ee70       ?GetCurveType@?$TAnimTrack@UISequenceKey@@@@UAE?AW4EAnimCurveType@@XZ 3401fe70 f i AnimNode.obj
 0001:0001ee70       ?GetValueType@?$TAnimTrack@UILookAtKey@@@@UAE?AW4EAnimValue@@XZ 3401fe70 f i AnimNode.obj
 0001:0001ee70       ?GetCurveType@?$TAnimTrack@UICharacterKey@@@@UAE?AW4EAnimCurveType@@XZ 3401fe70 f i AnimNode.obj
 0001:0001ee70       ?GetAnimationLayerIndex@IAnimTrack@@UBEHXZ 3401fe70 f i Movie.obj
 0001:0001ee70       ?GetCurveType@?$TAnimTrack@UIExprKey@@@@UAE?AW4EAnimCurveType@@XZ 3401fe70 f i AnimNode.obj
 0001:0001ee70       ?GetValueType@?$TAnimTrack@UIMusicKey@@@@UAE?AW4EAnimValue@@XZ 3401fe70 f i AnimNode.obj
 0001:0001ee70       ?GetCurveType@?$TAnimTrack@UIBoolKey@@@@UAE?AW4EAnimCurveType@@XZ 3401fe70 f i AnimNode.obj
 0001:0001ee70       ?GetValueType@?$TAnimTrack@UISoundKey@@@@UAE?AW4EAnimValue@@XZ 3401fe70 f i AnimNode.obj
 0001:0001ee70       ?GetCurveType@?$TAnimTrack@UISelectKey@@@@UAE?AW4EAnimCurveType@@XZ 3401fe70 f i AnimNode.obj
 0001:0001ee70       ?GetCurveType@?$TAnimTrack@UISoundKey@@@@UAE?AW4EAnimCurveType@@XZ 3401fe70 f i AnimNode.obj
 0001:0001ee70       ?GetCurveType@?$TAnimTrack@UIFaceSeqKey@@@@UAE?AW4EAnimCurveType@@XZ 3401fe70 f i AnimNode.obj
 0001:0001ee70       ?GetValueType@?$TAnimTrack@UIDiscreteFloatKey@@@@UAE?AW4EAnimValue@@XZ 3401fe70 f i GotoTrack.obj
 0001:0001ee70       ?GetCurveType@?$TAnimTrack@UIScreenFaderKey@@@@UAE?AW4EAnimCurveType@@XZ 3401fe70 f i ScreenFaderTrack.obj
 0001:0001ee70       ?GetValueType@?$TAnimTrack@UICaptureKey@@@@UAE?AW4EAnimValue@@XZ 3401fe70 f i AnimNode.obj
 0001:0001ee70       ?GetCurveType@?$TAnimTrack@UIConsoleKey@@@@UAE?AW4EAnimCurveType@@XZ 3401fe70 f i AnimNode.obj
 0001:0001ee70       ?GetValueType@?$TAnimTrack@UISelectKey@@@@UAE?AW4EAnimValue@@XZ 3401fe70 f i AnimNode.obj
 0001:0001ee70       ?GetCurveType@?$TAnimTrack@UILookAtKey@@@@UAE?AW4EAnimCurveType@@XZ 3401fe70 f i AnimNode.obj
 0001:0001ee70       ?GetCurveType@?$TAnimTrack@UICommentKey@@@@UAE?AW4EAnimCurveType@@XZ 3401fe70 f i CommentTrack.obj
 0001:0001ee70       ?GetValueType@?$TAnimTrack@UIFaceSeqKey@@@@UAE?AW4EAnimValue@@XZ 3401fe70 f i AnimNode.obj
 0001:0001ee70       ?GetValueType@?$TAnimTrack@UIEventKey@@@@UAE?AW4EAnimValue@@XZ 3401fe70 f i AnimNode.obj
 0001:0001ee70       ?GetCurveType@?$TAnimTrack@UICaptureKey@@@@UAE?AW4EAnimCurveType@@XZ 3401fe70 f i AnimNode.obj
 0001:0001ee70       ?GetValueType@?$TAnimTrack@UICommentKey@@@@UAE?AW4EAnimValue@@XZ 3401fe70 f i CommentTrack.obj
 0001:0001ee70       ?GetCurveType@?$TAnimTrack@UIMusicKey@@@@UAE?AW4EAnimCurveType@@XZ 3401fe70 f i AnimNode.obj
 0001:0001ee80       ?IsMasked@?$TAnimTrack@UICommentKey@@@@UBE_NI@Z 3401fe80 f i CommentTrack.obj
 0001:0001ee80       ?IsMasked@?$TAnimTrack@UISelectKey@@@@UBE_NI@Z 3401fe80 f i AnimNode.obj
 0001:0001ee80       ?IsMasked@?$TAnimTrack@UIScreenFaderKey@@@@UBE_NI@Z 3401fe80 f i ScreenFaderTrack.obj
 0001:0001ee80       ?IsMasked@?$TAnimTrack@UISoundKey@@@@UBE_NI@Z 3401fe80 f i AnimNode.obj
 0001:0001ee80       ?IsMasked@?$TAnimTrack@UICharacterKey@@@@UBE_NI@Z 3401fe80 f i AnimNode.obj
 0001:0001ee80       ?IsMasked@?$TAnimTrack@UIMusicKey@@@@UBE_NI@Z 3401fe80 f i AnimNode.obj
 0001:0001ee80       ?IsMasked@?$TAnimTrack@UIConsoleKey@@@@UBE_NI@Z 3401fe80 f i AnimNode.obj
 0001:0001ee80       ?IsMasked@?$TAnimTrack@UICaptureKey@@@@UBE_NI@Z 3401fe80 f i AnimNode.obj
 0001:0001ee80       ?IsMasked@?$TAnimTrack@UIBoolKey@@@@UBE_NI@Z 3401fe80 f i AnimNode.obj
 0001:0001ee80       ?IsMasked@?$TAnimTrack@UISequenceKey@@@@UBE_NI@Z 3401fe80 f i AnimNode.obj
 0001:0001ee80       ?IsMasked@?$TAnimTrack@UIExprKey@@@@UBE_NI@Z 3401fe80 f i AnimNode.obj
 0001:0001ee80       ?IsMasked@?$TAnimSplineTrack@M@@UBE_NI@Z 3401fe80 f i Movie.obj
 0001:0001ee80       ?IsMasked@?$TAnimTrack@UIFaceSeqKey@@@@UBE_NI@Z 3401fe80 f i AnimNode.obj
 0001:0001ee80       ?IsMasked@?$TAnimSplineTrack@U?$Vec3_tpl@M@@@@UBE_NI@Z 3401fe80 f i Movie.obj
 0001:0001ee80       ?IsMasked@?$TAnimTrack@UIDiscreteFloatKey@@@@UBE_NI@Z 3401fe80 f i GotoTrack.obj
 0001:0001ee80       ?IsMasked@?$TAnimTrack@UILookAtKey@@@@UBE_NI@Z 3401fe80 f i AnimNode.obj
 0001:0001ee80       ?IsMasked@?$TAnimSplineTrack@U?$Vec2_tpl@M@@@@UBE_NI@Z 3401fe80 f i CompoundSplineTrack.obj
 0001:0001ee80       ?IsMasked@?$TAnimSplineTrack@U?$Quat_tpl@M@@@@UBE_NI@Z 3401fe80 f i Movie.obj
 0001:0001ee80       ?IsMasked@?$TAnimTrack@UIEventKey@@@@UBE_NI@Z 3401fe80 f i AnimNode.obj
 0001:0001ee80       ?IsMasked@CCompoundSplineTrack@@UBE_NI@Z 3401fe80 f i CompoundSplineTrack.obj
 0001:0001ee90       ?AddLabel@CDummyMemReplay@@UAEXPBD@Z 3401fe90 f i AnimSequence.obj
 0001:0001ee90       ?SetEntityGuid@CAnimNode@@UAEXAB_K@Z 3401fe90 f i AnimSequence.obj
 0001:0001ee90       ?OffsetKeyPosition@?$TAnimTrack@UICommentKey@@@@UAEXABU?$Vec3_tpl@M@@@Z 3401fe90 f i CommentTrack.obj
 0001:0001ee90       ?AddSizerTree@CDummyMemReplay@@UAEXPBD@Z 3401fe90 f i AnimSequence.obj
 0001:0001ee90       ?SetAnimationLayerIndex@IAnimTrack@@UAEXH@Z 3401fe90 f i Movie.obj
 0001:0001ee90       ?OffsetKeyPosition@?$TAnimTrack@UIExprKey@@@@UAEXABU?$Vec3_tpl@M@@@Z 3401fe90 f i AnimNode.obj
 0001:0001ee90       ?SetDefault@?$TControlParam@M@CFXNodeDescription@@UAEX_N@Z 3401fe90 f i AnimPostFXNode.obj
 0001:0001ee90       ?OffsetKeyPosition@?$TAnimTrack@UIDiscreteFloatKey@@@@UAEXABU?$Vec3_tpl@M@@@Z 3401fe90 f i GotoTrack.obj
 0001:0001ee90       ?OffsetKeyPosition@?$TAnimTrack@UICharacterKey@@@@UAEXABU?$Vec3_tpl@M@@@Z 3401fe90 f i AnimNode.obj
 0001:0001ee90       ?OffsetKeyPosition@?$TAnimTrack@UICaptureKey@@@@UAEXABU?$Vec3_tpl@M@@@Z 3401fe90 f i AnimNode.obj
 0001:0001ee90       ?Animate@CAnimNode@@UAEXAAUSAnimContext@@@Z 3401fe90 f i AnimNode.obj
 0001:0001ee90       ?OffsetKeyPosition@?$TAnimTrack@UIScreenFaderKey@@@@UAEXABU?$Vec3_tpl@M@@@Z 3401fe90 f i ScreenFaderTrack.obj
 0001:0001ee90       ?SetDefault@?$TControlParam@_N@CFXNodeDescription@@UAEXM@Z 3401fe90 f i AnimPostFXNode.obj
 0001:0001ee90       ?OffsetKeyPosition@?$TAnimTrack@UIConsoleKey@@@@UAEXABU?$Vec3_tpl@M@@@Z 3401fe90 f i AnimNode.obj
 0001:0001ee90       ?OffsetKeyPosition@?$TAnimSplineTrack@U?$Vec2_tpl@M@@@@UAEXABU?$Vec3_tpl@M@@@Z 3401fe90 f i CompoundSplineTrack.obj
 0001:0001ee90       ?StartOnCommandLine@CDummyMemReplay@@UAEXPBD@Z 3401fe90 f i AnimSequence.obj
 0001:0001ee90       ?OffsetKeyPosition@?$TAnimSplineTrack@U?$Quat_tpl@M@@@@UAEXABU?$Vec3_tpl@M@@@Z 3401fe90 f i Movie.obj
 0001:0001ee90       ?EnableBoneLinkTransform@CAnimNode@@UAEX_N@Z 3401fe90 f i AnimSequence.obj
 0001:0001ee90       ?GetDefault@?$TControlParam@M@CFXNodeDescription@@UBEXAA_N@Z 3401fe90 f i AnimPostFXNode.obj
 0001:0001ee90       ?Activate@CAnimNode@@UAEX_N@Z 3401fe90 f i AnimNode.obj
 0001:0001ee90       ?SetNumKeys@CCompoundSplineTrack@@UAEXH@Z 3401fe90 f i CompoundSplineTrack.obj
 0001:0001ee90       ?OffsetKeyPosition@?$TAnimTrack@UISoundKey@@@@UAEXABU?$Vec3_tpl@M@@@Z 3401fe90 f i AnimNode.obj
 0001:0001ee90       ?GetInfo@CDummyMemReplay@@UAEXAAUCryReplayInfo@@@Z 3401fe90 f i AnimSequence.obj
 0001:0001ee90       ?OffsetKeyPosition@?$TAnimTrack@UIMusicKey@@@@UAEXABU?$Vec3_tpl@M@@@Z 3401fe90 f i AnimNode.obj
 0001:0001ee90       ?OffsetKeyPosition@?$TAnimTrack@UISelectKey@@@@UAEXABU?$Vec3_tpl@M@@@Z 3401fe90 f i AnimNode.obj
 0001:0001ee90       ?ExitScope_Free@CDummyMemReplay@@UAEXI@Z 3401fe90 f i AnimSequence.obj
 0001:0001ee90       ?OnStartAnimation@CAnimEntityNode@@MAEXPBD@Z 3401fe90 f i AnimLightNode.obj
 0001:0001ee90       ?GetDefault@?$TControlParam@_N@CFXNodeDescription@@UBEXAAM@Z 3401fe90 f i AnimPostFXNode.obj
 0001:0001ee90       ?OffsetKeyPosition@?$TAnimTrack@UIFaceSeqKey@@@@UAEXABU?$Vec3_tpl@M@@@Z 3401fe90 f i AnimNode.obj
 0001:0001ee90       ?RemoveAllocReference@CDummyMemReplay@@UAEXPAX@Z 3401fe90 f i AnimSequence.obj
 0001:0001ee90       ?OffsetKeyPosition@?$TAnimTrack@UIBoolKey@@@@UAEXABU?$Vec3_tpl@M@@@Z 3401fe90 f i AnimNode.obj
 0001:0001ee90       ?OffsetKeyPosition@?$TAnimTrack@UISequenceKey@@@@UAEXABU?$Vec3_tpl@M@@@Z 3401fe90 f i AnimNode.obj
 0001:0001ee90       ?OffsetKeyPosition@?$TAnimSplineTrack@M@@UAEXABU?$Vec3_tpl@M@@@Z 3401fe90 f i Movie.obj
 0001:0001ee90       ?Animate@IAnimTrack@@UAEXAAUSAnimContext@@@Z 3401fe90 f i Movie.obj
 0001:0001ee90       ?OffsetKeyPosition@?$TAnimTrack@UIEventKey@@@@UAEXABU?$Vec3_tpl@M@@@Z 3401fe90 f i AnimNode.obj
 0001:0001ee90       ?SetEntityGuidTarget@CAnimNode@@UAEXAB_K@Z 3401fe90 f i AnimSequence.obj
 0001:0001ee90       ?OffsetKeyPosition@?$TAnimTrack@UILookAtKey@@@@UAEXABU?$Vec3_tpl@M@@@Z 3401fe90 f i AnimNode.obj
 0001:0001ee90       ?UnregisterContainer@CDummyMemReplay@@UAEXPBX@Z 3401fe90 f i AnimSequence.obj
 0001:0001ee90       ?SetEntityGuidSource@CAnimNode@@UAEXAB_K@Z 3401fe90 f i AnimSequence.obj
 0001:0001eea0       ?GetNumKeys@?$TAnimTrack@UICommentKey@@@@UBEHXZ 3401fea0 f i CommentTrack.obj
 0001:0001eec0       ?GetKeyTime@?$TAnimTrack@UICommentKey@@@@UBEMH@Z 3401fec0 f i CommentTrack.obj
 0001:0001eee0       ?FindKey@?$TAnimTrack@UICommentKey@@@@UAEHM@Z 3401fee0 f i CommentTrack.obj
 0001:0001ef40       ?GetKeyFlags@?$TAnimTrack@UICommentKey@@@@UAEHH@Z 3401ff40 f i CommentTrack.obj
 0001:0001ef60       ?SetKeyTime@?$TAnimTrack@UICommentKey@@@@UAEXHM@Z 3401ff60 f i CommentTrack.obj
 0001:0001ef80       ?SetKeyFlags@?$TAnimTrack@UICommentKey@@@@UAEXHH@Z 3401ff80 f i CommentTrack.obj
 0001:0001efa0       ?Serialize@?$TAnimTrack@UICommentKey@@@@UAE_NAAVXmlNodeRef@@_N1@Z 3401ffa0 f i CommentTrack.obj
 0001:0001f250       ?SerializeSelection@?$TAnimTrack@UICommentKey@@@@UAE_NAAVXmlNodeRef@@_N1M@Z 34020250 f i CommentTrack.obj
 0001:0001f410       ?IsKeySelected@?$TAnimTrack@UICommentKey@@@@UBE_NH@Z 34020410 f i CommentTrack.obj
 0001:0001f430       ?SelectKey@?$TAnimTrack@UICommentKey@@@@UAEXH_N@Z 34020430 f i CommentTrack.obj
 0001:0001f470       ??4ICommentKey@@QAEAAU0@ABU0@@Z 34020470 f i CommentTrack.obj
 0001:0001f510       ??$__copy@PAUICommentKey@@PAU1@H@priv@stlpmtx_std@@YAPAUICommentKey@@PAU2@00ABUrandom_access_iterator_tag@1@PAH@Z 34020510 f i CommentTrack.obj
 0001:0001f640       ??$__copy_backward@PAUICommentKey@@PAU1@H@priv@stlpmtx_std@@YAPAUICommentKey@@PAU2@00ABUrandom_access_iterator_tag@1@PAH@Z 34020640 f i CommentTrack.obj
 0001:0001f770       ??$__fill@PAUICommentKey@@U1@H@priv@stlpmtx_std@@YAXPAUICommentKey@@0ABU2@ABUrandom_access_iterator_tag@1@PAH@Z 34020770 f i CommentTrack.obj
 0001:0001f8a0       ??$__unguarded_linear_insert@PAUICommentKey@@U1@U?$less@UICommentKey@@@stlpmtx_std@@@priv@stlpmtx_std@@YAXPAUICommentKey@@U2@U?$less@UICommentKey@@@1@@Z 340208a0 f i CommentTrack.obj
 0001:0001f900       ??$__push_heap@PAUICommentKey@@HU1@U?$less@UICommentKey@@@stlpmtx_std@@@stlpmtx_std@@YAXPAUICommentKey@@HHU1@U?$less@UICommentKey@@@0@@Z 34020900 f i CommentTrack.obj
 0001:0001f990       ??0ICommentKey@@QAE@ABU0@@Z 34020990 f i CommentTrack.obj
 0001:0001fa30       ?CreateKey@?$TAnimTrack@UICommentKey@@@@UAEHM@Z 34020a30 f i CommentTrack.obj
 0001:0001fbb0       ?CloneKey@?$TAnimTrack@UICommentKey@@@@UAEHH@Z 34020bb0 f i CommentTrack.obj
 0001:0001fca0       ?CopyKey@?$TAnimTrack@UICommentKey@@@@UAEHPAUIAnimTrack@@H@Z 34020ca0 f i CommentTrack.obj
 0001:0001fd90       ?GetKey@?$TAnimTrack@UICommentKey@@@@UBEXHPAUIKey@@@Z 34020d90 f i CommentTrack.obj
 0001:0001fdb0       ?SetKey@?$TAnimTrack@UICommentKey@@@@UAEXHPAUIKey@@@Z 34020db0 f i CommentTrack.obj
 0001:0001fde0       ??$__unguarded_insertion_sort_aux@PAUICommentKey@@U1@U?$less@UICommentKey@@@stlpmtx_std@@@priv@stlpmtx_std@@YAXPAUICommentKey@@00U?$less@UICommentKey@@@1@@Z 34020de0 f i CommentTrack.obj
 0001:0001fe60       ??$__adjust_heap@PAUICommentKey@@HU1@U?$less@UICommentKey@@@stlpmtx_std@@@stlpmtx_std@@YAXPAUICommentKey@@HHU1@U?$less@UICommentKey@@@0@@Z 34020e60 f i CommentTrack.obj
 0001:0001ff20       ??$__destroy_range_aux@PAUICommentKey@@U1@@stlpmtx_std@@YAXPAUICommentKey@@00ABU__false_type@0@@Z 34020f20 f i CommentTrack.obj
 0001:0001ff70       ?_M_erase@?$_Impl_vector@UICommentKey@@V?$allocator@UICommentKey@@@stlpmtx_std@@@priv@stlpmtx_std@@AAEPAUICommentKey@@PAU4@ABU__false_type@3@@Z 34020f70 f i CommentTrack.obj
 0001:0001fff0       ??$__linear_insert@PAUICommentKey@@U1@U?$less@UICommentKey@@@stlpmtx_std@@@priv@stlpmtx_std@@YAXPAUICommentKey@@0U2@U?$less@UICommentKey@@@1@@Z 34020ff0 f i CommentTrack.obj
 0001:00020080       ??$make_heap@PAUICommentKey@@U?$less@UICommentKey@@@stlpmtx_std@@@stlpmtx_std@@YAXPAUICommentKey@@0U?$less@UICommentKey@@@0@@Z 34021080 f i CommentTrack.obj
 0001:000200f0       ??$__uninitialized_fill_n@PAUICommentKey@@IU1@@priv@stlpmtx_std@@YAPAUICommentKey@@PAU2@IABU2@@Z 340210f0 f i CommentTrack.obj
 0001:00020140       ??$__unguarded_partition@PAUICommentKey@@U1@U?$less@UICommentKey@@@stlpmtx_std@@@priv@stlpmtx_std@@YAPAUICommentKey@@PAU2@0U2@U?$less@UICommentKey@@@1@@Z 34021140 f i CommentTrack.obj
 0001:000201f0       ??$sort_heap@PAUICommentKey@@U?$less@UICommentKey@@@stlpmtx_std@@@stlpmtx_std@@YAXPAUICommentKey@@0U?$less@UICommentKey@@@0@@Z 340211f0 f i CommentTrack.obj
 0001:000202c0       ?_M_fill_insert_aux@?$_Impl_vector@UICommentKey@@V?$allocator@UICommentKey@@@stlpmtx_std@@@priv@stlpmtx_std@@AAEXPAUICommentKey@@IABU4@ABU__false_type@3@@Z 340212c0 f i CommentTrack.obj
 0001:00020480       ??$__final_insertion_sort@PAUICommentKey@@U?$less@UICommentKey@@@stlpmtx_std@@@priv@stlpmtx_std@@YAXPAUICommentKey@@0U?$less@UICommentKey@@@1@@Z 34021480 f i CommentTrack.obj
 0001:00020540       ??$__partial_sort@PAUICommentKey@@U1@U?$less@UICommentKey@@@stlpmtx_std@@@priv@stlpmtx_std@@YAXPAUICommentKey@@000U?$less@UICommentKey@@@1@@Z 34021540 f i CommentTrack.obj
 0001:00020610       ?erase@?$_Impl_vector@UICommentKey@@V?$allocator@UICommentKey@@@stlpmtx_std@@@priv@stlpmtx_std@@QAEPAUICommentKey@@PAU4@0@Z 34021610 f i CommentTrack.obj
 0001:00020670       ?RemoveKey@?$TAnimTrack@UICommentKey@@@@UAEXH@Z 34021670 f i CommentTrack.obj
 0001:000206a0       ?_M_insert_overflow_aux@?$_Impl_vector@UICommentKey@@V?$allocator@UICommentKey@@@stlpmtx_std@@@priv@stlpmtx_std@@AAEXPAUICommentKey@@ABU4@ABU__false_type@3@I_N@Z 340216a0 f i CommentTrack.obj
 0001:00020890       ??1?$TAnimTrack@UICommentKey@@@@UAE@XZ 34021890 f i CommentTrack.obj
 0001:00020910       ??_G?$TAnimTrack@UICommentKey@@@@UAEPAXI@Z 34021910 f i CommentTrack.obj
 0001:00020910       ??_E?$TAnimTrack@UICommentKey@@@@UAEPAXI@Z 34021910 f i CommentTrack.obj
 0001:00020910       ??_GCCommentTrack@@UAEPAXI@Z 34021910 f i CommentTrack.obj
 0001:00020910       ??_ECCommentTrack@@UAEPAXI@Z 34021910 f i CommentTrack.obj
 0001:00020940       ??$__introsort_loop@PAUICommentKey@@U1@HU?$less@UICommentKey@@@stlpmtx_std@@@priv@stlpmtx_std@@YAXPAUICommentKey@@00HU?$less@UICommentKey@@@1@@Z 34021940 f i CommentTrack.obj
 0001:00020a40       ??0CCommentTrack@@QAE@XZ   34021a40 f   CommentTrack.obj
 0001:00020ab0       ??$sort@PAUICommentKey@@@stlpmtx_std@@YAXPAUICommentKey@@0@Z 34021ab0 f i CommentTrack.obj
 0001:00020b10       ?SortKeys@?$TAnimTrack@UICommentKey@@@@UAEXXZ 34021b10 f i CommentTrack.obj
 0001:00020b30       ?resize@?$_Impl_vector@UICommentKey@@V?$allocator@UICommentKey@@@stlpmtx_std@@@priv@stlpmtx_std@@QAEXIABUICommentKey@@@Z 34021b30 f i CommentTrack.obj
 0001:00020bd0       ?SetNumKeys@?$TAnimTrack@UICommentKey@@@@UAEXH@Z 34021bd0 f i CommentTrack.obj
 0001:00020c90       ??4CCryName@@QAEAAV0@PBD@Z 34021c90 f i CompoundSplineTrack.obj
 0001:00020d00       ?SetTimeRange@CCompoundSplineTrack@@UAEXABV?$TRange@M@@@Z 34021d00 f   CompoundSplineTrack.obj
 0001:00020d50       ?GetValue@CCompoundSplineTrack@@UAEXMAAM@Z 34021d50 f   CompoundSplineTrack.obj
 0001:00020da0       ?GetValue@CCompoundSplineTrack@@UAEXMAAU?$Vec3_tpl@M@@@Z 34021da0 f   CompoundSplineTrack.obj
 0001:00020da0       ?GetValue@CCompoundSplineTrack@@QAEXMAAU?$Vec4_tpl@M@@@Z 34021da0 f   CompoundSplineTrack.obj
 0001:00020e00       ?SetValue@CCompoundSplineTrack@@UAEXMABM_N@Z 34021e00 f   CompoundSplineTrack.obj
 0001:00020e40       ?SetValue@CCompoundSplineTrack@@UAEXMABU?$Vec3_tpl@M@@_N@Z 34021e40 f   CompoundSplineTrack.obj
 0001:00020e40       ?SetValue@CCompoundSplineTrack@@QAEXMABU?$Vec4_tpl@M@@_N@Z 34021e40 f   CompoundSplineTrack.obj
 0001:00020e90       ?OffsetKeyPosition@CCompoundSplineTrack@@UAEXABU?$Vec3_tpl@M@@@Z 34021e90 f   CompoundSplineTrack.obj
 0001:00020f40       ?SetSelected@CCompoundSplineTrack@@UAEX_N@Z 34021f40 f   CompoundSplineTrack.obj
 0001:00020f80       ?GetSubTrack@CCompoundSplineTrack@@UBEPAUIAnimTrack@@H@Z 34021f80 f   CompoundSplineTrack.obj
 0001:00020f90       ?GetSubTrackName@CCompoundSplineTrack@@UBEPBDH@Z 34021f90 f   CompoundSplineTrack.obj
 0001:00020fa0       ?GetNumKeys@CCompoundSplineTrack@@UBEHXZ 34021fa0 f   CompoundSplineTrack.obj
 0001:00020fe0       ?GetSubTrackIndex@CCompoundSplineTrack@@IBEHAAH@Z 34021fe0 f   CompoundSplineTrack.obj
 0001:00021040       ?RemoveKey@CCompoundSplineTrack@@UAEXH@Z 34022040 f   CompoundSplineTrack.obj
 0001:00021070       ?GetKeyInfo@CCompoundSplineTrack@@UAEXHAAPBDAAM@Z 34022070 f   CompoundSplineTrack.obj
 0001:00021210       ?GetKeyTime@CCompoundSplineTrack@@UBEMH@Z 34022210 f   CompoundSplineTrack.obj
 0001:00021240       ?SetKeyTime@CCompoundSplineTrack@@UAEXHM@Z 34022240 f   CompoundSplineTrack.obj
 0001:00021270       ?IsKeySelected@CCompoundSplineTrack@@UBE_NH@Z 34022270 f   CompoundSplineTrack.obj
 0001:000212a0       ?SelectKey@CCompoundSplineTrack@@UAEXH_N@Z 340222a0 f   CompoundSplineTrack.obj
 0001:00021340       ?NextKeyByTime@CCompoundSplineTrack@@UBEHH@Z 34022340 f   CompoundSplineTrack.obj
 0001:00021420       ?GetValue@CCompoundSplineTrack@@UAEXMAAU?$Quat_tpl@M@@@Z 34022420 f   CompoundSplineTrack.obj
 0001:000215d0       ?SetValue@CCompoundSplineTrack@@UAEXMABU?$Quat_tpl@M@@_N@Z 340225d0 f   CompoundSplineTrack.obj
 0001:000216e0       ?SetSubTrackName@CCompoundSplineTrack@@UAEXHPBD@Z 340226e0 f   CompoundSplineTrack.obj
 0001:00021720       ?SaveToColladaInFixedFPS@CCompoundSplineTrack@@UAEXABUSColladaExporterSaveProperties@@VXmlNodeRef@@PBD2@Z 34022720 f   CompoundSplineTrack.obj
 0001:000217e0       ??$AddContainer@U?$DynArray@U?$SplineKeyEx@U?$Vec2_tpl@M@@@spline@@HU?$SmallDynStorage@U?$SplineKeyEx@U?$Vec2_tpl@M@@@spline@@HUStandardAlloc@NAlloc@@@NArray@@@@@ICrySizer@@QAE_NABU?$DynArray@U?$SplineKeyEx@U?$Vec2_tpl@M@@@spline@@HU?$SmallDynStorage@U?$SplineKeyEx@U?$Vec2_tpl@M@@@spline@@HUStandardAlloc@NAlloc@@@NArray@@@@@Z 340227e0 f i CompoundSplineTrack.obj
 0001:00021860       ?GetMemoryUsage@?$TSpline@U?$SplineKeyEx@U?$Vec2_tpl@M@@@spline@@VBezierBasis@2@@spline@@UBEXPAVICrySizer@@_N@Z 34022860 f i CompoundSplineTrack.obj
 0001:000218a0       ??_E?$TSpline@U?$SplineKeyEx@U?$Vec2_tpl@M@@@spline@@VBezierBasis@2@@spline@@UAEPAXI@Z 340228a0 f i CompoundSplineTrack.obj
 0001:000218a0       ??_G?$BezierSpline@U?$Vec2_tpl@M@@U?$SplineKeyEx@U?$Vec2_tpl@M@@@spline@@@spline@@UAEPAXI@Z 340228a0 f i CompoundSplineTrack.obj
 0001:000218a0       ??_E?$BezierSpline@U?$Vec2_tpl@M@@U?$SplineKeyEx@U?$Vec2_tpl@M@@@spline@@@spline@@UAEPAXI@Z 340228a0 f i CompoundSplineTrack.obj
 0001:000218a0       ??_G?$TSpline@U?$SplineKeyEx@U?$Vec2_tpl@M@@@spline@@VBezierBasis@2@@spline@@UAEPAXI@Z 340228a0 f i CompoundSplineTrack.obj
 0001:000218f0       ??0?$TSpline@U?$SplineKeyEx@U?$Vec2_tpl@M@@@spline@@VBezierBasis@2@@spline@@QAE@XZ 340228f0 f i CompoundSplineTrack.obj
 0001:00021950       ?comp_deriv@?$BezierSpline@U?$Vec2_tpl@M@@U?$SplineKeyEx@U?$Vec2_tpl@M@@@spline@@@spline@@UAEXXZ 34022950 f i CompoundSplineTrack.obj
 0001:00021be0       ?interp_keys@?$BezierSpline@U?$Vec2_tpl@M@@U?$SplineKeyEx@U?$Vec2_tpl@M@@@spline@@@spline@@MAEXHHMAAU?$Vec2_tpl@M@@@Z 34022be0 f i CompoundSplineTrack.obj
 0001:00021d70       ?assign@?$Array@U?$SplineKeyEx@U?$Vec2_tpl@M@@@spline@@HU?$SmallDynStorage@U?$SplineKeyEx@U?$Vec2_tpl@M@@@spline@@HUStandardAlloc@NAlloc@@@NArray@@@@QAEXU?$Array@$$CBU?$SplineKeyEx@U?$Vec2_tpl@M@@@spline@@HU?$ArrayStorage@$$CBU?$SplineKeyEx@U?$Vec2_tpl@M@@@spline@@H@NArray@@@@@Z 34022d70 f i CompoundSplineTrack.obj
 0001:00021dc0       ??$move_init@U?$SplineKeyEx@U?$Vec2_tpl@M@@@spline@@@NArray@@YAXPAU?$SplineKeyEx@U?$Vec2_tpl@M@@@spline@@0I@Z 34022dc0 f i CompoundSplineTrack.obj
 0001:00021e00       ??$__push_heap@PAU?$SplineKeyEx@U?$Vec2_tpl@M@@@spline@@HU12@U?$less@U?$SplineKeyEx@U?$Vec2_tpl@M@@@spline@@@stlpmtx_std@@@stlpmtx_std@@YAXPAU?$SplineKeyEx@U?$Vec2_tpl@M@@@spline@@HHU12@U?$less@U?$SplineKeyEx@U?$Vec2_tpl@M@@@spline@@@0@@Z 34022e00 f i CompoundSplineTrack.obj
 0001:00021e90       ??$__copy_backward@PAU?$SplineKeyEx@U?$Vec2_tpl@M@@@spline@@PAU12@H@priv@stlpmtx_std@@YAPAU?$SplineKeyEx@U?$Vec2_tpl@M@@@spline@@PAU23@00ABUrandom_access_iterator_tag@1@PAH@Z 34022e90 f i CompoundSplineTrack.obj
 0001:00021f80       ?seek_key@?$TSpline@U?$SplineKeyEx@U?$Vec2_tpl@M@@@spline@@VBezierBasis@2@@spline@@IAEHM@Z 34022f80 f i CompoundSplineTrack.obj
 0001:00021ff0       ?init@?$DynArray@U?$SplineKeyEx@U?$Vec2_tpl@M@@@spline@@HU?$SmallDynStorage@U?$SplineKeyEx@U?$Vec2_tpl@M@@@spline@@HUStandardAlloc@NAlloc@@@NArray@@@@KAPAU?$SplineKeyEx@U?$Vec2_tpl@M@@@spline@@U?$Array@U?$SplineKeyEx@U?$Vec2_tpl@M@@@spline@@HU?$ArrayStorage@U?$SplineKeyEx@U?$Vec2_tpl@M@@@spline@@H@NArray@@@@PBU23@@Z 34022ff0 f i CompoundSplineTrack.obj
 0001:00022040       ??$__unguarded_insertion_sort_aux@PAU?$SplineKeyEx@U?$Vec2_tpl@M@@@spline@@U12@U?$less@U?$SplineKeyEx@U?$Vec2_tpl@M@@@spline@@@stlpmtx_std@@@priv@stlpmtx_std@@YAXPAU?$SplineKeyEx@U?$Vec2_tpl@M@@@spline@@00U?$less@U?$SplineKeyEx@U?$Vec2_tpl@M@@@spline@@@1@@Z 34023040 f i CompoundSplineTrack.obj
 0001:000220c0       ??$__adjust_heap@PAU?$SplineKeyEx@U?$Vec2_tpl@M@@@spline@@HU12@U?$less@U?$SplineKeyEx@U?$Vec2_tpl@M@@@spline@@@stlpmtx_std@@@stlpmtx_std@@YAXPAU?$SplineKeyEx@U?$Vec2_tpl@M@@@spline@@HHU12@U?$less@U?$SplineKeyEx@U?$Vec2_tpl@M@@@spline@@@0@@Z 340230c0 f i CompoundSplineTrack.obj
 0001:00022180       ?FindKeysInRange@?$CBaseSplineInterpolator@U?$Vec2_tpl@M@@V?$BezierSpline@U?$Vec2_tpl@M@@U?$SplineKeyEx@U?$Vec2_tpl@M@@@spline@@@spline@@@spline@@UAEXMMAAH0@Z 34023180 f i CompoundSplineTrack.obj
 0001:000222b0       ?GetKeyCount@?$CBaseSplineInterpolator@U?$Quat_tpl@M@@VTCBQuatSpline@spline@@@spline@@UAEHXZ 340232b0 f i Movie.obj
 0001:000222b0       ?GetKeyCount@?$CBaseSplineInterpolator@U?$Vec2_tpl@M@@V?$BezierSpline@U?$Vec2_tpl@M@@U?$SplineKeyEx@U?$Vec2_tpl@M@@@spline@@@spline@@@spline@@UAEHXZ 340232b0 f i CompoundSplineTrack.obj
 0001:000222b0       ?GetKeyCount@?$CBaseSplineInterpolator@MV?$TCBSpline@MU?$TCBSplineKeyEx@M@spline@@@spline@@@spline@@UAEHXZ 340232b0 f i Movie.obj
 0001:000222b0       ?GetKeyCount@?$CBaseSplineInterpolator@U?$Vec3_tpl@M@@V?$TCBSpline@U?$Vec3_tpl@M@@U?$TCBSplineKeyEx@U?$Vec3_tpl@M@@@spline@@@spline@@@spline@@UAEHXZ 340232b0 f i Movie.obj
 0001:000222c0       ?GetKeyTime@?$CBaseSplineInterpolator@U?$Vec2_tpl@M@@V?$BezierSpline@U?$Vec2_tpl@M@@U?$SplineKeyEx@U?$Vec2_tpl@M@@@spline@@@spline@@@spline@@UAEMH@Z 340232c0 f i CompoundSplineTrack.obj
 0001:000222f0       ?SetKeyTangents@?$CBaseSplineInterpolator@U?$Vec2_tpl@M@@V?$BezierSpline@U?$Vec2_tpl@M@@U?$SplineKeyEx@U?$Vec2_tpl@M@@@spline@@@spline@@@spline@@UAEXHQAM0@Z 340232f0 f i CompoundSplineTrack.obj
 0001:00022340       ?GetKeyTangents@?$CBaseSplineInterpolator@U?$Vec2_tpl@M@@V?$BezierSpline@U?$Vec2_tpl@M@@U?$SplineKeyEx@U?$Vec2_tpl@M@@@spline@@@spline@@@spline@@UAE_NHAAY03M0@Z 34023340 f i CompoundSplineTrack.obj
 0001:00022390       ?GetKeyFlags@?$CBaseSplineInterpolator@U?$Vec2_tpl@M@@V?$BezierSpline@U?$Vec2_tpl@M@@U?$SplineKeyEx@U?$Vec2_tpl@M@@@spline@@@spline@@@spline@@UAEHH@Z 34023390 f i CompoundSplineTrack.obj
 0001:000223c0       ?set_size@?$SmallDynStorage@U?$SplineKeyEx@U?$Vec2_tpl@M@@@spline@@HUStandardAlloc@NAlloc@@@NArray@@QAEXH@Z 340233c0 f i CompoundSplineTrack.obj
 0001:00022450       ?resize_raw@?$SmallDynStorage@U?$SplineKeyEx@U?$Vec2_tpl@M@@@spline@@HUStandardAlloc@NAlloc@@@NArray@@QAEXHH_N@Z 34023450 f i CompoundSplineTrack.obj
 0001:000225b0       ?expand_raw@?$DynArray@U?$SplineKeyEx@U?$Vec2_tpl@M@@@spline@@HU?$SmallDynStorage@U?$SplineKeyEx@U?$Vec2_tpl@M@@@spline@@HUStandardAlloc@NAlloc@@@NArray@@@@IAEPAU?$SplineKeyEx@U?$Vec2_tpl@M@@@spline@@PAU23@H@Z 340235b0 f i CompoundSplineTrack.obj
 0001:00022640       ??$__make_heap@PAU?$SplineKeyEx@U?$Vec2_tpl@M@@@spline@@U?$less@U?$SplineKeyEx@U?$Vec2_tpl@M@@@spline@@@stlpmtx_std@@U12@H@stlpmtx_std@@YAXPAU?$SplineKeyEx@U?$Vec2_tpl@M@@@spline@@0U?$less@U?$SplineKeyEx@U?$Vec2_tpl@M@@@spline@@@0@0PAH@Z 34023640 f i CompoundSplineTrack.obj
 0001:00022760       ?insert_raw@?$DynArray@U?$SplineKeyEx@U?$Vec2_tpl@M@@@spline@@HU?$SmallDynStorage@U?$SplineKeyEx@U?$Vec2_tpl@M@@@spline@@HUStandardAlloc@NAlloc@@@NArray@@@@QAE?AU?$Array@U?$SplineKeyEx@U?$Vec2_tpl@M@@@spline@@HU?$ArrayStorage@U?$SplineKeyEx@U?$Vec2_tpl@M@@@spline@@H@NArray@@@@PAU?$SplineKeyEx@U?$Vec2_tpl@M@@@spline@@H@Z 34023760 f i CompoundSplineTrack.obj
 0001:00022820       ??$__unguarded_partition@PAU?$SplineKeyEx@U?$Vec2_tpl@M@@@spline@@U12@U?$less@U?$SplineKeyEx@U?$Vec2_tpl@M@@@spline@@@stlpmtx_std@@@priv@stlpmtx_std@@YAPAU?$SplineKeyEx@U?$Vec2_tpl@M@@@spline@@PAU23@0U23@U?$less@U?$SplineKeyEx@U?$Vec2_tpl@M@@@spline@@@1@@Z 34023820 f i CompoundSplineTrack.obj
 0001:000228a0       ?erase@?$DynArray@U?$SplineKeyEx@U?$Vec2_tpl@M@@@spline@@HU?$SmallDynStorage@U?$SplineKeyEx@U?$Vec2_tpl@M@@@spline@@HUStandardAlloc@NAlloc@@@NArray@@@@QAEPAU?$SplineKeyEx@U?$Vec2_tpl@M@@@spline@@PAU23@0@Z 340238a0 f i CompoundSplineTrack.obj
 0001:000229f0       ??$sort_heap@PAU?$SplineKeyEx@U?$Vec2_tpl@M@@@spline@@U?$less@U?$SplineKeyEx@U?$Vec2_tpl@M@@@spline@@@stlpmtx_std@@@stlpmtx_std@@YAXPAU?$SplineKeyEx@U?$Vec2_tpl@M@@@spline@@0U?$less@U?$SplineKeyEx@U?$Vec2_tpl@M@@@spline@@@0@@Z 340239f0 f i CompoundSplineTrack.obj
 0001:00022ab0       ??4?$DynArray@U?$SplineKeyEx@U?$Vec2_tpl@M@@@spline@@HU?$SmallDynStorage@U?$SplineKeyEx@U?$Vec2_tpl@M@@@spline@@HUStandardAlloc@NAlloc@@@NArray@@@@QAEAAU0@U?$Array@$$CBU?$SplineKeyEx@U?$Vec2_tpl@M@@@spline@@HU?$ArrayStorage@$$CBU?$SplineKeyEx@U?$Vec2_tpl@M@@@spline@@H@NArray@@@@@Z 34023ab0 f i CompoundSplineTrack.obj
 0001:00022b50       ??0?$DynArray@U?$SplineKeyEx@U?$Vec2_tpl@M@@@spline@@HU?$SmallDynStorage@U?$SplineKeyEx@U?$Vec2_tpl@M@@@spline@@HUStandardAlloc@NAlloc@@@NArray@@@@QAE@ABU0@@Z 34023b50 f i CompoundSplineTrack.obj
 0001:00022c00       ??$__insertion_sort@PAU?$SplineKeyEx@U?$Vec2_tpl@M@@@spline@@U12@U?$less@U?$SplineKeyEx@U?$Vec2_tpl@M@@@spline@@@stlpmtx_std@@@priv@stlpmtx_std@@YAXPAU?$SplineKeyEx@U?$Vec2_tpl@M@@@spline@@00U?$less@U?$SplineKeyEx@U?$Vec2_tpl@M@@@spline@@@1@@Z 34023c00 f i CompoundSplineTrack.obj
 0001:00022ce0       ??$__partial_sort@PAU?$SplineKeyEx@U?$Vec2_tpl@M@@@spline@@U12@U?$less@U?$SplineKeyEx@U?$Vec2_tpl@M@@@spline@@@stlpmtx_std@@@priv@stlpmtx_std@@YAXPAU?$SplineKeyEx@U?$Vec2_tpl@M@@@spline@@000U?$less@U?$SplineKeyEx@U?$Vec2_tpl@M@@@spline@@@1@@Z 34023ce0 f i CompoundSplineTrack.obj
 0001:00022da0       ?RemoveKey@?$CBaseSplineInterpolator@U?$Vec2_tpl@M@@V?$BezierSpline@U?$Vec2_tpl@M@@U?$SplineKeyEx@U?$Vec2_tpl@M@@@spline@@@spline@@@spline@@UAEXH@Z 34023da0 f i CompoundSplineTrack.obj
 0001:00022df0       ?RemoveKeysInRange@?$CBaseSplineInterpolator@U?$Vec2_tpl@M@@V?$BezierSpline@U?$Vec2_tpl@M@@U?$SplineKeyEx@U?$Vec2_tpl@M@@@spline@@@spline@@@spline@@UAEXMM@Z 34023df0 f i CompoundSplineTrack.obj
 0001:00022f30       ??$__final_insertion_sort@PAU?$SplineKeyEx@U?$Vec2_tpl@M@@@spline@@U?$less@U?$SplineKeyEx@U?$Vec2_tpl@M@@@spline@@@stlpmtx_std@@@priv@stlpmtx_std@@YAXPAU?$SplineKeyEx@U?$Vec2_tpl@M@@@spline@@0U?$less@U?$SplineKeyEx@U?$Vec2_tpl@M@@@spline@@@1@@Z 34023f30 f i CompoundSplineTrack.obj
 0001:00022fa0       ?InsertKey@?$CBaseSplineInterpolator@U?$Vec2_tpl@M@@V?$BezierSpline@U?$Vec2_tpl@M@@U?$SplineKeyEx@U?$Vec2_tpl@M@@@spline@@@spline@@@spline@@UAEHMQAM@Z 34023fa0 f i CompoundSplineTrack.obj
 0001:00023100       ??$__introsort_loop@PAU?$SplineKeyEx@U?$Vec2_tpl@M@@@spline@@U12@HU?$less@U?$SplineKeyEx@U?$Vec2_tpl@M@@@spline@@@stlpmtx_std@@@priv@stlpmtx_std@@YAXPAU?$SplineKeyEx@U?$Vec2_tpl@M@@@spline@@00HU?$less@U?$SplineKeyEx@U?$Vec2_tpl@M@@@spline@@@1@@Z 34024100 f i CompoundSplineTrack.obj
 0001:00023200       ??0?$SSplineBackup@V?$BezierSpline@U?$Vec2_tpl@M@@U?$SplineKeyEx@U?$Vec2_tpl@M@@@spline@@@spline@@@spline@@QAE@ABV?$BezierSpline@U?$Vec2_tpl@M@@U?$SplineKeyEx@U?$Vec2_tpl@M@@@spline@@@1@@Z 34024200 f i CompoundSplineTrack.obj
 0001:00023270       ?AddRef@?$SSplineBackup@V?$TCBSpline@U?$Vec3_tpl@M@@U?$TCBSplineKeyEx@U?$Vec3_tpl@M@@@spline@@@spline@@@spline@@UAEXXZ 34024270 f i Movie.obj
 0001:00023270       ?AddRef@?$SSplineBackup@V?$BezierSpline@U?$Vec2_tpl@M@@U?$SplineKeyEx@U?$Vec2_tpl@M@@@spline@@@spline@@@spline@@UAEXXZ 34024270 f i CompoundSplineTrack.obj
 0001:00023270       ?AddRef@?$SSplineBackup@VTCBQuatSpline@spline@@@spline@@UAEXXZ 34024270 f i Movie.obj
 0001:00023270       ?AddRef@?$SSplineBackup@V?$TCBSpline@MU?$TCBSplineKeyEx@M@spline@@@spline@@@spline@@UAEXXZ 34024270 f i Movie.obj
 0001:00023280       ??_E?$SSplineBackup@V?$BezierSpline@U?$Vec2_tpl@M@@U?$SplineKeyEx@U?$Vec2_tpl@M@@@spline@@@spline@@@spline@@W3AEPAXI@Z 34024280 f i CompoundSplineTrack.obj
 0001:00023290       ??_E?$SSplineBackup@V?$BezierSpline@U?$Vec2_tpl@M@@U?$SplineKeyEx@U?$Vec2_tpl@M@@@spline@@@spline@@@spline@@UAEPAXI@Z 34024290 f i CompoundSplineTrack.obj
 0001:00023290       ??_G?$SSplineBackup@V?$BezierSpline@U?$Vec2_tpl@M@@U?$SplineKeyEx@U?$Vec2_tpl@M@@@spline@@@spline@@@spline@@UAEPAXI@Z 34024290 f i CompoundSplineTrack.obj
 0001:000232f0       ??$sort@PAU?$SplineKeyEx@U?$Vec2_tpl@M@@@spline@@@stlpmtx_std@@YAXPAU?$SplineKeyEx@U?$Vec2_tpl@M@@@spline@@0@Z 340242f0 f i CompoundSplineTrack.obj
 0001:00023350       ?Backup@?$CBaseSplineInterpolator@U?$Vec2_tpl@M@@V?$BezierSpline@U?$Vec2_tpl@M@@U?$SplineKeyEx@U?$Vec2_tpl@M@@@spline@@@spline@@@spline@@UAEPAUISplineBackup@@XZ 34024350 f i CompoundSplineTrack.obj
 0001:00023390       ?Restore@?$CBaseSplineInterpolator@U?$Vec2_tpl@M@@V?$BezierSpline@U?$Vec2_tpl@M@@U?$SplineKeyEx@U?$Vec2_tpl@M@@@spline@@@spline@@@spline@@UAEXPAUISplineBackup@@@Z 34024390 f i CompoundSplineTrack.obj
 0001:000233f0       ??_E?$TrackSplineInterpolator@U?$Vec2_tpl@M@@@spline@@W3AEPAXI@Z 340243f0 f i CompoundSplineTrack.obj
 0001:00023400       ?ComputeThetaAndScale@?$SplineKeyEx@U?$Vec2_tpl@M@@@spline@@QAEXXZ 34024400 f i CompoundSplineTrack.obj
 0001:00023510       ?SetOutTangentFromIn@?$SplineKeyEx@U?$Vec2_tpl@M@@@spline@@QAEXXZ 34024510 f i CompoundSplineTrack.obj
 0001:00023640       ?SetInTangentFromOut@?$SplineKeyEx@U?$Vec2_tpl@M@@@spline@@QAEXXZ 34024640 f i CompoundSplineTrack.obj
 0001:00023770       ?comp_time_deriv@?$TrackSplineInterpolator@U?$Vec2_tpl@M@@@spline@@ABEMHHM@Z 34024770 f i CompoundSplineTrack.obj
 0001:00023810       ?comp_value_deriv@?$TrackSplineInterpolator@U?$Vec2_tpl@M@@@spline@@ABEMHHM@Z 34024810 f i CompoundSplineTrack.obj
 0001:000238b0       ?ConstrainOutTangentsOf@?$TrackSplineInterpolator@U?$Vec2_tpl@M@@@spline@@QAEXH@Z 340248b0 f i CompoundSplineTrack.obj
 0001:00023920       ?SetKeyTime@?$TrackSplineInterpolator@U?$Vec2_tpl@M@@@spline@@UAEXHM@Z 34024920 f i CompoundSplineTrack.obj
 0001:000239a0       ?SetKeyValue@?$TrackSplineInterpolator@U?$Vec2_tpl@M@@@spline@@UAEXHQAM@Z 340249a0 f i CompoundSplineTrack.obj
 0001:00023a00       ?GetKeyValue@?$TrackSplineInterpolator@U?$Vec2_tpl@M@@@spline@@UAE_NHAAY03M@Z 34024a00 f i CompoundSplineTrack.obj
 0001:00023a50       ?SetKeyFlags@?$TrackSplineInterpolator@U?$Vec2_tpl@M@@@spline@@UAEXHH@Z 34024a50 f i CompoundSplineTrack.obj
 0001:00023ac0       ?SetKeyInTangent@?$TrackSplineInterpolator@U?$Vec2_tpl@M@@@spline@@UAEXHQAM@Z 34024ac0 f i CompoundSplineTrack.obj
 0001:00023b30       ?SetKeyOutTangent@?$TrackSplineInterpolator@U?$Vec2_tpl@M@@@spline@@UAEXHQAM@Z 34024b30 f i CompoundSplineTrack.obj
 0001:00023bf0       ?comp_deriv@?$TrackSplineInterpolator@U?$Vec2_tpl@M@@@spline@@UAEXXZ 34024bf0 f i CompoundSplineTrack.obj
 0001:00023ef0       ??_E?$TrackSplineInterpolator@U?$Vec2_tpl@M@@@spline@@UAEPAXI@Z 34024ef0 f i CompoundSplineTrack.obj
 0001:00023ef0       ??_G?$TrackSplineInterpolator@U?$Vec2_tpl@M@@@spline@@UAEPAXI@Z 34024ef0 f i CompoundSplineTrack.obj
 0001:00023f50       ?interpolate@?$TSpline@U?$SplineKeyEx@U?$Vec2_tpl@M@@@spline@@VBezierBasis@2@@spline@@QAE_NMAAU?$Vec2_tpl@M@@@Z 34024f50 f i CompoundSplineTrack.obj
 0001:00024080       ??0?$TAnimSplineTrack@U?$Vec2_tpl@M@@@@QAE@XZ 34025080 f i CompoundSplineTrack.obj
 0001:00024100       ?GetValue@?$TAnimSplineTrack@U?$Vec2_tpl@M@@@@UAEXMAAM@Z 34025100 f i CompoundSplineTrack.obj
 0001:00024150       ?CreateKey@?$TAnimSplineTrack@U?$Vec2_tpl@M@@@@UAEHM@Z 34025150 f i CompoundSplineTrack.obj
 0001:000241c0       ?GetKeyValueRange@?$TAnimSplineTrack@U?$Vec2_tpl@M@@@@UBEXAAM0@Z 340251c0 f i CompoundSplineTrack.obj
 0001:000241e0       ?SetKeyValueRange@?$TAnimSplineTrack@U?$Vec2_tpl@M@@@@UAEXMM@Z 340251e0 f i CompoundSplineTrack.obj
 0001:00024200       ?IsKeySelected@?$TAnimSplineTrack@U?$Quat_tpl@M@@@@UBE_NH@Z 34025200 f i Movie.obj
 0001:00024200       ?IsKeySelected@?$TAnimSplineTrack@U?$Vec2_tpl@M@@@@UBE_NH@Z 34025200 f i CompoundSplineTrack.obj
 0001:00024200       ?IsKeySelected@?$TAnimSplineTrack@M@@UBE_NH@Z 34025200 f i Movie.obj
 0001:00024200       ?IsKeySelected@?$TAnimSplineTrack@U?$Vec3_tpl@M@@@@UBE_NH@Z 34025200 f i Movie.obj
 0001:00024260       ?SelectKey@?$TAnimSplineTrack@U?$Vec3_tpl@M@@@@UAEXH_N@Z 34025260 f i Movie.obj
 0001:00024260       ?SelectKey@?$TAnimSplineTrack@M@@UAEXH_N@Z 34025260 f i Movie.obj
 0001:00024260       ?SelectKey@?$TAnimSplineTrack@U?$Vec2_tpl@M@@@@UAEXH_N@Z 34025260 f i CompoundSplineTrack.obj
 0001:00024260       ?SelectKey@?$TAnimSplineTrack@U?$Quat_tpl@M@@@@UAEXH_N@Z 34025260 f i Movie.obj
 0001:000242a0       ?SetSelected@?$TAnimSplineTrack@U?$Vec2_tpl@M@@@@UAEX_N@Z 340252a0 f i CompoundSplineTrack.obj
 0001:000242c0       ?GetFlags@?$TAnimSplineTrack@U?$Vec2_tpl@M@@@@UAEHXZ 340252c0 f i CompoundSplineTrack.obj
 0001:000242c0       ?GetNodeOwner@CAnimNode@@UAEPAUIAnimNodeOwner@@XZ 340252c0 f i AnimLightNode.obj
 0001:000242d0       ?GetCustomColor@?$TAnimSplineTrack@U?$Vec2_tpl@M@@@@UBE?AU?$Color_tpl@E@@XZ 340252d0 f i CompoundSplineTrack.obj
 0001:000242e0       ?HasCustomColor@?$TAnimSplineTrack@U?$Vec2_tpl@M@@@@UBE_NXZ 340252e0 f i CompoundSplineTrack.obj
 0001:000242f0       ?ClearCustomColor@?$TAnimSplineTrack@U?$Vec2_tpl@M@@@@UAEXXZ 340252f0 f i CompoundSplineTrack.obj
 0001:00024300       ?CryLog@@YAXPBDZZ          34025300 f i CompoundSplineTrack.obj
 0001:00024330       ??$__fill@PAMMH@priv@stlpmtx_std@@YAXPAM0ABMABUrandom_access_iterator_tag@1@PAH@Z 34025330 f i CompoundSplineTrack.obj
 0001:00024390       ?GetParameterType@?$TAnimSplineTrack@U?$Vec2_tpl@M@@@@UBE?AVAnimParamType@@XZ 34025390 f i CompoundSplineTrack.obj
 0001:000243b0       ?SetParameterType@?$TAnimSplineTrack@U?$Vec2_tpl@M@@@@UAEXVAnimParamType@@@Z 340253b0 f i CompoundSplineTrack.obj
 0001:00024420       ?SetFlags@?$TAnimSplineTrack@U?$Vec2_tpl@M@@@@UAEXH@Z 34025420 f i CompoundSplineTrack.obj
 0001:00024460       ?SetDefaultValue@?$TAnimSplineTrack@U?$Vec2_tpl@M@@@@UAEXABU?$Vec2_tpl@M@@@Z 34025460 f i CompoundSplineTrack.obj
 0001:00024480       ?SetCustomColor@?$TAnimSplineTrack@U?$Vec2_tpl@M@@@@UAEXU?$Color_tpl@E@@@Z 34025480 f i CompoundSplineTrack.obj
 0001:000244b0       ??$?9D@@YA_NABV?$CryStringT@D@@PBD@Z 340254b0 f i CompoundSplineTrack.obj
 0001:00024500       ?CopyKey@?$TAnimSplineTrack@U?$Vec2_tpl@M@@@@UAEHPAUIAnimTrack@@H@Z 34025500 f i CompoundSplineTrack.obj
 0001:00024580       ?GetKeyTime@?$TAnimSplineTrack@U?$Vec2_tpl@M@@@@UBEMH@Z 34025580 f i CompoundSplineTrack.obj
 0001:000245a0       ?SetKeyTime@?$TAnimSplineTrack@U?$Quat_tpl@M@@@@UAEXHM@Z 340255a0 f i Movie.obj
 0001:000245a0       ?SetKeyTime@?$TAnimSplineTrack@U?$Vec3_tpl@M@@@@UAEXHM@Z 340255a0 f i Movie.obj
 0001:000245a0       ?SetKeyTime@?$TAnimSplineTrack@U?$Vec2_tpl@M@@@@UAEXHM@Z 340255a0 f i CompoundSplineTrack.obj
 0001:000245a0       ?SetKeyTime@?$TAnimSplineTrack@M@@UAEXHM@Z 340255a0 f i Movie.obj
 0001:000245d0       ?GetKeyFlags@?$TAnimSplineTrack@U?$Vec2_tpl@M@@@@UAEHH@Z 340255d0 f i CompoundSplineTrack.obj
 0001:000245f0       ?SetKeyFlags@?$TAnimSplineTrack@U?$Vec2_tpl@M@@@@UAEXHH@Z 340255f0 f i CompoundSplineTrack.obj
 0001:00024610       ?FindKey@?$TAnimSplineTrack@U?$Vec2_tpl@M@@@@UAEHM@Z 34025610 f i CompoundSplineTrack.obj
 0001:00024660       ?SetKeyAtTime@?$TAnimSplineTrack@U?$Vec2_tpl@M@@@@QAEXMPAUIKey@@@Z 34025660 f i CompoundSplineTrack.obj
 0001:00024700       ?GetMemoryUsage@?$TAnimSplineTrack@U?$Vec2_tpl@M@@@@UBEXPAVICrySizer@@@Z 34025700 f i CompoundSplineTrack.obj
 0001:00024740       ?init@?$DynArray@U?$SplineKeyEx@U?$Vec2_tpl@M@@@spline@@HU?$SmallDynStorage@U?$SplineKeyEx@U?$Vec2_tpl@M@@@spline@@HUStandardAlloc@NAlloc@@@NArray@@@@KAPAU?$SplineKeyEx@U?$Vec2_tpl@M@@@spline@@U?$Array@U?$SplineKeyEx@U?$Vec2_tpl@M@@@spline@@HU?$ArrayStorage@U?$SplineKeyEx@U?$Vec2_tpl@M@@@spline@@H@NArray@@@@@Z 34025740 f i CompoundSplineTrack.obj
 0001:000247a0       ?SetValue@?$TAnimSplineTrack@U?$Vec2_tpl@M@@@@UAEXMABM_N@Z 340257a0 f i CompoundSplineTrack.obj
 0001:00024800       ?GetKey@?$TAnimSplineTrack@U?$Vec2_tpl@M@@@@UBEXHPAUIKey@@@Z 34025800 f i CompoundSplineTrack.obj
 0001:00024830       ?SetKey@?$TAnimSplineTrack@U?$Vec2_tpl@M@@@@UAEXHPAUIKey@@@Z 34025830 f i CompoundSplineTrack.obj
 0001:00024870       ?Serialize@?$TAnimSplineTrack@U?$Vec2_tpl@M@@@@UAE_NAAVXmlNodeRef@@_N1@Z 34025870 f i CompoundSplineTrack.obj
 0001:00024bf0       ?SerializeSelection@?$TAnimSplineTrack@U?$Vec2_tpl@M@@@@UAE_NAAVXmlNodeRef@@_N1M@Z 34025bf0 f i CompoundSplineTrack.obj
 0001:00024eb0       ??_E?$TAnimSplineTrack@U?$Vec2_tpl@M@@@@UAEPAXI@Z 34025eb0 f i CompoundSplineTrack.obj
 0001:00024eb0       ??_G?$TAnimSplineTrack@U?$Vec2_tpl@M@@@@UAEPAXI@Z 34025eb0 f i CompoundSplineTrack.obj
 0001:00024f10       ?GetKeyInfo@?$TAnimSplineTrack@U?$Vec2_tpl@M@@@@UAEXHAAPBDAAM@Z 34025f10 f i CompoundSplineTrack.obj
 0001:00024f60       ?_M_insert_overflow@?$_Impl_vector@MV?$allocator@M@stlpmtx_std@@@priv@stlpmtx_std@@AAEXPAMABMABU__true_type@3@I_N@Z 34025f60 f i CompoundSplineTrack.obj
 0001:000250b0       ?_M_fill_insert_aux@?$_Impl_vector@MV?$allocator@M@stlpmtx_std@@@priv@stlpmtx_std@@AAEXPAMIABMABU__false_type@3@@Z 340260b0 f i CompoundSplineTrack.obj
 0001:000251e0       ?RemoveKey@?$TAnimSplineTrack@U?$Vec2_tpl@M@@@@UAEXH@Z 340261e0 f i CompoundSplineTrack.obj
 0001:00025230       ?resize@?$_Impl_vector@MV?$allocator@M@stlpmtx_std@@@priv@stlpmtx_std@@QAEXIABM@Z 34026230 f i CompoundSplineTrack.obj
 0001:000252d0       ?SetNumKeys@?$TAnimSplineTrack@U?$Vec2_tpl@M@@@@UAEXH@Z 340262d0 f i CompoundSplineTrack.obj
 0001:00025340       ?LoadFromCollada@?$TAnimSplineTrack@U?$Vec2_tpl@M@@@@UAE_NVXmlNodeRef@@@Z 34026340 f i CompoundSplineTrack.obj
 0001:000269c0       ?SortKeys@?$TAnimSplineTrack@U?$Vec2_tpl@M@@@@UAEXXZ 340279c0 f i CompoundSplineTrack.obj
 0001:000269f0       ??0CCompoundSplineTrack@@QAE@HW4EAnimValue@@QAVAnimParamType@@@Z 340279f0 f   CompoundSplineTrack.obj
 0001:00026cc0       ?CopyKey@CCompoundSplineTrack@@UAEHPAUIAnimTrack@@H@Z 34027cc0 f i CompoundSplineTrack.obj
 0001:00026cd0       ?GetSubTrackName@?$TAnimTrack@UIBoolKey@@@@UBEPBDH@Z 34027cd0 f i AnimNode.obj
 0001:00026cd0       ?GetSubTrack@?$TAnimTrack@UICaptureKey@@@@UBEPAUIAnimTrack@@H@Z 34027cd0 f i AnimNode.obj
 0001:00026cd0       ?GetSubTrack@?$TAnimSplineTrack@U?$Vec2_tpl@M@@@@UBEPAUIAnimTrack@@H@Z 34027cd0 f i CompoundSplineTrack.obj
 0001:00026cd0       ?GetSubTrack@?$TAnimTrack@UIConsoleKey@@@@UBEPAUIAnimTrack@@H@Z 34027cd0 f i AnimNode.obj
 0001:00026cd0       ?GetSubTrackName@?$TAnimTrack@UISelectKey@@@@UBEPBDH@Z 34027cd0 f i AnimNode.obj
 0001:00026cd0       ?GetSubTrackName@?$TAnimSplineTrack@U?$Quat_tpl@M@@@@UBEPBDH@Z 34027cd0 f i Movie.obj
 0001:00026cd0       ?GetSubTrackName@?$TAnimTrack@UIExprKey@@@@UBEPBDH@Z 34027cd0 f i AnimNode.obj
 0001:00026cd0       ?GetSubTrackName@?$TAnimSplineTrack@M@@UBEPBDH@Z 34027cd0 f i Movie.obj
 0001:00026cd0       ?GetSubTrack@?$TAnimSplineTrack@U?$Vec3_tpl@M@@@@UBEPAUIAnimTrack@@H@Z 34027cd0 f i Movie.obj
 0001:00026cd0       ?CreateKey@CCompoundSplineTrack@@UAEHM@Z 34027cd0 f i CompoundSplineTrack.obj
 0001:00026cd0       ?QueryComposite@CEngineModule_CryMovie@@MBEPAXPBD@Z 34027cd0 f i CryMovie.obj
 0001:00026cd0       ?GetSubTrack@?$TAnimTrack@UIScreenFaderKey@@@@UBEPAUIAnimTrack@@H@Z 34027cd0 f i ScreenFaderTrack.obj
 0001:00026cd0       ?GetSubTrack@?$TAnimTrack@UIEventKey@@@@UBEPAUIAnimTrack@@H@Z 34027cd0 f i AnimNode.obj
 0001:00026cd0       ?GetSubTrack@?$TAnimTrack@UISelectKey@@@@UBEPAUIAnimTrack@@H@Z 34027cd0 f i AnimNode.obj
 0001:00026cd0       ?GetSubTrack@?$TAnimTrack@UICharacterKey@@@@UBEPAUIAnimTrack@@H@Z 34027cd0 f i AnimNode.obj
 0001:00026cd0       ?GetSubTrack@?$TAnimTrack@UIFaceSeqKey@@@@UBEPAUIAnimTrack@@H@Z 34027cd0 f i AnimNode.obj
 0001:00026cd0       ?GetKeyFlags@CCompoundSplineTrack@@UAEHH@Z 34027cd0 f i CompoundSplineTrack.obj
 0001:00026cd0       ?GetSubTrackName@?$TAnimTrack@UIConsoleKey@@@@UBEPBDH@Z 34027cd0 f i AnimNode.obj
 0001:00026cd0       ?GetSubTrackName@?$TAnimTrack@UICharacterKey@@@@UBEPBDH@Z 34027cd0 f i AnimNode.obj
 0001:00026cd0       ?get_deleter@?$sp_counted_impl_p@VCEngineModule_CryMovie@@@detail@boost@@UAEPAXABVsp_typeinfo@23@@Z 34027cd0 f i CryMovie.obj
 0001:00026cd0       ?GetSubTrack@?$TAnimTrack@UIMusicKey@@@@UBEPAUIAnimTrack@@H@Z 34027cd0 f i AnimNode.obj
 0001:00026cd0       ?GetSubTrack@?$TAnimTrack@UIBoolKey@@@@UBEPAUIAnimTrack@@H@Z 34027cd0 f i AnimNode.obj
 0001:00026cd0       ?GetSubTrack@?$TAnimTrack@UICommentKey@@@@UBEPAUIAnimTrack@@H@Z 34027cd0 f i CommentTrack.obj
 0001:00026cd0       ?GetSubTrackName@?$TAnimTrack@UIScreenFaderKey@@@@UBEPBDH@Z 34027cd0 f i ScreenFaderTrack.obj
 0001:00026cd0       ?FindKey@CCompoundSplineTrack@@UAEHM@Z 34027cd0 f i CompoundSplineTrack.obj
 0001:00026cd0       ?GetSubTrackName@?$TAnimTrack@UICaptureKey@@@@UBEPBDH@Z 34027cd0 f i AnimNode.obj
 0001:00026cd0       ?GetSubTrackName@?$TAnimTrack@UIDiscreteFloatKey@@@@UBEPBDH@Z 34027cd0 f i GotoTrack.obj
 0001:00026cd0       ?GetSubTrackName@?$TAnimTrack@UIEventKey@@@@UBEPBDH@Z 34027cd0 f i AnimNode.obj
 0001:00026cd0       ?GetSubTrackName@?$TAnimTrack@UICommentKey@@@@UBEPBDH@Z 34027cd0 f i CommentTrack.obj
 0001:00026cd0       ?GetSubTrackName@?$TAnimTrack@UILookAtKey@@@@UBEPBDH@Z 34027cd0 f i AnimNode.obj
 0001:00026cd0       ?GetSubTrackName@?$TAnimTrack@UISequenceKey@@@@UBEPBDH@Z 34027cd0 f i AnimNode.obj
 0001:00026cd0       ?GetSubTrackName@?$TAnimTrack@UISoundKey@@@@UBEPBDH@Z 34027cd0 f i AnimNode.obj
 0001:00026cd0       ?GetSubTrack@?$TAnimTrack@UISoundKey@@@@UBEPAUIAnimTrack@@H@Z 34027cd0 f i AnimNode.obj
 0001:00026cd0       ?GetSubTrackName@?$TAnimTrack@UIFaceSeqKey@@@@UBEPBDH@Z 34027cd0 f i AnimNode.obj
 0001:00026cd0       ?GetSubTrackName@?$TAnimSplineTrack@U?$Vec2_tpl@M@@@@UBEPBDH@Z 34027cd0 f i CompoundSplineTrack.obj
 0001:00026cd0       ?CloneKey@CCompoundSplineTrack@@UAEHH@Z 34027cd0 f i CompoundSplineTrack.obj
 0001:00026cd0       ?GetSubTrackName@?$TAnimTrack@UIMusicKey@@@@UBEPBDH@Z 34027cd0 f i AnimNode.obj
 0001:00026cd0       ?GetSubTrack@?$TAnimTrack@UISequenceKey@@@@UBEPAUIAnimTrack@@H@Z 34027cd0 f i AnimNode.obj
 0001:00026cd0       ?GetSubTrack@?$TAnimSplineTrack@U?$Quat_tpl@M@@@@UBEPAUIAnimTrack@@H@Z 34027cd0 f i Movie.obj
 0001:00026cd0       ?GetSubTrack@?$TAnimTrack@UIExprKey@@@@UBEPAUIAnimTrack@@H@Z 34027cd0 f i AnimNode.obj
 0001:00026cd0       ?GetSubTrack@?$TAnimTrack@UIDiscreteFloatKey@@@@UBEPAUIAnimTrack@@H@Z 34027cd0 f i GotoTrack.obj
 0001:00026cd0       ?GetSubTrack@?$TAnimTrack@UILookAtKey@@@@UBEPAUIAnimTrack@@H@Z 34027cd0 f i AnimNode.obj
 0001:00026cd0       ?GetSubTrackName@?$TAnimSplineTrack@U?$Vec3_tpl@M@@@@UBEPBDH@Z 34027cd0 f i Movie.obj
 0001:00026cd0       ?GetSubTrack@?$TAnimSplineTrack@M@@UBEPAUIAnimTrack@@H@Z 34027cd0 f i Movie.obj
 0001:00026ce0       ?SetFlags@CCompoundSplineTrack@@UAEXH@Z 34027ce0 f i CompoundSplineTrack.obj
 0001:00026cf0       ?GetCustomColor@CCompoundSplineTrack@@UBE?AU?$Color_tpl@E@@XZ 34027cf0 f i CompoundSplineTrack.obj
 0001:00026d00       ?HasCustomColor@CCompoundSplineTrack@@UBE_NXZ 34027d00 f i CompoundSplineTrack.obj
 0001:00026d10       ?GetParameterType@CCompoundSplineTrack@@UBE?AVAnimParamType@@XZ 34027d10 f i CompoundSplineTrack.obj
 0001:00026d30       ?SetCustomColor@CCompoundSplineTrack@@UAEXU?$Color_tpl@E@@@Z 34027d30 f i CompoundSplineTrack.obj
 0001:00026d60       ?GetKeyValueRange@CCompoundSplineTrack@@UBEXAAM0@Z 34027d60 f i CompoundSplineTrack.obj
 0001:00026d90       ?SetKeyValueRange@CCompoundSplineTrack@@UAEXMM@Z 34027d90 f i CompoundSplineTrack.obj
 0001:00026dd0       ?SetParameterType@CCompoundSplineTrack@@UAEXVAnimParamType@@@Z 34027dd0 f i CompoundSplineTrack.obj
 0001:00026e40       ?GetMemoryUsage@CCompoundSplineTrack@@UBEXPAVICrySizer@@@Z 34027e40 f i CompoundSplineTrack.obj
 0001:00026ea0       ??1CCompoundSplineTrack@@UAE@XZ 34027ea0 f i CompoundSplineTrack.obj
 0001:00026f30       ??_ECCompoundSplineTrack@@UAEPAXI@Z 34027f30 f i CompoundSplineTrack.obj
 0001:00026f30       ??_GCCompoundSplineTrack@@UAEPAXI@Z 34027f30 f i CompoundSplineTrack.obj
 0001:00026f60       ?PrepareNodeForSubTrackSerialization@CCompoundSplineTrack@@IAEXAAVXmlNodeRef@@0H_N@Z 34027f60 f   CompoundSplineTrack.obj
 0001:00027120       ?Serialize@CCompoundSplineTrack@@UAE_NAAVXmlNodeRef@@_N1@Z 34028120 f   CompoundSplineTrack.obj
 0001:00027240       ?SerializeSelection@CCompoundSplineTrack@@UAE_NAAVXmlNodeRef@@_N1M@Z 34028240 f   CompoundSplineTrack.obj
 0001:000272c0       ?search_u@?$TrackSplineInterpolator@U?$Vec2_tpl@M@@@spline@@AAEMMAAY03M@Z 340282c0 f i CompoundSplineTrack.obj
 0001:000274e0       ?interpolate_tangent@?$TrackSplineInterpolator@U?$Vec2_tpl@M@@@spline@@AAE?AU?$Vec2_tpl@M@@MAAM@Z 340284e0 f i CompoundSplineTrack.obj
 0001:00027570       ?Interpolate@?$TrackSplineInterpolator@U?$Vec2_tpl@M@@@spline@@UAEXMAAY03M@Z 34028570 f i CompoundSplineTrack.obj
 0001:000275f0       ?InsertKey@?$TrackSplineInterpolator@U?$Vec2_tpl@M@@@spline@@UAEHMQAM@Z 340285f0 f i CompoundSplineTrack.obj
 0001:00027980       ?SerializeKey@CConsoleTrack@@UAEXAAUIConsoleKey@@AAVXmlNodeRef@@_N@Z 34028980 f   ConsoleTrack.obj
 0001:000279f0       ?GetKeyInfo@CConsoleTrack@@UAEXHAAPBDAAM@Z 340289f0 f   ConsoleTrack.obj
 0001:00027a50       ?SerializeKey@CEventTrack@@UAEXAAUIEventKey@@AAVXmlNodeRef@@_N@Z 34028a50 f   EventTrack.obj
 0001:00027bb0       ?GetKeyInfo@CEventTrack@@UAEXHAAPBDAAM@Z 34028bb0 f   EventTrack.obj
 0001:00027c80       ?SerializeKey@CExprTrack@@UAEXAAUIExprKey@@AAVXmlNodeRef@@_N@Z 34028c80 f   ExprTrack.obj
 0001:00027db0       ?GetKeyInfo@CExprTrack@@UAEXHAAPBDAAM@Z 34028db0 f   ExprTrack.obj
 0001:00027e30       ?SerializeKey@CFaceSeqTrack@@UAEXAAUIFaceSeqKey@@AAVXmlNodeRef@@_N@Z 34028e30 f   FaceSeqTrack.obj
 0001:00027e90       ?GetKeyInfo@CFaceSeqTrack@@UAEXHAAPBDAAM@Z 34028e90 f   FaceSeqTrack.obj
 0001:00027ef0       ?SerializeKey@CGotoTrack@@UAEXAAUIDiscreteFloatKey@@AAVXmlNodeRef@@_N@Z 34028ef0 f   GotoTrack.obj
 0001:00027f90       ?GetValue@CGotoTrack@@UAEXMAAM@Z 34028f90 f   GotoTrack.obj
 0001:00028060       ?GetKeyInfo@CGotoTrack@@UAEXHAAPBDAAM@Z 34029060 f   GotoTrack.obj
 0001:000280a0       ?SetKeyAtTime@CGotoTrack@@IAEXMPAUIKey@@@Z 340290a0 f   GotoTrack.obj
 0001:00028150       ?SetValue@CGotoTrack@@UAEXMABM_N@Z 34029150 f   GotoTrack.obj
 0001:000281a0       ?CreateKey@?$TAnimTrack@UIDiscreteFloatKey@@@@UAEHM@Z 340291a0 f i GotoTrack.obj
 0001:00028200       ?CloneKey@?$TAnimTrack@UIDiscreteFloatKey@@@@UAEHH@Z 34029200 f i GotoTrack.obj
 0001:00028270       ?CopyKey@?$TAnimTrack@UIDiscreteFloatKey@@@@UAEHPAUIAnimTrack@@H@Z 34029270 f i GotoTrack.obj
 0001:000282e0       ??$fill@PAUIDiscreteFloatKey@@U1@@stlpmtx_std@@YAXPAUIDiscreteFloatKey@@0ABU1@@Z 340292e0 f i GotoTrack.obj
 0001:00028320       ??$__push_heap@PAUIDiscreteFloatKey@@HU1@U?$less@UIDiscreteFloatKey@@@stlpmtx_std@@@stlpmtx_std@@YAXPAUIDiscreteFloatKey@@HHU1@U?$less@UIDiscreteFloatKey@@@0@@Z 34029320 f i GotoTrack.obj
 0001:00028390       ?GetNumKeys@?$TAnimTrack@UIDiscreteFloatKey@@@@UBEHXZ 34029390 f i GotoTrack.obj
 0001:000283b0       ?GetKey@?$TAnimTrack@UIDiscreteFloatKey@@@@UBEXHPAUIKey@@@Z 340293b0 f i GotoTrack.obj
 0001:000283e0       ?GetKeyTime@?$TAnimTrack@UIDiscreteFloatKey@@@@UBEMH@Z 340293e0 f i GotoTrack.obj
 0001:00028400       ?FindKey@?$TAnimTrack@UIDiscreteFloatKey@@@@UAEHM@Z 34029400 f i GotoTrack.obj
 0001:00028460       ?GetKeyFlags@?$TAnimTrack@UIDiscreteFloatKey@@@@UAEHH@Z 34029460 f i GotoTrack.obj
 0001:00028480       ?SetKey@?$TAnimTrack@UIDiscreteFloatKey@@@@UAEXHPAUIKey@@@Z 34029480 f i GotoTrack.obj
 0001:000284b0       ?SetKeyTime@?$TAnimTrack@UIDiscreteFloatKey@@@@UAEXHM@Z 340294b0 f i GotoTrack.obj
 0001:000284d0       ?SetKeyFlags@?$TAnimTrack@UIDiscreteFloatKey@@@@UAEXHH@Z 340294d0 f i GotoTrack.obj
 0001:000284f0       ?Serialize@?$TAnimTrack@UIDiscreteFloatKey@@@@UAE_NAAVXmlNodeRef@@_N1@Z 340294f0 f i GotoTrack.obj
 0001:000287a0       ?SerializeSelection@?$TAnimTrack@UIDiscreteFloatKey@@@@UAE_NAAVXmlNodeRef@@_N1M@Z 340297a0 f i GotoTrack.obj
 0001:00028970       ??$__unguarded_insertion_sort_aux@PAUIDiscreteFloatKey@@U1@U?$less@UIDiscreteFloatKey@@@stlpmtx_std@@@priv@stlpmtx_std@@YAXPAUIDiscreteFloatKey@@00U?$less@UIDiscreteFloatKey@@@1@@Z 34029970 f i GotoTrack.obj
 0001:000289e0       ??$__adjust_heap@PAUIDiscreteFloatKey@@HU1@U?$less@UIDiscreteFloatKey@@@stlpmtx_std@@@stlpmtx_std@@YAXPAUIDiscreteFloatKey@@HHU1@U?$less@UIDiscreteFloatKey@@@0@@Z 340299e0 f i GotoTrack.obj
 0001:00028a90       ?IsKeySelected@?$TAnimTrack@UIDiscreteFloatKey@@@@UBE_NH@Z 34029a90 f i GotoTrack.obj
 0001:00028ab0       ?SelectKey@?$TAnimTrack@UIDiscreteFloatKey@@@@UAEXH_N@Z 34029ab0 f i GotoTrack.obj
 0001:00028af0       ??$__uninitialized_fill_n@PAUIDiscreteFloatKey@@IU1@@priv@stlpmtx_std@@YAPAUIDiscreteFloatKey@@PAU2@IABU2@@Z 34029af0 f i GotoTrack.obj
 0001:00028b50       ??$__unguarded_partition@PAUIDiscreteFloatKey@@U1@U?$less@UIDiscreteFloatKey@@@stlpmtx_std@@@priv@stlpmtx_std@@YAPAUIDiscreteFloatKey@@PAU2@0U2@U?$less@UIDiscreteFloatKey@@@1@@Z 34029b50 f i GotoTrack.obj
 0001:00028bb0       ??$__make_heap@PAUIDiscreteFloatKey@@U?$less@UIDiscreteFloatKey@@@stlpmtx_std@@U1@H@stlpmtx_std@@YAXPAUIDiscreteFloatKey@@0U?$less@UIDiscreteFloatKey@@@0@0PAH@Z 34029bb0 f i GotoTrack.obj
 0001:00028cc0       ?_M_insert_overflow@?$_Impl_vector@UIDiscreteFloatKey@@V?$allocator@UIDiscreteFloatKey@@@stlpmtx_std@@@priv@stlpmtx_std@@AAEXPAUIDiscreteFloatKey@@ABU4@ABU__true_type@3@I_N@Z 34029cc0 f i GotoTrack.obj
 0001:00028e40       ?_M_fill_insert_aux@?$_Impl_vector@UIDiscreteFloatKey@@V?$allocator@UIDiscreteFloatKey@@@stlpmtx_std@@@priv@stlpmtx_std@@AAEXPAUIDiscreteFloatKey@@IABU4@ABU__false_type@3@@Z 34029e40 f i GotoTrack.obj
 0001:00028f60       ??$__insertion_sort@PAUIDiscreteFloatKey@@U1@U?$less@UIDiscreteFloatKey@@@stlpmtx_std@@@priv@stlpmtx_std@@YAXPAUIDiscreteFloatKey@@00U?$less@UIDiscreteFloatKey@@@1@@Z 34029f60 f i GotoTrack.obj
 0001:00029030       ?RemoveKey@?$TAnimTrack@UIDiscreteFloatKey@@@@UAEXH@Z 3402a030 f i GotoTrack.obj
 0001:00029090       ??$__final_insertion_sort@PAUIDiscreteFloatKey@@U?$less@UIDiscreteFloatKey@@@stlpmtx_std@@@priv@stlpmtx_std@@YAXPAUIDiscreteFloatKey@@0U?$less@UIDiscreteFloatKey@@@1@@Z 3402a090 f i GotoTrack.obj
 0001:00029100       ??$sort_heap@PAUIDiscreteFloatKey@@U?$less@UIDiscreteFloatKey@@@stlpmtx_std@@@stlpmtx_std@@YAXPAUIDiscreteFloatKey@@0U?$less@UIDiscreteFloatKey@@@0@@Z 3402a100 f i GotoTrack.obj
 0001:000291b0       ??$__partial_sort@PAUIDiscreteFloatKey@@U1@U?$less@UIDiscreteFloatKey@@@stlpmtx_std@@@priv@stlpmtx_std@@YAXPAUIDiscreteFloatKey@@000U?$less@UIDiscreteFloatKey@@@1@@Z 3402a1b0 f i GotoTrack.obj
 0001:00029250       ??0CGotoTrack@@QAE@XZ      3402a250 f   GotoTrack.obj
 0001:000292c0       ?GetValueType@CGotoTrack@@UAE?AW4EAnimValue@@XZ 3402a2c0 f i GotoTrack.obj
 0001:000292c0       ?GetType@CCommentNode@@UBE?AW4EAnimNodeType@@XZ 3402a2c0 f i CommentNode.obj
 0001:000292d0       ?GetMemoryUsage@CGotoTrack@@UBEXPAVICrySizer@@@Z 3402a2d0 f i GotoTrack.obj
 0001:000292d0       ?GetMemoryUsage@CLookAtTrack@@UBEXPAVICrySizer@@@Z 3402a2d0 f i AnimNode.obj
 0001:000292d0       ?GetMemoryUsage@CCharacterTrack@@UBEXPAVICrySizer@@@Z 3402a2d0 f i AnimNode.obj
 0001:000292f0       ?resize@?$_Impl_vector@UIDiscreteFloatKey@@V?$allocator@UIDiscreteFloatKey@@@stlpmtx_std@@@priv@stlpmtx_std@@QAEXIABUIDiscreteFloatKey@@@Z 3402a2f0 f i GotoTrack.obj
 0001:000293a0       ??$__introsort_loop@PAUIDiscreteFloatKey@@U1@HU?$less@UIDiscreteFloatKey@@@stlpmtx_std@@@priv@stlpmtx_std@@YAXPAUIDiscreteFloatKey@@00HU?$less@UIDiscreteFloatKey@@@1@@Z 3402a3a0 f i GotoTrack.obj
 0001:000294a0       ?SetNumKeys@?$TAnimTrack@UIDiscreteFloatKey@@@@UAEXH@Z 3402a4a0 f i GotoTrack.obj
 0001:000294e0       ??$sort@PAUIDiscreteFloatKey@@@stlpmtx_std@@YAXPAUIDiscreteFloatKey@@0@Z 3402a4e0 f i GotoTrack.obj
 0001:00029540       ?SortKeys@?$TAnimTrack@UIDiscreteFloatKey@@@@UAEXXZ 3402a540 f i GotoTrack.obj
 0001:00029560       ?SerializeKey@CLookAtTrack@@UAEXAAUILookAtKey@@AAVXmlNodeRef@@_N@Z 3402a560 f   LookAtTrack.obj
 0001:00029650       ?Serialize@?$TAnimTrack@UILookAtKey@@@@UAE_NAAVXmlNodeRef@@_N1@Z 3402a650 f i LookAtTrack.obj
 0001:00029900       ?Serialize@CLookAtTrack@@UAE_NAAVXmlNodeRef@@_N1@Z 3402a900 f   LookAtTrack.obj
 0001:00029960       ?GetKeyInfo@CLookAtTrack@@UAEXHAAPBDAAM@Z 3402a960 f   LookAtTrack.obj
 0001:000299c0       ?SerializeKey@CMusicTrack@@UAEXAAUIMusicKey@@AAVXmlNodeRef@@_N@Z 3402a9c0 f   MusicTrack.obj
 0001:00029aa0       ?GetKeyInfo@CMusicTrack@@UAEXHAAPBDAAM@Z 3402aaa0 f   MusicTrack.obj
 0001:00029b10       ?GetMemoryUsage@CScreenFaderTrack@@UBEXPAVICrySizer@@@Z 3402ab10 f   ScreenFaderTrack.obj
 0001:00029b30       ?SerializeKey@CScreenFaderTrack@@UAEXAAUIScreenFaderKey@@AAVXmlNodeRef@@_N@Z 3402ab30 f   ScreenFaderTrack.obj
 0001:00029cd0       ?GetKeyInfo@CScreenFaderTrack@@UAEXHAAPBDAAM@Z 3402acd0 f   ScreenFaderTrack.obj
 0001:00029d30       ?GetActiveTexture@CScreenFaderTrack@@QBEPAVITexture@@XZ 3402ad30 f   ScreenFaderTrack.obj
 0001:00029d50       ??$_M_allocate_and_copy@PAPAX@?$_Impl_vector@PAXV?$allocator@PAX@stlpmtx_std@@@priv@stlpmtx_std@@AAEPAPAXAAIPAPAX1@Z 3402ad50 f i ScreenFaderTrack.obj
 0001:00029d50       ??$_M_allocate_and_copy@PAI@?$_Impl_vector@IV?$allocator@I@stlpmtx_std@@@priv@stlpmtx_std@@AAEPAIAAIPAI1@Z 3402ad50 f i EntityNode.obj
 0001:00029dc0       ?erase@?$_Impl_vector@PAXV?$allocator@PAX@stlpmtx_std@@@priv@stlpmtx_std@@QAEPAPAXPAPAX0@Z 3402adc0 f i ScreenFaderTrack.obj
 0001:00029e10       ?reserve@?$_Impl_vector@PAXV?$allocator@PAX@stlpmtx_std@@@priv@stlpmtx_std@@QAEXI@Z 3402ae10 f i ScreenFaderTrack.obj
 0001:00029ea0       ?_M_fill_insert_aux@?$_Impl_vector@PAXV?$allocator@PAX@stlpmtx_std@@@priv@stlpmtx_std@@AAEXPAPAXIABQAXABU__false_type@3@@Z 3402aea0 f i ScreenFaderTrack.obj
 0001:00029ea0       ?_M_fill_insert_aux@?$_Impl_vector@IV?$allocator@I@stlpmtx_std@@@priv@stlpmtx_std@@AAEXPAIIABIABU__false_type@3@@Z 3402aea0 f i EntityNode.obj
 0001:00029fe0       ?SetFlags@?$TAnimTrack@UILookAtKey@@@@UAEXH@Z 3402afe0 f i AnimNode.obj
 0001:00029fe0       ?SetFlags@?$TAnimTrack@UIDiscreteFloatKey@@@@UAEXH@Z 3402afe0 f i GotoTrack.obj
 0001:00029fe0       ?SetFlags@?$TAnimTrack@UIBoolKey@@@@UAEXH@Z 3402afe0 f i AnimNode.obj
 0001:00029fe0       ?SetFlags@?$TAnimTrack@UISoundKey@@@@UAEXH@Z 3402afe0 f i AnimNode.obj
 0001:00029fe0       ?SetFlags@?$TAnimTrack@UISelectKey@@@@UAEXH@Z 3402afe0 f i AnimNode.obj
 0001:00029fe0       ?SetFlags@?$TAnimTrack@UIFaceSeqKey@@@@UAEXH@Z 3402afe0 f i AnimNode.obj
 0001:00029fe0       ?SetFlags@?$TAnimTrack@UIScreenFaderKey@@@@UAEXH@Z 3402afe0 f i ScreenFaderTrack.obj
 0001:00029fe0       ?SetFlags@?$TAnimTrack@UIMusicKey@@@@UAEXH@Z 3402afe0 f i AnimNode.obj
 0001:00029fe0       ?SetFlags@?$TAnimTrack@UISequenceKey@@@@UAEXH@Z 3402afe0 f i AnimNode.obj
 0001:00029fe0       ?SetFlags@?$TAnimTrack@UICharacterKey@@@@UAEXH@Z 3402afe0 f i AnimNode.obj
 0001:00029fe0       ?SetFlags@?$TAnimTrack@UIConsoleKey@@@@UAEXH@Z 3402afe0 f i AnimNode.obj
 0001:00029fe0       ?SetFlags@?$TAnimTrack@UICaptureKey@@@@UAEXH@Z 3402afe0 f i AnimNode.obj
 0001:00029fe0       ?SetFlags@?$TAnimTrack@UIEventKey@@@@UAEXH@Z 3402afe0 f i AnimNode.obj
 0001:00029fe0       ?SetFlags@?$TAnimTrack@UIExprKey@@@@UAEXH@Z 3402afe0 f i AnimNode.obj
 0001:00029fe0       ?SetFlags@?$TAnimTrack@UICommentKey@@@@UAEXH@Z 3402afe0 f i CommentTrack.obj
 0001:00029ff0       ?GetParameterType@?$TAnimTrack@UISoundKey@@@@UBE?AVAnimParamType@@XZ 3402aff0 f i AnimNode.obj
 0001:00029ff0       ?GetParameterType@?$TAnimTrack@UISequenceKey@@@@UBE?AVAnimParamType@@XZ 3402aff0 f i AnimNode.obj
 0001:00029ff0       ?GetParameterType@?$TAnimTrack@UICommentKey@@@@UBE?AVAnimParamType@@XZ 3402aff0 f i CommentTrack.obj
 0001:00029ff0       ?GetParameterType@?$TAnimTrack@UICaptureKey@@@@UBE?AVAnimParamType@@XZ 3402aff0 f i AnimNode.obj
 0001:00029ff0       ?GetParameterType@?$TAnimTrack@UIFaceSeqKey@@@@UBE?AVAnimParamType@@XZ 3402aff0 f i AnimNode.obj
 0001:00029ff0       ?GetParameterType@?$TAnimTrack@UIEventKey@@@@UBE?AVAnimParamType@@XZ 3402aff0 f i AnimNode.obj
 0001:00029ff0       ?GetParameterType@?$TAnimTrack@UIConsoleKey@@@@UBE?AVAnimParamType@@XZ 3402aff0 f i AnimNode.obj
 0001:00029ff0       ?GetParameterType@?$TAnimTrack@UICharacterKey@@@@UBE?AVAnimParamType@@XZ 3402aff0 f i AnimNode.obj
 0001:00029ff0       ?GetParameterType@?$TAnimTrack@UIExprKey@@@@UBE?AVAnimParamType@@XZ 3402aff0 f i AnimNode.obj
 0001:00029ff0       ?GetParameterType@?$TAnimTrack@UIDiscreteFloatKey@@@@UBE?AVAnimParamType@@XZ 3402aff0 f i GotoTrack.obj
 0001:00029ff0       ?GetParameterType@?$TAnimTrack@UIScreenFaderKey@@@@UBE?AVAnimParamType@@XZ 3402aff0 f i ScreenFaderTrack.obj
 0001:00029ff0       ?GetParameterType@?$TAnimSplineTrack@U?$Vec3_tpl@M@@@@UBE?AVAnimParamType@@XZ 3402aff0 f i Movie.obj
 0001:00029ff0       ?GetParameterType@?$TAnimTrack@UIBoolKey@@@@UBE?AVAnimParamType@@XZ 3402aff0 f i AnimNode.obj
 0001:00029ff0       ?GetParameterType@?$TAnimTrack@UILookAtKey@@@@UBE?AVAnimParamType@@XZ 3402aff0 f i AnimNode.obj
 0001:00029ff0       ?GetParameterType@?$TAnimTrack@UISelectKey@@@@UBE?AVAnimParamType@@XZ 3402aff0 f i AnimNode.obj
 0001:00029ff0       ?GetParameterType@?$TAnimTrack@UIMusicKey@@@@UBE?AVAnimParamType@@XZ 3402aff0 f i AnimNode.obj
 0001:0002a010       ??4IScreenFaderKey@@QAEAAU0@ABU0@@Z 3402b010 f i ScreenFaderTrack.obj
 0001:0002a080       ??$__copy@PAUIScreenFaderKey@@PAU1@H@priv@stlpmtx_std@@YAPAUIScreenFaderKey@@PAU2@00ABUrandom_access_iterator_tag@1@PAH@Z 3402b080 f i ScreenFaderTrack.obj
 0001:0002a120       ??$__copy_backward@PAUIScreenFaderKey@@PAU1@H@priv@stlpmtx_std@@YAPAUIScreenFaderKey@@PAU2@00ABUrandom_access_iterator_tag@1@PAH@Z 3402b120 f i ScreenFaderTrack.obj
 0001:0002a1c0       ??$__fill@PAUIScreenFaderKey@@U1@H@priv@stlpmtx_std@@YAXPAUIScreenFaderKey@@0ABU2@ABUrandom_access_iterator_tag@1@PAH@Z 3402b1c0 f i ScreenFaderTrack.obj
 0001:0002a250       ??$__unguarded_linear_insert@PAUIScreenFaderKey@@U1@U?$less@UIScreenFaderKey@@@stlpmtx_std@@@priv@stlpmtx_std@@YAXPAUIScreenFaderKey@@U2@U?$less@UIScreenFaderKey@@@1@@Z 3402b250 f i ScreenFaderTrack.obj
 0001:0002a2e0       ??$__push_heap@PAUIScreenFaderKey@@HU1@U?$less@UIScreenFaderKey@@@stlpmtx_std@@@stlpmtx_std@@YAXPAUIScreenFaderKey@@HHU1@U?$less@UIScreenFaderKey@@@0@@Z 3402b2e0 f i ScreenFaderTrack.obj
 0001:0002a390       ??0IScreenFaderKey@@QAE@ABU0@@Z 3402b390 f i ScreenFaderTrack.obj
 0001:0002a3f0       ?GetNumKeys@?$TAnimTrack@UIScreenFaderKey@@@@UBEHXZ 3402b3f0 f i ScreenFaderTrack.obj
 0001:0002a410       ?CreateKey@?$TAnimTrack@UIScreenFaderKey@@@@UAEHM@Z 3402b410 f i ScreenFaderTrack.obj
 0001:0002a4a0       ?CloneKey@?$TAnimTrack@UIScreenFaderKey@@@@UAEHH@Z 3402b4a0 f i ScreenFaderTrack.obj
 0001:0002a540       ?CopyKey@?$TAnimTrack@UIScreenFaderKey@@@@UAEHPAUIAnimTrack@@H@Z 3402b540 f i ScreenFaderTrack.obj
 0001:0002a5e0       ?GetKey@?$TAnimTrack@UIScreenFaderKey@@@@UBEXHPAUIKey@@@Z 3402b5e0 f i ScreenFaderTrack.obj
 0001:0002a600       ?GetKeyTime@?$TAnimTrack@UIScreenFaderKey@@@@UBEMH@Z 3402b600 f i ScreenFaderTrack.obj
 0001:0002a620       ?FindKey@?$TAnimTrack@UIScreenFaderKey@@@@UAEHM@Z 3402b620 f i ScreenFaderTrack.obj
 0001:0002a680       ?GetKeyFlags@?$TAnimTrack@UIScreenFaderKey@@@@UAEHH@Z 3402b680 f i ScreenFaderTrack.obj
 0001:0002a6a0       ?SetKey@?$TAnimTrack@UIScreenFaderKey@@@@UAEXHPAUIKey@@@Z 3402b6a0 f i ScreenFaderTrack.obj
 0001:0002a6d0       ?SetKeyTime@?$TAnimTrack@UIScreenFaderKey@@@@UAEXHM@Z 3402b6d0 f i ScreenFaderTrack.obj
 0001:0002a6f0       ?SetKeyFlags@?$TAnimTrack@UIScreenFaderKey@@@@UAEXHH@Z 3402b6f0 f i ScreenFaderTrack.obj
 0001:0002a710       ?Serialize@?$TAnimTrack@UIScreenFaderKey@@@@UAE_NAAVXmlNodeRef@@_N1@Z 3402b710 f i ScreenFaderTrack.obj
 0001:0002a9c0       ?SerializeSelection@?$TAnimTrack@UIScreenFaderKey@@@@UAE_NAAVXmlNodeRef@@_N1M@Z 3402b9c0 f i ScreenFaderTrack.obj
 0001:0002ab80       ??$__unguarded_insertion_sort_aux@PAUIScreenFaderKey@@U1@U?$less@UIScreenFaderKey@@@stlpmtx_std@@@priv@stlpmtx_std@@YAXPAUIScreenFaderKey@@00U?$less@UIScreenFaderKey@@@1@@Z 3402bb80 f i ScreenFaderTrack.obj
 0001:0002ac10       ??$__adjust_heap@PAUIScreenFaderKey@@HU1@U?$less@UIScreenFaderKey@@@stlpmtx_std@@@stlpmtx_std@@YAXPAUIScreenFaderKey@@HHU1@U?$less@UIScreenFaderKey@@@0@@Z 3402bc10 f i ScreenFaderTrack.obj
 0001:0002ad60       ?IsKeySelected@?$TAnimTrack@UIScreenFaderKey@@@@UBE_NH@Z 3402bd60 f i ScreenFaderTrack.obj
 0001:0002ad80       ?SelectKey@?$TAnimTrack@UIScreenFaderKey@@@@UAEXH_N@Z 3402bd80 f i ScreenFaderTrack.obj
 0001:0002adc0       ??$__make_heap@PAUIScreenFaderKey@@U?$less@UIScreenFaderKey@@@stlpmtx_std@@U1@H@stlpmtx_std@@YAXPAUIScreenFaderKey@@0U?$less@UIScreenFaderKey@@@0@0PAH@Z 3402bdc0 f i ScreenFaderTrack.obj
 0001:0002ae80       ??$__ufill@PAUIScreenFaderKey@@U1@H@priv@stlpmtx_std@@YAXPAUIScreenFaderKey@@0ABU2@ABUrandom_access_iterator_tag@1@PAH@Z 3402be80 f i ScreenFaderTrack.obj
 0001:0002af20       ??$__ucopy@PAUIScreenFaderKey@@PAU1@H@priv@stlpmtx_std@@YAPAUIScreenFaderKey@@PAU2@00ABUrandom_access_iterator_tag@1@PAH@Z 3402bf20 f i ScreenFaderTrack.obj
 0001:0002afc0       ?RemoveKey@?$TAnimTrack@UIScreenFaderKey@@@@UAEXH@Z 3402bfc0 f i ScreenFaderTrack.obj
 0001:0002b020       ??$__unguarded_partition@PAUIScreenFaderKey@@U1@U?$less@UIScreenFaderKey@@@stlpmtx_std@@@priv@stlpmtx_std@@YAPAUIScreenFaderKey@@PAU2@0U2@U?$less@UIScreenFaderKey@@@1@@Z 3402c020 f i ScreenFaderTrack.obj
 0001:0002b180       ??$__insertion_sort@PAUIScreenFaderKey@@U1@U?$less@UIScreenFaderKey@@@stlpmtx_std@@@priv@stlpmtx_std@@YAXPAUIScreenFaderKey@@00U?$less@UIScreenFaderKey@@@1@@Z 3402c180 f i ScreenFaderTrack.obj
 0001:0002b2c0       ??$sort_heap@PAUIScreenFaderKey@@U?$less@UIScreenFaderKey@@@stlpmtx_std@@@stlpmtx_std@@YAXPAUIScreenFaderKey@@0U?$less@UIScreenFaderKey@@@0@@Z 3402c2c0 f i ScreenFaderTrack.obj
 0001:0002b490       ?_M_fill_insert_aux@?$_Impl_vector@UIScreenFaderKey@@V?$allocator@UIScreenFaderKey@@@stlpmtx_std@@@priv@stlpmtx_std@@AAEXPAUIScreenFaderKey@@IABU4@ABU__false_type@3@@Z 3402c490 f i ScreenFaderTrack.obj
 0001:0002b5a0       ??$__final_insertion_sort@PAUIScreenFaderKey@@U?$less@UIScreenFaderKey@@@stlpmtx_std@@@priv@stlpmtx_std@@YAXPAUIScreenFaderKey@@0U?$less@UIScreenFaderKey@@@1@@Z 3402c5a0 f i ScreenFaderTrack.obj
 0001:0002b610       ??$__partial_sort@PAUIScreenFaderKey@@U1@U?$less@UIScreenFaderKey@@@stlpmtx_std@@@priv@stlpmtx_std@@YAXPAUIScreenFaderKey@@000U?$less@UIScreenFaderKey@@@1@@Z 3402c610 f i ScreenFaderTrack.obj
 0001:0002b780       ??0CScreenFaderTrack@@QAE@XZ 3402c780 f   ScreenFaderTrack.obj
 0001:0002b830       ?resize@?$_Impl_vector@PAXV?$allocator@PAX@stlpmtx_std@@@priv@stlpmtx_std@@QAEXIABQAX@Z 3402c830 f i ScreenFaderTrack.obj
 0001:0002b830       ?resize@?$_Impl_vector@IV?$allocator@I@stlpmtx_std@@@priv@stlpmtx_std@@QAEXIABI@Z 3402c830 f i EntityNode.obj
 0001:0002b8d0       ?_M_insert_overflow_aux@?$_Impl_vector@UIScreenFaderKey@@V?$allocator@UIScreenFaderKey@@@stlpmtx_std@@@priv@stlpmtx_std@@AAEXPAUIScreenFaderKey@@ABU4@ABU__false_type@3@I_N@Z 3402c8d0 f i ScreenFaderTrack.obj
 0001:0002ba60       ??$__introsort_loop@PAUIScreenFaderKey@@U1@HU?$less@UIScreenFaderKey@@@stlpmtx_std@@@priv@stlpmtx_std@@YAXPAUIScreenFaderKey@@00HU?$less@UIScreenFaderKey@@@1@@Z 3402ca60 f i ScreenFaderTrack.obj
 0001:0002bba0       ?ReleasePreloadedTextures@CScreenFaderTrack@@AAEXXZ 3402cba0 f   ScreenFaderTrack.obj
 0001:0002bc00       ??$sort@PAUIScreenFaderKey@@@stlpmtx_std@@YAXPAUIScreenFaderKey@@0@Z 3402cc00 f i ScreenFaderTrack.obj
 0001:0002bc60       ??1CScreenFaderTrack@@UAE@XZ 3402cc60 f   ScreenFaderTrack.obj
 0001:0002bcf0       ?PreloadTextures@CScreenFaderTrack@@QAEXXZ 3402ccf0 f   ScreenFaderTrack.obj
 0001:0002be30       ?SetActiveTexture@CScreenFaderTrack@@QAE_NH@Z 3402ce30 f   ScreenFaderTrack.obj
 0001:0002bf60       ?SortKeys@?$TAnimTrack@UIScreenFaderKey@@@@UAEXXZ 3402cf60 f i ScreenFaderTrack.obj
 0001:0002bf80       ??_GCScreenFaderTrack@@UAEPAXI@Z 3402cf80 f i ScreenFaderTrack.obj
 0001:0002bf80       ??_ECScreenFaderTrack@@UAEPAXI@Z 3402cf80 f i ScreenFaderTrack.obj
 0001:0002bfb0       ?resize@?$_Impl_vector@UIScreenFaderKey@@V?$allocator@UIScreenFaderKey@@@stlpmtx_std@@@priv@stlpmtx_std@@QAEXIABUIScreenFaderKey@@@Z 3402cfb0 f i ScreenFaderTrack.obj
 0001:0002c060       ?SetNumKeys@?$TAnimTrack@UIScreenFaderKey@@@@UAEXH@Z 3402d060 f i ScreenFaderTrack.obj
 0001:0002c0d0       ?SerializeKey@CSelectTrack@@UAEXAAUISelectKey@@AAVXmlNodeRef@@_N@Z 3402d0d0 f   SelectTrack.obj
 0001:0002c160       ?GetKeyInfo@CSelectTrack@@UAEXHAAPBDAAM@Z 3402d160 f   SelectTrack.obj
 0001:0002c1c0       ?SerializeKey@CSequenceTrack@@UAEXAAUISequenceKey@@AAVXmlNodeRef@@_N@Z 3402d1c0 f   SequenceTrack.obj
 0001:0002c340       ?GetKeyInfo@CSequenceTrack@@UAEXHAAPBDAAM@Z 3402d340 f   SequenceTrack.obj
 0001:0002c3a0       ?SerializeKey@CSoundTrack@@UAEXAAUISoundKey@@AAVXmlNodeRef@@_N@Z 3402d3a0 f   SoundTrack.obj
 0001:0002c800       ?GetKeyInfo@CSoundTrack@@UAEXHAAPBDAAM@Z 3402d800 f   SoundTrack.obj
 0001:0002c8b0       ?SerializeKey@CTrackEventTrack@@UAEXAAUIEventKey@@AAVXmlNodeRef@@_N@Z 3402d8b0 f   TrackEventTrack.obj
 0001:0002c970       ?GetKeyInfo@CTrackEventTrack@@UAEXHAAPBDAAM@Z 3402d970 f   TrackEventTrack.obj
 0001:0002ca40       ?GetMemoryUsage@CAnimCameraNode@@UBEXPAVICrySizer@@@Z 3402da40 f i AnimCameraNode.obj
 0001:0002ca60       ?Reset@CAnimCameraNode@@UAEXXZ 3402da60 f   AnimCameraNode.obj
 0001:0002caa0       ?ApplyFocusKey@CAnimCameraNode@@QAEXAAUISelectKey@@AAUSAnimContext@@@Z 3402daa0 f   AnimCameraNode.obj
 0001:0002caf0       ?Activate@CAnimCameraNode@@UAEX_N@Z 3402daf0 f   AnimCameraNode.obj
 0001:0002cb20       ??_ECAnimCameraNode@@$4PPPPPPPM@A@AEPAXI@Z 3402db20 f i AnimCameraNode.obj
 0001:0002cb30       ?Release@CAnimNode@@$4PPPPPPPM@CCA@AEXXZ 3402db30 f i AnimCameraNode.obj
 0001:0002cb40       ?CreateTrack@CAnimCameraNode@@UAEPAUIAnimTrack@@ABVAnimParamType@@@Z 3402db40 f   AnimCameraNode.obj
 0001:0002cc00       ?Serialize@CAnimCameraNode@@UAEXAAVXmlNodeRef@@_N1@Z 3402dc00 f   AnimCameraNode.obj
 0001:0002cf40       ??$?9D@@YA_NABV?$CryStringT@D@@0@Z 3402df40 f i AnimCameraNode.obj
 0001:0002cf90       ??_GCAnimCameraNode@@UAEPAXI@Z 3402df90 f i AnimCameraNode.obj
 0001:0002cf90       ??_ECAnimCameraNode@@UAEPAXI@Z 3402df90 f i AnimCameraNode.obj
 0001:0002cff0       ?GetParamCount@CAnimCameraNode@@UBEHXZ 3402dff0 f   AnimCameraNode.obj
 0001:0002d010       ?CreateDefaultTracks@CAnimCameraNode@@UAEXXZ 3402e010 f   AnimCameraNode.obj
 0001:0002d0e0       ?SetParamValue@CAnimCameraNode@@UAE_NMVAnimParamType@@M@Z 3402e0e0 f   AnimCameraNode.obj
 0001:0002d180       ?SetParamValue@CAnimCameraNode@@UAE_NMVAnimParamType@@ABU?$Vec3_tpl@M@@@Z 3402e180 f   AnimCameraNode.obj
 0001:0002d2e0       ?SetParamValue@CAnimCameraNode@@UAE_NMVAnimParamType@@ABU?$Vec4_tpl@M@@@Z 3402e2e0 f   AnimCameraNode.obj
 0001:0002d3d0       ?GetParamValue@CAnimCameraNode@@UAE_NMVAnimParamType@@AAM@Z 3402e3d0 f   AnimCameraNode.obj
 0001:0002d4b0       ?GetParamValue@CAnimCameraNode@@UAE_NMVAnimParamType@@AAU?$Vec3_tpl@M@@@Z 3402e4b0 f   AnimCameraNode.obj
 0001:0002d5c0       ?GetParamValue@CAnimCameraNode@@UAE_NMVAnimParamType@@AAU?$Vec4_tpl@M@@@Z 3402e5c0 f   AnimCameraNode.obj
 0001:0002d6e0       ?find@?$CryStringT@D@@QBEIPBDI@Z 3402e6e0 f i AnimCameraNode.obj
 0001:0002d720       ?GetActiveKey@?$TAnimTrack@UISelectKey@@@@QAEHMPAUISelectKey@@@Z 3402e720 f i AnimCameraNode.obj
 0001:0002d8d0       ?_M_set@?$_Impl_vector@USParamInfo@IAnimNode@@V?$allocator@USParamInfo@IAnimNode@@@stlpmtx_std@@@priv@stlpmtx_std@@AAEXPAUSParamInfo@IAnimNode@@00@Z 3402e8d0 f i AnimCameraNode.obj
 0001:0002d8d0       ?_M_set@?$_Impl_vector@V?$_smart_ptr@VCControlParamBase@CFXNodeDescription@@@@V?$allocator@V?$_smart_ptr@VCControlParamBase@CFXNodeDescription@@@@@stlpmtx_std@@@priv@stlpmtx_std@@AAEXPAV?$_smart_ptr@VCControlParamBase@CFXNodeDescription@@@@00@Z 3402e8d0 f i AnimPostFXNode.obj
 0001:0002d8d0       ?_M_set@?$_Impl_vector@PAXV?$allocator@PAX@stlpmtx_std@@@priv@stlpmtx_std@@AAEXPAPAX00@Z 3402e8d0 f i Movie.obj
 0001:0002d8d0       ?_M_set@?$_Impl_vector@USkelAnimUpdateCMD@CMovieSystem@@V?$allocator@USkelAnimUpdateCMD@CMovieSystem@@@stlpmtx_std@@@priv@stlpmtx_std@@AAEXPAUSkelAnimUpdateCMD@CMovieSystem@@00@Z 3402e8d0 f i Movie.obj
 0001:0002d8d0       ?_M_set@?$_Impl_vector@IV?$allocator@I@stlpmtx_std@@@priv@stlpmtx_std@@AAEXPAI00@Z 3402e8d0 f i EntityNode.obj
 0001:0002d930       ?allocate@?$_STLP_alloc_proxy@PAUSParamInfo@IAnimNode@@U12@V?$allocator@USParamInfo@IAnimNode@@@stlpmtx_std@@@priv@stlpmtx_std@@QAEPAUSParamInfo@IAnimNode@@IAAI@Z 3402e930 f i AnimCameraNode.obj
 0001:0002d990       ?GetParamInfo@CAnimCameraNode@@UBE_NHAAUSParamInfo@IAnimNode@@@Z 3402e990 f   AnimCameraNode.obj
 0001:0002d9e0       ?GetParamInfoFromId@CAnimCameraNode@@UBE_NABVAnimParamType@@AAUSParamInfo@IAnimNode@@@Z 3402e9e0 f   AnimCameraNode.obj
 0001:0002daa0       ?insert@?$CryStringT@D@@QAEAAV1@IPBDI@Z 3402eaa0 f i AnimCameraNode.obj
 0001:0002db80       ??$__ufill@PAUSParamInfo@IAnimNode@@U12@H@priv@stlpmtx_std@@YAXPAUSParamInfo@IAnimNode@@0ABU23@ABUrandom_access_iterator_tag@1@PAH@Z 3402eb80 f i AnimCameraNode.obj
 0001:0002dbe0       ??$__destroy_range_aux@V?$reverse_iterator@PAUSParamInfo@IAnimNode@@@stlpmtx_std@@USParamInfo@IAnimNode@@@stlpmtx_std@@YAXV?$reverse_iterator@PAUSParamInfo@IAnimNode@@@0@0PAUSParamInfo@IAnimNode@@ABU__false_type@0@@Z 3402ebe0 f i AnimCameraNode.obj
 0001:0002dc30       ??$__ucopy@PAUSParamInfo@IAnimNode@@PAU12@H@priv@stlpmtx_std@@YAPAUSParamInfo@IAnimNode@@PAU23@00ABUrandom_access_iterator_tag@1@PAH@Z 3402ec30 f i AnimCameraNode.obj
 0001:0002dca0       ?MakeLower@?$CryStringT@D@@QAEAAV1@XZ 3402eca0 f i AnimCameraNode.obj
 0001:0002dce0       ?comp_area@?$TrackSplineInterpolator@U?$Vec2_tpl@M@@@spline@@ABEMHHM@Z 3402ece0 f i AnimCameraNode.obj
 0001:0002df20       ?ShowCameraShakeDebug@ShakeParam@CAnimCameraNode@@QBEXIHM@Z 3402ef20 f   AnimCameraNode.obj
 0001:0002e070       ?insert@?$CryStringT@D@@QAEAAV1@IPBD@Z 3402f070 f i AnimCameraNode.obj
 0001:0002e0b0       ?FixCameraNodeForExport@CAnimCameraNode@@QBEXVXmlNodeRef@@ABUSColladaExporterSaveProperties@@@Z 3402f0b0 f   AnimCameraNode.obj
 0001:0002e490       ?SaveToColladaInFixedFPS@CAnimCameraNode@@UBE?AVXmlNodeRef@@ABUSColladaExporterSaveProperties@@@Z 3402f490 f   AnimCameraNode.obj
 0001:0002ea30       ?LoadFromCollada@CAnimCameraNode@@UAE_NVXmlNodeRef@@@Z 3402fa30 f   AnimCameraNode.obj
 0001:0002f800       ?_M_insert_overflow_aux@?$_Impl_vector@USParamInfo@IAnimNode@@V?$allocator@USParamInfo@IAnimNode@@@stlpmtx_std@@@priv@stlpmtx_std@@AAEXPAUSParamInfo@IAnimNode@@ABU45@ABU__false_type@3@I_N@Z 34030800 f i AnimCameraNode.obj
 0001:0002f9c0       ??$_M_allocate_and_copy@PAUSParamInfo@IAnimNode@@@?$_Impl_vector@USParamInfo@IAnimNode@@V?$allocator@USParamInfo@IAnimNode@@@stlpmtx_std@@@priv@stlpmtx_std@@AAEPAUSParamInfo@IAnimNode@@AAIPAU34@1@Z 340309c0 f i AnimCameraNode.obj
 0001:0002fa30       ?reserve@?$_Impl_vector@USParamInfo@IAnimNode@@V?$allocator@USParamInfo@IAnimNode@@@stlpmtx_std@@@priv@stlpmtx_std@@QAEXI@Z 34030a30 f i AnimCameraNode.obj
 0001:0002fb00       ?push_back@?$_Impl_vector@USParamInfo@IAnimNode@@V?$allocator@USParamInfo@IAnimNode@@@stlpmtx_std@@@priv@stlpmtx_std@@QAEXABUSParamInfo@IAnimNode@@@Z 34030b00 f i AnimCameraNode.obj
 0001:0002fb80       ?Initialize@CAnimCameraNode@@SAXXZ 34030b80 f   AnimCameraNode.obj
 0001:0002fe00       ??0CAnimCameraNode@@QAE@XZ 34030e00 f   AnimCameraNode.obj
 0001:0002ffe0       ?Integrate@?$TrackSplineInterpolator@U?$Vec2_tpl@M@@@spline@@QAEMM@Z 34030fe0 f i AnimCameraNode.obj
 0001:000300c0       ?ApplyCameraShake@ShakeParam@CAnimCameraNode@@QAE?AU?$Ang3_tpl@M@@MU3@PAV?$TAnimSplineTrack@U?$Vec2_tpl@M@@@@IH@Z 340310c0 f   AnimCameraNode.obj
 0001:00030740       ?Animate@CAnimCameraNode@@UAEXAAUSAnimContext@@@Z 34031740 f   AnimCameraNode.obj
 0001:00031230       ?SetFlags@CAnimNode@@UAEXH@Z 34032230 f   AnimNode.obj
 0001:00031240       ?LoadFromCollada@CAnimNode@@UAE_NVXmlNodeRef@@@Z 34032240 f   AnimNode.obj
 0001:00031320       ?SetNodeOwner@CAnimNode@@UAEXPAUIAnimNodeOwner@@@Z 34032320 f   AnimNode.obj
 0001:00031340       ?PostLoad@CAnimNode@@UAEXXZ 34032340 f   AnimNode.obj
 0001:00031360       ?HasDirectorAsParent@CAnimNode@@UBEPAUIAnimNode@@XZ 34032360 f   AnimNode.obj
 0001:000313c0       ?TrackOrder@CAnimNode@@CA_NABUTrackDesc@1@0@Z 340323c0 f   AnimNode.obj
 0001:00031400       ?SetParamValue@CAnimNode@@UAE_NMVAnimParamType@@M@Z 34032400 f   AnimNode.obj
 0001:00031500       ?SetParamValue@CAnimNode@@UAE_NMVAnimParamType@@ABU?$Vec3_tpl@M@@@Z 34032500 f   AnimNode.obj
 0001:00031600       ?SetParamValue@CAnimNode@@UAE_NMVAnimParamType@@ABU?$Vec4_tpl@M@@@Z 34032600 f   AnimNode.obj
 0001:000316f0       ?GetParamValue@CAnimNode@@UAE_NMVAnimParamType@@AAM@Z 340326f0 f   AnimNode.obj
 0001:00031790       ?GetParamValue@CAnimNode@@UAE_NMVAnimParamType@@AAU?$Vec3_tpl@M@@@Z 34032790 f   AnimNode.obj
 0001:00031830       ?GetParamValue@CAnimNode@@UAE_NMVAnimParamType@@AAU?$Vec4_tpl@M@@@Z 34032830 f   AnimNode.obj
 0001:000318d0       ?Serialize@CAnimNode@@UAEXAAVXmlNodeRef@@_N1@Z 340328d0 f   AnimNode.obj
 0001:00031a10       ??0ISoundKey@@QAE@XZ       34032a10 f i AnimNode.obj
 0001:00031a90       ??4TrackDesc@CAnimNode@@QAEAAU01@ABU01@@Z 34032a90 f i AnimNode.obj
 0001:00031b00       ??$__unguarded_linear_insert@PAUTrackDesc@CAnimNode@@U12@P6A_NABU12@0@Z@priv@stlpmtx_std@@YAXPAUTrackDesc@CAnimNode@@U23@P6A_NABU23@2@Z@Z 34032b00 f i AnimNode.obj
 0001:00031bd0       ??$__lower_bound@PAUTrackDesc@CAnimNode@@U12@P6A_NABU12@0@ZP6A_N00@ZH@priv@stlpmtx_std@@YAPAUTrackDesc@CAnimNode@@PAU23@0ABU23@P6A_N11@Z2PAH@Z 34032bd0 f i AnimNode.obj
 0001:00031c40       ??$__upper_bound@PAUTrackDesc@CAnimNode@@U12@P6A_NABU12@0@ZP6A_N00@ZH@priv@stlpmtx_std@@YAPAUTrackDesc@CAnimNode@@PAU23@0ABU23@P6A_N11@Z2PAH@Z 34032c40 f i AnimNode.obj
 0001:00031cb0       ??$swap@UTrackDesc@CAnimNode@@@stlpmtx_std@@YAXAAUTrackDesc@CAnimNode@@0@Z 34032cb0 f i AnimNode.obj
 0001:00031d30       ??$__copy_backward@PAUTrackDesc@CAnimNode@@PAU12@H@priv@stlpmtx_std@@YAPAUTrackDesc@CAnimNode@@PAU23@00ABUrandom_access_iterator_tag@1@PAH@Z 34032d30 f i AnimNode.obj
 0001:00031de0       ?GetTrackCount@CAnimNode@@UBEHXZ 34032de0 f   AnimNode.obj
 0001:00031e00       ?GetParamName@CAnimNode@@UBEPBDVAnimParamType@@@Z 34032e00 f   AnimNode.obj
 0001:00031ee0       ?SetTimeRange@CAnimNode@@UAEXV?$TRange@M@@@Z 34032ee0 f   AnimNode.obj
 0001:00031f50       ?IsParamValid@CAnimNode@@UBE_NABVAnimParamType@@@Z 34032f50 f   AnimNode.obj
 0001:00031ff0       ?GetReferenceMatrix@CAnimNode@@UBE?AU?$Matrix34_tpl@M@@XZ 34032ff0 f   AnimNode.obj
 0001:00032120       ?CreateTrackInternalVector4@CAnimNode@@IBEPAUIAnimTrack@@ABVAnimParamType@@@Z 34033120 f   AnimNode.obj
 0001:00032260       ??_GIAnimNode@@MAEPAXI@Z   34033260 f i AnimNode.obj
 0001:00032260       ??_EIAnimNode@@MAEPAXI@Z   34033260 f i AnimNode.obj
 0001:000322a0       ??$__copy@PAUTrackDesc@CAnimNode@@PAU12@H@priv@stlpmtx_std@@YAPAUTrackDesc@CAnimNode@@PAU23@00ABUrandom_access_iterator_tag@1@PAH@Z 340332a0 f i AnimNode.obj
 0001:00032340       ?_M_allocate_buffer@?$_Temporary_buffer@PAUTrackDesc@CAnimNode@@U12@@stlpmtx_std@@AAEXXZ 34033340 f i AnimNode.obj
 0001:00032480       ??$__destroy_range_aux@PAUTrackDesc@CAnimNode@@U12@@stlpmtx_std@@YAXPAUTrackDesc@CAnimNode@@00ABU__false_type@0@@Z 34033480 f i AnimNode.obj
 0001:000324d0       ?GetTrackForParameter@CAnimNode@@UBEPAUIAnimTrack@@ABVAnimParamType@@@Z 340334d0 f   AnimNode.obj
 0001:00032610       ?GetTrackForParameter@CAnimNode@@UBEPAUIAnimTrack@@ABVAnimParamType@@I@Z 34033610 f   AnimNode.obj
 0001:00032740       ?GetTrackParamIndex@CAnimNode@@UBEIPBUIAnimTrack@@@Z 34033740 f   AnimNode.obj
 0001:000328d0       ?GetTrackByIndex@CAnimNode@@UBEPAUIAnimTrack@@H@Z 340338d0 f   AnimNode.obj
 0001:00032910       ?Serialize@AnimParamType@@QAEXAAVXmlNodeRef@@_N@Z 34033910 f i AnimNode.obj
 0001:00032a20       ??$__ufill@PAUTrackDesc@CAnimNode@@U12@H@priv@stlpmtx_std@@YAXPAUTrackDesc@CAnimNode@@0ABU23@ABUrandom_access_iterator_tag@1@PAH@Z 34033a20 f i AnimNode.obj
 0001:00032a80       ??$__destroy_range_aux@V?$reverse_iterator@PAUTrackDesc@CAnimNode@@@stlpmtx_std@@UTrackDesc@CAnimNode@@@stlpmtx_std@@YAXV?$reverse_iterator@PAUTrackDesc@CAnimNode@@@0@0PAUTrackDesc@CAnimNode@@ABU__false_type@0@@Z 34033a80 f i AnimNode.obj
 0001:00032ae0       ??$__ucopy@PAUTrackDesc@CAnimNode@@PAU12@H@priv@stlpmtx_std@@YAPAUTrackDesc@CAnimNode@@PAU23@00ABUrandom_access_iterator_tag@1@PAH@Z 34033ae0 f i AnimNode.obj
 0001:00032b50       ??$swap_ranges@PAUTrackDesc@CAnimNode@@PAU12@@stlpmtx_std@@YAPAUTrackDesc@CAnimNode@@PAU12@00@Z 34033b50 f i AnimNode.obj
 0001:00032cb0       ?_M_erase@?$_Impl_vector@UTrackDesc@CAnimNode@@V?$allocator@UTrackDesc@CAnimNode@@@stlpmtx_std@@@priv@stlpmtx_std@@AAEPAUTrackDesc@CAnimNode@@PAU45@ABU__false_type@3@@Z 34033cb0 f i AnimNode.obj
 0001:00032d40       ??$merge@PAUTrackDesc@CAnimNode@@PAU12@PAU12@P6A_NABU12@0@Z@stlpmtx_std@@YAPAUTrackDesc@CAnimNode@@PAU12@0000P6A_NABU12@1@Z@Z 34033d40 f i AnimNode.obj
 0001:00032e70       ??$__rotate_aux@PAUTrackDesc@CAnimNode@@HU12@@priv@stlpmtx_std@@YAPAUTrackDesc@CAnimNode@@PAU23@00PAH0@Z 34033e70 f i AnimNode.obj
 0001:00033220       ?SaveToColladaInFixedFPS@CAnimNode@@UBE?AVXmlNodeRef@@ABUSColladaExporterSaveProperties@@@Z 34034220 f   AnimNode.obj
 0001:00033840       ??$__linear_insert@PAUTrackDesc@CAnimNode@@U12@P6A_NABU12@0@Z@priv@stlpmtx_std@@YAXPAUTrackDesc@CAnimNode@@0U23@P6A_NABU23@2@Z@Z 34034840 f i AnimNode.obj
 0001:000338f0       ??$__merge_sort_loop@PAUTrackDesc@CAnimNode@@PAU12@HP6A_NABU12@0@Z@priv@stlpmtx_std@@YAXPAUTrackDesc@CAnimNode@@00HP6A_NABU23@1@Z@Z 340348f0 f i AnimNode.obj
 0001:000339e0       ??$__merge_backward@PAUTrackDesc@CAnimNode@@PAU12@PAU12@P6A_NABU12@0@Z@priv@stlpmtx_std@@YAPAUTrackDesc@CAnimNode@@PAU23@0000P6A_NABU23@1@Z@Z 340349e0 f i AnimNode.obj
 0001:00033aa0       ?_M_insert_overflow_aux@?$_Impl_vector@UTrackDesc@CAnimNode@@V?$allocator@UTrackDesc@CAnimNode@@@stlpmtx_std@@@priv@stlpmtx_std@@AAEXPAUTrackDesc@CAnimNode@@ABU45@ABU__false_type@3@I_N@Z 34034aa0 f i AnimNode.obj
 0001:00033c60       ?SetValue@?$TAnimTrack@UIScreenFaderKey@@@@UAEXMABU?$Quat_tpl@M@@_N@Z 34034c60 f i ScreenFaderTrack.obj
 0001:00033c60       ?SetValue@?$TAnimTrack@UICommentKey@@@@UAEXMABU?$Vec3_tpl@M@@_N@Z 34034c60 f i CommentTrack.obj
 0001:00033c60       ?SetValue@?$TAnimTrack@UISelectKey@@@@UAEXMABU?$Vec3_tpl@M@@_N@Z 34034c60 f i AnimNode.obj
 0001:00033c60       ?SetValue@?$TAnimTrack@UICaptureKey@@@@UAEXMAB_N_N@Z 34034c60 f i AnimNode.obj
 0001:00033c60       ?SetValue@?$TAnimTrack@UILookAtKey@@@@UAEXMABU?$Vec3_tpl@M@@_N@Z 34034c60 f i AnimNode.obj
 0001:00033c60       ?SetValue@?$TAnimTrack@UIFaceSeqKey@@@@UAEXMAB_N_N@Z 34034c60 f i AnimNode.obj
 0001:00033c60       ?SetValue@?$TAnimTrack@UIConsoleKey@@@@UAEXMABU?$Quat_tpl@M@@_N@Z 34034c60 f i AnimNode.obj
 0001:00033c60       ?SetValue@?$TAnimTrack@UIBoolKey@@@@UAEXMABM_N@Z 34034c60 f i AnimNode.obj
 0001:00033c60       ?SetValue@?$TAnimTrack@UISequenceKey@@@@UAEXMABU?$Vec3_tpl@M@@_N@Z 34034c60 f i AnimNode.obj
 0001:00033c60       ?SetValue@?$TAnimTrack@UICaptureKey@@@@UAEXMABU?$Quat_tpl@M@@_N@Z 34034c60 f i AnimNode.obj
 0001:00033c60       ?SetValue@?$TAnimTrack@UICaptureKey@@@@UAEXMABU?$Vec3_tpl@M@@_N@Z 34034c60 f i AnimNode.obj
 0001:00033c60       ?SetValue@?$TAnimTrack@UISequenceKey@@@@UAEXMAB_N_N@Z 34034c60 f i AnimNode.obj
 0001:00033c60       ?SetValue@?$TAnimTrack@UIEventKey@@@@UAEXMABU?$Vec3_tpl@M@@_N@Z 34034c60 f i AnimNode.obj
 0001:00033c60       ?SetValue@?$TAnimTrack@UIScreenFaderKey@@@@UAEXMAB_N_N@Z 34034c60 f i ScreenFaderTrack.obj
 0001:00033c60       ?SetValue@?$TAnimTrack@UILookAtKey@@@@UAEXMAB_N_N@Z 34034c60 f i AnimNode.obj
 0001:00033c60       ?SetValue@?$TAnimTrack@UIConsoleKey@@@@UAEXMAB_N_N@Z 34034c60 f i AnimNode.obj
 0001:00033c60       ?SetValue@?$TAnimTrack@UIFaceSeqKey@@@@UAEXMABM_N@Z 34034c60 f i AnimNode.obj
 0001:00033c60       ?SetValue@?$TAnimTrack@UIFaceSeqKey@@@@UAEXMABU?$Quat_tpl@M@@_N@Z 34034c60 f i AnimNode.obj
 0001:00033c60       ?SetValue@?$TAnimTrack@UIMusicKey@@@@UAEXMABU?$Quat_tpl@M@@_N@Z 34034c60 f i AnimNode.obj
 0001:00033c60       ?SetValue@?$TAnimSplineTrack@M@@UAEXMABU?$Quat_tpl@M@@_N@Z 34034c60 f i Movie.obj
 0001:00033c60       ?SetValue@?$TAnimSplineTrack@U?$Vec3_tpl@M@@@@UAEXMABU?$Quat_tpl@M@@_N@Z 34034c60 f i Movie.obj
 0001:00033c60       ?ExitScope_Alloc@CDummyMemReplay@@UAEXIII@Z 34034c60 f i AnimSequence.obj
 0001:00033c60       ?SetValue@?$TAnimTrack@UISelectKey@@@@UAEXMABU?$Quat_tpl@M@@_N@Z 34034c60 f i AnimNode.obj
 0001:00033c60       ?SetValue@?$TAnimTrack@UIScreenFaderKey@@@@UAEXMABM_N@Z 34034c60 f i ScreenFaderTrack.obj
 0001:00033c60       ?SetValue@?$TAnimTrack@UIBoolKey@@@@UAEXMABU?$Vec3_tpl@M@@_N@Z 34034c60 f i AnimNode.obj
 0001:00033c60       ?SetValue@?$TAnimTrack@UIDiscreteFloatKey@@@@UAEXMABU?$Quat_tpl@M@@_N@Z 34034c60 f i GotoTrack.obj
 0001:00033c60       ?SetValue@?$TAnimTrack@UIConsoleKey@@@@UAEXMABU?$Vec3_tpl@M@@_N@Z 34034c60 f i AnimNode.obj
 0001:00033c60       ?SetValue@CCompoundSplineTrack@@UAEXMAB_N_N@Z 34034c60 f i CompoundSplineTrack.obj
 0001:00033c60       ?SetValue@?$TAnimTrack@UICharacterKey@@@@UAEXMABU?$Vec3_tpl@M@@_N@Z 34034c60 f i AnimNode.obj
 0001:00033c60       ?SetValue@?$TAnimTrack@UIFaceSeqKey@@@@UAEXMABU?$Vec3_tpl@M@@_N@Z 34034c60 f i AnimNode.obj
 0001:00033c60       ?SetValue@?$TAnimSplineTrack@U?$Quat_tpl@M@@@@UAEXMAB_N_N@Z 34034c60 f i Movie.obj
 0001:00033c60       ?SetValue@?$TAnimTrack@UIScreenFaderKey@@@@UAEXMABU?$Vec3_tpl@M@@_N@Z 34034c60 f i ScreenFaderTrack.obj
 0001:00033c60       ?SetValue@?$TAnimTrack@UICaptureKey@@@@UAEXMABM_N@Z 34034c60 f i AnimNode.obj
 0001:00033c60       ?SetValue@?$TAnimTrack@UICharacterKey@@@@UAEXMAB_N_N@Z 34034c60 f i AnimNode.obj
 0001:00033c60       ?SetValue@?$TAnimTrack@UIDiscreteFloatKey@@@@UAEXMABM_N@Z 34034c60 f i GotoTrack.obj
 0001:00033c60       ?SetValue@?$TAnimTrack@UISoundKey@@@@UAEXMAB_N_N@Z 34034c60 f i AnimNode.obj
 0001:00033c60       ?SetValue@?$TAnimSplineTrack@U?$Vec2_tpl@M@@@@UAEXMABU?$Vec3_tpl@M@@_N@Z 34034c60 f i CompoundSplineTrack.obj
 0001:00033c60       ?SetValue@?$TAnimTrack@UISelectKey@@@@UAEXMAB_N_N@Z 34034c60 f i AnimNode.obj
 0001:00033c60       ?SetValue@?$TAnimSplineTrack@M@@UAEXMAB_N_N@Z 34034c60 f i Movie.obj
 0001:00033c60       ?SetValue@?$TAnimTrack@UILookAtKey@@@@UAEXMABM_N@Z 34034c60 f i AnimNode.obj
 0001:00033c60       ?SetValue@?$TAnimTrack@UIMusicKey@@@@UAEXMAB_N_N@Z 34034c60 f i AnimNode.obj
 0001:00033c60       ?SetValue@?$TAnimTrack@UISequenceKey@@@@UAEXMABM_N@Z 34034c60 f i AnimNode.obj
 0001:00033c60       ?SetValue@?$TAnimTrack@UIExprKey@@@@UAEXMABM_N@Z 34034c60 f i AnimNode.obj
 0001:00033c60       ?SetValue@?$TAnimTrack@UIBoolKey@@@@UAEXMAB_N_N@Z 34034c60 f i AnimNode.obj
 0001:00033c60       ?SetValue@?$TAnimTrack@UISoundKey@@@@UAEXMABU?$Vec3_tpl@M@@_N@Z 34034c60 f i AnimNode.obj
 0001:00033c60       ?SetValue@?$TAnimTrack@UIEventKey@@@@UAEXMABM_N@Z 34034c60 f i AnimNode.obj
 0001:00033c60       ?SetValue@?$TAnimTrack@UIEventKey@@@@UAEXMABU?$Quat_tpl@M@@_N@Z 34034c60 f i AnimNode.obj
 0001:00033c60       ?SetValue@?$TAnimTrack@UIMusicKey@@@@UAEXMABM_N@Z 34034c60 f i AnimNode.obj
 0001:00033c60       ?SetValue@?$TAnimTrack@UIExprKey@@@@UAEXMABU?$Vec3_tpl@M@@_N@Z 34034c60 f i AnimNode.obj
 0001:00033c60       ?SerializeKey@CBoolTrack@@UAEXAAUIBoolKey@@AAVXmlNodeRef@@_N@Z 34034c60 f i AnimNode.obj
 0001:00033c60       ?AddContext@CDummyMemReplay@@UAEXHIPBD@Z 34034c60 f i AnimSequence.obj
 0001:00033c60       ?SetValue@?$TAnimTrack@UIExprKey@@@@UAEXMABU?$Quat_tpl@M@@_N@Z 34034c60 f i AnimNode.obj
 0001:00033c60       ?SetValue@?$TAnimSplineTrack@M@@UAEXMABU?$Vec3_tpl@M@@_N@Z 34034c60 f i Movie.obj
 0001:00033c60       ?SetValue@?$TAnimTrack@UISoundKey@@@@UAEXMABM_N@Z 34034c60 f i AnimNode.obj
 0001:00033c60       ?SetValue@?$TAnimTrack@UILookAtKey@@@@UAEXMABU?$Quat_tpl@M@@_N@Z 34034c60 f i AnimNode.obj
 0001:00033c60       ?SetValue@?$TAnimTrack@UIExprKey@@@@UAEXMAB_N_N@Z 34034c60 f i AnimNode.obj
 0001:00033c60       ?SetValue@?$TAnimTrack@UIDiscreteFloatKey@@@@UAEXMABU?$Vec3_tpl@M@@_N@Z 34034c60 f i GotoTrack.obj
 0001:00033c60       ?SetValue@?$TAnimTrack@UISelectKey@@@@UAEXMABM_N@Z 34034c60 f i AnimNode.obj
 0001:00033c60       ?SetValue@?$TAnimTrack@UIConsoleKey@@@@UAEXMABM_N@Z 34034c60 f i AnimNode.obj
 0001:00033c60       ?SetValue@?$TAnimSplineTrack@U?$Quat_tpl@M@@@@UAEXMABU?$Vec3_tpl@M@@_N@Z 34034c60 f i Movie.obj
 0001:00033c60       ?SetValue@?$TAnimSplineTrack@U?$Vec3_tpl@M@@@@UAEXMAB_N_N@Z 34034c60 f i Movie.obj
 0001:00033c60       ?SetValue@?$TAnimTrack@UICharacterKey@@@@UAEXMABU?$Quat_tpl@M@@_N@Z 34034c60 f i AnimNode.obj
 0001:00033c60       ?SetValue@?$TAnimTrack@UICommentKey@@@@UAEXMABM_N@Z 34034c60 f i CommentTrack.obj
 0001:00033c60       ?RegisterFixedAddressRange@CDummyMemReplay@@UAEXPAXIPBD@Z 34034c60 f i AnimSequence.obj
 0001:00033c60       ?SetValue@?$TAnimTrack@UIEventKey@@@@UAEXMAB_N_N@Z 34034c60 f i AnimNode.obj
 0001:00033c60       ?SetValue@?$TAnimTrack@UISoundKey@@@@UAEXMABU?$Quat_tpl@M@@_N@Z 34034c60 f i AnimNode.obj
 0001:00033c60       ?SetValue@?$TAnimTrack@UIMusicKey@@@@UAEXMABU?$Vec3_tpl@M@@_N@Z 34034c60 f i AnimNode.obj
 0001:00033c60       ?SetValue@?$TAnimTrack@UIBoolKey@@@@UAEXMABU?$Quat_tpl@M@@_N@Z 34034c60 f i AnimNode.obj
 0001:00033c60       ?SetValue@?$TAnimSplineTrack@U?$Quat_tpl@M@@@@UAEXMABM_N@Z 34034c60 f i Movie.obj
 0001:00033c60       ?SetValue@?$TAnimTrack@UIDiscreteFloatKey@@@@UAEXMAB_N_N@Z 34034c60 f i GotoTrack.obj
 0001:00033c60       ?SetValue@?$TAnimTrack@UICommentKey@@@@UAEXMAB_N_N@Z 34034c60 f i CommentTrack.obj
 0001:00033c60       ?SetValue@?$TAnimSplineTrack@U?$Vec3_tpl@M@@@@UAEXMABM_N@Z 34034c60 f i Movie.obj
 0001:00033c60       ?SetValue@?$TAnimTrack@UICommentKey@@@@UAEXMABU?$Quat_tpl@M@@_N@Z 34034c60 f i CommentTrack.obj
 0001:00033c60       ?SetValue@?$TAnimTrack@UICharacterKey@@@@UAEXMABM_N@Z 34034c60 f i AnimNode.obj
 0001:00033c60       ?SetValue@?$TAnimSplineTrack@U?$Vec2_tpl@M@@@@UAEXMAB_N_N@Z 34034c60 f i CompoundSplineTrack.obj
 0001:00033c60       ?AllocUsage@CDummyMemReplay@@UAEXW4Class@EMemReplayAllocClass@@II@Z 34034c60 f i AnimSequence.obj
 0001:00033c60       ?SetValue@?$TAnimTrack@UISequenceKey@@@@UAEXMABU?$Quat_tpl@M@@_N@Z 34034c60 f i AnimNode.obj
 0001:00033c60       ?SetValue@?$TAnimSplineTrack@U?$Vec2_tpl@M@@@@UAEXMABU?$Quat_tpl@M@@_N@Z 34034c60 f i CompoundSplineTrack.obj
 0001:00033c70       ?CreateKey@?$TAnimTrack@UICharacterKey@@@@UAEHM@Z 34034c70 f i AnimNode.obj
 0001:00033cf0       ?CloneKey@?$TAnimTrack@UICharacterKey@@@@UAEHH@Z 34034cf0 f i AnimNode.obj
 0001:00033d70       ?CopyKey@?$TAnimTrack@UICharacterKey@@@@UAEHPAUIAnimTrack@@H@Z 34034d70 f i AnimNode.obj
 0001:00033df0       ?FindKey@?$TAnimTrack@UICharacterKey@@@@UAEHM@Z 34034df0 f i AnimNode.obj
 0001:00033e50       ?GetKeyFlags@?$TAnimTrack@UICharacterKey@@@@UAEHH@Z 34034e50 f i AnimNode.obj
 0001:00033e70       ?SetKey@?$TAnimTrack@UICharacterKey@@@@UAEXHPAUIKey@@@Z 34034e70 f i AnimNode.obj
 0001:00033ea0       ?SetKeyTime@?$TAnimTrack@UICharacterKey@@@@UAEXHM@Z 34034ea0 f i AnimNode.obj
 0001:00033ec0       ?SetKeyFlags@?$TAnimTrack@UICharacterKey@@@@UAEXHH@Z 34034ec0 f i AnimNode.obj
 0001:00033ee0       ?SerializeSelection@?$TAnimTrack@UICharacterKey@@@@UAE_NAAVXmlNodeRef@@_N1M@Z 34034ee0 f i AnimNode.obj
 0001:000340a0       ??$fill@PAUICharacterKey@@U1@@stlpmtx_std@@YAXPAUICharacterKey@@0ABU1@@Z 340350a0 f i AnimNode.obj
 0001:000340e0       ??$__push_heap@PAUICharacterKey@@HU1@U?$less@UICharacterKey@@@stlpmtx_std@@@stlpmtx_std@@YAXPAUICharacterKey@@HHU1@U?$less@UICharacterKey@@@0@@Z 340350e0 f i AnimNode.obj
 0001:00034140       ?SelectKey@?$TAnimTrack@UICharacterKey@@@@UAEXH_N@Z 34035140 f i AnimNode.obj
 0001:00034180       ?GetNumKeys@?$TAnimTrack@UICharacterKey@@@@UBEHXZ 34035180 f i AnimNode.obj
 0001:000341a0       ?GetKey@?$TAnimTrack@UICharacterKey@@@@UBEXHPAUIKey@@@Z 340351a0 f i AnimNode.obj
 0001:000341c0       ?GetKeyTime@?$TAnimTrack@UICharacterKey@@@@UBEMH@Z 340351c0 f i AnimNode.obj
 0001:000341e0       ??$__unguarded_insertion_sort_aux@PAUICharacterKey@@U1@U?$less@UICharacterKey@@@stlpmtx_std@@@priv@stlpmtx_std@@YAXPAUICharacterKey@@00U?$less@UICharacterKey@@@1@@Z 340351e0 f i AnimNode.obj
 0001:00034240       ??$__adjust_heap@PAUICharacterKey@@HU1@U?$less@UICharacterKey@@@stlpmtx_std@@@stlpmtx_std@@YAXPAUICharacterKey@@HHU1@U?$less@UICharacterKey@@@0@@Z 34035240 f i AnimNode.obj
 0001:000342e0       ?IsKeySelected@?$TAnimTrack@UICharacterKey@@@@UBE_NH@Z 340352e0 f i AnimNode.obj
 0001:00034300       ?_M_insert_overflow@?$_Impl_vector@UICharacterKey@@V?$allocator@UICharacterKey@@@stlpmtx_std@@@priv@stlpmtx_std@@AAEXPAUICharacterKey@@ABU4@ABU__true_type@3@I_N@Z 34035300 f i AnimNode.obj
 0001:00034480       ??$__uninitialized_fill_n@PAUICharacterKey@@IU1@@priv@stlpmtx_std@@YAPAUICharacterKey@@PAU2@IABU2@@Z 34035480 f i AnimNode.obj
 0001:000344e0       ??$__unguarded_partition@PAUICharacterKey@@U1@U?$less@UICharacterKey@@@stlpmtx_std@@@priv@stlpmtx_std@@YAPAUICharacterKey@@PAU2@0U2@U?$less@UICharacterKey@@@1@@Z 340354e0 f i AnimNode.obj
 0001:00034540       ??$__make_heap@PAUICharacterKey@@U?$less@UICharacterKey@@@stlpmtx_std@@U1@H@stlpmtx_std@@YAXPAUICharacterKey@@0U?$less@UICharacterKey@@@0@0PAH@Z 34035540 f i AnimNode.obj
 0001:00034660       ?_M_fill_insert_aux@?$_Impl_vector@UICharacterKey@@V?$allocator@UICharacterKey@@@stlpmtx_std@@@priv@stlpmtx_std@@AAEXPAUICharacterKey@@IABU4@ABU__false_type@3@@Z 34035660 f i AnimNode.obj
 0001:00034780       ??$__insertion_sort@PAUICharacterKey@@U1@U?$less@UICharacterKey@@@stlpmtx_std@@@priv@stlpmtx_std@@YAXPAUICharacterKey@@00U?$less@UICharacterKey@@@1@@Z 34035780 f i AnimNode.obj
 0001:00034840       ?RemoveKey@?$TAnimTrack@UICharacterKey@@@@UAEXH@Z 34035840 f i AnimNode.obj
 0001:000348a0       ??$__final_insertion_sort@PAUICharacterKey@@U?$less@UICharacterKey@@@stlpmtx_std@@@priv@stlpmtx_std@@YAXPAUICharacterKey@@0U?$less@UICharacterKey@@@1@@Z 340358a0 f i AnimNode.obj
 0001:00034910       ??$sort_heap@PAUICharacterKey@@U?$less@UICharacterKey@@@stlpmtx_std@@@stlpmtx_std@@YAXPAUICharacterKey@@0U?$less@UICharacterKey@@@0@@Z 34035910 f i AnimNode.obj
 0001:000349d0       ?insert@?$_Impl_vector@UICharacterKey@@V?$allocator@UICharacterKey@@@stlpmtx_std@@@priv@stlpmtx_std@@QAEXPAUICharacterKey@@IABU4@@Z 340359d0 f i AnimNode.obj
 0001:00034a30       ?CreateKey@?$TAnimTrack@UIBoolKey@@@@UAEHM@Z 34035a30 f i AnimNode.obj
 0001:00034a90       ?CloneKey@?$TAnimTrack@UIBoolKey@@@@UAEHH@Z 34035a90 f i AnimNode.obj
 0001:00034af0       ?CopyKey@?$TAnimTrack@UIBoolKey@@@@UAEHPAUIAnimTrack@@H@Z 34035af0 f i AnimNode.obj
 0001:00034b50       ?FindKey@?$TAnimTrack@UIBoolKey@@@@UAEHM@Z 34035b50 f i AnimNode.obj
 0001:00034ba0       ?GetKeyFlags@?$TAnimTrack@UIBoolKey@@@@UAEHH@Z 34035ba0 f i AnimNode.obj
 0001:00034bc0       ?SetKey@?$TAnimTrack@UIBoolKey@@@@UAEXHPAUIKey@@@Z 34035bc0 f i AnimNode.obj
 0001:00034bf0       ?SetKeyTime@?$TAnimTrack@UIBoolKey@@@@UAEXHM@Z 34035bf0 f i AnimNode.obj
 0001:00034c10       ?SetKeyFlags@?$TAnimTrack@UIBoolKey@@@@UAEXHH@Z 34035c10 f i AnimNode.obj
 0001:00034c30       ?Serialize@?$TAnimTrack@UIBoolKey@@@@UAE_NAAVXmlNodeRef@@_N1@Z 34035c30 f i AnimNode.obj
 0001:00034ef0       ?SerializeSelection@?$TAnimTrack@UIBoolKey@@@@UAE_NAAVXmlNodeRef@@_N1M@Z 34035ef0 f i AnimNode.obj
 0001:000350c0       ?SelectKey@?$TAnimTrack@UIBoolKey@@@@UAEXH_N@Z 340360c0 f i AnimNode.obj
 0001:000350f0       ?GetNumKeys@?$TAnimTrack@UIBoolKey@@@@UBEHXZ 340360f0 f i AnimNode.obj
 0001:00035100       ?GetKey@?$TAnimTrack@UIBoolKey@@@@UBEXHPAUIKey@@@Z 34036100 f i AnimNode.obj
 0001:00035120       ?GetKeyTime@?$TAnimTrack@UIBoolKey@@@@UBEMH@Z 34036120 f i AnimNode.obj
 0001:00035130       ??$__unguarded_insertion_sort_aux@PAUIBoolKey@@U1@U?$less@UIBoolKey@@@stlpmtx_std@@@priv@stlpmtx_std@@YAXPAUIBoolKey@@00U?$less@UIBoolKey@@@1@@Z 34036130 f i AnimNode.obj
 0001:00035190       ??$__adjust_heap@PAUIBoolKey@@HU1@U?$less@UIBoolKey@@@stlpmtx_std@@@stlpmtx_std@@YAXPAUIBoolKey@@HHU1@U?$less@UIBoolKey@@@0@@Z 34036190 f i AnimNode.obj
 0001:00035240       ?IsKeySelected@?$TAnimTrack@UIBoolKey@@@@UBE_NH@Z 34036240 f i AnimNode.obj
 0001:00035260       ?_M_insert_overflow@?$_Impl_vector@UIBoolKey@@V?$allocator@UIBoolKey@@@stlpmtx_std@@@priv@stlpmtx_std@@AAEXPAUIBoolKey@@ABU4@ABU__true_type@3@I_N@Z 34036260 f i AnimNode.obj
 0001:000353c0       ??$__uninitialized_fill_n@PAUIBoolKey@@IU1@@priv@stlpmtx_std@@YAPAUIBoolKey@@PAU2@IABU2@@Z 340363c0 f i AnimNode.obj
 0001:00035400       ??$__make_heap@PAUIBoolKey@@U?$less@UIBoolKey@@@stlpmtx_std@@U1@H@stlpmtx_std@@YAXPAUIBoolKey@@0U?$less@UIBoolKey@@@0@0PAH@Z 34036400 f i AnimNode.obj
 0001:000354f0       ?_M_fill_insert_aux@?$_Impl_vector@UIBoolKey@@V?$allocator@UIBoolKey@@@stlpmtx_std@@@priv@stlpmtx_std@@AAEXPAUIBoolKey@@IABU4@ABU__false_type@3@@Z 340364f0 f i AnimNode.obj
 0001:00035630       ??$__insertion_sort@PAUIBoolKey@@U1@U?$less@UIBoolKey@@@stlpmtx_std@@@priv@stlpmtx_std@@YAXPAUIBoolKey@@00U?$less@UIBoolKey@@@1@@Z 34036630 f i AnimNode.obj
 0001:000356e0       ?RemoveKey@?$TAnimTrack@UIBoolKey@@@@UAEXH@Z 340366e0 f i AnimNode.obj
 0001:00035740       ??$sort_heap@PAUIBoolKey@@U?$less@UIBoolKey@@@stlpmtx_std@@@stlpmtx_std@@YAXPAUIBoolKey@@0U?$less@UIBoolKey@@@0@@Z 34036740 f i AnimNode.obj
 0001:000357a0       ?SetSelected@?$TAnimTrack@UISoundKey@@@@UAEX_N@Z 340367a0 f i AnimNode.obj
 0001:000357a0       ?SetSelected@?$TAnimTrack@UIDiscreteFloatKey@@@@UAEX_N@Z 340367a0 f i GotoTrack.obj
 0001:000357a0       ?SetSelected@?$TAnimTrack@UIScreenFaderKey@@@@UAEX_N@Z 340367a0 f i ScreenFaderTrack.obj
 0001:000357a0       ?SetSelected@?$TAnimTrack@UIMusicKey@@@@UAEX_N@Z 340367a0 f i AnimNode.obj
 0001:000357a0       ?SetSelected@?$TAnimTrack@UISelectKey@@@@UAEX_N@Z 340367a0 f i AnimNode.obj
 0001:000357a0       ?SetSelected@?$TAnimTrack@UIBoolKey@@@@UAEX_N@Z 340367a0 f i AnimNode.obj
 0001:000357a0       ?SetSelected@?$TAnimTrack@UICharacterKey@@@@UAEX_N@Z 340367a0 f i AnimNode.obj
 0001:000357a0       ?SetSelected@?$TAnimTrack@UISequenceKey@@@@UAEX_N@Z 340367a0 f i AnimNode.obj
 0001:000357a0       ?SetSelected@?$TAnimTrack@UIExprKey@@@@UAEX_N@Z 340367a0 f i AnimNode.obj
 0001:000357a0       ?SetSelected@?$TAnimTrack@UIEventKey@@@@UAEX_N@Z 340367a0 f i AnimNode.obj
 0001:000357a0       ?SetSelected@?$TAnimTrack@UICaptureKey@@@@UAEX_N@Z 340367a0 f i AnimNode.obj
 0001:000357a0       ?SetSelected@?$TAnimTrack@UILookAtKey@@@@UAEX_N@Z 340367a0 f i AnimNode.obj
 0001:000357a0       ?SetSelected@?$TAnimTrack@UIConsoleKey@@@@UAEX_N@Z 340367a0 f i AnimNode.obj
 0001:000357a0       ?SetSelected@?$TAnimTrack@UIFaceSeqKey@@@@UAEX_N@Z 340367a0 f i AnimNode.obj
 0001:000357a0       ?SetSelected@?$TAnimTrack@UICommentKey@@@@UAEX_N@Z 340367a0 f i CommentTrack.obj
 0001:000357c0       ?CreateKey@?$TAnimTrack@UISelectKey@@@@UAEHM@Z 340367c0 f i AnimNode.obj
 0001:00035830       ?CloneKey@?$TAnimTrack@UISelectKey@@@@UAEHH@Z 34036830 f i AnimNode.obj
 0001:000358b0       ?CopyKey@?$TAnimTrack@UISelectKey@@@@UAEHPAUIAnimTrack@@H@Z 340368b0 f i AnimNode.obj
 0001:00035930       ?SetCustomColor@?$TAnimTrack@UISequenceKey@@@@UAEXU?$Color_tpl@E@@@Z 34036930 f i AnimNode.obj
 0001:00035930       ?SetCustomColor@?$TAnimTrack@UISelectKey@@@@UAEXU?$Color_tpl@E@@@Z 34036930 f i AnimNode.obj
 0001:00035930       ?SetCustomColor@?$TAnimTrack@UICommentKey@@@@UAEXU?$Color_tpl@E@@@Z 34036930 f i CommentTrack.obj
 0001:00035930       ?SetCustomColor@?$TAnimTrack@UIScreenFaderKey@@@@UAEXU?$Color_tpl@E@@@Z 34036930 f i ScreenFaderTrack.obj
 0001:00035930       ?SetCustomColor@?$TAnimTrack@UIExprKey@@@@UAEXU?$Color_tpl@E@@@Z 34036930 f i AnimNode.obj
 0001:00035930       ?SetCustomColor@?$TAnimTrack@UIDiscreteFloatKey@@@@UAEXU?$Color_tpl@E@@@Z 34036930 f i GotoTrack.obj
 0001:00035930       ?SetCustomColor@?$TAnimTrack@UIFaceSeqKey@@@@UAEXU?$Color_tpl@E@@@Z 34036930 f i AnimNode.obj
 0001:00035930       ?SetCustomColor@?$TAnimTrack@UICharacterKey@@@@UAEXU?$Color_tpl@E@@@Z 34036930 f i AnimNode.obj
 0001:00035930       ?SetCustomColor@?$TAnimTrack@UICaptureKey@@@@UAEXU?$Color_tpl@E@@@Z 34036930 f i AnimNode.obj
 0001:00035930       ?SetCustomColor@?$TAnimTrack@UISoundKey@@@@UAEXU?$Color_tpl@E@@@Z 34036930 f i AnimNode.obj
 0001:00035930       ?SetCustomColor@?$TAnimTrack@UIEventKey@@@@UAEXU?$Color_tpl@E@@@Z 34036930 f i AnimNode.obj
 0001:00035930       ?SetCustomColor@?$TAnimTrack@UIMusicKey@@@@UAEXU?$Color_tpl@E@@@Z 34036930 f i AnimNode.obj
 0001:00035930       ?SetCustomColor@?$TAnimTrack@UIConsoleKey@@@@UAEXU?$Color_tpl@E@@@Z 34036930 f i AnimNode.obj
 0001:00035930       ?SetCustomColor@?$TAnimTrack@UIBoolKey@@@@UAEXU?$Color_tpl@E@@@Z 34036930 f i AnimNode.obj
 0001:00035930       ?SetCustomColor@?$TAnimTrack@UILookAtKey@@@@UAEXU?$Color_tpl@E@@@Z 34036930 f i AnimNode.obj
 0001:00035960       ?FindKey@?$TAnimTrack@UISelectKey@@@@UAEHM@Z 34036960 f i AnimNode.obj
 0001:000359c0       ?GetKeyFlags@?$TAnimTrack@UISelectKey@@@@UAEHH@Z 340369c0 f i AnimNode.obj
 0001:000359e0       ?SetKey@?$TAnimTrack@UISelectKey@@@@UAEXHPAUIKey@@@Z 340369e0 f i AnimNode.obj
 0001:00035a10       ?SetKeyTime@?$TAnimTrack@UISelectKey@@@@UAEXHM@Z 34036a10 f i AnimNode.obj
 0001:00035a30       ?SetKeyFlags@?$TAnimTrack@UISelectKey@@@@UAEXHH@Z 34036a30 f i AnimNode.obj
 0001:00035a50       ?Serialize@?$TAnimTrack@UISelectKey@@@@UAE_NAAVXmlNodeRef@@_N1@Z 34036a50 f i AnimNode.obj
 0001:00035d00       ?SerializeSelection@?$TAnimTrack@UISelectKey@@@@UAE_NAAVXmlNodeRef@@_N1M@Z 34036d00 f i AnimNode.obj
 0001:00035ee0       ??$fill@PAUISelectKey@@U1@@stlpmtx_std@@YAXPAUISelectKey@@0ABU1@@Z 34036ee0 f i AnimNode.obj
 0001:00035f30       ??$__push_heap@PAUISelectKey@@HU1@U?$less@UISelectKey@@@stlpmtx_std@@@stlpmtx_std@@YAXPAUISelectKey@@HHU1@U?$less@UISelectKey@@@0@@Z 34036f30 f i AnimNode.obj
 0001:00035f90       ?SelectKey@?$TAnimTrack@UISelectKey@@@@UAEXH_N@Z 34036f90 f i AnimNode.obj
 0001:00035fd0       ?GetNumKeys@?$TAnimTrack@UISelectKey@@@@UBEHXZ 34036fd0 f i AnimNode.obj
 0001:00035ff0       ?GetKey@?$TAnimTrack@UISelectKey@@@@UBEXHPAUIKey@@@Z 34036ff0 f i AnimNode.obj
 0001:00036020       ?GetKeyTime@?$TAnimTrack@UISelectKey@@@@UBEMH@Z 34037020 f i AnimNode.obj
 0001:00036040       ??$__unguarded_insertion_sort_aux@PAUISelectKey@@U1@U?$less@UISelectKey@@@stlpmtx_std@@@priv@stlpmtx_std@@YAXPAUISelectKey@@00U?$less@UISelectKey@@@1@@Z 34037040 f i AnimNode.obj
 0001:000360c0       ??$__adjust_heap@PAUISelectKey@@HU1@U?$less@UISelectKey@@@stlpmtx_std@@@stlpmtx_std@@YAXPAUISelectKey@@HHU1@U?$less@UISelectKey@@@0@@Z 340370c0 f i AnimNode.obj
 0001:00036170       ?IsKeySelected@?$TAnimTrack@UISelectKey@@@@UBE_NH@Z 34037170 f i AnimNode.obj
 0001:00036190       ?_M_insert_overflow@?$_Impl_vector@UISelectKey@@V?$allocator@UISelectKey@@@stlpmtx_std@@@priv@stlpmtx_std@@AAEXPAUISelectKey@@ABU4@ABU__true_type@3@I_N@Z 34037190 f i AnimNode.obj
 0001:00036310       ??$__uninitialized_fill_n@PAUISelectKey@@IU1@@priv@stlpmtx_std@@YAPAUISelectKey@@PAU2@IABU2@@Z 34037310 f i AnimNode.obj
 0001:00036370       ??$__unguarded_partition@PAUISelectKey@@U1@U?$less@UISelectKey@@@stlpmtx_std@@@priv@stlpmtx_std@@YAPAUISelectKey@@PAU2@0U2@U?$less@UISelectKey@@@1@@Z 34037370 f i AnimNode.obj
 0001:000363e0       ??$__make_heap@PAUISelectKey@@U?$less@UISelectKey@@@stlpmtx_std@@U1@H@stlpmtx_std@@YAXPAUISelectKey@@0U?$less@UISelectKey@@@0@0PAH@Z 340373e0 f i AnimNode.obj
 0001:00036530       ?_M_fill_insert_aux@?$_Impl_vector@UISelectKey@@V?$allocator@UISelectKey@@@stlpmtx_std@@@priv@stlpmtx_std@@AAEXPAUISelectKey@@IABU4@ABU__false_type@3@@Z 34037530 f i AnimNode.obj
 0001:00036660       ??$__insertion_sort@PAUISelectKey@@U1@U?$less@UISelectKey@@@stlpmtx_std@@@priv@stlpmtx_std@@YAXPAUISelectKey@@00U?$less@UISelectKey@@@1@@Z 34037660 f i AnimNode.obj
 0001:00036740       ?RemoveKey@?$TAnimTrack@UISelectKey@@@@UAEXH@Z 34037740 f i AnimNode.obj
 0001:000367a0       ??$__final_insertion_sort@PAUISelectKey@@U?$less@UISelectKey@@@stlpmtx_std@@@priv@stlpmtx_std@@YAXPAUISelectKey@@0U?$less@UISelectKey@@@1@@Z 340377a0 f i AnimNode.obj
 0001:00036810       ??$sort_heap@PAUISelectKey@@U?$less@UISelectKey@@@stlpmtx_std@@@stlpmtx_std@@YAXPAUISelectKey@@0U?$less@UISelectKey@@@0@@Z 34037810 f i AnimNode.obj
 0001:000368f0       ?Release@CAnimSequenceGroup@@UAEXXZ 340378f0 f i AnimSequenceGroup.obj
 0001:000368f0       ?Release@?$TAnimTrack@UIFaceSeqKey@@@@UAEXXZ 340378f0 f i AnimNode.obj
 0001:000368f0       ?Release@?$TAnimTrack@UICharacterKey@@@@UAEXXZ 340378f0 f i AnimNode.obj
 0001:000368f0       ?Release@?$TAnimTrack@UIDiscreteFloatKey@@@@UAEXXZ 340378f0 f i GotoTrack.obj
 0001:000368f0       ?Release@?$TAnimSplineTrack@M@@UAEXXZ 340378f0 f i Movie.obj
 0001:000368f0       ?Release@?$TAnimSplineTrack@U?$Vec2_tpl@M@@@@UAEXXZ 340378f0 f i CompoundSplineTrack.obj
 0001:000368f0       ?Release@?$TAnimTrack@UIExprKey@@@@UAEXXZ 340378f0 f i AnimNode.obj
 0001:000368f0       ?Release@?$TAnimTrack@UILookAtKey@@@@UAEXXZ 340378f0 f i AnimNode.obj
 0001:000368f0       ?Release@?$TAnimTrack@UISoundKey@@@@UAEXXZ 340378f0 f i AnimNode.obj
 0001:000368f0       ?Release@?$TAnimTrack@UICommentKey@@@@UAEXXZ 340378f0 f i CommentTrack.obj
 0001:000368f0       ?Release@?$TAnimTrack@UIConsoleKey@@@@UAEXXZ 340378f0 f i AnimNode.obj
 0001:000368f0       ?Release@?$TAnimTrack@UIScreenFaderKey@@@@UAEXXZ 340378f0 f i ScreenFaderTrack.obj
 0001:000368f0       ?Release@?$TAnimSplineTrack@U?$Vec3_tpl@M@@@@UAEXXZ 340378f0 f i Movie.obj
 0001:000368f0       ?Release@?$TAnimSplineTrack@U?$Quat_tpl@M@@@@UAEXXZ 340378f0 f i Movie.obj
 0001:000368f0       ?Release@?$TAnimTrack@UIMusicKey@@@@UAEXXZ 340378f0 f i AnimNode.obj
 0001:000368f0       ?Release@?$TAnimTrack@UICaptureKey@@@@UAEXXZ 340378f0 f i AnimNode.obj
 0001:000368f0       ?Release@CAnimSequence@@UAEXXZ 340378f0 f i AnimSequence.obj
 0001:000368f0       ?Release@CCompoundSplineTrack@@UAEXXZ 340378f0 f i CompoundSplineTrack.obj
 0001:000368f0       ?Release@?$TAnimTrack@UISequenceKey@@@@UAEXXZ 340378f0 f i AnimNode.obj
 0001:000368f0       ?Release@?$TAnimTrack@UIEventKey@@@@UAEXXZ 340378f0 f i AnimNode.obj
 0001:000368f0       ?Release@?$TAnimTrack@UISelectKey@@@@UAEXXZ 340378f0 f i AnimNode.obj
 0001:000368f0       ?Release@?$TAnimTrack@UIBoolKey@@@@UAEXXZ 340378f0 f i AnimNode.obj
 0001:00036910       ?CreateKey@?$TAnimTrack@UIEventKey@@@@UAEHM@Z 34037910 f i AnimNode.obj
 0001:00036990       ?CloneKey@?$TAnimTrack@UIEventKey@@@@UAEHH@Z 34037990 f i AnimNode.obj
 0001:00036a10       ?CopyKey@?$TAnimTrack@UIEventKey@@@@UAEHPAUIAnimTrack@@H@Z 34037a10 f i AnimNode.obj
 0001:00036a90       ?FindKey@?$TAnimTrack@UIEventKey@@@@UAEHM@Z 34037a90 f i AnimNode.obj
 0001:00036af0       ?GetKeyFlags@?$TAnimTrack@UIEventKey@@@@UAEHH@Z 34037af0 f i AnimNode.obj
 0001:00036b10       ?SetKey@?$TAnimTrack@UIEventKey@@@@UAEXHPAUIKey@@@Z 34037b10 f i AnimNode.obj
 0001:00036b40       ?SetKeyTime@?$TAnimTrack@UIEventKey@@@@UAEXHM@Z 34037b40 f i AnimNode.obj
 0001:00036b70       ?SetKeyFlags@?$TAnimTrack@UIEventKey@@@@UAEXHH@Z 34037b70 f i AnimNode.obj
 0001:00036b90       ?Serialize@?$TAnimTrack@UIEventKey@@@@UAE_NAAVXmlNodeRef@@_N1@Z 34037b90 f i AnimNode.obj
 0001:00036e40       ?SerializeSelection@?$TAnimTrack@UIEventKey@@@@UAE_NAAVXmlNodeRef@@_N1M@Z 34037e40 f i AnimNode.obj
 0001:00037010       ??$fill@PAUIEventKey@@U1@@stlpmtx_std@@YAXPAUIEventKey@@0ABU1@@Z 34038010 f i AnimNode.obj
 0001:00037060       ??$__push_heap@PAUIEventKey@@HU1@U?$less@UIEventKey@@@stlpmtx_std@@@stlpmtx_std@@YAXPAUIEventKey@@HHU1@U?$less@UIEventKey@@@0@@Z 34038060 f i AnimNode.obj
 0001:000370d0       ?SelectKey@?$TAnimTrack@UIEventKey@@@@UAEXH_N@Z 340380d0 f i AnimNode.obj
 0001:00037110       ?GetNumKeys@?$TAnimTrack@UIEventKey@@@@UBEHXZ 34038110 f i AnimNode.obj
 0001:00037130       ?GetKey@?$TAnimTrack@UIEventKey@@@@UBEXHPAUIKey@@@Z 34038130 f i AnimNode.obj
 0001:00037160       ?GetKeyTime@?$TAnimTrack@UIEventKey@@@@UBEMH@Z 34038160 f i AnimNode.obj
 0001:00037180       ??$__unguarded_insertion_sort_aux@PAUIEventKey@@U1@U?$less@UIEventKey@@@stlpmtx_std@@@priv@stlpmtx_std@@YAXPAUIEventKey@@00U?$less@UIEventKey@@@1@@Z 34038180 f i AnimNode.obj
 0001:00037200       ??$__adjust_heap@PAUIEventKey@@HU1@U?$less@UIEventKey@@@stlpmtx_std@@@stlpmtx_std@@YAXPAUIEventKey@@HHU1@U?$less@UIEventKey@@@0@@Z 34038200 f i AnimNode.obj
 0001:000372b0       ?IsKeySelected@?$TAnimTrack@UIEventKey@@@@UBE_NH@Z 340382b0 f i AnimNode.obj
 0001:000372d0       ?_M_insert_overflow@?$_Impl_vector@UIEventKey@@V?$allocator@UIEventKey@@@stlpmtx_std@@@priv@stlpmtx_std@@AAEXPAUIEventKey@@ABU4@ABU__true_type@3@I_N@Z 340382d0 f i AnimNode.obj
 0001:00037450       ??$__uninitialized_fill_n@PAUIEventKey@@IU1@@priv@stlpmtx_std@@YAPAUIEventKey@@PAU2@IABU2@@Z 34038450 f i AnimNode.obj
 0001:000374b0       ??$__unguarded_partition@PAUIEventKey@@U1@U?$less@UIEventKey@@@stlpmtx_std@@@priv@stlpmtx_std@@YAPAUIEventKey@@PAU2@0U2@U?$less@UIEventKey@@@1@@Z 340384b0 f i AnimNode.obj
 0001:00037520       ??$__make_heap@PAUIEventKey@@U?$less@UIEventKey@@@stlpmtx_std@@U1@H@stlpmtx_std@@YAXPAUIEventKey@@0U?$less@UIEventKey@@@0@0PAH@Z 34038520 f i AnimNode.obj
 0001:00037650       ?_M_fill_insert_aux@?$_Impl_vector@UIEventKey@@V?$allocator@UIEventKey@@@stlpmtx_std@@@priv@stlpmtx_std@@AAEXPAUIEventKey@@IABU4@ABU__false_type@3@@Z 34038650 f i AnimNode.obj
 0001:00037780       ??$__insertion_sort@PAUIEventKey@@U1@U?$less@UIEventKey@@@stlpmtx_std@@@priv@stlpmtx_std@@YAXPAUIEventKey@@00U?$less@UIEventKey@@@1@@Z 34038780 f i AnimNode.obj
 0001:00037860       ?RemoveKey@?$TAnimTrack@UIEventKey@@@@UAEXH@Z 34038860 f i AnimNode.obj
 0001:000378c0       ??$__final_insertion_sort@PAUIEventKey@@U?$less@UIEventKey@@@stlpmtx_std@@@priv@stlpmtx_std@@YAXPAUIEventKey@@0U?$less@UIEventKey@@@1@@Z 340388c0 f i AnimNode.obj
 0001:00037930       ??$sort_heap@PAUIEventKey@@U?$less@UIEventKey@@@stlpmtx_std@@@stlpmtx_std@@YAXPAUIEventKey@@0U?$less@UIEventKey@@@0@@Z 34038930 f i AnimNode.obj
 0001:00037a10       ?GetParamCount@CAnimNodeGroup@@UBEHXZ 34038a10 f i AnimSequence.obj
 0001:00037a10       ?GetSubTrackCount@?$TAnimTrack@UISelectKey@@@@UBEHXZ 34038a10 f i AnimNode.obj
 0001:00037a10       ?GetSubTrackCount@?$TAnimTrack@UICaptureKey@@@@UBEHXZ 34038a10 f i AnimNode.obj
 0001:00037a10       ?GetSubTrackCount@?$TAnimTrack@UIBoolKey@@@@UBEHXZ 34038a10 f i AnimNode.obj
 0001:00037a10       ?GetValueType@?$TAnimSplineTrack@U?$Vec2_tpl@M@@@@UAE?AW4EAnimValue@@XZ 34038a10 f i CompoundSplineTrack.obj
 0001:00037a10       ?GetSubTrackCount@?$TAnimTrack@UIDiscreteFloatKey@@@@UBEHXZ 34038a10 f i GotoTrack.obj
 0001:00037a10       ?GetSubTrackCount@?$TAnimTrack@UILookAtKey@@@@UBEHXZ 34038a10 f i AnimNode.obj
 0001:00037a10       ?GetSubTrackCount@?$TAnimTrack@UIConsoleKey@@@@UBEHXZ 34038a10 f i AnimNode.obj
 0001:00037a10       ?GetEntityGuid@CAnimNode@@UAEPA_KXZ 34038a10 f i AnimSequence.obj
 0001:00037a10       ?GetSubTrackCount@?$TAnimTrack@UISoundKey@@@@UBEHXZ 34038a10 f i AnimNode.obj
 0001:00037a10       ?GetSubTrackCount@?$TAnimTrack@UIFaceSeqKey@@@@UBEHXZ 34038a10 f i AnimNode.obj
 0001:00037a10       ?GetSubTrackCount@?$TAnimTrack@UIScreenFaderKey@@@@UBEHXZ 34038a10 f i ScreenFaderTrack.obj
 0001:00037a10       ?GetSpline@IAnimTrack@@UBEPAUISplineInterpolator@@XZ 34038a10 f i Movie.obj
 0001:00037a10       ?GetSubTrackCount@?$TAnimTrack@UISequenceKey@@@@UBEHXZ 34038a10 f i AnimNode.obj
 0001:00037a10       ?GetSubTrackCount@?$TAnimSplineTrack@U?$Vec3_tpl@M@@@@UBEHXZ 34038a10 f i Movie.obj
 0001:00037a10       ?GetSubTrackCount@?$TAnimSplineTrack@U?$Vec2_tpl@M@@@@UBEHXZ 34038a10 f i CompoundSplineTrack.obj
 0001:00037a10       ?GetSubTrackCount@?$TAnimTrack@UIExprKey@@@@UBEHXZ 34038a10 f i AnimNode.obj
 0001:00037a10       ?GetSubTrackCount@?$TAnimTrack@UICharacterKey@@@@UBEHXZ 34038a10 f i AnimNode.obj
 0001:00037a10       ?GetSubTrackCount@?$TAnimTrack@UIEventKey@@@@UBEHXZ 34038a10 f i AnimNode.obj
 0001:00037a10       ?GetSubTrackCount@?$TAnimSplineTrack@U?$Quat_tpl@M@@@@UBEHXZ 34038a10 f i Movie.obj
 0001:00037a10       ?GetValueType@?$TAnimSplineTrack@M@@UAE?AW4EAnimValue@@XZ 34038a10 f i Movie.obj
 0001:00037a10       ?GetSubTrackCount@?$TAnimTrack@UICommentKey@@@@UBEHXZ 34038a10 f i CommentTrack.obj
 0001:00037a10       ?GetSubTrackCount@?$TAnimTrack@UIMusicKey@@@@UBEHXZ 34038a10 f i AnimNode.obj
 0001:00037a10       ?GetEntity@CAnimNode@@UAEPAUIEntity@@XZ 34038a10 f i AnimSequence.obj
 0001:00037a10       ?GetSubTrackCount@?$TAnimSplineTrack@M@@UBEHXZ 34038a10 f i Movie.obj
 0001:00037a20       ?SetSubTrackName@?$TAnimTrack@UIConsoleKey@@@@UAEXHPBD@Z 34038a20 f i AnimNode.obj
 0001:00037a20       ?GetValue@?$TAnimSplineTrack@U?$Vec2_tpl@M@@@@UAEXMAA_N@Z 34038a20 f i CompoundSplineTrack.obj
 0001:00037a20       ?GetValue@?$TAnimTrack@UIFaceSeqKey@@@@UAEXMAAM@Z 34038a20 f i AnimNode.obj
 0001:00037a20       ?GetValue@?$TAnimTrack@UIDiscreteFloatKey@@@@UAEXMAAM@Z 34038a20 f i GotoTrack.obj
 0001:00037a20       ?GetValue@?$TAnimSplineTrack@U?$Vec3_tpl@M@@@@UAEXMAAM@Z 34038a20 f i Movie.obj
 0001:00037a20       ?GetValue@?$TAnimTrack@UIScreenFaderKey@@@@UAEXMAAM@Z 34038a20 f i ScreenFaderTrack.obj
 0001:00037a20       ?GetValue@?$TAnimTrack@UISequenceKey@@@@UAEXMAAU?$Quat_tpl@M@@@Z 34038a20 f i AnimNode.obj
 0001:00037a20       ?GetValue@?$TAnimTrack@UICaptureKey@@@@UAEXMAA_N@Z 34038a20 f i AnimNode.obj
 0001:00037a20       ?GetValue@?$TAnimTrack@UISoundKey@@@@UAEXMAAM@Z 34038a20 f i AnimNode.obj
 0001:00037a20       ?SetPos@CAnimNode@@UAEXMABU?$Vec3_tpl@M@@@Z 34038a20 f i AnimSequence.obj
 0001:00037a20       ?SetSubTrackName@?$TAnimTrack@UIExprKey@@@@UAEXHPBD@Z 34038a20 f i AnimNode.obj
 0001:00037a20       ?UnMarkBucket@CDummyMemReplay@@UAEXHPAX@Z 34038a20 f i AnimSequence.obj
 0001:00037a20       ?SetSubTrackName@?$TAnimTrack@UICaptureKey@@@@UAEXHPBD@Z 34038a20 f i AnimNode.obj
 0001:00037a20       ?SetSubTrackName@?$TAnimTrack@UIBoolKey@@@@UAEXHPBD@Z 34038a20 f i AnimNode.obj
 0001:00037a20       ?GetValue@?$TAnimTrack@UIDiscreteFloatKey@@@@UAEXMAAU?$Vec3_tpl@M@@@Z 34038a20 f i GotoTrack.obj
 0001:00037a20       ?GetValue@?$TAnimTrack@UIExprKey@@@@UAEXMAAM@Z 34038a20 f i AnimNode.obj
 0001:00037a20       ?GetValue@?$TAnimTrack@UIDiscreteFloatKey@@@@UAEXMAA_N@Z 34038a20 f i GotoTrack.obj
 0001:00037a20       ?SetSubTrackName@?$TAnimTrack@UIFaceSeqKey@@@@UAEXHPBD@Z 34038a20 f i AnimNode.obj
 0001:00037a20       ?Start@CDummyMemReplay@@UAEX_NPBD@Z 34038a20 f i AnimSequence.obj
 0001:00037a20       ?GetValue@?$TAnimTrack@UISelectKey@@@@UAEXMAAM@Z 34038a20 f i AnimNode.obj
 0001:00037a20       ?GetValue@?$TAnimTrack@UICommentKey@@@@UAEXMAAU?$Quat_tpl@M@@@Z 34038a20 f i CommentTrack.obj
 0001:00037a20       ?SerializeSpline@?$TrackSplineInterpolator@U?$Quat_tpl@M@@@spline@@UAEXAAVXmlNodeRef@@_N@Z 34038a20 f i Movie.obj
 0001:00037a20       ?SetSubTrackName@?$TAnimSplineTrack@M@@UAEXHPBD@Z 34038a20 f i Movie.obj
 0001:00037a20       ?SetKeyFlags@CCompoundSplineTrack@@UAEXHH@Z 34038a20 f i CompoundSplineTrack.obj
 0001:00037a20       ?GetValue@?$TAnimSplineTrack@U?$Quat_tpl@M@@@@UAEXMAAU?$Vec3_tpl@M@@@Z 34038a20 f i Movie.obj
 0001:00037a20       ?GetValue@?$TAnimTrack@UISoundKey@@@@UAEXMAA_N@Z 34038a20 f i AnimNode.obj
 0001:00037a20       ?GetValue@?$TAnimSplineTrack@U?$Vec2_tpl@M@@@@UAEXMAAU?$Vec3_tpl@M@@@Z 34038a20 f i CompoundSplineTrack.obj
 0001:00037a20       ?GetValue@?$TAnimTrack@UILookAtKey@@@@UAEXMAA_N@Z 34038a20 f i AnimNode.obj
 0001:00037a20       ?SerializeSpline@?$TrackSplineInterpolator@U?$Vec3_tpl@M@@@spline@@UAEXAAVXmlNodeRef@@_N@Z 34038a20 f i Movie.obj
 0001:00037a20       ?GetValue@?$TAnimTrack@UILookAtKey@@@@UAEXMAAM@Z 34038a20 f i AnimNode.obj
 0001:00037a20       ?GetValue@?$TAnimTrack@UIEventKey@@@@UAEXMAAU?$Vec3_tpl@M@@@Z 34038a20 f i AnimNode.obj
 0001:00037a20       ?GetValue@?$TAnimTrack@UIExprKey@@@@UAEXMAAU?$Quat_tpl@M@@@Z 34038a20 f i AnimNode.obj
 0001:00037a20       ?GetValue@?$TAnimSplineTrack@U?$Vec2_tpl@M@@@@UAEXMAAU?$Quat_tpl@M@@@Z 34038a20 f i CompoundSplineTrack.obj
 0001:00037a20       ?GetValue@?$TAnimTrack@UICharacterKey@@@@UAEXMAAU?$Quat_tpl@M@@@Z 34038a20 f i AnimNode.obj
 0001:00037a20       ?SetRotate@CAnimNode@@UAEXMABU?$Quat_tpl@M@@@Z 34038a20 f i AnimSequence.obj
 0001:00037a20       ?GetValue@?$TAnimTrack@UIExprKey@@@@UAEXMAAU?$Vec3_tpl@M@@@Z 34038a20 f i AnimNode.obj
 0001:00037a20       ?SetSubTrackName@?$TAnimTrack@UICharacterKey@@@@UAEXHPBD@Z 34038a20 f i AnimNode.obj
 0001:00037a20       ?UnMapPage@CDummyMemReplay@@UAEXPAXI@Z 34038a20 f i AnimSequence.obj
 0001:00037a20       ?GetValue@?$TAnimSplineTrack@M@@UAEXMAAU?$Vec3_tpl@M@@@Z 34038a20 f i Movie.obj
 0001:00037a20       ?SetSubTrackName@?$TAnimTrack@UICommentKey@@@@UAEXHPBD@Z 34038a20 f i CommentTrack.obj
 0001:00037a20       ?SetSubTrackName@?$TAnimTrack@UISoundKey@@@@UAEXHPBD@Z 34038a20 f i AnimNode.obj
 0001:00037a20       ?GetValue@?$TAnimTrack@UIDiscreteFloatKey@@@@UAEXMAAU?$Quat_tpl@M@@@Z 34038a20 f i GotoTrack.obj
 0001:00037a20       ?SetSubTrackName@?$TAnimTrack@UIScreenFaderKey@@@@UAEXHPBD@Z 34038a20 f i ScreenFaderTrack.obj
 0001:00037a20       ?GetKey@CCompoundSplineTrack@@UBEXHPAUIKey@@@Z 34038a20 f i CompoundSplineTrack.obj
 0001:00037a20       ?SetKey@CCompoundSplineTrack@@UAEXHPAUIKey@@@Z 34038a20 f i CompoundSplineTrack.obj
 0001:00037a20       ?UnMarkPool@CDummyMemReplay@@UAEXHPAX@Z 34038a20 f i AnimSequence.obj
 0001:00037a20       ?GetValue@?$TAnimTrack@UIConsoleKey@@@@UAEXMAAU?$Quat_tpl@M@@@Z 34038a20 f i AnimNode.obj
 0001:00037a20       ?GetValue@?$TAnimTrack@UIScreenFaderKey@@@@UAEXMAA_N@Z 34038a20 f i ScreenFaderTrack.obj
 0001:00037a20       ?SetSubTrackName@?$TAnimTrack@UISequenceKey@@@@UAEXHPBD@Z 34038a20 f i AnimNode.obj
 0001:00037a20       ?GetValue@?$TAnimTrack@UICaptureKey@@@@UAEXMAAU?$Vec3_tpl@M@@@Z 34038a20 f i AnimNode.obj
 0001:00037a20       ?SetSubTrackName@?$TAnimTrack@UIMusicKey@@@@UAEXHPBD@Z 34038a20 f i AnimNode.obj
 0001:00037a20       ?GetValue@?$TAnimTrack@UISequenceKey@@@@UAEXMAAM@Z 34038a20 f i AnimNode.obj
 0001:00037a20       ?SetSubTrackName@?$TAnimSplineTrack@U?$Quat_tpl@M@@@@UAEXHPBD@Z 34038a20 f i Movie.obj
 0001:00037a20       ?GetValue@?$TAnimTrack@UICommentKey@@@@UAEXMAAM@Z 34038a20 f i CommentTrack.obj
 0001:00037a20       ?GetValue@?$TAnimTrack@UICaptureKey@@@@UAEXMAAM@Z 34038a20 f i AnimNode.obj
 0001:00037a20       ?GetValue@?$TAnimSplineTrack@U?$Quat_tpl@M@@@@UAEXMAAM@Z 34038a20 f i Movie.obj
 0001:00037a20       ?GetValue@?$TAnimTrack@UISoundKey@@@@UAEXMAAU?$Vec3_tpl@M@@@Z 34038a20 f i AnimNode.obj
 0001:00037a20       ?GetValue@CCompoundSplineTrack@@UAEXMAA_N@Z 34038a20 f i CompoundSplineTrack.obj
 0001:00037a20       ?AddAllocReference@CDummyMemReplay@@UAEXPAX0@Z 34038a20 f i AnimSequence.obj
 0001:00037a20       ?SetSubTrackName@?$TAnimSplineTrack@U?$Vec2_tpl@M@@@@UAEXHPBD@Z 34038a20 f i CompoundSplineTrack.obj
 0001:00037a20       ?GetValue@?$TAnimTrack@UIBoolKey@@@@UAEXMAAU?$Quat_tpl@M@@@Z 34038a20 f i AnimNode.obj
 0001:00037a20       ?GetValue@?$TAnimTrack@UIMusicKey@@@@UAEXMAA_N@Z 34038a20 f i AnimNode.obj
 0001:00037a20       ?GetValue@?$TAnimTrack@UISoundKey@@@@UAEXMAAU?$Quat_tpl@M@@@Z 34038a20 f i AnimNode.obj
 0001:00037a20       ?BucketEnableCleanups@CDummyMemReplay@@UAEXPAX_N@Z 34038a20 f i AnimSequence.obj
 0001:00037a20       ?GetValue@?$TAnimTrack@UIMusicKey@@@@UAEXMAAU?$Vec3_tpl@M@@@Z 34038a20 f i AnimNode.obj
 0001:00037a20       ?BindToContainer@CDummyMemReplay@@UAEXPBX0@Z 34038a20 f i AnimSequence.obj
 0001:00037a20       ?GetValue@?$TAnimTrack@UIExprKey@@@@UAEXMAA_N@Z 34038a20 f i AnimNode.obj
 0001:00037a20       ?GetValue@?$TAnimSplineTrack@U?$Quat_tpl@M@@@@UAEXMAA_N@Z 34038a20 f i Movie.obj
 0001:00037a20       ?GetValue@?$TAnimTrack@UISelectKey@@@@UAEXMAA_N@Z 34038a20 f i AnimNode.obj
 0001:00037a20       ?GetValue@?$TAnimTrack@UIEventKey@@@@UAEXMAA_N@Z 34038a20 f i AnimNode.obj
 0001:00037a20       ?SetSubTrackName@?$TAnimTrack@UISelectKey@@@@UAEXHPBD@Z 34038a20 f i AnimNode.obj
 0001:00037a20       ?GetValue@?$TAnimTrack@UIScreenFaderKey@@@@UAEXMAAU?$Quat_tpl@M@@@Z 34038a20 f i ScreenFaderTrack.obj
 0001:00037a20       ?GetValue@?$TAnimTrack@UILookAtKey@@@@UAEXMAAU?$Vec3_tpl@M@@@Z 34038a20 f i AnimNode.obj
 0001:00037a20       ?GetValue@?$TAnimTrack@UISequenceKey@@@@UAEXMAA_N@Z 34038a20 f i AnimNode.obj
 0001:00037a20       ?GetValue@?$TAnimTrack@UISequenceKey@@@@UAEXMAAU?$Vec3_tpl@M@@@Z 34038a20 f i AnimNode.obj
 0001:00037a20       ?GetValue@?$TAnimTrack@UILookAtKey@@@@UAEXMAAU?$Quat_tpl@M@@@Z 34038a20 f i AnimNode.obj
 0001:00037a20       ?GetValue@?$TAnimTrack@UIScreenFaderKey@@@@UAEXMAAU?$Vec3_tpl@M@@@Z 34038a20 f i ScreenFaderTrack.obj
 0001:00037a20       ?SwapContainers@CDummyMemReplay@@UAEXPBX0@Z 34038a20 f i AnimSequence.obj
 0001:00037a20       ?GetValue@?$TAnimTrack@UIBoolKey@@@@UAEXMAAU?$Vec3_tpl@M@@@Z 34038a20 f i AnimNode.obj
 0001:00037a20       ?SerializeSpline@?$TrackSplineInterpolator@M@spline@@UAEXAAVXmlNodeRef@@_N@Z 34038a20 f i Movie.obj
 0001:00037a20       ?SetScale@CAnimNode@@UAEXMABU?$Vec3_tpl@M@@@Z 34038a20 f i AnimSequence.obj
 0001:00037a20       ?GetValue@?$TAnimTrack@UIMusicKey@@@@UAEXMAAM@Z 34038a20 f i AnimNode.obj
 0001:00037a20       ?GetValue@?$TAnimTrack@UISelectKey@@@@UAEXMAAU?$Quat_tpl@M@@@Z 34038a20 f i AnimNode.obj
 0001:00037a20       ?GetValue@?$TAnimTrack@UIConsoleKey@@@@UAEXMAA_N@Z 34038a20 f i AnimNode.obj
 0001:00037a20       ?GetValue@?$TAnimTrack@UIFaceSeqKey@@@@UAEXMAA_N@Z 34038a20 f i AnimNode.obj
 0001:00037a20       ?GetValue@?$TAnimTrack@UIMusicKey@@@@UAEXMAAU?$Quat_tpl@M@@@Z 34038a20 f i AnimNode.obj
 0001:00037a20       ?GetValue@?$TAnimTrack@UIConsoleKey@@@@UAEXMAAU?$Vec3_tpl@M@@@Z 34038a20 f i AnimNode.obj
 0001:00037a20       ?GetValue@?$TAnimTrack@UIEventKey@@@@UAEXMAAM@Z 34038a20 f i AnimNode.obj
 0001:00037a20       ?GetValue@?$TAnimTrack@UISelectKey@@@@UAEXMAAU?$Vec3_tpl@M@@@Z 34038a20 f i AnimNode.obj
 0001:00037a20       ?GetValue@?$TAnimTrack@UICharacterKey@@@@UAEXMAAU?$Vec3_tpl@M@@@Z 34038a20 f i AnimNode.obj
 0001:00037a20       ?GetValue@?$TAnimSplineTrack@M@@UAEXMAA_N@Z 34038a20 f i Movie.obj
 0001:00037a20       ?GetValue@?$TAnimTrack@UICommentKey@@@@UAEXMAAU?$Vec3_tpl@M@@@Z 34038a20 f i CommentTrack.obj
 0001:00037a20       ?GetValue@?$TAnimSplineTrack@U?$Vec3_tpl@M@@@@UAEXMAAU?$Quat_tpl@M@@@Z 34038a20 f i Movie.obj
 0001:00037a20       ?GetValue@?$TAnimTrack@UIBoolKey@@@@UAEXMAA_N@Z 34038a20 f i AnimNode.obj
 0001:00037a20       ?GetValue@?$TAnimTrack@UIConsoleKey@@@@UAEXMAAM@Z 34038a20 f i AnimNode.obj
 0001:00037a20       ?GetValue@?$TAnimSplineTrack@U?$Vec3_tpl@M@@@@UAEXMAA_N@Z 34038a20 f i Movie.obj
 0001:00037a20       ?SetSubTrackName@?$TAnimTrack@UIDiscreteFloatKey@@@@UAEXHPBD@Z 34038a20 f i GotoTrack.obj
 0001:00037a20       ?UnbindFromContainer@CDummyMemReplay@@UAEXPBX0@Z 34038a20 f i AnimSequence.obj
 0001:00037a20       ?GetValue@?$TAnimTrack@UIFaceSeqKey@@@@UAEXMAAU?$Vec3_tpl@M@@@Z 34038a20 f i AnimNode.obj
 0001:00037a20       ?SetSubTrackName@?$TAnimSplineTrack@U?$Vec3_tpl@M@@@@UAEXHPBD@Z 34038a20 f i Movie.obj
 0001:00037a20       ?GetValue@?$TAnimTrack@UICaptureKey@@@@UAEXMAAU?$Quat_tpl@M@@@Z 34038a20 f i AnimNode.obj
 0001:00037a20       ?GetValue@?$TAnimTrack@UICommentKey@@@@UAEXMAA_N@Z 34038a20 f i CommentTrack.obj
 0001:00037a20       ?GetValue@?$TAnimTrack@UICharacterKey@@@@UAEXMAAM@Z 34038a20 f i AnimNode.obj
 0001:00037a20       ?MapPage@CDummyMemReplay@@UAEXPAXI@Z 34038a20 f i AnimSequence.obj
 0001:00037a20       ?RegisterContainer@CDummyMemReplay@@UAEXPBXH@Z 34038a20 f i AnimSequence.obj
 0001:00037a20       ?SerializeSpline@?$TrackSplineInterpolator@U?$Vec2_tpl@M@@@spline@@UAEXAAVXmlNodeRef@@_N@Z 34038a20 f i CompoundSplineTrack.obj
 0001:00037a20       ?SetSubTrackName@?$TAnimTrack@UIEventKey@@@@UAEXHPBD@Z 34038a20 f i AnimNode.obj
 0001:00037a20       ?SetSubTrackName@?$TAnimTrack@UILookAtKey@@@@UAEXHPBD@Z 34038a20 f i AnimNode.obj
 0001:00037a20       ?GetValue@?$TAnimTrack@UIEventKey@@@@UAEXMAAU?$Quat_tpl@M@@@Z 34038a20 f i AnimNode.obj
 0001:00037a20       ?GetValue@?$TAnimSplineTrack@M@@UAEXMAAU?$Quat_tpl@M@@@Z 34038a20 f i Movie.obj
 0001:00037a20       ?GetValue@?$TAnimTrack@UIFaceSeqKey@@@@UAEXMAAU?$Quat_tpl@M@@@Z 34038a20 f i AnimNode.obj
 0001:00037a20       ?GetValue@?$TAnimTrack@UIBoolKey@@@@UAEXMAAM@Z 34038a20 f i AnimNode.obj
 0001:00037a20       ?GetValue@?$TAnimTrack@UICharacterKey@@@@UAEXMAA_N@Z 34038a20 f i AnimNode.obj
 0001:00037a30       ?HasCustomColor@?$TAnimTrack@UIFaceSeqKey@@@@UBE_NXZ 34038a30 f i AnimNode.obj
 0001:00037a30       ?HasCustomColor@?$TAnimTrack@UISoundKey@@@@UBE_NXZ 34038a30 f i AnimNode.obj
 0001:00037a30       ?HasCustomColor@?$TAnimTrack@UILookAtKey@@@@UBE_NXZ 34038a30 f i AnimNode.obj
 0001:00037a30       ?HasCustomColor@?$TAnimTrack@UIBoolKey@@@@UBE_NXZ 34038a30 f i AnimNode.obj
 0001:00037a30       ?HasCustomColor@?$TAnimTrack@UICharacterKey@@@@UBE_NXZ 34038a30 f i AnimNode.obj
 0001:00037a30       ?HasCustomColor@?$TAnimTrack@UIConsoleKey@@@@UBE_NXZ 34038a30 f i AnimNode.obj
 0001:00037a30       ?HasCustomColor@?$TAnimTrack@UICaptureKey@@@@UBE_NXZ 34038a30 f i AnimNode.obj
 0001:00037a30       ?HasCustomColor@?$TAnimTrack@UISequenceKey@@@@UBE_NXZ 34038a30 f i AnimNode.obj
 0001:00037a30       ?HasCustomColor@?$TAnimTrack@UIEventKey@@@@UBE_NXZ 34038a30 f i AnimNode.obj
 0001:00037a30       ?HasCustomColor@?$TAnimTrack@UISelectKey@@@@UBE_NXZ 34038a30 f i AnimNode.obj
 0001:00037a30       ?HasCustomColor@?$TAnimTrack@UIScreenFaderKey@@@@UBE_NXZ 34038a30 f i ScreenFaderTrack.obj
 0001:00037a30       ?HasCustomColor@?$TAnimTrack@UIMusicKey@@@@UBE_NXZ 34038a30 f i AnimNode.obj
 0001:00037a30       ?HasCustomColor@?$TAnimTrack@UICommentKey@@@@UBE_NXZ 34038a30 f i CommentTrack.obj
 0001:00037a30       ?HasCustomColor@?$TAnimTrack@UIDiscreteFloatKey@@@@UBE_NXZ 34038a30 f i GotoTrack.obj
 0001:00037a30       ?HasCustomColor@?$TAnimTrack@UIExprKey@@@@UBE_NXZ 34038a30 f i AnimNode.obj
 0001:00037a40       ?CreateKey@?$TAnimTrack@UISoundKey@@@@UAEHM@Z 34038a40 f i AnimNode.obj
 0001:00037af0       ?CloneKey@?$TAnimTrack@UISoundKey@@@@UAEHH@Z 34038af0 f i AnimNode.obj
 0001:00037bb0       ?CopyKey@?$TAnimTrack@UISoundKey@@@@UAEHPAUIAnimTrack@@H@Z 34038bb0 f i AnimNode.obj
 0001:00037c70       ?FindKey@?$TAnimTrack@UISoundKey@@@@UAEHM@Z 34038c70 f i AnimNode.obj
 0001:00037cd0       ?GetKeyFlags@?$TAnimTrack@UISoundKey@@@@UAEHH@Z 34038cd0 f i AnimNode.obj
 0001:00037cf0       ?SetKey@?$TAnimTrack@UISoundKey@@@@UAEXHPAUIKey@@@Z 34038cf0 f i AnimNode.obj
 0001:00037d20       ?SetKeyTime@?$TAnimTrack@UISoundKey@@@@UAEXHM@Z 34038d20 f i AnimNode.obj
 0001:00037d50       ?SetKeyFlags@?$TAnimTrack@UISoundKey@@@@UAEXHH@Z 34038d50 f i AnimNode.obj
 0001:00037d70       ?Serialize@?$TAnimTrack@UISoundKey@@@@UAE_NAAVXmlNodeRef@@_N1@Z 34038d70 f i AnimNode.obj
 0001:00038020       ?SerializeSelection@?$TAnimTrack@UISoundKey@@@@UAE_NAAVXmlNodeRef@@_N1M@Z 34039020 f i AnimNode.obj
 0001:000381f0       ??$fill@PAUISoundKey@@U1@@stlpmtx_std@@YAXPAUISoundKey@@0ABU1@@Z 340391f0 f i AnimNode.obj
 0001:00038240       ??$__push_heap@PAUISoundKey@@HU1@U?$less@UISoundKey@@@stlpmtx_std@@@stlpmtx_std@@YAXPAUISoundKey@@HHU1@U?$less@UISoundKey@@@0@@Z 34039240 f i AnimNode.obj
 0001:000382b0       ?SelectKey@?$TAnimTrack@UISoundKey@@@@UAEXH_N@Z 340392b0 f i AnimNode.obj
 0001:000382f0       ?GetNumKeys@?$TAnimTrack@UISoundKey@@@@UBEHXZ 340392f0 f i AnimNode.obj
 0001:00038310       ?GetKey@?$TAnimTrack@UISoundKey@@@@UBEXHPAUIKey@@@Z 34039310 f i AnimNode.obj
 0001:00038340       ?GetKeyTime@?$TAnimTrack@UISoundKey@@@@UBEMH@Z 34039340 f i AnimNode.obj
 0001:00038360       ??$__unguarded_insertion_sort_aux@PAUISoundKey@@U1@U?$less@UISoundKey@@@stlpmtx_std@@@priv@stlpmtx_std@@YAXPAUISoundKey@@00U?$less@UISoundKey@@@1@@Z 34039360 f i AnimNode.obj
 0001:000383e0       ??$__adjust_heap@PAUISoundKey@@HU1@U?$less@UISoundKey@@@stlpmtx_std@@@stlpmtx_std@@YAXPAUISoundKey@@HHU1@U?$less@UISoundKey@@@0@@Z 340393e0 f i AnimNode.obj
 0001:00038490       ?IsKeySelected@?$TAnimTrack@UISoundKey@@@@UBE_NH@Z 34039490 f i AnimNode.obj
 0001:000384b0       ?_M_insert_overflow@?$_Impl_vector@UISoundKey@@V?$allocator@UISoundKey@@@stlpmtx_std@@@priv@stlpmtx_std@@AAEXPAUISoundKey@@ABU4@ABU__true_type@3@I_N@Z 340394b0 f i AnimNode.obj
 0001:00038640       ??$__uninitialized_fill_n@PAUISoundKey@@IU1@@priv@stlpmtx_std@@YAPAUISoundKey@@PAU2@IABU2@@Z 34039640 f i AnimNode.obj
 0001:000386a0       ??$__unguarded_partition@PAUISoundKey@@U1@U?$less@UISoundKey@@@stlpmtx_std@@@priv@stlpmtx_std@@YAPAUISoundKey@@PAU2@0U2@U?$less@UISoundKey@@@1@@Z 340396a0 f i AnimNode.obj
 0001:00038710       ??$__make_heap@PAUISoundKey@@U?$less@UISoundKey@@@stlpmtx_std@@U1@H@stlpmtx_std@@YAXPAUISoundKey@@0U?$less@UISoundKey@@@0@0PAH@Z 34039710 f i AnimNode.obj
 0001:00038840       ?_M_fill_insert_aux@?$_Impl_vector@UISoundKey@@V?$allocator@UISoundKey@@@stlpmtx_std@@@priv@stlpmtx_std@@AAEXPAUISoundKey@@IABU4@ABU__false_type@3@@Z 34039840 f i AnimNode.obj
 0001:00038970       ??$__insertion_sort@PAUISoundKey@@U1@U?$less@UISoundKey@@@stlpmtx_std@@@priv@stlpmtx_std@@YAXPAUISoundKey@@00U?$less@UISoundKey@@@1@@Z 34039970 f i AnimNode.obj
 0001:00038a50       ?RemoveKey@?$TAnimTrack@UISoundKey@@@@UAEXH@Z 34039a50 f i AnimNode.obj
 0001:00038ab0       ??$__final_insertion_sort@PAUISoundKey@@U?$less@UISoundKey@@@stlpmtx_std@@@priv@stlpmtx_std@@YAXPAUISoundKey@@0U?$less@UISoundKey@@@1@@Z 34039ab0 f i AnimNode.obj
 0001:00038b20       ??$sort_heap@PAUISoundKey@@U?$less@UISoundKey@@@stlpmtx_std@@@stlpmtx_std@@YAXPAUISoundKey@@0U?$less@UISoundKey@@@0@@Z 34039b20 f i AnimNode.obj
 0001:00038c00       ?GetCustomColor@?$TAnimTrack@UICharacterKey@@@@UBE?AU?$Color_tpl@E@@XZ 34039c00 f i AnimNode.obj
 0001:00038c00       ?GetCustomColor@?$TAnimTrack@UIMusicKey@@@@UBE?AU?$Color_tpl@E@@XZ 34039c00 f i AnimNode.obj
 0001:00038c00       ?GetCustomColor@?$TAnimTrack@UISoundKey@@@@UBE?AU?$Color_tpl@E@@XZ 34039c00 f i AnimNode.obj
 0001:00038c00       ?GetCustomColor@?$TAnimTrack@UIScreenFaderKey@@@@UBE?AU?$Color_tpl@E@@XZ 34039c00 f i ScreenFaderTrack.obj
 0001:00038c00       ?GetCustomColor@?$TAnimTrack@UIDiscreteFloatKey@@@@UBE?AU?$Color_tpl@E@@XZ 34039c00 f i GotoTrack.obj
 0001:00038c00       ?GetCustomColor@?$TAnimTrack@UIExprKey@@@@UBE?AU?$Color_tpl@E@@XZ 34039c00 f i AnimNode.obj
 0001:00038c00       ?GetCustomColor@?$TAnimTrack@UICaptureKey@@@@UBE?AU?$Color_tpl@E@@XZ 34039c00 f i AnimNode.obj
 0001:00038c00       ?GetCustomColor@?$TAnimTrack@UISelectKey@@@@UBE?AU?$Color_tpl@E@@XZ 34039c00 f i AnimNode.obj
 0001:00038c00       ?GetCustomColor@?$TAnimTrack@UIFaceSeqKey@@@@UBE?AU?$Color_tpl@E@@XZ 34039c00 f i AnimNode.obj
 0001:00038c00       ?GetCustomColor@?$TAnimTrack@UIConsoleKey@@@@UBE?AU?$Color_tpl@E@@XZ 34039c00 f i AnimNode.obj
 0001:00038c00       ?GetCustomColor@?$TAnimTrack@UIBoolKey@@@@UBE?AU?$Color_tpl@E@@XZ 34039c00 f i AnimNode.obj
 0001:00038c00       ?GetCustomColor@?$TAnimTrack@UILookAtKey@@@@UBE?AU?$Color_tpl@E@@XZ 34039c00 f i AnimNode.obj
 0001:00038c00       ?GetCustomColor@?$TAnimTrack@UIEventKey@@@@UBE?AU?$Color_tpl@E@@XZ 34039c00 f i AnimNode.obj
 0001:00038c00       ?GetCustomColor@?$TAnimTrack@UISequenceKey@@@@UBE?AU?$Color_tpl@E@@XZ 34039c00 f i AnimNode.obj
 0001:00038c00       ?GetCustomColor@?$TAnimTrack@UICommentKey@@@@UBE?AU?$Color_tpl@E@@XZ 34039c00 f i CommentTrack.obj
 0001:00038c10       ?ClearCustomColor@?$TAnimTrack@UIDiscreteFloatKey@@@@UAEXXZ 34039c10 f i GotoTrack.obj
 0001:00038c10       ?ClearCustomColor@?$TAnimTrack@UICaptureKey@@@@UAEXXZ 34039c10 f i AnimNode.obj
 0001:00038c10       ?ClearCustomColor@?$TAnimTrack@UISequenceKey@@@@UAEXXZ 34039c10 f i AnimNode.obj
 0001:00038c10       ?ClearCustomColor@?$TAnimTrack@UICommentKey@@@@UAEXXZ 34039c10 f i CommentTrack.obj
 0001:00038c10       ?ClearCustomColor@?$TAnimTrack@UIEventKey@@@@UAEXXZ 34039c10 f i AnimNode.obj
 0001:00038c10       ?ClearCustomColor@?$TAnimTrack@UIConsoleKey@@@@UAEXXZ 34039c10 f i AnimNode.obj
 0001:00038c10       ?ClearCustomColor@?$TAnimTrack@UISelectKey@@@@UAEXXZ 34039c10 f i AnimNode.obj
 0001:00038c10       ?ClearCustomColor@?$TAnimTrack@UIBoolKey@@@@UAEXXZ 34039c10 f i AnimNode.obj
 0001:00038c10       ?ClearCustomColor@?$TAnimTrack@UICharacterKey@@@@UAEXXZ 34039c10 f i AnimNode.obj
 0001:00038c10       ?ClearCustomColor@?$TAnimTrack@UIScreenFaderKey@@@@UAEXXZ 34039c10 f i ScreenFaderTrack.obj
 0001:00038c10       ?ClearCustomColor@?$TAnimTrack@UIMusicKey@@@@UAEXXZ 34039c10 f i AnimNode.obj
 0001:00038c10       ?ClearCustomColor@?$TAnimTrack@UILookAtKey@@@@UAEXXZ 34039c10 f i AnimNode.obj
 0001:00038c10       ?ClearCustomColor@?$TAnimTrack@UIFaceSeqKey@@@@UAEXXZ 34039c10 f i AnimNode.obj
 0001:00038c10       ?ClearCustomColor@?$TAnimTrack@UIExprKey@@@@UAEXXZ 34039c10 f i AnimNode.obj
 0001:00038c10       ?ClearCustomColor@?$TAnimTrack@UISoundKey@@@@UAEXXZ 34039c10 f i AnimNode.obj
 0001:00038c20       ?CreateKey@?$TAnimTrack@UIExprKey@@@@UAEHM@Z 34039c20 f i AnimNode.obj
 0001:00038cb0       ?CloneKey@?$TAnimTrack@UIExprKey@@@@UAEHH@Z 34039cb0 f i AnimNode.obj
 0001:00038d50       ?CopyKey@?$TAnimTrack@UIExprKey@@@@UAEHPAUIAnimTrack@@H@Z 34039d50 f i AnimNode.obj
 0001:00038df0       ?SetParameterType@?$TAnimTrack@UIEventKey@@@@UAEXVAnimParamType@@@Z 34039df0 f i AnimNode.obj
 0001:00038df0       ?SetParameterType@?$TAnimTrack@UIScreenFaderKey@@@@UAEXVAnimParamType@@@Z 34039df0 f i ScreenFaderTrack.obj
 0001:00038df0       ?SetParameterType@?$TAnimTrack@UICaptureKey@@@@UAEXVAnimParamType@@@Z 34039df0 f i AnimNode.obj
 0001:00038df0       ?SetParameterType@?$TAnimTrack@UICharacterKey@@@@UAEXVAnimParamType@@@Z 34039df0 f i AnimNode.obj
 0001:00038df0       ?SetParameterType@?$TAnimTrack@UICommentKey@@@@UAEXVAnimParamType@@@Z 34039df0 f i CommentTrack.obj
 0001:00038df0       ?SetParameterType@?$TAnimTrack@UIDiscreteFloatKey@@@@UAEXVAnimParamType@@@Z 34039df0 f i GotoTrack.obj
 0001:00038df0       ?SetParameterType@?$TAnimTrack@UIConsoleKey@@@@UAEXVAnimParamType@@@Z 34039df0 f i AnimNode.obj
 0001:00038df0       ?SetParameterType@?$TAnimTrack@UIFaceSeqKey@@@@UAEXVAnimParamType@@@Z 34039df0 f i AnimNode.obj
 0001:00038df0       ?SetParameterType@?$TAnimTrack@UIBoolKey@@@@UAEXVAnimParamType@@@Z 34039df0 f i AnimNode.obj
 0001:00038df0       ?SetParameterType@?$TAnimTrack@UISequenceKey@@@@UAEXVAnimParamType@@@Z 34039df0 f i AnimNode.obj
 0001:00038df0       ?SetParameterType@?$TAnimSplineTrack@U?$Vec3_tpl@M@@@@UAEXVAnimParamType@@@Z 34039df0 f i Movie.obj
 0001:00038df0       ?SetParameterType@?$TAnimTrack@UILookAtKey@@@@UAEXVAnimParamType@@@Z 34039df0 f i AnimNode.obj
 0001:00038df0       ?SetParameterType@?$TAnimTrack@UISoundKey@@@@UAEXVAnimParamType@@@Z 34039df0 f i AnimNode.obj
 0001:00038df0       ?SetParameterType@?$TAnimTrack@UIExprKey@@@@UAEXVAnimParamType@@@Z 34039df0 f i AnimNode.obj
 0001:00038df0       ?SetParameterType@?$TAnimTrack@UIMusicKey@@@@UAEXVAnimParamType@@@Z 34039df0 f i AnimNode.obj
 0001:00038df0       ?SetParameterType@?$TAnimTrack@UISelectKey@@@@UAEXVAnimParamType@@@Z 34039df0 f i AnimNode.obj
 0001:00038e60       ?FindKey@?$TAnimTrack@UIExprKey@@@@UAEHM@Z 34039e60 f i AnimNode.obj
 0001:00038e60       ?FindKey@?$TAnimTrack@UISequenceKey@@@@UAEHM@Z 34039e60 f i AnimNode.obj
 0001:00038ec0       ?SetKeyTime@?$TAnimTrack@UISequenceKey@@@@UAEXHM@Z 34039ec0 f i AnimNode.obj
 0001:00038ec0       ?SetKeyTime@?$TAnimTrack@UIExprKey@@@@UAEXHM@Z 34039ec0 f i AnimNode.obj
 0001:00038ef0       ?SetKeyFlags@?$TAnimTrack@UISequenceKey@@@@UAEXHH@Z 34039ef0 f i AnimNode.obj
 0001:00038ef0       ?SetKeyFlags@?$TAnimTrack@UIExprKey@@@@UAEXHH@Z 34039ef0 f i AnimNode.obj
 0001:00038f10       ?Serialize@?$TAnimTrack@UIExprKey@@@@UAE_NAAVXmlNodeRef@@_N1@Z 34039f10 f i AnimNode.obj
 0001:00038f10       ?Serialize@?$TAnimTrack@UISequenceKey@@@@UAE_NAAVXmlNodeRef@@_N1@Z 34039f10 f i AnimNode.obj
 0001:000391c0       ?SerializeSelection@?$TAnimTrack@UISequenceKey@@@@UAE_NAAVXmlNodeRef@@_N1M@Z 3403a1c0 f i AnimNode.obj
 0001:000391c0       ?SerializeSelection@?$TAnimTrack@UIExprKey@@@@UAE_NAAVXmlNodeRef@@_N1M@Z 3403a1c0 f i AnimNode.obj
 0001:00039390       ?GetKeyTime@?$TAnimTrack@UISequenceKey@@@@UBEMH@Z 3403a390 f i AnimNode.obj
 0001:00039390       ?GetKeyTime@?$TAnimTrack@UIExprKey@@@@UBEMH@Z 3403a390 f i AnimNode.obj
 0001:000393b0       ??$__unguarded_insertion_sort_aux@PAUISequenceKey@@U1@U?$less@UISequenceKey@@@stlpmtx_std@@@priv@stlpmtx_std@@YAXPAUISequenceKey@@00U?$less@UISequenceKey@@@1@@Z 3403a3b0 f i AnimNode.obj
 0001:000393b0       ??$__unguarded_insertion_sort_aux@PAUIExprKey@@U1@U?$less@UIExprKey@@@stlpmtx_std@@@priv@stlpmtx_std@@YAXPAUIExprKey@@00U?$less@UIExprKey@@@1@@Z 3403a3b0 f i AnimNode.obj
 0001:00039430       ??$__unguarded_partition@PAUIExprKey@@U1@U?$less@UIExprKey@@@stlpmtx_std@@@priv@stlpmtx_std@@YAPAUIExprKey@@PAU2@0U2@U?$less@UIExprKey@@@1@@Z 3403a430 f i AnimNode.obj
 0001:00039430       ??$__unguarded_partition@PAUISequenceKey@@U1@U?$less@UISequenceKey@@@stlpmtx_std@@@priv@stlpmtx_std@@YAPAUISequenceKey@@PAU2@0U2@U?$less@UISequenceKey@@@1@@Z 3403a430 f i AnimNode.obj
 0001:000394a0       ??$__final_insertion_sort@PAUIExprKey@@U?$less@UIExprKey@@@stlpmtx_std@@@priv@stlpmtx_std@@YAXPAUIExprKey@@0U?$less@UIExprKey@@@1@@Z 3403a4a0 f i AnimNode.obj
 0001:000394a0       ??$__final_insertion_sort@PAUISequenceKey@@U?$less@UISequenceKey@@@stlpmtx_std@@@priv@stlpmtx_std@@YAXPAUISequenceKey@@0U?$less@UISequenceKey@@@1@@Z 3403a4a0 f i AnimNode.obj
 0001:00039510       ??$sort_heap@PAUISequenceKey@@U?$less@UISequenceKey@@@stlpmtx_std@@@stlpmtx_std@@YAXPAUISequenceKey@@0U?$less@UISequenceKey@@@0@@Z 3403a510 f i AnimNode.obj
 0001:00039510       ??$sort_heap@PAUIExprKey@@U?$less@UIExprKey@@@stlpmtx_std@@@stlpmtx_std@@YAXPAUIExprKey@@0U?$less@UIExprKey@@@0@@Z 3403a510 f i AnimNode.obj
 0001:000395f0       ?CreateKey@?$TAnimTrack@UIConsoleKey@@@@UAEHM@Z 3403a5f0 f i AnimNode.obj
 0001:00039650       ?CloneKey@?$TAnimTrack@UIConsoleKey@@@@UAEHH@Z 3403a650 f i AnimNode.obj
 0001:000396b0       ?CopyKey@?$TAnimTrack@UIConsoleKey@@@@UAEHPAUIAnimTrack@@H@Z 3403a6b0 f i AnimNode.obj
 0001:00039710       ?FindKey@?$TAnimTrack@UIConsoleKey@@@@UAEHM@Z 3403a710 f i AnimNode.obj
 0001:00039770       ?GetKeyFlags@?$TAnimTrack@UIConsoleKey@@@@UAEHH@Z 3403a770 f i AnimNode.obj
 0001:00039790       ?SetKey@?$TAnimTrack@UIConsoleKey@@@@UAEXHPAUIKey@@@Z 3403a790 f i AnimNode.obj
 0001:000397c0       ?SetKeyTime@?$TAnimTrack@UIConsoleKey@@@@UAEXHM@Z 3403a7c0 f i AnimNode.obj
 0001:000397e0       ?SetKeyFlags@?$TAnimTrack@UIConsoleKey@@@@UAEXHH@Z 3403a7e0 f i AnimNode.obj
 0001:00039800       ?Serialize@?$TAnimTrack@UIConsoleKey@@@@UAE_NAAVXmlNodeRef@@_N1@Z 3403a800 f i AnimNode.obj
 0001:00039ab0       ?SerializeSelection@?$TAnimTrack@UIConsoleKey@@@@UAE_NAAVXmlNodeRef@@_N1M@Z 3403aab0 f i AnimNode.obj
 0001:00039c80       ??$fill@PAUIConsoleKey@@U1@@stlpmtx_std@@YAXPAUIConsoleKey@@0ABU1@@Z 3403ac80 f i AnimNode.obj
 0001:00039cc0       ??$__push_heap@PAUIConsoleKey@@HU1@U?$less@UIConsoleKey@@@stlpmtx_std@@@stlpmtx_std@@YAXPAUIConsoleKey@@HHU1@U?$less@UIConsoleKey@@@0@@Z 3403acc0 f i AnimNode.obj
 0001:00039d20       ?SelectKey@?$TAnimTrack@UIConsoleKey@@@@UAEXH_N@Z 3403ad20 f i AnimNode.obj
 0001:00039d60       ?GetNumKeys@?$TAnimTrack@UIConsoleKey@@@@UBEHXZ 3403ad60 f i AnimNode.obj
 0001:00039d80       ?GetKey@?$TAnimTrack@UIConsoleKey@@@@UBEXHPAUIKey@@@Z 3403ad80 f i AnimNode.obj
 0001:00039db0       ?GetKeyTime@?$TAnimTrack@UIConsoleKey@@@@UBEMH@Z 3403adb0 f i AnimNode.obj
 0001:00039dd0       ??$__unguarded_insertion_sort_aux@PAUIConsoleKey@@U1@U?$less@UIConsoleKey@@@stlpmtx_std@@@priv@stlpmtx_std@@YAXPAUIConsoleKey@@00U?$less@UIConsoleKey@@@1@@Z 3403add0 f i AnimNode.obj
 0001:00039e30       ??$__adjust_heap@PAUIConsoleKey@@HU1@U?$less@UIConsoleKey@@@stlpmtx_std@@@stlpmtx_std@@YAXPAUIConsoleKey@@HHU1@U?$less@UIConsoleKey@@@0@@Z 3403ae30 f i AnimNode.obj
 0001:00039ec0       ?IsKeySelected@?$TAnimTrack@UIConsoleKey@@@@UBE_NH@Z 3403aec0 f i AnimNode.obj
 0001:00039ee0       ?_M_insert_overflow@?$_Impl_vector@UIConsoleKey@@V?$allocator@UIConsoleKey@@@stlpmtx_std@@@priv@stlpmtx_std@@AAEXPAUIConsoleKey@@ABU4@ABU__true_type@3@I_N@Z 3403aee0 f i AnimNode.obj
 0001:0003a060       ??$__uninitialized_fill_n@PAUIConsoleKey@@IU1@@priv@stlpmtx_std@@YAPAUIConsoleKey@@PAU2@IABU2@@Z 3403b060 f i AnimNode.obj
 0001:0003a0c0       ??$__unguarded_partition@PAUIConsoleKey@@U1@U?$less@UIConsoleKey@@@stlpmtx_std@@@priv@stlpmtx_std@@YAPAUIConsoleKey@@PAU2@0U2@U?$less@UIConsoleKey@@@1@@Z 3403b0c0 f i AnimNode.obj
 0001:0003a120       ??$__make_heap@PAUIConsoleKey@@U?$less@UIConsoleKey@@@stlpmtx_std@@U1@H@stlpmtx_std@@YAXPAUIConsoleKey@@0U?$less@UIConsoleKey@@@0@0PAH@Z 3403b120 f i AnimNode.obj
 0001:0003a250       ?_M_fill_insert_aux@?$_Impl_vector@UIConsoleKey@@V?$allocator@UIConsoleKey@@@stlpmtx_std@@@priv@stlpmtx_std@@AAEXPAUIConsoleKey@@IABU4@ABU__false_type@3@@Z 3403b250 f i AnimNode.obj
 0001:0003a370       ??$__insertion_sort@PAUIConsoleKey@@U1@U?$less@UIConsoleKey@@@stlpmtx_std@@@priv@stlpmtx_std@@YAXPAUIConsoleKey@@00U?$less@UIConsoleKey@@@1@@Z 3403b370 f i AnimNode.obj
 0001:0003a430       ?RemoveKey@?$TAnimTrack@UIConsoleKey@@@@UAEXH@Z 3403b430 f i AnimNode.obj
 0001:0003a490       ??$__final_insertion_sort@PAUIConsoleKey@@U?$less@UIConsoleKey@@@stlpmtx_std@@@priv@stlpmtx_std@@YAXPAUIConsoleKey@@0U?$less@UIConsoleKey@@@1@@Z 3403b490 f i AnimNode.obj
 0001:0003a500       ??$sort_heap@PAUIConsoleKey@@U?$less@UIConsoleKey@@@stlpmtx_std@@@stlpmtx_std@@YAXPAUIConsoleKey@@0U?$less@UIConsoleKey@@@0@@Z 3403b500 f i AnimNode.obj
 0001:0003a5b0       ?CreateKey@?$TAnimTrack@UIMusicKey@@@@UAEHM@Z 3403b5b0 f i AnimNode.obj
 0001:0003a620       ?CloneKey@?$TAnimTrack@UIMusicKey@@@@UAEHH@Z 3403b620 f i AnimNode.obj
 0001:0003a690       ?CopyKey@?$TAnimTrack@UIMusicKey@@@@UAEHPAUIAnimTrack@@H@Z 3403b690 f i AnimNode.obj
 0001:0003a700       ?FindKey@?$TAnimTrack@UIMusicKey@@@@UAEHM@Z 3403b700 f i AnimNode.obj
 0001:0003a760       ?GetKeyFlags@?$TAnimTrack@UIMusicKey@@@@UAEHH@Z 3403b760 f i AnimNode.obj
 0001:0003a780       ?SetKey@?$TAnimTrack@UIMusicKey@@@@UAEXHPAUIKey@@@Z 3403b780 f i AnimNode.obj
 0001:0003a7b0       ?SetKeyTime@?$TAnimTrack@UIMusicKey@@@@UAEXHM@Z 3403b7b0 f i AnimNode.obj
 0001:0003a7d0       ?SetKeyFlags@?$TAnimTrack@UIMusicKey@@@@UAEXHH@Z 3403b7d0 f i AnimNode.obj
 0001:0003a7f0       ?Serialize@?$TAnimTrack@UIMusicKey@@@@UAE_NAAVXmlNodeRef@@_N1@Z 3403b7f0 f i AnimNode.obj
 0001:0003aaa0       ?SerializeSelection@?$TAnimTrack@UIMusicKey@@@@UAE_NAAVXmlNodeRef@@_N1M@Z 3403baa0 f i AnimNode.obj
 0001:0003ac60       ??$fill@PAUIMusicKey@@U1@@stlpmtx_std@@YAXPAUIMusicKey@@0ABU1@@Z 3403bc60 f i AnimNode.obj
 0001:0003aca0       ??$__push_heap@PAUIMusicKey@@HU1@U?$less@UIMusicKey@@@stlpmtx_std@@@stlpmtx_std@@YAXPAUIMusicKey@@HHU1@U?$less@UIMusicKey@@@0@@Z 3403bca0 f i AnimNode.obj
 0001:0003ad00       ?SelectKey@?$TAnimTrack@UIMusicKey@@@@UAEXH_N@Z 3403bd00 f i AnimNode.obj
 0001:0003ad40       ?GetNumKeys@?$TAnimTrack@UIMusicKey@@@@UBEHXZ 3403bd40 f i AnimNode.obj
 0001:0003ad60       ?GetKey@?$TAnimTrack@UIMusicKey@@@@UBEXHPAUIKey@@@Z 3403bd60 f i AnimNode.obj
 0001:0003ad80       ?GetKeyTime@?$TAnimTrack@UIMusicKey@@@@UBEMH@Z 3403bd80 f i AnimNode.obj
 0001:0003ada0       ??$__unguarded_insertion_sort_aux@PAUIMusicKey@@U1@U?$less@UIMusicKey@@@stlpmtx_std@@@priv@stlpmtx_std@@YAXPAUIMusicKey@@00U?$less@UIMusicKey@@@1@@Z 3403bda0 f i AnimNode.obj
 0001:0003ae00       ??$__adjust_heap@PAUIMusicKey@@HU1@U?$less@UIMusicKey@@@stlpmtx_std@@@stlpmtx_std@@YAXPAUIMusicKey@@HHU1@U?$less@UIMusicKey@@@0@@Z 3403be00 f i AnimNode.obj
 0001:0003aea0       ?IsKeySelected@?$TAnimTrack@UIMusicKey@@@@UBE_NH@Z 3403bea0 f i AnimNode.obj
 0001:0003aec0       ?_M_insert_overflow@?$_Impl_vector@UIMusicKey@@V?$allocator@UIMusicKey@@@stlpmtx_std@@@priv@stlpmtx_std@@AAEXPAUIMusicKey@@ABU4@ABU__true_type@3@I_N@Z 3403bec0 f i AnimNode.obj
 0001:0003b040       ??$__uninitialized_fill_n@PAUIMusicKey@@IU1@@priv@stlpmtx_std@@YAPAUIMusicKey@@PAU2@IABU2@@Z 3403c040 f i AnimNode.obj
 0001:0003b0a0       ??$__unguarded_partition@PAUIMusicKey@@U1@U?$less@UIMusicKey@@@stlpmtx_std@@@priv@stlpmtx_std@@YAPAUIMusicKey@@PAU2@0U2@U?$less@UIMusicKey@@@1@@Z 3403c0a0 f i AnimNode.obj
 0001:0003b100       ??$__make_heap@PAUIMusicKey@@U?$less@UIMusicKey@@@stlpmtx_std@@U1@H@stlpmtx_std@@YAXPAUIMusicKey@@0U?$less@UIMusicKey@@@0@0PAH@Z 3403c100 f i AnimNode.obj
 0001:0003b220       ?_M_fill_insert_aux@?$_Impl_vector@UIMusicKey@@V?$allocator@UIMusicKey@@@stlpmtx_std@@@priv@stlpmtx_std@@AAEXPAUIMusicKey@@IABU4@ABU__false_type@3@@Z 3403c220 f i AnimNode.obj
 0001:0003b340       ??$__insertion_sort@PAUIMusicKey@@U1@U?$less@UIMusicKey@@@stlpmtx_std@@@priv@stlpmtx_std@@YAXPAUIMusicKey@@00U?$less@UIMusicKey@@@1@@Z 3403c340 f i AnimNode.obj
 0001:0003b400       ?RemoveKey@?$TAnimTrack@UIMusicKey@@@@UAEXH@Z 3403c400 f i AnimNode.obj
 0001:0003b460       ??_E?$TAnimTrack@UICharacterKey@@@@UAEPAXI@Z 3403c460 f i AnimNode.obj
 0001:0003b460       ??_ECEventTrack@@UAEPAXI@Z 3403c460 f i AnimNode.obj
 0001:0003b460       ??_ECExprTrack@@UAEPAXI@Z  3403c460 f i AnimNode.obj
 0001:0003b460       ??_G?$TAnimTrack@UIBoolKey@@@@UAEPAXI@Z 3403c460 f i AnimNode.obj
 0001:0003b460       ??_G?$TAnimTrack@UIExprKey@@@@UAEPAXI@Z 3403c460 f i AnimNode.obj
 0001:0003b460       ??_E?$TAnimTrack@UIConsoleKey@@@@UAEPAXI@Z 3403c460 f i AnimNode.obj
 0001:0003b460       ??_E?$TAnimTrack@UIScreenFaderKey@@@@UAEPAXI@Z 3403c460 f i ScreenFaderTrack.obj
 0001:0003b460       ??_GCCaptureTrack@@UAEPAXI@Z 3403c460 f i AnimNode.obj
 0001:0003b460       ??_GCLookAtTrack@@UAEPAXI@Z 3403c460 f i AnimNode.obj
 0001:0003b460       ??_G?$TAnimTrack@UISequenceKey@@@@UAEPAXI@Z 3403c460 f i AnimNode.obj
 0001:0003b460       ??_E?$TAnimTrack@UIBoolKey@@@@UAEPAXI@Z 3403c460 f i AnimNode.obj
 0001:0003b460       ??_G?$TAnimTrack@UIScreenFaderKey@@@@UAEPAXI@Z 3403c460 f i ScreenFaderTrack.obj
 0001:0003b460       ??_ECCharacterTrack@@UAEPAXI@Z 3403c460 f i AnimNode.obj
 0001:0003b460       ??_G?$TAnimTrack@UIDiscreteFloatKey@@@@UAEPAXI@Z 3403c460 f i GotoTrack.obj
 0001:0003b460       ??_ECGotoTrack@@UAEPAXI@Z  3403c460 f i GotoTrack.obj
 0001:0003b460       ??_ECTrackEventTrack@@UAEPAXI@Z 3403c460 f i AnimNode.obj
 0001:0003b460       ??_E?$TAnimTrack@UIMusicKey@@@@UAEPAXI@Z 3403c460 f i AnimNode.obj
 0001:0003b460       ??_ECSelectTrack@@UAEPAXI@Z 3403c460 f i AnimNode.obj
 0001:0003b460       ??_ECSequenceTrack@@UAEPAXI@Z 3403c460 f i AnimNode.obj
 0001:0003b460       ??_E?$TAnimTrack@UIEventKey@@@@UAEPAXI@Z 3403c460 f i AnimNode.obj
 0001:0003b460       ??_G?$TAnimTrack@UISoundKey@@@@UAEPAXI@Z 3403c460 f i AnimNode.obj
 0001:0003b460       ??_E?$TAnimTrack@UIDiscreteFloatKey@@@@UAEPAXI@Z 3403c460 f i GotoTrack.obj
 0001:0003b460       ??_G?$TAnimTrack@UICharacterKey@@@@UAEPAXI@Z 3403c460 f i AnimNode.obj
 0001:0003b460       ??_E?$TAnimTrack@UIFaceSeqKey@@@@UAEPAXI@Z 3403c460 f i AnimNode.obj
 0001:0003b460       ??_ECLookAtTrack@@UAEPAXI@Z 3403c460 f i AnimNode.obj
 0001:0003b460       ??_GCExprTrack@@UAEPAXI@Z  3403c460 f i AnimNode.obj
 0001:0003b460       ??_E?$TAnimTrack@UICaptureKey@@@@UAEPAXI@Z 3403c460 f i AnimNode.obj
 0001:0003b460       ??_GCSoundTrack@@UAEPAXI@Z 3403c460 f i AnimNode.obj
 0001:0003b460       ??_GCSelectTrack@@UAEPAXI@Z 3403c460 f i AnimNode.obj
 0001:0003b460       ??_ECFaceSeqTrack@@UAEPAXI@Z 3403c460 f i AnimNode.obj
 0001:0003b460       ??_GCFaceSeqTrack@@UAEPAXI@Z 3403c460 f i AnimNode.obj
 0001:0003b460       ??_GCMusicTrack@@UAEPAXI@Z 3403c460 f i AnimNode.obj
 0001:0003b460       ??_G?$TAnimTrack@UICaptureKey@@@@UAEPAXI@Z 3403c460 f i AnimNode.obj
 0001:0003b460       ??_GCCharacterTrack@@UAEPAXI@Z 3403c460 f i AnimNode.obj
 0001:0003b460       ??_E?$TAnimTrack@UIExprKey@@@@UAEPAXI@Z 3403c460 f i AnimNode.obj
 0001:0003b460       ??_ECCaptureTrack@@UAEPAXI@Z 3403c460 f i AnimNode.obj
 0001:0003b460       ??_G?$TAnimTrack@UIMusicKey@@@@UAEPAXI@Z 3403c460 f i AnimNode.obj
 0001:0003b460       ??_GCConsoleTrack@@UAEPAXI@Z 3403c460 f i AnimNode.obj
 0001:0003b460       ??_G?$TAnimTrack@UIFaceSeqKey@@@@UAEPAXI@Z 3403c460 f i AnimNode.obj
 0001:0003b460       ??_ECConsoleTrack@@UAEPAXI@Z 3403c460 f i AnimNode.obj
 0001:0003b460       ??_GCSequenceTrack@@UAEPAXI@Z 3403c460 f i AnimNode.obj
 0001:0003b460       ??_ECMusicTrack@@UAEPAXI@Z 3403c460 f i AnimNode.obj
 0001:0003b460       ??_GCEventTrack@@UAEPAXI@Z 3403c460 f i AnimNode.obj
 0001:0003b460       ??_ECSoundTrack@@UAEPAXI@Z 3403c460 f i AnimNode.obj
 0001:0003b460       ??_E?$TAnimTrack@UILookAtKey@@@@UAEPAXI@Z 3403c460 f i AnimNode.obj
 0001:0003b460       ??_E?$TAnimTrack@UISelectKey@@@@UAEPAXI@Z 3403c460 f i AnimNode.obj
 0001:0003b460       ??_E?$TAnimTrack@UISequenceKey@@@@UAEPAXI@Z 3403c460 f i AnimNode.obj
 0001:0003b460       ??_E?$TAnimTrack@UISoundKey@@@@UAEPAXI@Z 3403c460 f i AnimNode.obj
 0001:0003b460       ??_G?$TAnimTrack@UISelectKey@@@@UAEPAXI@Z 3403c460 f i AnimNode.obj
 0001:0003b460       ??_GCBoolTrack@@UAEPAXI@Z  3403c460 f i AnimNode.obj
 0001:0003b460       ??_GCTrackEventTrack@@UAEPAXI@Z 3403c460 f i AnimNode.obj
 0001:0003b460       ??_GCGotoTrack@@UAEPAXI@Z  3403c460 f i GotoTrack.obj
 0001:0003b460       ??_G?$TAnimTrack@UILookAtKey@@@@UAEPAXI@Z 3403c460 f i AnimNode.obj
 0001:0003b460       ??_ECBoolTrack@@UAEPAXI@Z  3403c460 f i AnimNode.obj
 0001:0003b460       ??_G?$TAnimTrack@UIEventKey@@@@UAEPAXI@Z 3403c460 f i AnimNode.obj
 0001:0003b460       ??_G?$TAnimTrack@UIConsoleKey@@@@UAEPAXI@Z 3403c460 f i AnimNode.obj
 0001:0003b4d0       ??$__final_insertion_sort@PAUIMusicKey@@U?$less@UIMusicKey@@@stlpmtx_std@@@priv@stlpmtx_std@@YAXPAUIMusicKey@@0U?$less@UIMusicKey@@@1@@Z 3403c4d0 f i AnimNode.obj
 0001:0003b540       ??$sort_heap@PAUIMusicKey@@U?$less@UIMusicKey@@@stlpmtx_std@@@stlpmtx_std@@YAXPAUIMusicKey@@0U?$less@UIMusicKey@@@0@@Z 3403c540 f i AnimNode.obj
 0001:0003b600       ?insert@?$_Impl_vector@UIMusicKey@@V?$allocator@UIMusicKey@@@stlpmtx_std@@@priv@stlpmtx_std@@QAEXPAUIMusicKey@@IABU4@@Z 3403c600 f i AnimNode.obj
 0001:0003b660       ?GetFlags@?$TAnimTrack@UISequenceKey@@@@UAEHXZ 3403c660 f i AnimNode.obj
 0001:0003b660       ?GetFlags@?$TAnimTrack@UIEventKey@@@@UAEHXZ 3403c660 f i AnimNode.obj
 0001:0003b660       ?GetFlags@?$TAnimTrack@UISelectKey@@@@UAEHXZ 3403c660 f i AnimNode.obj
 0001:0003b660       ?GetFlags@?$TAnimTrack@UICharacterKey@@@@UAEHXZ 3403c660 f i AnimNode.obj
 0001:0003b660       ?GetFlags@?$TAnimTrack@UISoundKey@@@@UAEHXZ 3403c660 f i AnimNode.obj
 0001:0003b660       ?GetFlags@?$TAnimTrack@UIScreenFaderKey@@@@UAEHXZ 3403c660 f i ScreenFaderTrack.obj
 0001:0003b660       ?GetFlags@?$TAnimTrack@UICommentKey@@@@UAEHXZ 3403c660 f i CommentTrack.obj
 0001:0003b660       ?GetFlags@?$TAnimTrack@UIFaceSeqKey@@@@UAEHXZ 3403c660 f i AnimNode.obj
 0001:0003b660       ?GetFlags@?$TAnimTrack@UIConsoleKey@@@@UAEHXZ 3403c660 f i AnimNode.obj
 0001:0003b660       ?GetFlags@?$TAnimTrack@UICaptureKey@@@@UAEHXZ 3403c660 f i AnimNode.obj
 0001:0003b660       ?GetFlags@?$TAnimTrack@UIBoolKey@@@@UAEHXZ 3403c660 f i AnimNode.obj
 0001:0003b660       ?GetFlags@?$TAnimTrack@UILookAtKey@@@@UAEHXZ 3403c660 f i AnimNode.obj
 0001:0003b660       ?GetFlags@?$TAnimTrack@UIMusicKey@@@@UAEHXZ 3403c660 f i AnimNode.obj
 0001:0003b660       ?GetFlags@?$TAnimTrack@UIDiscreteFloatKey@@@@UAEHXZ 3403c660 f i GotoTrack.obj
 0001:0003b660       ?GetFlags@?$TAnimTrack@UIExprKey@@@@UAEHXZ 3403c660 f i AnimNode.obj
 0001:0003b670       ?CreateKey@?$TAnimTrack@UIFaceSeqKey@@@@UAEHM@Z 3403c670 f i AnimNode.obj
 0001:0003b6e0       ?CloneKey@?$TAnimTrack@UIFaceSeqKey@@@@UAEHH@Z 3403c6e0 f i AnimNode.obj
 0001:0003b760       ?CopyKey@?$TAnimTrack@UIFaceSeqKey@@@@UAEHPAUIAnimTrack@@H@Z 3403c760 f i AnimNode.obj
 0001:0003b7e0       ?FindKey@?$TAnimTrack@UIFaceSeqKey@@@@UAEHM@Z 3403c7e0 f i AnimNode.obj
 0001:0003b840       ?GetKeyFlags@?$TAnimTrack@UIFaceSeqKey@@@@UAEHH@Z 3403c840 f i AnimNode.obj
 0001:0003b860       ?SetKey@?$TAnimTrack@UIFaceSeqKey@@@@UAEXHPAUIKey@@@Z 3403c860 f i AnimNode.obj
 0001:0003b890       ?SetKeyTime@?$TAnimTrack@UIFaceSeqKey@@@@UAEXHM@Z 3403c890 f i AnimNode.obj
 0001:0003b8c0       ?SetKeyFlags@?$TAnimTrack@UIFaceSeqKey@@@@UAEXHH@Z 3403c8c0 f i AnimNode.obj
 0001:0003b8e0       ?Serialize@?$TAnimTrack@UIFaceSeqKey@@@@UAE_NAAVXmlNodeRef@@_N1@Z 3403c8e0 f i AnimNode.obj
 0001:0003bb90       ?SerializeSelection@?$TAnimTrack@UIFaceSeqKey@@@@UAE_NAAVXmlNodeRef@@_N1M@Z 3403cb90 f i AnimNode.obj
 0001:0003bd60       ??$fill@PAUIFaceSeqKey@@U1@@stlpmtx_std@@YAXPAUIFaceSeqKey@@0ABU1@@Z 3403cd60 f i AnimNode.obj
 0001:0003bdb0       ??$__push_heap@PAUIFaceSeqKey@@HU1@U?$less@UIFaceSeqKey@@@stlpmtx_std@@@stlpmtx_std@@YAXPAUIFaceSeqKey@@HHU1@U?$less@UIFaceSeqKey@@@0@@Z 3403cdb0 f i AnimNode.obj
 0001:0003be20       ?SelectKey@?$TAnimTrack@UIFaceSeqKey@@@@UAEXH_N@Z 3403ce20 f i AnimNode.obj
 0001:0003be60       ?GetNumKeys@?$TAnimTrack@UIFaceSeqKey@@@@UBEHXZ 3403ce60 f i AnimNode.obj
 0001:0003be80       ?GetKey@?$TAnimTrack@UIFaceSeqKey@@@@UBEXHPAUIKey@@@Z 3403ce80 f i AnimNode.obj
 0001:0003beb0       ?GetKeyTime@?$TAnimTrack@UIFaceSeqKey@@@@UBEMH@Z 3403ceb0 f i AnimNode.obj
 0001:0003bed0       ??$__unguarded_insertion_sort_aux@PAUIFaceSeqKey@@U1@U?$less@UIFaceSeqKey@@@stlpmtx_std@@@priv@stlpmtx_std@@YAXPAUIFaceSeqKey@@00U?$less@UIFaceSeqKey@@@1@@Z 3403ced0 f i AnimNode.obj
 0001:0003bf50       ??$__adjust_heap@PAUIFaceSeqKey@@HU1@U?$less@UIFaceSeqKey@@@stlpmtx_std@@@stlpmtx_std@@YAXPAUIFaceSeqKey@@HHU1@U?$less@UIFaceSeqKey@@@0@@Z 3403cf50 f i AnimNode.obj
 0001:0003c000       ?IsKeySelected@?$TAnimTrack@UIFaceSeqKey@@@@UBE_NH@Z 3403d000 f i AnimNode.obj
 0001:0003c020       ?_M_insert_overflow@?$_Impl_vector@UIFaceSeqKey@@V?$allocator@UIFaceSeqKey@@@stlpmtx_std@@@priv@stlpmtx_std@@AAEXPAUIFaceSeqKey@@ABU4@ABU__true_type@3@I_N@Z 3403d020 f i AnimNode.obj
 0001:0003c1b0       ??$__uninitialized_fill_n@PAUIFaceSeqKey@@IU1@@priv@stlpmtx_std@@YAPAUIFaceSeqKey@@PAU2@IABU2@@Z 3403d1b0 f i AnimNode.obj
 0001:0003c210       ??$__unguarded_partition@PAUIFaceSeqKey@@U1@U?$less@UIFaceSeqKey@@@stlpmtx_std@@@priv@stlpmtx_std@@YAPAUIFaceSeqKey@@PAU2@0U2@U?$less@UIFaceSeqKey@@@1@@Z 3403d210 f i AnimNode.obj
 0001:0003c280       ??$__make_heap@PAUIFaceSeqKey@@U?$less@UIFaceSeqKey@@@stlpmtx_std@@U1@H@stlpmtx_std@@YAXPAUIFaceSeqKey@@0U?$less@UIFaceSeqKey@@@0@0PAH@Z 3403d280 f i AnimNode.obj
 0001:0003c3b0       ?_M_fill_insert_aux@?$_Impl_vector@UIFaceSeqKey@@V?$allocator@UIFaceSeqKey@@@stlpmtx_std@@@priv@stlpmtx_std@@AAEXPAUIFaceSeqKey@@IABU4@ABU__false_type@3@@Z 3403d3b0 f i AnimNode.obj
 0001:0003c4e0       ??$__insertion_sort@PAUIFaceSeqKey@@U1@U?$less@UIFaceSeqKey@@@stlpmtx_std@@@priv@stlpmtx_std@@YAXPAUIFaceSeqKey@@00U?$less@UIFaceSeqKey@@@1@@Z 3403d4e0 f i AnimNode.obj
 0001:0003c5c0       ?RemoveKey@?$TAnimTrack@UIFaceSeqKey@@@@UAEXH@Z 3403d5c0 f i AnimNode.obj
 0001:0003c620       ??$__final_insertion_sort@PAUIFaceSeqKey@@U?$less@UIFaceSeqKey@@@stlpmtx_std@@@priv@stlpmtx_std@@YAXPAUIFaceSeqKey@@0U?$less@UIFaceSeqKey@@@1@@Z 3403d620 f i AnimNode.obj
 0001:0003c690       ??$sort_heap@PAUIFaceSeqKey@@U?$less@UIFaceSeqKey@@@stlpmtx_std@@@stlpmtx_std@@YAXPAUIFaceSeqKey@@0U?$less@UIFaceSeqKey@@@0@@Z 3403d690 f i AnimNode.obj
 0001:0003c770       ?insert@?$_Impl_vector@UIFaceSeqKey@@V?$allocator@UIFaceSeqKey@@@stlpmtx_std@@@priv@stlpmtx_std@@QAEXPAUIFaceSeqKey@@IABU4@@Z 3403d770 f i AnimNode.obj
 0001:0003c7d0       ?CreateKey@?$TAnimTrack@UILookAtKey@@@@UAEHM@Z 3403d7d0 f i AnimNode.obj
 0001:0003c850       ?CloneKey@?$TAnimTrack@UILookAtKey@@@@UAEHH@Z 3403d850 f i AnimNode.obj
 0001:0003c8e0       ?CopyKey@?$TAnimTrack@UILookAtKey@@@@UAEHPAUIAnimTrack@@H@Z 3403d8e0 f i AnimNode.obj
 0001:0003c970       ?FindKey@?$TAnimTrack@UILookAtKey@@@@UAEHM@Z 3403d970 f i AnimNode.obj
 0001:0003c9d0       ?GetKeyFlags@?$TAnimTrack@UILookAtKey@@@@UAEHH@Z 3403d9d0 f i AnimNode.obj
 0001:0003c9f0       ?SetKey@?$TAnimTrack@UILookAtKey@@@@UAEXHPAUIKey@@@Z 3403d9f0 f i AnimNode.obj
 0001:0003ca20       ?SetKeyTime@?$TAnimTrack@UILookAtKey@@@@UAEXHM@Z 3403da20 f i AnimNode.obj
 0001:0003ca50       ?SetKeyFlags@?$TAnimTrack@UILookAtKey@@@@UAEXHH@Z 3403da50 f i AnimNode.obj
 0001:0003ca70       ?SerializeSelection@?$TAnimTrack@UILookAtKey@@@@UAE_NAAVXmlNodeRef@@_N1M@Z 3403da70 f i AnimNode.obj
 0001:0003cc40       ??$fill@PAUILookAtKey@@U1@@stlpmtx_std@@YAXPAUILookAtKey@@0ABU1@@Z 3403dc40 f i AnimNode.obj
 0001:0003cc90       ??$__push_heap@PAUILookAtKey@@HU1@U?$less@UILookAtKey@@@stlpmtx_std@@@stlpmtx_std@@YAXPAUILookAtKey@@HHU1@U?$less@UILookAtKey@@@0@@Z 3403dc90 f i AnimNode.obj
 0001:0003cd00       ?SelectKey@?$TAnimTrack@UILookAtKey@@@@UAEXH_N@Z 3403dd00 f i AnimNode.obj
 0001:0003cd40       ?GetNumKeys@?$TAnimTrack@UILookAtKey@@@@UBEHXZ 3403dd40 f i AnimNode.obj
 0001:0003cd60       ?GetKey@?$TAnimTrack@UILookAtKey@@@@UBEXHPAUIKey@@@Z 3403dd60 f i AnimNode.obj
 0001:0003cd90       ?GetKeyTime@?$TAnimTrack@UILookAtKey@@@@UBEMH@Z 3403dd90 f i AnimNode.obj
 0001:0003cdb0       ??$__unguarded_insertion_sort_aux@PAUILookAtKey@@U1@U?$less@UILookAtKey@@@stlpmtx_std@@@priv@stlpmtx_std@@YAXPAUILookAtKey@@00U?$less@UILookAtKey@@@1@@Z 3403ddb0 f i AnimNode.obj
 0001:0003ce30       ??$__adjust_heap@PAUILookAtKey@@HU1@U?$less@UILookAtKey@@@stlpmtx_std@@@stlpmtx_std@@YAXPAUILookAtKey@@HHU1@U?$less@UILookAtKey@@@0@@Z 3403de30 f i AnimNode.obj
 0001:0003cee0       ?IsKeySelected@?$TAnimTrack@UILookAtKey@@@@UBE_NH@Z 3403dee0 f i AnimNode.obj
 0001:0003cf00       ?_M_insert_overflow@?$_Impl_vector@UILookAtKey@@V?$allocator@UILookAtKey@@@stlpmtx_std@@@priv@stlpmtx_std@@AAEXPAUILookAtKey@@ABU4@ABU__true_type@3@I_N@Z 3403df00 f i AnimNode.obj
 0001:0003d080       ??$__uninitialized_fill_n@PAUILookAtKey@@IU1@@priv@stlpmtx_std@@YAPAUILookAtKey@@PAU2@IABU2@@Z 3403e080 f i AnimNode.obj
 0001:0003d0e0       ??$__unguarded_partition@PAUILookAtKey@@U1@U?$less@UILookAtKey@@@stlpmtx_std@@@priv@stlpmtx_std@@YAPAUILookAtKey@@PAU2@0U2@U?$less@UILookAtKey@@@1@@Z 3403e0e0 f i AnimNode.obj
 0001:0003d150       ??$__make_heap@PAUILookAtKey@@U?$less@UILookAtKey@@@stlpmtx_std@@U1@H@stlpmtx_std@@YAXPAUILookAtKey@@0U?$less@UILookAtKey@@@0@0PAH@Z 3403e150 f i AnimNode.obj
 0001:0003d280       ?_M_fill_insert_aux@?$_Impl_vector@UILookAtKey@@V?$allocator@UILookAtKey@@@stlpmtx_std@@@priv@stlpmtx_std@@AAEXPAUILookAtKey@@IABU4@ABU__false_type@3@@Z 3403e280 f i AnimNode.obj
 0001:0003d3b0       ??$__insertion_sort@PAUILookAtKey@@U1@U?$less@UILookAtKey@@@stlpmtx_std@@@priv@stlpmtx_std@@YAXPAUILookAtKey@@00U?$less@UILookAtKey@@@1@@Z 3403e3b0 f i AnimNode.obj
 0001:0003d490       ?RemoveKey@?$TAnimTrack@UILookAtKey@@@@UAEXH@Z 3403e490 f i AnimNode.obj
 0001:0003d4f0       ??$__final_insertion_sort@PAUILookAtKey@@U?$less@UILookAtKey@@@stlpmtx_std@@@priv@stlpmtx_std@@YAXPAUILookAtKey@@0U?$less@UILookAtKey@@@1@@Z 3403e4f0 f i AnimNode.obj
 0001:0003d560       ??$sort_heap@PAUILookAtKey@@U?$less@UILookAtKey@@@stlpmtx_std@@@stlpmtx_std@@YAXPAUILookAtKey@@0U?$less@UILookAtKey@@@0@@Z 3403e560 f i AnimNode.obj
 0001:0003d640       ?CreateKey@?$TAnimTrack@UISequenceKey@@@@UAEHM@Z 3403e640 f i AnimNode.obj
 0001:0003d6c0       ?CloneKey@?$TAnimTrack@UISequenceKey@@@@UAEHH@Z 3403e6c0 f i AnimNode.obj
 0001:0003d740       ?CopyKey@?$TAnimTrack@UISequenceKey@@@@UAEHPAUIAnimTrack@@H@Z 3403e740 f i AnimNode.obj
 0001:0003d7d0       ?SetTimeRange@?$TAnimTrack@UICharacterKey@@@@UAEXABV?$TRange@M@@@Z 3403e7d0 f i AnimNode.obj
 0001:0003d7d0       ?SetTimeRange@?$TAnimTrack@UIEventKey@@@@UAEXABV?$TRange@M@@@Z 3403e7d0 f i AnimNode.obj
 0001:0003d7d0       ?SetTimeRange@?$TAnimTrack@UILookAtKey@@@@UAEXABV?$TRange@M@@@Z 3403e7d0 f i AnimNode.obj
 0001:0003d7d0       ?SetTimeRange@?$TAnimTrack@UICaptureKey@@@@UAEXABV?$TRange@M@@@Z 3403e7d0 f i AnimNode.obj
 0001:0003d7d0       ?SetTimeRange@?$TAnimTrack@UISoundKey@@@@UAEXABV?$TRange@M@@@Z 3403e7d0 f i AnimNode.obj
 0001:0003d7d0       ?SetTimeRange@?$TAnimTrack@UISelectKey@@@@UAEXABV?$TRange@M@@@Z 3403e7d0 f i AnimNode.obj
 0001:0003d7d0       ?SetTimeRange@?$TAnimTrack@UICommentKey@@@@UAEXABV?$TRange@M@@@Z 3403e7d0 f i CommentTrack.obj
 0001:0003d7d0       ?SetTimeRange@?$TAnimTrack@UIDiscreteFloatKey@@@@UAEXABV?$TRange@M@@@Z 3403e7d0 f i GotoTrack.obj
 0001:0003d7d0       ?SetTimeRange@?$TAnimTrack@UIMusicKey@@@@UAEXABV?$TRange@M@@@Z 3403e7d0 f i AnimNode.obj
 0001:0003d7d0       ?SetTimeRange@?$TAnimTrack@UIConsoleKey@@@@UAEXABV?$TRange@M@@@Z 3403e7d0 f i AnimNode.obj
 0001:0003d7d0       ?SetTimeRange@?$TAnimTrack@UIScreenFaderKey@@@@UAEXABV?$TRange@M@@@Z 3403e7d0 f i ScreenFaderTrack.obj
 0001:0003d7d0       ?SetTimeRange@?$TAnimTrack@UIFaceSeqKey@@@@UAEXABV?$TRange@M@@@Z 3403e7d0 f i AnimNode.obj
 0001:0003d7d0       ?SetTimeRange@?$TAnimTrack@UIBoolKey@@@@UAEXABV?$TRange@M@@@Z 3403e7d0 f i AnimNode.obj
 0001:0003d7d0       ?SetTimeRange@?$TAnimTrack@UISequenceKey@@@@UAEXABV?$TRange@M@@@Z 3403e7d0 f i AnimNode.obj
 0001:0003d7d0       ?SetTimeRange@?$TAnimTrack@UIExprKey@@@@UAEXABV?$TRange@M@@@Z 3403e7d0 f i AnimNode.obj
 0001:0003d7f0       ?GetKeyFlags@?$TAnimTrack@UIExprKey@@@@UAEHH@Z 3403e7f0 f i AnimNode.obj
 0001:0003d7f0       ?GetKeyFlags@?$TAnimTrack@UISequenceKey@@@@UAEHH@Z 3403e7f0 f i AnimNode.obj
 0001:0003d810       ?SetKey@?$TAnimTrack@UISequenceKey@@@@UAEXHPAUIKey@@@Z 3403e810 f i AnimNode.obj
 0001:0003d810       ?SetKey@?$TAnimTrack@UIExprKey@@@@UAEXHPAUIKey@@@Z 3403e810 f i AnimNode.obj
 0001:0003d840       ??$fill@PAUIExprKey@@U1@@stlpmtx_std@@YAXPAUIExprKey@@0ABU1@@Z 3403e840 f i AnimNode.obj
 0001:0003d840       ??$fill@PAUISequenceKey@@U1@@stlpmtx_std@@YAXPAUISequenceKey@@0ABU1@@Z 3403e840 f i AnimNode.obj
 0001:0003d890       ??$__push_heap@PAUIExprKey@@HU1@U?$less@UIExprKey@@@stlpmtx_std@@@stlpmtx_std@@YAXPAUIExprKey@@HHU1@U?$less@UIExprKey@@@0@@Z 3403e890 f i AnimNode.obj
 0001:0003d890       ??$__push_heap@PAUISequenceKey@@HU1@U?$less@UISequenceKey@@@stlpmtx_std@@@stlpmtx_std@@YAXPAUISequenceKey@@HHU1@U?$less@UISequenceKey@@@0@@Z 3403e890 f i AnimNode.obj
 0001:0003d900       ?SelectKey@?$TAnimTrack@UISequenceKey@@@@UAEXH_N@Z 3403e900 f i AnimNode.obj
 0001:0003d900       ?SelectKey@?$TAnimTrack@UIExprKey@@@@UAEXH_N@Z 3403e900 f i AnimNode.obj
 0001:0003d940       ?GetNumKeys@?$TAnimTrack@UISequenceKey@@@@UBEHXZ 3403e940 f i AnimNode.obj
 0001:0003d940       ?GetNumKeys@?$TAnimTrack@UIExprKey@@@@UBEHXZ 3403e940 f i AnimNode.obj
 0001:0003d960       ?GetKey@?$TAnimTrack@UISequenceKey@@@@UBEXHPAUIKey@@@Z 3403e960 f i AnimNode.obj
 0001:0003d960       ?GetKey@?$TAnimTrack@UIExprKey@@@@UBEXHPAUIKey@@@Z 3403e960 f i AnimNode.obj
 0001:0003d990       ??$__adjust_heap@PAUISequenceKey@@HU1@U?$less@UISequenceKey@@@stlpmtx_std@@@stlpmtx_std@@YAXPAUISequenceKey@@HHU1@U?$less@UISequenceKey@@@0@@Z 3403e990 f i AnimNode.obj
 0001:0003d990       ??$__adjust_heap@PAUIExprKey@@HU1@U?$less@UIExprKey@@@stlpmtx_std@@@stlpmtx_std@@YAXPAUIExprKey@@HHU1@U?$less@UIExprKey@@@0@@Z 3403e990 f i AnimNode.obj
 0001:0003da40       ?IsKeySelected@?$TAnimTrack@UIExprKey@@@@UBE_NH@Z 3403ea40 f i AnimNode.obj
 0001:0003da40       ?IsKeySelected@?$TAnimTrack@UISequenceKey@@@@UBE_NH@Z 3403ea40 f i AnimNode.obj
 0001:0003da60       ?_M_insert_overflow@?$_Impl_vector@UISequenceKey@@V?$allocator@UISequenceKey@@@stlpmtx_std@@@priv@stlpmtx_std@@AAEXPAUISequenceKey@@ABU4@ABU__true_type@3@I_N@Z 3403ea60 f i AnimNode.obj
 0001:0003da60       ?_M_insert_overflow@?$_Impl_vector@UIExprKey@@V?$allocator@UIExprKey@@@stlpmtx_std@@@priv@stlpmtx_std@@AAEXPAUIExprKey@@ABU4@ABU__true_type@3@I_N@Z 3403ea60 f i AnimNode.obj
 0001:0003dbf0       ??$__uninitialized_fill_n@PAUISequenceKey@@IU1@@priv@stlpmtx_std@@YAPAUISequenceKey@@PAU2@IABU2@@Z 3403ebf0 f i AnimNode.obj
 0001:0003dbf0       ??$__uninitialized_fill_n@PAUIExprKey@@IU1@@priv@stlpmtx_std@@YAPAUIExprKey@@PAU2@IABU2@@Z 3403ebf0 f i AnimNode.obj
 0001:0003dc50       ??$__make_heap@PAUIExprKey@@U?$less@UIExprKey@@@stlpmtx_std@@U1@H@stlpmtx_std@@YAXPAUIExprKey@@0U?$less@UIExprKey@@@0@0PAH@Z 3403ec50 f i AnimNode.obj
 0001:0003dc50       ??$__make_heap@PAUISequenceKey@@U?$less@UISequenceKey@@@stlpmtx_std@@U1@H@stlpmtx_std@@YAXPAUISequenceKey@@0U?$less@UISequenceKey@@@0@0PAH@Z 3403ec50 f i AnimNode.obj
 0001:0003dd80       ?_M_fill_insert_aux@?$_Impl_vector@UISequenceKey@@V?$allocator@UISequenceKey@@@stlpmtx_std@@@priv@stlpmtx_std@@AAEXPAUISequenceKey@@IABU4@ABU__false_type@3@@Z 3403ed80 f i AnimNode.obj
 0001:0003dd80       ?_M_fill_insert_aux@?$_Impl_vector@UIExprKey@@V?$allocator@UIExprKey@@@stlpmtx_std@@@priv@stlpmtx_std@@AAEXPAUIExprKey@@IABU4@ABU__false_type@3@@Z 3403ed80 f i AnimNode.obj
 0001:0003deb0       ??$__insertion_sort@PAUIExprKey@@U1@U?$less@UIExprKey@@@stlpmtx_std@@@priv@stlpmtx_std@@YAXPAUIExprKey@@00U?$less@UIExprKey@@@1@@Z 3403eeb0 f i AnimNode.obj
 0001:0003deb0       ??$__insertion_sort@PAUISequenceKey@@U1@U?$less@UISequenceKey@@@stlpmtx_std@@@priv@stlpmtx_std@@YAXPAUISequenceKey@@00U?$less@UISequenceKey@@@1@@Z 3403eeb0 f i AnimNode.obj
 0001:0003df90       ?RemoveKey@?$TAnimTrack@UIExprKey@@@@UAEXH@Z 3403ef90 f i AnimNode.obj
 0001:0003df90       ?RemoveKey@?$TAnimTrack@UISequenceKey@@@@UAEXH@Z 3403ef90 f i AnimNode.obj
 0001:0003dff0       ?SetKeyValueRange@?$TAnimTrack@UISequenceKey@@@@UAEXMM@Z 3403eff0 f i AnimNode.obj
 0001:0003dff0       ?SetKeyValueRange@?$TAnimTrack@UICaptureKey@@@@UAEXMM@Z 3403eff0 f i AnimNode.obj
 0001:0003dff0       ?SetKeyValueRange@?$TAnimTrack@UIExprKey@@@@UAEXMM@Z 3403eff0 f i AnimNode.obj
 0001:0003dff0       ?SetKeyValueRange@?$TAnimTrack@UICharacterKey@@@@UAEXMM@Z 3403eff0 f i AnimNode.obj
 0001:0003dff0       ?SetKeyValueRange@?$TAnimTrack@UILookAtKey@@@@UAEXMM@Z 3403eff0 f i AnimNode.obj
 0001:0003dff0       ?SetKeyValueRange@?$TAnimTrack@UIDiscreteFloatKey@@@@UAEXMM@Z 3403eff0 f i GotoTrack.obj
 0001:0003dff0       ?SetKeyValueRange@?$TAnimTrack@UISelectKey@@@@UAEXMM@Z 3403eff0 f i AnimNode.obj
 0001:0003dff0       ?SetKeyValueRange@?$TAnimTrack@UISoundKey@@@@UAEXMM@Z 3403eff0 f i AnimNode.obj
 0001:0003dff0       ?SetKeyValueRange@CAnimMaterialNode@@UAEXMM@Z 3403eff0 f i MaterialNode.obj
 0001:0003dff0       ?SetKeyValueRange@?$TAnimTrack@UIMusicKey@@@@UAEXMM@Z 3403eff0 f i AnimNode.obj
 0001:0003dff0       ?SetKeyValueRange@?$TAnimTrack@UIScreenFaderKey@@@@UAEXMM@Z 3403eff0 f i ScreenFaderTrack.obj
 0001:0003dff0       ?SetKeyValueRange@?$TAnimTrack@UIConsoleKey@@@@UAEXMM@Z 3403eff0 f i AnimNode.obj
 0001:0003dff0       ?SetKeyValueRange@?$TAnimTrack@UIEventKey@@@@UAEXMM@Z 3403eff0 f i AnimNode.obj
 0001:0003dff0       ?SetKeyValueRange@?$TAnimTrack@UICommentKey@@@@UAEXMM@Z 3403eff0 f i CommentTrack.obj
 0001:0003dff0       ?SetKeyValueRange@?$TAnimTrack@UIBoolKey@@@@UAEXMM@Z 3403eff0 f i AnimNode.obj
 0001:0003dff0       ?SetKeyValueRange@?$TAnimTrack@UIFaceSeqKey@@@@UAEXMM@Z 3403eff0 f i AnimNode.obj
 0001:0003e010       ??0ICaptureKey@@QAE@ABU0@@Z 3403f010 f i AnimNode.obj
 0001:0003e090       ?CreateKey@?$TAnimTrack@UICaptureKey@@@@UAEHM@Z 3403f090 f i AnimNode.obj
 0001:0003e100       ?CloneKey@?$TAnimTrack@UICaptureKey@@@@UAEHH@Z 3403f100 f i AnimNode.obj
 0001:0003e160       ?CopyKey@?$TAnimTrack@UICaptureKey@@@@UAEHPAUIAnimTrack@@H@Z 3403f160 f i AnimNode.obj
 0001:0003e1c0       ?FindKey@?$TAnimTrack@UICaptureKey@@@@UAEHM@Z 3403f1c0 f i AnimNode.obj
 0001:0003e220       ?GetKeyFlags@?$TAnimTrack@UICaptureKey@@@@UAEHH@Z 3403f220 f i AnimNode.obj
 0001:0003e240       ?SetKey@?$TAnimTrack@UICaptureKey@@@@UAEXHPAUIKey@@@Z 3403f240 f i AnimNode.obj
 0001:0003e270       ?SetKeyTime@?$TAnimTrack@UICaptureKey@@@@UAEXHM@Z 3403f270 f i AnimNode.obj
 0001:0003e2a0       ?SetKeyFlags@?$TAnimTrack@UICaptureKey@@@@UAEXHH@Z 3403f2a0 f i AnimNode.obj
 0001:0003e2c0       ?Serialize@?$TAnimTrack@UICaptureKey@@@@UAE_NAAVXmlNodeRef@@_N1@Z 3403f2c0 f i AnimNode.obj
 0001:0003e570       ?SerializeSelection@?$TAnimTrack@UICaptureKey@@@@UAE_NAAVXmlNodeRef@@_N1M@Z 3403f570 f i AnimNode.obj
 0001:0003e740       ??$fill@PAUICaptureKey@@U1@@stlpmtx_std@@YAXPAUICaptureKey@@0ABU1@@Z 3403f740 f i AnimNode.obj
 0001:0003e790       ??$__push_heap@PAUICaptureKey@@HU1@U?$less@UICaptureKey@@@stlpmtx_std@@@stlpmtx_std@@YAXPAUICaptureKey@@HHU1@U?$less@UICaptureKey@@@0@@Z 3403f790 f i AnimNode.obj
 0001:0003e800       ?SelectKey@?$TAnimTrack@UICaptureKey@@@@UAEXH_N@Z 3403f800 f i AnimNode.obj
 0001:0003e840       ?GetNumKeys@?$TAnimTrack@UICaptureKey@@@@UBEHXZ 3403f840 f i AnimNode.obj
 0001:0003e860       ?GetKey@?$TAnimTrack@UICaptureKey@@@@UBEXHPAUIKey@@@Z 3403f860 f i AnimNode.obj
 0001:0003e890       ?GetKeyTime@?$TAnimTrack@UICaptureKey@@@@UBEMH@Z 3403f890 f i AnimNode.obj
 0001:0003e8b0       ??$__unguarded_insertion_sort_aux@PAUICaptureKey@@U1@U?$less@UICaptureKey@@@stlpmtx_std@@@priv@stlpmtx_std@@YAXPAUICaptureKey@@00U?$less@UICaptureKey@@@1@@Z 3403f8b0 f i AnimNode.obj
 0001:0003e9a0       ??$__adjust_heap@PAUICaptureKey@@HU1@U?$less@UICaptureKey@@@stlpmtx_std@@@stlpmtx_std@@YAXPAUICaptureKey@@HHU1@U?$less@UICaptureKey@@@0@@Z 3403f9a0 f i AnimNode.obj
 0001:0003ea50       ?IsKeySelected@?$TAnimTrack@UICaptureKey@@@@UBE_NH@Z 3403fa50 f i AnimNode.obj
 0001:0003ea70       ?_M_insert_overflow@?$_Impl_vector@UICaptureKey@@V?$allocator@UICaptureKey@@@stlpmtx_std@@@priv@stlpmtx_std@@AAEXPAUICaptureKey@@ABU4@ABU__true_type@3@I_N@Z 3403fa70 f i AnimNode.obj
 0001:0003ebf0       ??$__linear_insert@PAUICaptureKey@@U1@U?$less@UICaptureKey@@@stlpmtx_std@@@priv@stlpmtx_std@@YAXPAUICaptureKey@@0U2@U?$less@UICaptureKey@@@1@@Z 3403fbf0 f i AnimNode.obj
 0001:0003ec90       ??$__make_heap@PAUICaptureKey@@U?$less@UICaptureKey@@@stlpmtx_std@@U1@H@stlpmtx_std@@YAXPAUICaptureKey@@0U?$less@UICaptureKey@@@0@0PAH@Z 3403fc90 f i AnimNode.obj
 0001:0003ed70       ??$__uninitialized_fill_n@PAUICaptureKey@@IU1@@priv@stlpmtx_std@@YAPAUICaptureKey@@PAU2@IABU2@@Z 3403fd70 f i AnimNode.obj
 0001:0003edd0       ??$__unguarded_partition@PAUICaptureKey@@U1@U?$less@UICaptureKey@@@stlpmtx_std@@@priv@stlpmtx_std@@YAPAUICaptureKey@@PAU2@0U2@U?$less@UICaptureKey@@@1@@Z 3403fdd0 f i AnimNode.obj
 0001:0003eec0       ??$__insertion_sort@PAUICaptureKey@@U1@U?$less@UICaptureKey@@@stlpmtx_std@@@priv@stlpmtx_std@@YAXPAUICaptureKey@@00U?$less@UICaptureKey@@@1@@Z 3403fec0 f i AnimNode.obj
 0001:0003ef10       ?RemoveKey@?$TAnimTrack@UICaptureKey@@@@UAEXH@Z 3403ff10 f i AnimNode.obj
 0001:0003ef70       ?_M_fill_insert_aux@?$_Impl_vector@UICaptureKey@@V?$allocator@UICaptureKey@@@stlpmtx_std@@@priv@stlpmtx_std@@AAEXPAUICaptureKey@@IABU4@ABU__false_type@3@@Z 3403ff70 f i AnimNode.obj
 0001:0003f110       ??$__final_insertion_sort@PAUICaptureKey@@U?$less@UICaptureKey@@@stlpmtx_std@@@priv@stlpmtx_std@@YAXPAUICaptureKey@@0U?$less@UICaptureKey@@@1@@Z 34040110 f i AnimNode.obj
 0001:0003f180       ??$sort_heap@PAUICaptureKey@@U?$less@UICaptureKey@@@stlpmtx_std@@@stlpmtx_std@@YAXPAUICaptureKey@@0U?$less@UICaptureKey@@@0@@Z 34040180 f i AnimNode.obj
 0001:0003f330       ??$__insertion_sort@PAUTrackDesc@CAnimNode@@U12@P6A_NABU12@0@Z@priv@stlpmtx_std@@YAXPAUTrackDesc@CAnimNode@@00P6A_NABU23@1@Z@Z 34040330 f i AnimNode.obj
 0001:0003f3a0       ??$__partial_sort@PAUICharacterKey@@U1@U?$less@UICharacterKey@@@stlpmtx_std@@@priv@stlpmtx_std@@YAXPAUICharacterKey@@000U?$less@UICharacterKey@@@1@@Z 340403a0 f i AnimNode.obj
 0001:0003f450       ??$__partial_sort@PAUIBoolKey@@U1@U?$less@UIBoolKey@@@stlpmtx_std@@@priv@stlpmtx_std@@YAXPAUIBoolKey@@000U?$less@UIBoolKey@@@1@@Z 34040450 f i AnimNode.obj
 0001:0003f4d0       ??$__partial_sort@PAUISelectKey@@U1@U?$less@UISelectKey@@@stlpmtx_std@@@priv@stlpmtx_std@@YAXPAUISelectKey@@000U?$less@UISelectKey@@@1@@Z 340404d0 f i AnimNode.obj
 0001:0003f590       ??$__partial_sort@PAUIEventKey@@U1@U?$less@UIEventKey@@@stlpmtx_std@@@priv@stlpmtx_std@@YAXPAUIEventKey@@000U?$less@UIEventKey@@@1@@Z 34040590 f i AnimNode.obj
 0001:0003f650       ??$__partial_sort@PAUISoundKey@@U1@U?$less@UISoundKey@@@stlpmtx_std@@@priv@stlpmtx_std@@YAXPAUISoundKey@@000U?$less@UISoundKey@@@1@@Z 34040650 f i AnimNode.obj
 0001:0003f710       ??$__partial_sort@PAUISequenceKey@@U1@U?$less@UISequenceKey@@@stlpmtx_std@@@priv@stlpmtx_std@@YAXPAUISequenceKey@@000U?$less@UISequenceKey@@@1@@Z 34040710 f i AnimNode.obj
 0001:0003f710       ??$__partial_sort@PAUIExprKey@@U1@U?$less@UIExprKey@@@stlpmtx_std@@@priv@stlpmtx_std@@YAXPAUIExprKey@@000U?$less@UIExprKey@@@1@@Z 34040710 f i AnimNode.obj
 0001:0003f7d0       ??$__partial_sort@PAUIConsoleKey@@U1@U?$less@UIConsoleKey@@@stlpmtx_std@@@priv@stlpmtx_std@@YAXPAUIConsoleKey@@000U?$less@UIConsoleKey@@@1@@Z 340407d0 f i AnimNode.obj
 0001:0003f880       ??$__partial_sort@PAUIMusicKey@@U1@U?$less@UIMusicKey@@@stlpmtx_std@@@priv@stlpmtx_std@@YAXPAUIMusicKey@@000U?$less@UIMusicKey@@@1@@Z 34040880 f i AnimNode.obj
 0001:0003f930       ??$__partial_sort@PAUIFaceSeqKey@@U1@U?$less@UIFaceSeqKey@@@stlpmtx_std@@@priv@stlpmtx_std@@YAXPAUIFaceSeqKey@@000U?$less@UIFaceSeqKey@@@1@@Z 34040930 f i AnimNode.obj
 0001:0003f9f0       ??$__partial_sort@PAUILookAtKey@@U1@U?$less@UILookAtKey@@@stlpmtx_std@@@priv@stlpmtx_std@@YAXPAUILookAtKey@@000U?$less@UILookAtKey@@@1@@Z 340409f0 f i AnimNode.obj
 0001:0003fab0       ??$__partial_sort@PAUICaptureKey@@U1@U?$less@UICaptureKey@@@stlpmtx_std@@@priv@stlpmtx_std@@YAXPAUICaptureKey@@000U?$less@UICaptureKey@@@1@@Z 34040ab0 f i AnimNode.obj
 0001:0003fbe0       ??$__chunk_insertion_sort@PAUTrackDesc@CAnimNode@@HP6A_NABU12@0@Z@priv@stlpmtx_std@@YAXPAUTrackDesc@CAnimNode@@0HP6A_NABU23@1@Z@Z 34040be0 f i AnimNode.obj
 0001:0003fcd0       ??$__rotate_adaptive@PAUTrackDesc@CAnimNode@@PAU12@H@priv@stlpmtx_std@@YAPAUTrackDesc@CAnimNode@@PAU23@00HH0H@Z 34040cd0 f i AnimNode.obj
 0001:0003fd90       ??0CCharacterTrack@@QAE@XZ 34040d90 f i AnimNode.obj
 0001:0003fe00       ?GetAnimationLayerIndex@CCharacterTrack@@UBEHXZ 34040e00 f i AnimNode.obj
 0001:0003fe00       ?GetAnimationLayerIndex@CLookAtTrack@@UBEHXZ 34040e00 f i AnimNode.obj
 0001:0003fe10       ??0CLookAtTrack@@QAE@XZ    34040e10 f i AnimNode.obj
 0001:0003fe80       ?SetAnimationLayerIndex@CLookAtTrack@@UAEXH@Z 34040e80 f i AnimNode.obj
 0001:0003fe80       ?SetAnimationLayerIndex@CCharacterTrack@@UAEXH@Z 34040e80 f i AnimNode.obj
 0001:0003fe90       ?RemoveTrack@CAnimNode@@UAE_NPAUIAnimTrack@@@Z 34040e90 f   AnimNode.obj
 0001:0003fef0       ??0CEventTrack@@QAE@XZ     34040ef0 f i AnimNode.obj
 0001:0003ff60       ?GetMemoryUsage@CCommentTrack@@UBEXPAVICrySizer@@@Z 34040f60 f i CommentTrack.obj
 0001:0003ff60       ?GetMemoryUsage@CTrackEventTrack@@UBEXPAVICrySizer@@@Z 34040f60 f i AnimNode.obj
 0001:0003ff60       ?GetMemoryUsage@CSoundTrack@@UBEXPAVICrySizer@@@Z 34040f60 f i AnimNode.obj
 0001:0003ff60       ?GetMemoryUsage@CExprTrack@@UBEXPAVICrySizer@@@Z 34040f60 f i AnimNode.obj
 0001:0003ff60       ?GetMemoryUsage@CSelectTrack@@UBEXPAVICrySizer@@@Z 34040f60 f i AnimNode.obj
 0001:0003ff60       ?GetMemoryUsage@CBoolTrack@@UBEXPAVICrySizer@@@Z 34040f60 f i AnimNode.obj
 0001:0003ff60       ?GetMemoryUsage@CMusicTrack@@UBEXPAVICrySizer@@@Z 34040f60 f i AnimNode.obj
 0001:0003ff60       ?GetMemoryUsage@CFaceSeqTrack@@UBEXPAVICrySizer@@@Z 34040f60 f i AnimNode.obj
 0001:0003ff60       ?GetMemoryUsage@CSequenceTrack@@UBEXPAVICrySizer@@@Z 34040f60 f i AnimNode.obj
 0001:0003ff60       ?GetMemoryUsage@CEventTrack@@UBEXPAVICrySizer@@@Z 34040f60 f i AnimNode.obj
 0001:0003ff60       ?GetMemoryUsage@CConsoleTrack@@UBEXPAVICrySizer@@@Z 34040f60 f i AnimNode.obj
 0001:0003ff60       ?GetMemoryUsage@CCaptureTrack@@UBEXPAVICrySizer@@@Z 34040f60 f i AnimNode.obj
 0001:0003ff80       ??0CSoundTrack@@QAE@XZ     34040f80 f i AnimNode.obj
 0001:0003fff0       ?IsMasked@CSoundTrack@@UBE_NI@Z 34040ff0 f i AnimNode.obj
 0001:00040000       ??0CExprTrack@@QAE@XZ      34041000 f i AnimNode.obj
 0001:00040070       ??0CConsoleTrack@@QAE@XZ   34041070 f i AnimNode.obj
 0001:000400e0       ??0CMusicTrack@@QAE@XZ     340410e0 f i AnimNode.obj
 0001:00040150       ?IsMasked@CMusicTrack@@UBE_NI@Z 34041150 f i AnimNode.obj
 0001:00040160       ??0CFaceSeqTrack@@QAE@XZ   34041160 f i AnimNode.obj
 0001:000401d0       ??0CTrackEventTrack@@QAE@XZ 340411d0 f i AnimNode.obj
 0001:00040240       ??0CSequenceTrack@@QAE@XZ  34041240 f i AnimNode.obj
 0001:000402b0       ??0CCaptureTrack@@QAE@XZ   340412b0 f i AnimNode.obj
 0001:00040320       ??0CBoolTrack@@QAE@XZ      34041320 f i AnimNode.obj
 0001:00040390       ??0CSelectTrack@@QAE@XZ    34041390 f i AnimNode.obj
 0001:00040400       ??1CAnimNode@@UAE@XZ       34041400 f   AnimNode.obj
 0001:000404c0       ?resize@?$_Impl_vector@UICharacterKey@@V?$allocator@UICharacterKey@@@stlpmtx_std@@@priv@stlpmtx_std@@QAEXIABUICharacterKey@@@Z 340414c0 f i AnimNode.obj
 0001:00040550       ?resize@?$_Impl_vector@UIBoolKey@@V?$allocator@UIBoolKey@@@stlpmtx_std@@@priv@stlpmtx_std@@QAEXIABUIBoolKey@@@Z 34041550 f i AnimNode.obj
 0001:000405f0       ?resize@?$_Impl_vector@UISelectKey@@V?$allocator@UISelectKey@@@stlpmtx_std@@@priv@stlpmtx_std@@QAEXIABUISelectKey@@@Z 340415f0 f i AnimNode.obj
 0001:000406b0       ?resize@?$_Impl_vector@UIEventKey@@V?$allocator@UIEventKey@@@stlpmtx_std@@@priv@stlpmtx_std@@QAEXIABUIEventKey@@@Z 340416b0 f i AnimNode.obj
 0001:00040770       ?resize@?$_Impl_vector@UISoundKey@@V?$allocator@UISoundKey@@@stlpmtx_std@@@priv@stlpmtx_std@@QAEXIABUISoundKey@@@Z 34041770 f i AnimNode.obj
 0001:00040830       ?resize@?$_Impl_vector@UIConsoleKey@@V?$allocator@UIConsoleKey@@@stlpmtx_std@@@priv@stlpmtx_std@@QAEXIABUIConsoleKey@@@Z 34041830 f i AnimNode.obj
 0001:000408f0       ?resize@?$_Impl_vector@UIMusicKey@@V?$allocator@UIMusicKey@@@stlpmtx_std@@@priv@stlpmtx_std@@QAEXIABUIMusicKey@@@Z 340418f0 f i AnimNode.obj
 0001:00040980       ?resize@?$_Impl_vector@UIFaceSeqKey@@V?$allocator@UIFaceSeqKey@@@stlpmtx_std@@@priv@stlpmtx_std@@QAEXIABUIFaceSeqKey@@@Z 34041980 f i AnimNode.obj
 0001:00040a10       ?resize@?$_Impl_vector@UILookAtKey@@V?$allocator@UILookAtKey@@@stlpmtx_std@@@priv@stlpmtx_std@@QAEXIABUILookAtKey@@@Z 34041a10 f i AnimNode.obj
 0001:00040ad0       ?resize@?$_Impl_vector@UIExprKey@@V?$allocator@UIExprKey@@@stlpmtx_std@@@priv@stlpmtx_std@@QAEXIABUIExprKey@@@Z 34041ad0 f i AnimNode.obj
 0001:00040ad0       ?resize@?$_Impl_vector@UISequenceKey@@V?$allocator@UISequenceKey@@@stlpmtx_std@@@priv@stlpmtx_std@@QAEXIABUISequenceKey@@@Z 34041ad0 f i AnimNode.obj
 0001:00040b90       ??$__merge_without_buffer@PAUTrackDesc@CAnimNode@@HP6A_NABU12@0@Z@priv@stlpmtx_std@@YAXPAUTrackDesc@CAnimNode@@00HHP6A_NABU23@1@Z@Z 34041b90 f i AnimNode.obj
 0001:00040cb0       ??$__merge_sort_with_buffer@PAUTrackDesc@CAnimNode@@PAU12@HP6A_NABU12@0@Z@priv@stlpmtx_std@@YAXPAUTrackDesc@CAnimNode@@00PAHP6A_NABU23@2@Z@Z 34041cb0 f i AnimNode.obj
 0001:00040d30       ??$__merge_adaptive@PAUTrackDesc@CAnimNode@@HPAU12@P6A_NABU12@0@Z@priv@stlpmtx_std@@YAXPAUTrackDesc@CAnimNode@@00HH0HP6A_NABU23@1@Z@Z 34041d30 f i AnimNode.obj
 0001:00040ea0       ??0CAnimNode@@QAE@XZ       34041ea0 f   AnimNode.obj
 0001:00040f50       ?push_back@?$_Impl_vector@UTrackDesc@CAnimNode@@V?$allocator@UTrackDesc@CAnimNode@@@stlpmtx_std@@@priv@stlpmtx_std@@QAEXABUTrackDesc@CAnimNode@@@Z 34041f50 f i AnimNode.obj
 0001:00040fd0       ?resize@?$_Impl_vector@UICaptureKey@@V?$allocator@UICaptureKey@@@stlpmtx_std@@@priv@stlpmtx_std@@QAEXIABUICaptureKey@@@Z 34041fd0 f i AnimNode.obj
 0001:00041090       ??$reconstruct@V?$vector@UTrackDesc@CAnimNode@@V?$allocator@UTrackDesc@CAnimNode@@@stlpmtx_std@@@stlpmtx_std@@@stl@@YAXAAV?$vector@UTrackDesc@CAnimNode@@V?$allocator@UTrackDesc@CAnimNode@@@stlpmtx_std@@@stlpmtx_std@@@Z 34042090 f i AnimNode.obj
 0001:00041110       ??$__introsort_loop@PAUICharacterKey@@U1@HU?$less@UICharacterKey@@@stlpmtx_std@@@priv@stlpmtx_std@@YAXPAUICharacterKey@@00HU?$less@UICharacterKey@@@1@@Z 34042110 f i AnimNode.obj
 0001:00041210       ??$__introsort_loop@PAUIBoolKey@@U1@HU?$less@UIBoolKey@@@stlpmtx_std@@@priv@stlpmtx_std@@YAXPAUIBoolKey@@00HU?$less@UIBoolKey@@@1@@Z 34042210 f i AnimNode.obj
 0001:00041320       ??$__introsort_loop@PAUISelectKey@@U1@HU?$less@UISelectKey@@@stlpmtx_std@@@priv@stlpmtx_std@@YAXPAUISelectKey@@00HU?$less@UISelectKey@@@1@@Z 34042320 f i AnimNode.obj
 0001:00041430       ??$__introsort_loop@PAUIEventKey@@U1@HU?$less@UIEventKey@@@stlpmtx_std@@@priv@stlpmtx_std@@YAXPAUIEventKey@@00HU?$less@UIEventKey@@@1@@Z 34042430 f i AnimNode.obj
 0001:00041540       ??$__introsort_loop@PAUISoundKey@@U1@HU?$less@UISoundKey@@@stlpmtx_std@@@priv@stlpmtx_std@@YAXPAUISoundKey@@00HU?$less@UISoundKey@@@1@@Z 34042540 f i AnimNode.obj
 0001:00041650       ??$__introsort_loop@PAUIConsoleKey@@U1@HU?$less@UIConsoleKey@@@stlpmtx_std@@@priv@stlpmtx_std@@YAXPAUIConsoleKey@@00HU?$less@UIConsoleKey@@@1@@Z 34042650 f i AnimNode.obj
 0001:00041750       ??$__introsort_loop@PAUIMusicKey@@U1@HU?$less@UIMusicKey@@@stlpmtx_std@@@priv@stlpmtx_std@@YAXPAUIMusicKey@@00HU?$less@UIMusicKey@@@1@@Z 34042750 f i AnimNode.obj
 0001:00041860       ??$__introsort_loop@PAUIFaceSeqKey@@U1@HU?$less@UIFaceSeqKey@@@stlpmtx_std@@@priv@stlpmtx_std@@YAXPAUIFaceSeqKey@@00HU?$less@UIFaceSeqKey@@@1@@Z 34042860 f i AnimNode.obj
 0001:00041970       ??$__introsort_loop@PAUILookAtKey@@U1@HU?$less@UILookAtKey@@@stlpmtx_std@@@priv@stlpmtx_std@@YAXPAUILookAtKey@@00HU?$less@UILookAtKey@@@1@@Z 34042970 f i AnimNode.obj
 0001:00041a80       ??$__introsort_loop@PAUIExprKey@@U1@HU?$less@UIExprKey@@@stlpmtx_std@@@priv@stlpmtx_std@@YAXPAUIExprKey@@00HU?$less@UIExprKey@@@1@@Z 34042a80 f i AnimNode.obj
 0001:00041a80       ??$__introsort_loop@PAUISequenceKey@@U1@HU?$less@UISequenceKey@@@stlpmtx_std@@@priv@stlpmtx_std@@YAXPAUISequenceKey@@00HU?$less@UISequenceKey@@@1@@Z 34042a80 f i AnimNode.obj
 0001:00041b90       ??$__introsort_loop@PAUICaptureKey@@U1@HU?$less@UICaptureKey@@@stlpmtx_std@@@priv@stlpmtx_std@@YAXPAUICaptureKey@@00HU?$less@UICaptureKey@@@1@@Z 34042b90 f i AnimNode.obj
 0001:00041d00       ??$__inplace_stable_sort@PAUTrackDesc@CAnimNode@@P6A_NABU12@0@Z@priv@stlpmtx_std@@YAXPAUTrackDesc@CAnimNode@@0P6A_NABU23@1@Z@Z 34042d00 f i AnimNode.obj
 0001:00041da0       ??$__stable_sort_adaptive@PAUTrackDesc@CAnimNode@@PAU12@HP6A_NABU12@0@Z@priv@stlpmtx_std@@YAXPAUTrackDesc@CAnimNode@@00HP6A_NABU23@1@Z@Z 34042da0 f i AnimNode.obj
 0001:00041e70       ?SetNumKeys@?$TAnimTrack@UICharacterKey@@@@UAEXH@Z 34042e70 f i AnimNode.obj
 0001:00041ec0       ?SetNumKeys@?$TAnimTrack@UIBoolKey@@@@UAEXH@Z 34042ec0 f i AnimNode.obj
 0001:00041ef0       ?SetNumKeys@?$TAnimTrack@UISelectKey@@@@UAEXH@Z 34042ef0 f i AnimNode.obj
 0001:00041f40       ?SetNumKeys@?$TAnimTrack@UIEventKey@@@@UAEXH@Z 34042f40 f i AnimNode.obj
 0001:00041f90       ?SetNumKeys@?$TAnimTrack@UISoundKey@@@@UAEXH@Z 34042f90 f i AnimNode.obj
 0001:00042010       ?SetNumKeys@?$TAnimTrack@UIExprKey@@@@UAEXH@Z 34043010 f i AnimNode.obj
 0001:00042070       ?SetNumKeys@?$TAnimTrack@UIConsoleKey@@@@UAEXH@Z 34043070 f i AnimNode.obj
 0001:000420a0       ?SetNumKeys@?$TAnimTrack@UIMusicKey@@@@UAEXH@Z 340430a0 f i AnimNode.obj
 0001:000420e0       ?SetNumKeys@?$TAnimTrack@UIFaceSeqKey@@@@UAEXH@Z 340430e0 f i AnimNode.obj
 0001:00042120       ?SetNumKeys@?$TAnimTrack@UILookAtKey@@@@UAEXH@Z 34043120 f i AnimNode.obj
 0001:00042180       ?SetNumKeys@?$TAnimTrack@UISequenceKey@@@@UAEXH@Z 34043180 f i AnimNode.obj
 0001:000421d0       ??$sort@PAUICharacterKey@@@stlpmtx_std@@YAXPAUICharacterKey@@0@Z 340431d0 f i AnimNode.obj
 0001:00042230       ??$sort@PAUIBoolKey@@@stlpmtx_std@@YAXPAUIBoolKey@@0@Z 34043230 f i AnimNode.obj
 0001:000422b0       ??$sort@PAUISelectKey@@@stlpmtx_std@@YAXPAUISelectKey@@0@Z 340432b0 f i AnimNode.obj
 0001:00042310       ??$sort@PAUIEventKey@@@stlpmtx_std@@YAXPAUIEventKey@@0@Z 34043310 f i AnimNode.obj
 0001:00042370       ??$sort@PAUISoundKey@@@stlpmtx_std@@YAXPAUISoundKey@@0@Z 34043370 f i AnimNode.obj
 0001:000423d0       ??$sort@PAUIConsoleKey@@@stlpmtx_std@@YAXPAUIConsoleKey@@0@Z 340433d0 f i AnimNode.obj
 0001:00042430       ??$sort@PAUIMusicKey@@@stlpmtx_std@@YAXPAUIMusicKey@@0@Z 34043430 f i AnimNode.obj
 0001:00042490       ??$sort@PAUIFaceSeqKey@@@stlpmtx_std@@YAXPAUIFaceSeqKey@@0@Z 34043490 f i AnimNode.obj
 0001:000424f0       ??$sort@PAUILookAtKey@@@stlpmtx_std@@YAXPAUILookAtKey@@0@Z 340434f0 f i AnimNode.obj
 0001:00042550       ??$sort@PAUISequenceKey@@@stlpmtx_std@@YAXPAUISequenceKey@@0@Z 34043550 f i AnimNode.obj
 0001:00042550       ??$sort@PAUIExprKey@@@stlpmtx_std@@YAXPAUIExprKey@@0@Z 34043550 f i AnimNode.obj
 0001:000425b0       ??$sort@PAUICaptureKey@@@stlpmtx_std@@YAXPAUICaptureKey@@0@Z 340435b0 f i AnimNode.obj
 0001:00042610       ??$__stable_sort_aux@PAUTrackDesc@CAnimNode@@U12@HP6A_NABU12@0@Z@priv@stlpmtx_std@@YAXPAUTrackDesc@CAnimNode@@00PAHP6A_NABU23@2@Z@Z 34043610 f i AnimNode.obj
 0001:000426e0       ?SetNumKeys@?$TAnimTrack@UICaptureKey@@@@UAEXH@Z 340436e0 f i AnimNode.obj
 0001:00042710       ?SortKeys@?$TAnimTrack@UICharacterKey@@@@UAEXXZ 34043710 f i AnimNode.obj
 0001:00042730       ?SortKeys@?$TAnimTrack@UIBoolKey@@@@UAEXXZ 34043730 f i AnimNode.obj
 0001:00042750       ?SortKeys@?$TAnimTrack@UISelectKey@@@@UAEXXZ 34043750 f i AnimNode.obj
 0001:00042770       ?SortKeys@?$TAnimTrack@UIEventKey@@@@UAEXXZ 34043770 f i AnimNode.obj
 0001:00042790       ?SortKeys@?$TAnimTrack@UISoundKey@@@@UAEXXZ 34043790 f i AnimNode.obj
 0001:000427b0       ?SortKeys@?$TAnimTrack@UIConsoleKey@@@@UAEXXZ 340437b0 f i AnimNode.obj
 0001:000427d0       ?SortKeys@?$TAnimTrack@UIMusicKey@@@@UAEXXZ 340437d0 f i AnimNode.obj
 0001:000427f0       ?SortKeys@?$TAnimTrack@UIFaceSeqKey@@@@UAEXXZ 340437f0 f i AnimNode.obj
 0001:00042810       ?SortKeys@?$TAnimTrack@UILookAtKey@@@@UAEXXZ 34043810 f i AnimNode.obj
 0001:00042830       ?SortKeys@?$TAnimTrack@UISequenceKey@@@@UAEXXZ 34043830 f i AnimNode.obj
 0001:00042830       ?SortKeys@?$TAnimTrack@UIExprKey@@@@UAEXXZ 34043830 f i AnimNode.obj
 0001:00042850       ?SortKeys@?$TAnimTrack@UICaptureKey@@@@UAEXXZ 34043850 f i AnimNode.obj
 0001:00042870       ?AddTrack@CAnimNode@@IAEXABVAnimParamType@@PAUIAnimTrack@@@Z 34043870 f   AnimNode.obj
 0001:00042960       ?SetTrack@CAnimNode@@UAEXABVAnimParamType@@PAUIAnimTrack@@@Z 34043960 f   AnimNode.obj
 0001:00042a70       ?CreateTrackInternalFloat@CAnimNode@@IBEPAUIAnimTrack@@H@Z 34043a70 f   AnimNode.obj
 0001:00042ac0       ?CreateTrackInternalVector@CAnimNode@@IBEPAUIAnimTrack@@W4EAnimCurveType@@ABVAnimParamType@@W4EAnimValue@@@Z 34043ac0 f   AnimNode.obj
 0001:00042e70       ?CreateTrackInternalQuat@CAnimNode@@IBEPAUIAnimTrack@@W4EAnimCurveType@@ABVAnimParamType@@@Z 34043e70 f   AnimNode.obj
 0001:00042f50       ?CreateTrackInternal@CAnimNode@@IAEPAUIAnimTrack@@ABVAnimParamType@@W4EAnimCurveType@@W4EAnimValue@@@Z 34043f50 f   AnimNode.obj
 0001:000432f0       ?CreateTrack@CAnimNode@@UAEPAUIAnimTrack@@ABVAnimParamType@@@Z 340442f0 f   AnimNode.obj
 0001:00043310       ?SerializeAnims@CAnimNode@@UAEXAAVXmlNodeRef@@_N1@Z 34044310 f   AnimNode.obj
 0001:00043990       ?GetType@CAnimPostFXNode@@UBE?AW4EAnimNodeType@@XZ 34044990 f   AnimPostFXNode.obj
 0001:000439a0       ?Release@CAnimNode@@$4PPPPPPPM@3AEXXZ 340449a0 f i AnimPostFXNode.obj
 0001:000439b0       ??F?$_Rb_tree_iterator@V?$CryStringT@D@@U?$_SetTraitsT@V?$CryStringT@D@@@priv@stlpmtx_std@@@priv@stlpmtx_std@@QAEAAU012@XZ 340449b0 f i EntityNode.obj
 0001:000439b0       ??F?$_Rb_tree_iterator@U?$pair@$$CBHPAUIAnimNode@@@stlpmtx_std@@U?$_MapTraitsT@U?$pair@$$CBHPAUIAnimNode@@@stlpmtx_std@@@priv@2@@priv@stlpmtx_std@@QAEAAU012@XZ 340449b0 f i AnimSequence.obj
 0001:000439b0       ??F?$_Rb_tree_iterator@U?$pair@$$CBV?$CryStringT@D@@V?$_smart_ptr@UIFacialAnimSequence@@@@@stlpmtx_std@@U?$_MapTraitsT@U?$pair@$$CBV?$CryStringT@D@@V?$_smart_ptr@UIFacialAnimSequence@@@@@stlpmtx_std@@@priv@2@@priv@stlpmtx_std@@QAEAAU012@XZ 340449b0 f i EntityNode.obj
 0001:000439b0       ??F?$_Rb_tree_iterator@U?$pair@QAUIEntity@@PAUIAnimNode@@@stlpmtx_std@@U?$_MapTraitsT@U?$pair@QAUIEntity@@PAUIAnimNode@@@stlpmtx_std@@@priv@2@@priv@stlpmtx_std@@QAEAAU012@XZ 340449b0 f i Movie.obj
 0001:000439b0       ??F?$_Rb_tree_iterator@U?$pair@$$CBW4EAnimNodeType@@V?$_smart_ptr@VCFXNodeDescription@@@@@stlpmtx_std@@U?$_MapTraitsT@U?$pair@$$CBW4EAnimNodeType@@V?$_smart_ptr@VCFXNodeDescription@@@@@stlpmtx_std@@@priv@2@@priv@stlpmtx_std@@QAEAAU012@XZ 340449b0 f i AnimPostFXNode.obj
 0001:000439b0       ??F?$_Rb_tree_iterator@U?$pair@QAUIAnimSequence@@V?$vector@PAUIMovieListener@@V?$allocator@PAUIMovieListener@@@stlpmtx_std@@@stlpmtx_std@@@stlpmtx_std@@U?$_MapTraitsT@U?$pair@QAUIAnimSequence@@V?$vector@PAUIMovieListener@@V?$allocator@PAUIMovieListener@@@stlpmtx_std@@@stlpmtx_std@@@stlpmtx_std@@@priv@2@@priv@stlpmtx_std@@QAEAAU012@XZ 340449b0 f i Movie.obj
 0001:000439b0       ??F?$_Rb_tree_iterator@U?$pair@$$CBV?$CryStringT@D@@PAVCLightAnimWrapper@@@stlpmtx_std@@U?$_MapTraitsT@U?$pair@$$CBV?$CryStringT@D@@PAVCLightAnimWrapper@@@stlpmtx_std@@@priv@2@@priv@stlpmtx_std@@QAEAAU012@XZ 340449b0 f i Movie.obj
 0001:00043a00       ?GetParamCount@CAnimPostFXNode@@UBEHXZ 34044a00 f   AnimPostFXNode.obj
 0001:00043a20       ?allocate@?$_STLP_alloc_proxy@PAPAXPAXV?$allocator@PAX@stlpmtx_std@@@priv@stlpmtx_std@@QAEPAPAXIAAI@Z 34044a20 f i Movie.obj
 0001:00043a20       ?allocate@?$_STLP_alloc_proxy@PAIIV?$allocator@I@stlpmtx_std@@@priv@stlpmtx_std@@QAEPAIIAAI@Z 34044a20 f i EntityNode.obj
 0001:00043a20       ?allocate@?$_STLP_alloc_proxy@PAV?$_smart_ptr@VCControlParamBase@CFXNodeDescription@@@@V1@V?$allocator@V?$_smart_ptr@VCControlParamBase@CFXNodeDescription@@@@@stlpmtx_std@@@priv@stlpmtx_std@@QAEPAV?$_smart_ptr@VCControlParamBase@CFXNodeDescription@@@@IAAI@Z 34044a20 f i AnimPostFXNode.obj
 0001:00043a70       ?GetParamInfo@CAnimPostFXNode@@UBE_NHAAUSParamInfo@IAnimNode@@@Z 34044a70 f   AnimPostFXNode.obj
 0001:00043ac0       ?GetParamInfoFromId@CAnimPostFXNode@@UBE_NABVAnimParamType@@AAUSParamInfo@IAnimNode@@@Z 34044ac0 f   AnimPostFXNode.obj
 0001:00043ba0       ?CreateDefaultTracks@CAnimPostFXNode@@UAEXXZ 34044ba0 f   AnimPostFXNode.obj
 0001:00043c70       ?Animate@CAnimPostFXNode@@UAEXAAUSAnimContext@@@Z 34044c70 f   AnimPostFXNode.obj
 0001:00043e00       ?Reset@CAnimPostFXNode@@UAEXXZ 34044e00 f   AnimPostFXNode.obj
 0001:00043f50       ?SetDefault@?$TControlParam@M@CFXNodeDescription@@UAEXM@Z 34044f50 f i AnimPostFXNode.obj
 0001:00043f70       ?GetDefault@?$TControlParam@M@CFXNodeDescription@@UBEXAAM@Z 34044f70 f i AnimPostFXNode.obj
 0001:00043f80       ??_E?$TControlParam@M@CFXNodeDescription@@MAEPAXI@Z 34044f80 f i AnimPostFXNode.obj
 0001:00043f80       ??_G?$TControlParam@M@CFXNodeDescription@@MAEPAXI@Z 34044f80 f i AnimPostFXNode.obj
 0001:00043f80       ??_ECControlParamBase@CFXNodeDescription@@MAEPAXI@Z 34044f80 f i AnimPostFXNode.obj
 0001:00043f80       ??_GCControlParamBase@CFXNodeDescription@@MAEPAXI@Z 34044f80 f i AnimPostFXNode.obj
 0001:00043f80       ??_G?$TControlParam@_N@CFXNodeDescription@@MAEPAXI@Z 34044f80 f i AnimPostFXNode.obj
 0001:00043f80       ??_E?$TControlParam@_N@CFXNodeDescription@@MAEPAXI@Z 34044f80 f i AnimPostFXNode.obj
 0001:00043fe0       ?SetDefault@?$TControlParam@_N@CFXNodeDescription@@UAEX_N@Z 34044fe0 f i AnimPostFXNode.obj
 0001:00043ff0       ?GetDefault@?$TControlParam@_N@CFXNodeDescription@@UBEXAA_N@Z 34044ff0 f i AnimPostFXNode.obj
 0001:00044000       ?_M_create_node@?$_Rb_tree@W4EAnimNodeType@@U?$less@W4EAnimNodeType@@@stlpmtx_std@@U?$pair@$$CBW4EAnimNodeType@@V?$_smart_ptr@VCFXNodeDescription@@@@@3@U?$_Select1st@U?$pair@$$CBW4EAnimNodeType@@V?$_smart_ptr@VCFXNodeDescription@@@@@stlpmtx_std@@@priv@3@U?$_MapTraitsT@U?$pair@$$CBW4EAnimNodeType@@V?$_smart_ptr@VCFXNodeDescription@@@@@stlpmtx_std@@@63@V?$allocator@U?$pair@$$CBW4EAnimNodeType@@V?$_smart_ptr@VCFXNodeDescription@@@@@stlpmtx_std@@@3@@priv@stlpmtx_std@@IAEPAU_Rb_tree_node_base@23@ABU?$pair@$$CBW4EAnimNodeType@@V?$_smart_ptr@VCFXNodeDescription@@@@@3@@Z 34045000 f i AnimPostFXNode.obj
 0001:00044060       ?SerializeAnims@CAnimPostFXNode@@UAEXAAVXmlNodeRef@@_N1@Z 34045060 f   AnimPostFXNode.obj
 0001:00044180       ?_M_erase@?$_Rb_tree@W4EAnimNodeType@@U?$less@W4EAnimNodeType@@@stlpmtx_std@@U?$pair@$$CBW4EAnimNodeType@@V?$_smart_ptr@VCFXNodeDescription@@@@@3@U?$_Select1st@U?$pair@$$CBW4EAnimNodeType@@V?$_smart_ptr@VCFXNodeDescription@@@@@stlpmtx_std@@@priv@3@U?$_MapTraitsT@U?$pair@$$CBW4EAnimNodeType@@V?$_smart_ptr@VCFXNodeDescription@@@@@stlpmtx_std@@@63@V?$allocator@U?$pair@$$CBW4EAnimNodeType@@V?$_smart_ptr@VCFXNodeDescription@@@@@stlpmtx_std@@@3@@priv@stlpmtx_std@@AAEXPAU_Rb_tree_node_base@23@@Z 34045180 f i AnimPostFXNode.obj
 0001:000441d0       ?_M_insert@?$_Rb_tree@W4EAnimNodeType@@U?$less@W4EAnimNodeType@@@stlpmtx_std@@U?$pair@$$CBW4EAnimNodeType@@V?$_smart_ptr@VCFXNodeDescription@@@@@3@U?$_Select1st@U?$pair@$$CBW4EAnimNodeType@@V?$_smart_ptr@VCFXNodeDescription@@@@@stlpmtx_std@@@priv@3@U?$_MapTraitsT@U?$pair@$$CBW4EAnimNodeType@@V?$_smart_ptr@VCFXNodeDescription@@@@@stlpmtx_std@@@63@V?$allocator@U?$pair@$$CBW4EAnimNodeType@@V?$_smart_ptr@VCFXNodeDescription@@@@@stlpmtx_std@@@3@@priv@stlpmtx_std@@AAE?AU?$_Rb_tree_iterator@U?$pair@$$CBW4EAnimNodeType@@V?$_smart_ptr@VCFXNodeDescription@@@@@stlpmtx_std@@U?$_MapTraitsT@U?$pair@$$CBW4EAnimNodeType@@V?$_smart_ptr@VCFXNodeDescription@@@@@stlpmtx_std@@@priv@2@@23@PAU_Rb_tree_node_base@23@ABU?$pair@$$CBW4EAnimNodeType@@V?$_smart_ptr@VCFXNodeDescription@@@@@3@00@Z 340451d0 f i AnimPostFXNode.obj
 0001:00044260       ?insert_unique@?$_Rb_tree@W4EAnimNodeType@@U?$less@W4EAnimNodeType@@@stlpmtx_std@@U?$pair@$$CBW4EAnimNodeType@@V?$_smart_ptr@VCFXNodeDescription@@@@@3@U?$_Select1st@U?$pair@$$CBW4EAnimNodeType@@V?$_smart_ptr@VCFXNodeDescription@@@@@stlpmtx_std@@@priv@3@U?$_MapTraitsT@U?$pair@$$CBW4EAnimNodeType@@V?$_smart_ptr@VCFXNodeDescription@@@@@stlpmtx_std@@@63@V?$allocator@U?$pair@$$CBW4EAnimNodeType@@V?$_smart_ptr@VCFXNodeDescription@@@@@stlpmtx_std@@@3@@priv@stlpmtx_std@@QAE?AU?$pair@U?$_Rb_tree_iterator@U?$pair@$$CBW4EAnimNodeType@@V?$_smart_ptr@VCFXNodeDescription@@@@@stlpmtx_std@@U?$_MapTraitsT@U?$pair@$$CBW4EAnimNodeType@@V?$_smart_ptr@VCFXNodeDescription@@@@@stlpmtx_std@@@priv@2@@priv@stlpmtx_std@@_N@3@ABU?$pair@$$CBW4EAnimNodeType@@V?$_smart_ptr@VCFXNodeDescription@@@@@3@@Z 34045260 f i AnimPostFXNode.obj
 0001:00044370       ?_M_clear@?$_Impl_vector@V?$_smart_ptr@VCControlParamBase@CFXNodeDescription@@@@V?$allocator@V?$_smart_ptr@VCControlParamBase@CFXNodeDescription@@@@@stlpmtx_std@@@priv@stlpmtx_std@@AAEXXZ 34045370 f i AnimPostFXNode.obj
 0001:000443b0       ?insert_unique@?$_Rb_tree@W4EAnimNodeType@@U?$less@W4EAnimNodeType@@@stlpmtx_std@@U?$pair@$$CBW4EAnimNodeType@@V?$_smart_ptr@VCFXNodeDescription@@@@@3@U?$_Select1st@U?$pair@$$CBW4EAnimNodeType@@V?$_smart_ptr@VCFXNodeDescription@@@@@stlpmtx_std@@@priv@3@U?$_MapTraitsT@U?$pair@$$CBW4EAnimNodeType@@V?$_smart_ptr@VCFXNodeDescription@@@@@stlpmtx_std@@@63@V?$allocator@U?$pair@$$CBW4EAnimNodeType@@V?$_smart_ptr@VCFXNodeDescription@@@@@stlpmtx_std@@@3@@priv@stlpmtx_std@@QAE?AU?$_Rb_tree_iterator@U?$pair@$$CBW4EAnimNodeType@@V?$_smart_ptr@VCFXNodeDescription@@@@@stlpmtx_std@@U?$_MapTraitsT@U?$pair@$$CBW4EAnimNodeType@@V?$_smart_ptr@VCFXNodeDescription@@@@@stlpmtx_std@@@priv@2@@23@U423@ABU?$pair@$$CBW4EAnimNodeType@@V?$_smart_ptr@VCFXNodeDescription@@@@@3@@Z 340453b0 f i AnimPostFXNode.obj
 0001:000445a0       ??$_M_allocate_and_copy@PAV?$_smart_ptr@VCControlParamBase@CFXNodeDescription@@@@@?$_Impl_vector@V?$_smart_ptr@VCControlParamBase@CFXNodeDescription@@@@V?$allocator@V?$_smart_ptr@VCControlParamBase@CFXNodeDescription@@@@@stlpmtx_std@@@priv@stlpmtx_std@@AAEPAV?$_smart_ptr@VCControlParamBase@CFXNodeDescription@@@@AAIPAV3@1@Z 340455a0 f i AnimPostFXNode.obj
 0001:00044630       ?_M_insert_overflow_aux@?$_Impl_vector@V?$_smart_ptr@UIAnimSequence@@@@V?$allocator@V?$_smart_ptr@UIAnimSequence@@@@@stlpmtx_std@@@priv@stlpmtx_std@@AAEXPAV?$_smart_ptr@UIAnimSequence@@@@ABV4@ABU__false_type@3@I_N@Z 34045630 f i AnimSequenceGroup.obj
 0001:00044630       ?_M_insert_overflow_aux@?$_Impl_vector@V?$_smart_ptr@UIAnimSequenceGroup@@@@V?$allocator@V?$_smart_ptr@UIAnimSequenceGroup@@@@@stlpmtx_std@@@priv@stlpmtx_std@@AAEXPAV?$_smart_ptr@UIAnimSequenceGroup@@@@ABV4@ABU__false_type@3@I_N@Z 34045630 f i AnimSequenceGroup.obj
 0001:00044630       ?_M_insert_overflow_aux@?$_Impl_vector@V?$_smart_ptr@VCControlParamBase@CFXNodeDescription@@@@V?$allocator@V?$_smart_ptr@VCControlParamBase@CFXNodeDescription@@@@@stlpmtx_std@@@priv@stlpmtx_std@@AAEXPAV?$_smart_ptr@VCControlParamBase@CFXNodeDescription@@@@ABV4@ABU__false_type@3@I_N@Z 34045630 f i AnimPostFXNode.obj
 0001:00044810       ??$?AW4EAnimNodeType@@@?$map@W4EAnimNodeType@@V?$_smart_ptr@VCFXNodeDescription@@@@U?$less@W4EAnimNodeType@@@stlpmtx_std@@V?$allocator@U?$pair@$$CBW4EAnimNodeType@@V?$_smart_ptr@VCFXNodeDescription@@@@@stlpmtx_std@@@4@@stlpmtx_std@@QAEAAV?$_smart_ptr@VCFXNodeDescription@@@@ABW4EAnimNodeType@@@Z 34045810 f i AnimPostFXNode.obj
 0001:00044890       ??0CFXNodeDescription@@QAE@W4EAnimNodeType@@@Z 34045890 f i AnimPostFXNode.obj
 0001:000448f0       ??_ECFXNodeDescription@@UAEPAXI@Z 340458f0 f i AnimPostFXNode.obj
 0001:000448f0       ??_GCFXNodeDescription@@UAEPAXI@Z 340458f0 f i AnimPostFXNode.obj
 0001:00044960       ??$AddSupportedParam@M@CFXNodeDescription@@QAEXPBDW4EAnimValue@@0M@Z 34045960 f i AnimPostFXNode.obj
 0001:00044a90       ??$AddSupportedParam@_N@CFXNodeDescription@@QAEXPBDW4EAnimValue@@0_N@Z 34045a90 f i AnimPostFXNode.obj
 0001:00044bc0       ?Initialize@CAnimPostFXNode@@SAXXZ 34045bc0 f   AnimPostFXNode.obj
 0001:00045190       ?CreateNode@CAnimPostFXNode@@SAPAVCAnimNode@@W4EAnimNodeType@@@Z 34046190 f   AnimPostFXNode.obj
 0001:00045250       ?GetType@CAnimScreenFaderNode@@UBE?AW4EAnimNodeType@@XZ 34046250 f i AnimScreenFaderNode.obj
 0001:00045260       ?NeedToRender@CAnimScreenFaderNode@@MBE_NXZ 34046260 f i AnimScreenFaderNode.obj
 0001:00045270       ?Reset@CAnimScreenFaderNode@@UAEXXZ 34046270 f   AnimScreenFaderNode.obj
 0001:00045270       ?ClearCustomColor@CCompoundSplineTrack@@UAEXXZ 34046270 f   CompoundSplineTrack.obj
 0001:00045280       ?Release@CAnimNode@@$4PPPPPPPM@CE@AEXXZ 34046280 f i AnimScreenFaderNode.obj
 0001:00045290       ??_ECAnimScreenFaderNode@@$4PPPPPPPM@A@AEPAXI@Z 34046290 f i AnimScreenFaderNode.obj
 0001:000452a0       ?CalculateIsolatedKeyColor@@YA_NABUIScreenFaderKey@@MAAU?$Vec4_tpl@M@@@Z 340462a0 f   AnimScreenFaderNode.obj
 0001:00045340       ??_GCAnimScreenFaderNode@@UAEPAXI@Z 34046340 f i AnimScreenFaderNode.obj
 0001:00045340       ??_ECAnimScreenFaderNode@@UAEPAXI@Z 34046340 f i AnimScreenFaderNode.obj
 0001:00045390       ?CreateDefaultTracks@CAnimScreenFaderNode@@UAEXXZ 34046390 f   AnimScreenFaderNode.obj
 0001:000453e0       ?GetParamCount@CAnimScreenFaderNode@@UBEHXZ 340463e0 f   AnimScreenFaderNode.obj
 0001:00045400       ?Render@CAnimScreenFaderNode@@UAEXXZ 34046400 f   AnimScreenFaderNode.obj
 0001:000455d0       ?IsAnyTextureVisible@CAnimScreenFaderNode@@QBE_NXZ 340465d0 f   AnimScreenFaderNode.obj
 0001:00045670       ?GetActiveKey@?$TAnimTrack@UIScreenFaderKey@@@@QAEHMPAUIScreenFaderKey@@@Z 34046670 f i AnimScreenFaderNode.obj
 0001:00045800       ?Animate@CAnimScreenFaderNode@@UAEXAAUSAnimContext@@@Z 34046800 f   AnimScreenFaderNode.obj
 0001:00045c00       ?GetParamInfo@CAnimScreenFaderNode@@UBE_NHAAUSParamInfo@IAnimNode@@@Z 34046c00 f   AnimScreenFaderNode.obj
 0001:00045c50       ?GetParamInfoFromId@CAnimScreenFaderNode@@UBE_NABVAnimParamType@@AAUSParamInfo@IAnimNode@@@Z 34046c50 f   AnimScreenFaderNode.obj
 0001:00045d10       ?PrecacheTexData@CAnimScreenFaderNode@@AAEXXZ 34046d10 f   AnimScreenFaderNode.obj
 0001:00045d60       ?Activate@CAnimScreenFaderNode@@UAEX_N@Z 34046d60 f   AnimScreenFaderNode.obj
 0001:00045d80       ?Serialize@CAnimScreenFaderNode@@UAEXAAVXmlNodeRef@@_N1@Z 34046d80 f   AnimScreenFaderNode.obj
 0001:00045db0       ?Initialize@CAnimScreenFaderNode@@SAXXZ 34046db0 f   AnimScreenFaderNode.obj
 0001:00045e30       ??0CAnimScreenFaderNode@@QAE@XZ 34046e30 f   AnimScreenFaderNode.obj
 0001:00045ee0       ?Animate@CCommentNode@@UAEXAAUSAnimContext@@@Z 34046ee0 f   CommentNode.obj
 0001:00045f50       ?CreateDefaultTracks@CCommentNode@@UAEXXZ 34046f50 f   CommentNode.obj
 0001:00046080       ?GetParamCount@CCommentNode@@UBEHXZ 34047080 f   CommentNode.obj
 0001:000460a0       ?GetParamInfo@CCommentNode@@UBE_NHAAUSParamInfo@IAnimNode@@@Z 340470a0 f   CommentNode.obj
 0001:000460f0       ?GetParamInfoFromId@CCommentNode@@UBE_NABVAnimParamType@@AAUSParamInfo@IAnimNode@@@Z 340470f0 f   CommentNode.obj
 0001:000461b0       ?Initialize@CCommentNode@@SAXXZ 340471b0 f   CommentNode.obj
 0001:000462c0       ??0CCommentNode@@QAE@XZ    340472c0 f   CommentNode.obj
 0001:00046320       ??_ECAnimNodeGroup@@$4PPPPPPPM@A@AEPAXI@Z 34047320 f i AnimSequence.obj
 0001:00046320       ??_ECAnimNode@@$4PPPPPPPM@A@AEPAXI@Z 34047320 f i AnimNode.obj
 0001:00046320       ??_ECCommentNode@@$4PPPPPPPM@A@AEPAXI@Z 34047320 f i CommentNode.obj
 0001:00046330       ??_GCCommentNode@@UAEPAXI@Z 34047330 f i CommentNode.obj
 0001:00046330       ??_GCAnimNode@@UAEPAXI@Z   34047330 f i AnimNode.obj
 0001:00046330       ??_ECAnimNode@@UAEPAXI@Z   34047330 f i AnimNode.obj
 0001:00046330       ??_ECCommentNode@@UAEPAXI@Z 34047330 f i CommentNode.obj
 0001:00046330       ??_GCAnimNodeGroup@@UAEPAXI@Z 34047330 f i AnimSequence.obj
 0001:00046330       ??_ECAnimNodeGroup@@UAEPAXI@Z 34047330 f i AnimSequence.obj
 0001:00046360       ?Reset@CAnimScriptVarNode@@UAEXXZ 34047360 f   ScriptVarNode.obj
 0001:00046360       ?Reset@CAnimCVarNode@@UAEXXZ 34047360 f   CVarNode.obj
 0001:00046370       ??0CAnimCVarNode@@QAE@XZ   34047370 f   CVarNode.obj
 0001:000463e0       ?GetParamInfoFromId@CAnimScriptVarNode@@UBE_NABVAnimParamType@@AAUSParamInfo@IAnimNode@@@Z 340473e0 f   ScriptVarNode.obj
 0001:000463e0       ?GetParamInfoFromId@CAnimCVarNode@@UBE_NABVAnimParamType@@AAUSParamInfo@IAnimNode@@@Z 340473e0 f   CVarNode.obj
 0001:00046410       ?Animate@CAnimCVarNode@@UAEXAAUSAnimContext@@@Z 34047410 f   CVarNode.obj
 0001:000464f0       ?SetName@CAnimCVarNode@@UAEXPBD@Z 340474f0 f   CVarNode.obj
 0001:00046560       ?CryWarning@@YAXW4EValidatorModule@@W4EValidatorSeverity@@PBDZZ 34047560 f i EntityNode.obj
 0001:000465a0       ?GetEntity@CAnimEntityNode@@UAEPAUIEntity@@XZ 340475a0 f   EntityNode.obj
 0001:000465e0       ?SetEntityGuid@CAnimEntityNode@@UAEXAB_K@Z 340475e0 f   EntityNode.obj
 0001:00046620       ?SetEntityGuidTarget@CAnimEntityNode@@UAEXAB_K@Z 34047620 f   EntityNode.obj
 0001:00046660       ?SetEntityGuidSource@CAnimEntityNode@@UAEXAB_K@Z 34047660 f   EntityNode.obj
 0001:000466a0       ?ResetHard@CAnimEntityNode@@UAEXXZ 340476a0 f   EntityNode.obj
 0001:000466c0       ?Serialize@CAnimEntityNode@@UAEXAAVXmlNodeRef@@_N1@Z 340476c0 f   EntityNode.obj
 0001:00046860       ?CheckTimeJumpingOrOtherChanges@CAnimEntityNode@@IAE_NABUSAnimContext@@QAHHPAUICharacterInstance@@HH@Z 34047860 f   EntityNode.obj
 0001:00046970       ?ManualSeekAnimationInFIFO@CAnimEntityNode@@IAEXPAUICharacterInstance@@IIM_N@Z 34047970 f   EntityNode.obj
 0001:000469d0       ?SetLayerTime@CAnimEntityNode@@IAEXPAUICharacterInstance@@IM@Z 340479d0 f   EntityNode.obj
 0001:00046a20       ??4?$_smart_ptr@UISound@@@@QAEAAV0@PAUISound@@@Z 34047a20 f i EntityNode.obj
 0001:00046a50       ??4SmartScriptTable@@QAEAAV0@PAUIScriptTable@@@Z 34047a50 f i EntityNode.obj
 0001:00046a80       ??$GetValue@M@IScriptTable@@QAE_NPBDAAM@Z 34047a80 f i EntityNode.obj
 0001:00046b10       ??$GetValue@U?$Vec3_tpl@M@@@IScriptTable@@QAE_NPBDAAU?$Vec3_tpl@M@@@Z 34047b10 f i EntityNode.obj
 0001:00046bb0       ??$GetValue@_N@IScriptTable@@QAE_NPBDAA_N@Z 34047bb0 f i EntityNode.obj
 0001:00046c30       ??$SetValue@H@IScriptTable@@QAEXPBDABH@Z 34047c30 f i EntityNode.obj
 0001:00046ca0       ??$SetValue@_N@IScriptTable@@QAEXPBDAB_N@Z 34047ca0 f i EntityNode.obj
 0001:00046d10       ??$GetValue@VSmartScriptTable@@@IScriptTable@@QAE_NPBDAAVSmartScriptTable@@@Z 34047d10 f i EntityNode.obj
 0001:00046dd0       ??$PushFuncParam@PAUIScriptTable@@@IScriptSystem@@QAEXABQAUIScriptTable@@@Z 34047dd0 f i EntityNode.obj
 0001:00046e40       ??1Iterator@IScriptTable@@QAE@XZ 34047e40 f i EntityNode.obj
 0001:00046ed0       ?ApplyEventKey@CAnimEntityNode@@IAEXPAVCEventTrack@@HAAUIEventKey@@@Z 34047ed0 f   EntityNode.obj
 0001:00047470       ?AnimateExpressionTrack@CAnimEntityNode@@IAEXPAVCExprTrack@@AAUSAnimContext@@@Z 34048470 f   EntityNode.obj
 0001:00047520       ?SaveToColladaInFixedFPS@CAnimEntityNode@@UBE?AVXmlNodeRef@@ABUSColladaExporterSaveProperties@@@Z 34048520 f   EntityNode.obj
 0001:000478d0       ??0?$QuatT_tpl@M@@QAE@ABU0@@Z 340488d0 f i EntityNode.obj
 0001:00047910       ?ApplyAnimKey@CAnimEntityNode@@IAEXHPAVCCharacterTrack@@MPAUICharacterInstance@@HH_N@Z 34048910 f   EntityNode.obj
 0001:00047a60       ?UpdateAnimTimeJumped@CAnimEntityNode@@IAEXHPAVCCharacterTrack@@MPAUICharacterInstance@@H_NH@Z 34048a60 f   EntityNode.obj
 0001:00047bd0       ?UpdateAnimRegular@CAnimEntityNode@@IAEXHQAHPAVCCharacterTrack@@MPAUICharacterInstance@@H_N@Z 34048bd0 f   EntityNode.obj
 0001:00047d40       ?UpdateAnimBlendGap@CAnimEntityNode@@IAEXQAHPAVCCharacterTrack@@MPAUICharacterInstance@@H@Z 34048d40 f   EntityNode.obj
 0001:00047f60       ?Get@Noise@CAnimEntityNode@@QBE?AU?$Vec3_tpl@M@@M@Z 34048f60 f   EntityNode.obj
 0001:000481c0       ?Adjust3DSoundOffset@CAnimEntityNode@@IBE?AU?$Vec3_tpl@M@@_NPAUIEntity@@AAU2@@Z 340491c0 f   EntityNode.obj
 0001:00048360       ?HaveValue@IScriptTable@@QAE_NPBD@Z 34049360 f i EntityNode.obj
 0001:000483f0       ?GetActiveKey@?$TAnimTrack@UILookAtKey@@@@QAEHMPAUILookAtKey@@@Z 340493f0 f i EntityNode.obj
 0001:000485a0       ??$_M_find@V?$CryStringT@D@@@?$_Rb_tree@V?$CryStringT@D@@U?$less_stricmp@V?$CryStringT@D@@@stl@@U?$pair@$$CBV?$CryStringT@D@@V?$_smart_ptr@UIFacialAnimSequence@@@@@stlpmtx_std@@U?$_Select1st@U?$pair@$$CBV?$CryStringT@D@@V?$_smart_ptr@UIFacialAnimSequence@@@@@stlpmtx_std@@@priv@5@U?$_MapTraitsT@U?$pair@$$CBV?$CryStringT@D@@V?$_smart_ptr@UIFacialAnimSequence@@@@@stlpmtx_std@@@75@V?$allocator@U?$pair@$$CBV?$CryStringT@D@@V?$_smart_ptr@UIFacialAnimSequence@@@@@stlpmtx_std@@@5@@priv@stlpmtx_std@@ABEPAU_Rb_tree_node_base@12@ABV?$CryStringT@D@@@Z 340495a0 f i EntityNode.obj
 0001:00048620       ??R?$hash_stricmp@V?$CryStringT@D@@@stl@@QBEIABV?$CryStringT@D@@@Z 34049620 f i EntityNode.obj
 0001:00048660       ??0CMemStatContextFormat@@QAA@W4Type@EMemStatContextTypes@@IPBDZZ 34049660 f i EntityNode.obj
 0001:00048690       ?CreateDefaultTracks@CAnimEntityNode@@UAEXXZ 34049690 f   EntityNode.obj
 0001:00048770       ?GetParamCountStatic@CAnimEntityNode@@SAHXZ 34049770 f   EntityNode.obj
 0001:00048790       ?GetParamName@CAnimEntityNode@@UBEPBDVAnimParamType@@@Z 34049790 f   EntityNode.obj
 0001:000488e0       ?SetPos@CAnimEntityNode@@UAEXMABU?$Vec3_tpl@M@@@Z 340498e0 f   EntityNode.obj
 0001:000489b0       ?SetRotate@CAnimEntityNode@@UAEXMABU?$Quat_tpl@M@@@Z 340499b0 f   EntityNode.obj
 0001:00048a80       ?SetScale@CAnimEntityNode@@UAEXMABU?$Vec3_tpl@M@@@Z 34049a80 f   EntityNode.obj
 0001:00048b50       ?IsBoneLinkTransformEnabled@CAnimEntityNode@@UBE_NXZ 34049b50 f   EntityNode.obj
 0001:00048b60       ?GetActiveKey@?$TAnimTrack@UISoundKey@@@@QAEHMPAUISoundKey@@@Z 34049b60 f i EntityNode.obj
 0001:00048d10       ?GetActiveKey@?$TAnimTrack@UIEventKey@@@@QAEHMPAUIEventKey@@@Z 34049d10 f i EntityNode.obj
 0001:00048ec0       ?CallMethod@Script@@SA_NPAUIScriptTable@@PBD@Z 34049ec0 f i EntityNode.obj
 0001:00048f40       ?GetActiveKey@?$TAnimTrack@UIFaceSeqKey@@@@QAEHMPAUIFaceSeqKey@@@Z 34049f40 f i EntityNode.obj
 0001:000490f0       ??$__lower_bound@PBIIU?$less@I@stlpmtx_std@@U12@H@priv@stlpmtx_std@@YAPBIPBI0ABIU?$less@I@1@2PAH@Z 3404a0f0 f i EntityNode.obj
 0001:00049130       ??0SScriptPropertyParamInfo@CAnimEntityNode@@QAE@ABU01@@Z 3404a130 f i EntityNode.obj
 0001:000491b0       ??$__copy_backward@PAUSSoundInfo@@PAU1@H@priv@stlpmtx_std@@YAPAUSSoundInfo@@PAU2@00ABUrandom_access_iterator_tag@1@PAH@Z 3404a1b0 f i EntityNode.obj
 0001:000492a0       ??$__fill@PAUSSoundInfo@@U1@H@priv@stlpmtx_std@@YAXPAUSSoundInfo@@0ABU2@ABUrandom_access_iterator_tag@1@PAH@Z 3404a2a0 f i EntityNode.obj
 0001:00049390       ?NotifyEntityScript@?A0x6681eb95@@YAXPBUIEntity@@PBD@Z 3404a390 f   EntityNode.obj
 0001:000493e0       ??1SScriptPropertyParamInfo@CAnimEntityNode@@QAE@XZ 3404a3e0 f i EntityNode.obj
 0001:00049470       ?GetParamCount@CAnimEntityNode@@UBEHXZ 3404a470 f   EntityNode.obj
 0001:000494b0       ?GetParamInfoStatic@CAnimEntityNode@@SA_NHAAUSParamInfo@IAnimNode@@@Z 3404a4b0 f   EntityNode.obj
 0001:00049500       ?GetParamInfoFromId@CAnimEntityNode@@UBE_NABVAnimParamType@@AAUSParamInfo@IAnimNode@@@Z 3404a500 f   EntityNode.obj
 0001:00049680       ??1SSoundInfo@@QAE@XZ      3404a680 f i EntityNode.obj
 0001:000496b0       ?UpdateEntityPosRotVel@CAnimEntityNode@@KAXPAUIEntity@@ABU?$Vec3_tpl@M@@ABU?$Quat_tpl@M@@_NEAAU3@4@Z 3404a6b0 f   EntityNode.obj
 0001:00049a10       ?reserve@?$CryStringT@D@@QAEXI@Z 3404aa10 f i EntityNode.obj
 0001:00049b10       ??$__copy@PAUSSoundInfo@@PAU1@H@priv@stlpmtx_std@@YAPAUSSoundInfo@@PAU2@00ABUrandom_access_iterator_tag@1@PAH@Z 3404ab10 f i EntityNode.obj
 0001:00049c00       ??$__copy@PAUSScriptPropertyParamInfo@CAnimEntityNode@@PAU12@H@priv@stlpmtx_std@@YAPAUSScriptPropertyParamInfo@CAnimEntityNode@@PAU23@00ABUrandom_access_iterator_tag@1@PAH@Z 3404ac00 f i EntityNode.obj
 0001:00049de0       ?_M_create_node@?$_Rb_tree@V?$CryStringT@D@@U?$less@V?$CryStringT@D@@@stlpmtx_std@@V1@U?$_Identity@V?$CryStringT@D@@@priv@3@U?$_SetTraitsT@V?$CryStringT@D@@@53@V?$allocator@V?$CryStringT@D@@@3@@priv@stlpmtx_std@@IAEPAU_Rb_tree_node_base@23@ABV?$CryStringT@D@@@Z 3404ade0 f i EntityNode.obj
 0001:00049e40       ??$_M_find@PBD@?$_Rb_tree@V?$CryStringT@D@@U?$less@V?$CryStringT@D@@@stlpmtx_std@@V1@U?$_Identity@V?$CryStringT@D@@@priv@3@U?$_SetTraitsT@V?$CryStringT@D@@@53@V?$allocator@V?$CryStringT@D@@@3@@priv@stlpmtx_std@@ABEPAU_Rb_tree_node_base@12@ABQBD@Z 3404ae40 f i EntityNode.obj
 0001:00049fc0       ??$_M_bkt_num_key@PBD@?$hashtable@U?$pair@$$CBV?$CryStringT@D@@I@stlpmtx_std@@V?$CryStringT@D@@V?$hash_stricmp@V?$CryStringT@D@@@stl@@U?$_HashMapTraitsT@U?$pair@$$CBV?$CryStringT@D@@I@stlpmtx_std@@@priv@2@U?$_Select1st@U?$pair@$$CBV?$CryStringT@D@@I@stlpmtx_std@@@72@U?$stlport_hash_equal@V?$CryStringT@D@@V?$hash_stricmp@V?$CryStringT@D@@@stl@@@5@V?$allocator@U?$pair@V?$CryStringT@D@@I@stlpmtx_std@@@2@@stlpmtx_std@@ABEIABQBDI@Z 3404afc0 f i EntityNode.obj
 0001:0004a040       ?GetParamInfo@CAnimEntityNode@@UBE_NHAAUSParamInfo@IAnimNode@@@Z 3404b040 f   EntityNode.obj
 0001:0004a0f0       ?ReleaseSounds@CAnimEntityNode@@IAEXXZ 3404b0f0 f   EntityNode.obj
 0001:0004a1d0       ?Pause@CAnimEntityNode@@UAEXXZ 3404b1d0 f   EntityNode.obj
 0001:0004a1e0       ?ApplySoundKey@CAnimEntityNode@@IAEXPAUIAnimTrack@@HHAAUISoundKey@@AAUSAnimContext@@@Z 3404b1e0 f   EntityNode.obj
 0001:0004a7a0       ?AnimateLookAt@CAnimEntityNode@@IAEXPAVCLookAtTrack@@AAUSAnimContext@@@Z 3404b7a0 f   EntityNode.obj
 0001:0004ad90       ?EnableBoneLinkTransform@CAnimEntityNode@@UAEX_N@Z 3404bd90 f   EntityNode.obj
 0001:0004ae10       ?_M_insert@?$_Rb_tree@V?$CryStringT@D@@U?$less@V?$CryStringT@D@@@stlpmtx_std@@V1@U?$_Identity@V?$CryStringT@D@@@priv@3@U?$_SetTraitsT@V?$CryStringT@D@@@53@V?$allocator@V?$CryStringT@D@@@3@@priv@stlpmtx_std@@AAE?AU?$_Rb_tree_iterator@V?$CryStringT@D@@U?$_SetTraitsT@V?$CryStringT@D@@@priv@stlpmtx_std@@@23@PAU_Rb_tree_node_base@23@ABV?$CryStringT@D@@00@Z 3404be10 f i EntityNode.obj
 0001:0004aeb0       ??$_M_find@V?$CryStringT@D@@@?$hashtable@U?$pair@$$CBV?$CryStringT@D@@I@stlpmtx_std@@V?$CryStringT@D@@V?$hash_stricmp@V?$CryStringT@D@@@stl@@U?$_HashMapTraitsT@U?$pair@$$CBV?$CryStringT@D@@I@stlpmtx_std@@@priv@2@U?$_Select1st@U?$pair@$$CBV?$CryStringT@D@@I@stlpmtx_std@@@72@U?$stlport_hash_equal@V?$CryStringT@D@@V?$hash_stricmp@V?$CryStringT@D@@@stl@@@5@V?$allocator@U?$pair@V?$CryStringT@D@@I@stlpmtx_std@@@2@@stlpmtx_std@@ABE?AV?$_Slist_iterator@U?$pair@$$CBV?$CryStringT@D@@I@stlpmtx_std@@U?$_Nonconst_traits@U?$pair@$$CBV?$CryStringT@D@@I@stlpmtx_std@@@2@@priv@1@ABV?$CryStringT@D@@@Z 3404beb0 f i EntityNode.obj
 0001:0004af40       ??$__ufill@PAUSSoundInfo@@U1@H@priv@stlpmtx_std@@YAXPAUSSoundInfo@@0ABU2@ABUrandom_access_iterator_tag@1@PAH@Z 3404bf40 f i EntityNode.obj
 0001:0004afc0       ??$__ucopy@PAUSSoundInfo@@PAU1@H@priv@stlpmtx_std@@YAPAUSSoundInfo@@PAU2@00ABUrandom_access_iterator_tag@1@PAH@Z 3404bfc0 f i EntityNode.obj
 0001:0004b030       ?StillUpdate@CAnimEntityNode@@UAEXXZ 3404c030 f   EntityNode.obj
 0001:0004b0d0       ?UpdateBoneLink@CAnimEntityNode@@IAEXPBU?$Vec3_tpl@M@@PBU?$Quat_tpl@M@@@Z 3404c0d0 f   EntityNode.obj
 0001:0004b260       ?erase@?$_Rb_tree@V?$CryStringT@D@@U?$less@V?$CryStringT@D@@@stlpmtx_std@@V1@U?$_Identity@V?$CryStringT@D@@@priv@3@U?$_SetTraitsT@V?$CryStringT@D@@@53@V?$allocator@V?$CryStringT@D@@@3@@priv@stlpmtx_std@@QAEXU?$_Rb_tree_iterator@V?$CryStringT@D@@U?$_SetTraitsT@V?$CryStringT@D@@@priv@stlpmtx_std@@@23@@Z 3404c260 f i EntityNode.obj
 0001:0004b260       ?erase@?$_Rb_tree@V?$CryStringT@D@@U?$less@V?$CryStringT@D@@@stlpmtx_std@@U?$pair@$$CBV?$CryStringT@D@@PAVCLightAnimWrapper@@@3@U?$_Select1st@U?$pair@$$CBV?$CryStringT@D@@PAVCLightAnimWrapper@@@stlpmtx_std@@@priv@3@U?$_MapTraitsT@U?$pair@$$CBV?$CryStringT@D@@PAVCLightAnimWrapper@@@stlpmtx_std@@@63@V?$allocator@U?$pair@$$CBV?$CryStringT@D@@PAVCLightAnimWrapper@@@stlpmtx_std@@@3@@priv@stlpmtx_std@@QAEXU?$_Rb_tree_iterator@U?$pair@$$CBV?$CryStringT@D@@PAVCLightAnimWrapper@@@stlpmtx_std@@U?$_MapTraitsT@U?$pair@$$CBV?$CryStringT@D@@PAVCLightAnimWrapper@@@stlpmtx_std@@@priv@2@@23@@Z 3404c260 f i Movie.obj
 0001:0004b2d0       ?insert_unique@?$_Rb_tree@V?$CryStringT@D@@U?$less@V?$CryStringT@D@@@stlpmtx_std@@V1@U?$_Identity@V?$CryStringT@D@@@priv@3@U?$_SetTraitsT@V?$CryStringT@D@@@53@V?$allocator@V?$CryStringT@D@@@3@@priv@stlpmtx_std@@QAE?AU?$pair@U?$_Rb_tree_iterator@V?$CryStringT@D@@U?$_SetTraitsT@V?$CryStringT@D@@@priv@stlpmtx_std@@@priv@stlpmtx_std@@_N@3@ABV?$CryStringT@D@@@Z 3404c2d0 f i EntityNode.obj
 0001:0004b450       ??$?HD@@YA?AV?$CryStringT@D@@PBDABV0@@Z 3404c450 f i EntityNode.obj
 0001:0004b4c0       ?_M_fill_assign@?$_Impl_vector@PAXV?$allocator@PAX@stlpmtx_std@@@priv@stlpmtx_std@@QAEXIABQAX@Z 3404c4c0 f i EntityNode.obj
 0001:0004b630       ??$__uninitialized_fill_n@PAUSScriptPropertyParamInfo@CAnimEntityNode@@IU12@@priv@stlpmtx_std@@YAPAUSScriptPropertyParamInfo@CAnimEntityNode@@PAU23@IABU23@@Z 3404c630 f i EntityNode.obj
 0001:0004b680       ?_M_create_node@?$_Rb_tree@V?$CryStringT@D@@U?$less_stricmp@V?$CryStringT@D@@@stl@@U?$pair@$$CBV?$CryStringT@D@@V?$_smart_ptr@UIFacialAnimSequence@@@@@stlpmtx_std@@U?$_Select1st@U?$pair@$$CBV?$CryStringT@D@@V?$_smart_ptr@UIFacialAnimSequence@@@@@stlpmtx_std@@@priv@5@U?$_MapTraitsT@U?$pair@$$CBV?$CryStringT@D@@V?$_smart_ptr@UIFacialAnimSequence@@@@@stlpmtx_std@@@75@V?$allocator@U?$pair@$$CBV?$CryStringT@D@@V?$_smart_ptr@UIFacialAnimSequence@@@@@stlpmtx_std@@@5@@priv@stlpmtx_std@@IAEPAU_Rb_tree_node_base@23@ABU?$pair@$$CBV?$CryStringT@D@@V?$_smart_ptr@UIFacialAnimSequence@@@@@3@@Z 3404c680 f i EntityNode.obj
 0001:0004b6f0       ??$_M_find@PBD@?$hashtable@U?$pair@$$CBV?$CryStringT@D@@I@stlpmtx_std@@V?$CryStringT@D@@V?$hash_stricmp@V?$CryStringT@D@@@stl@@U?$_HashMapTraitsT@U?$pair@$$CBV?$CryStringT@D@@I@stlpmtx_std@@@priv@2@U?$_Select1st@U?$pair@$$CBV?$CryStringT@D@@I@stlpmtx_std@@@72@U?$stlport_hash_equal@V?$CryStringT@D@@V?$hash_stricmp@V?$CryStringT@D@@@stl@@@5@V?$allocator@U?$pair@V?$CryStringT@D@@I@stlpmtx_std@@@2@@stlpmtx_std@@ABE?AV?$_Slist_iterator@U?$pair@$$CBV?$CryStringT@D@@I@stlpmtx_std@@U?$_Nonconst_traits@U?$pair@$$CBV?$CryStringT@D@@I@stlpmtx_std@@@2@@priv@1@ABQBD@Z 3404c6f0 f i EntityNode.obj
 0001:0004b830       ??$__destroy_range_aux@V?$reverse_iterator@PAUSSoundInfo@@@stlpmtx_std@@USSoundInfo@@@stlpmtx_std@@YAXV?$reverse_iterator@PAUSSoundInfo@@@0@0PAUSSoundInfo@@ABU__false_type@0@@Z 3404c830 f i EntityNode.obj
 0001:0004b880       ??$__destroy_range_aux@PAUSSoundInfo@@U1@@stlpmtx_std@@YAXPAUSSoundInfo@@00ABU__false_type@0@@Z 3404c880 f i EntityNode.obj
 0001:0004b8d0       ??0CAnimationCacher@@QAE@XZ 3404c8d0 f i EntityNode.obj
 0001:0004b980       ?LoadFromCollada@CAnimEntityNode@@UAE_NVXmlNodeRef@@@Z 3404c980 f   EntityNode.obj
 0001:0004c270       ?_M_erase@?$_Rb_tree@V?$CryStringT@D@@U?$less_stricmp@V?$CryStringT@D@@@stl@@U?$pair@$$CBV?$CryStringT@D@@V?$_smart_ptr@UIFacialAnimSequence@@@@@stlpmtx_std@@U?$_Select1st@U?$pair@$$CBV?$CryStringT@D@@V?$_smart_ptr@UIFacialAnimSequence@@@@@stlpmtx_std@@@priv@5@U?$_MapTraitsT@U?$pair@$$CBV?$CryStringT@D@@V?$_smart_ptr@UIFacialAnimSequence@@@@@stlpmtx_std@@@75@V?$allocator@U?$pair@$$CBV?$CryStringT@D@@V?$_smart_ptr@UIFacialAnimSequence@@@@@stlpmtx_std@@@5@@priv@stlpmtx_std@@AAEXPAU_Rb_tree_node_base@23@@Z 3404d270 f i EntityNode.obj
 0001:0004c2e0       ?_M_erase_after@?$_Slist_base@U?$pair@$$CBV?$CryStringT@D@@I@stlpmtx_std@@V?$allocator@U?$pair@$$CBV?$CryStringT@D@@I@stlpmtx_std@@@2@@priv@stlpmtx_std@@IAEPAU_Slist_node_base@23@PAU423@0@Z 3404d2e0 f i EntityNode.obj
 0001:0004c350       ?_M_fill_insert_aux@?$_Impl_vector@USSoundInfo@@V?$allocator@USSoundInfo@@@stlpmtx_std@@@priv@stlpmtx_std@@AAEXPAUSSoundInfo@@IABU4@ABU__false_type@3@@Z 3404d350 f i EntityNode.obj
 0001:0004c4d0       ?_M_insert@?$_Rb_tree@V?$CryStringT@D@@U?$less_stricmp@V?$CryStringT@D@@@stl@@U?$pair@$$CBV?$CryStringT@D@@V?$_smart_ptr@UIFacialAnimSequence@@@@@stlpmtx_std@@U?$_Select1st@U?$pair@$$CBV?$CryStringT@D@@V?$_smart_ptr@UIFacialAnimSequence@@@@@stlpmtx_std@@@priv@5@U?$_MapTraitsT@U?$pair@$$CBV?$CryStringT@D@@V?$_smart_ptr@UIFacialAnimSequence@@@@@stlpmtx_std@@@75@V?$allocator@U?$pair@$$CBV?$CryStringT@D@@V?$_smart_ptr@UIFacialAnimSequence@@@@@stlpmtx_std@@@5@@priv@stlpmtx_std@@AAE?AU?$_Rb_tree_iterator@U?$pair@$$CBV?$CryStringT@D@@V?$_smart_ptr@UIFacialAnimSequence@@@@@stlpmtx_std@@U?$_MapTraitsT@U?$pair@$$CBV?$CryStringT@D@@V?$_smart_ptr@UIFacialAnimSequence@@@@@stlpmtx_std@@@priv@2@@23@PAU_Rb_tree_node_base@23@ABU?$pair@$$CBV?$CryStringT@D@@V?$_smart_ptr@UIFacialAnimSequence@@@@@3@00@Z 3404d4d0 f i EntityNode.obj
 0001:0004c570       ?OnEndAnimation@CAnimEntityNode@@MAEXPBD@Z 3404d570 f   EntityNode.obj
 0001:0004c5d0       ?AnimateCharacterTrack@CAnimEntityNode@@IAEXPAVCCharacterTrack@@AAUSAnimContext@@HH@Z 3404d5d0 f   EntityNode.obj
 0001:0004cab0       ?AddToCache@CAnimationCacher@@QAEXI@Z 3404dab0 f   EntityNode.obj
 0001:0004cb90       ?insert_unique@?$_Rb_tree@V?$CryStringT@D@@U?$less_stricmp@V?$CryStringT@D@@@stl@@U?$pair@$$CBV?$CryStringT@D@@V?$_smart_ptr@UIFacialAnimSequence@@@@@stlpmtx_std@@U?$_Select1st@U?$pair@$$CBV?$CryStringT@D@@V?$_smart_ptr@UIFacialAnimSequence@@@@@stlpmtx_std@@@priv@5@U?$_MapTraitsT@U?$pair@$$CBV?$CryStringT@D@@V?$_smart_ptr@UIFacialAnimSequence@@@@@stlpmtx_std@@@75@V?$allocator@U?$pair@$$CBV?$CryStringT@D@@V?$_smart_ptr@UIFacialAnimSequence@@@@@stlpmtx_std@@@5@@priv@stlpmtx_std@@QAE?AU?$pair@U?$_Rb_tree_iterator@U?$pair@$$CBV?$CryStringT@D@@V?$_smart_ptr@UIFacialAnimSequence@@@@@stlpmtx_std@@U?$_MapTraitsT@U?$pair@$$CBV?$CryStringT@D@@V?$_smart_ptr@UIFacialAnimSequence@@@@@stlpmtx_std@@@priv@2@@priv@stlpmtx_std@@_N@3@ABU?$pair@$$CBV?$CryStringT@D@@V?$_smart_ptr@UIFacialAnimSequence@@@@@3@@Z 3404db90 f i EntityNode.obj
 0001:0004ccd0       ?CreateTrack@CAnimEntityNode@@MAEPAUIAnimTrack@@ABVAnimParamType@@@Z 3404dcd0 f   EntityNode.obj
 0001:0004ced0       ?ReleaseAllAnims@CAnimEntityNode@@IAEXXZ 3404ded0 f   EntityNode.obj
 0001:0004d0a0       ?StopExpressions@CAnimEntityNode@@IAEXXZ 3404e0a0 f   EntityNode.obj
 0001:0004d100       ?AnimateScriptTableProperty@CAnimEntityNode@@IAEXPAUIAnimTrack@@AAUSAnimContext@@PBD@Z 3404e100 f   EntityNode.obj
 0001:0004d310       ?_M_erase@?$_Impl_vector@USScriptPropertyParamInfo@CAnimEntityNode@@V?$allocator@USScriptPropertyParamInfo@CAnimEntityNode@@@stlpmtx_std@@@priv@stlpmtx_std@@AAEPAUSScriptPropertyParamInfo@CAnimEntityNode@@PAU45@0ABU__false_type@3@@Z 3404e310 f i EntityNode.obj
 0001:0004d380       ?_M_insert_overflow_aux@?$_Impl_vector@USScriptPropertyParamInfo@CAnimEntityNode@@V?$allocator@USScriptPropertyParamInfo@CAnimEntityNode@@@stlpmtx_std@@@priv@stlpmtx_std@@AAEXPAUSScriptPropertyParamInfo@CAnimEntityNode@@ABU45@ABU__false_type@3@I_N@Z 3404e380 f i EntityNode.obj
 0001:0004d570       ?_M_insert_overflow_aux@?$_Impl_vector@USSoundInfo@@V?$allocator@USSoundInfo@@@stlpmtx_std@@@priv@stlpmtx_std@@AAEXPAUSSoundInfo@@ABU4@ABU__false_type@3@I_N@Z 3404e570 f i EntityNode.obj
 0001:0004d750       ?_M_insert_noresize@?$hashtable@U?$pair@$$CBV?$CryStringT@D@@I@stlpmtx_std@@V?$CryStringT@D@@V?$hash_stricmp@V?$CryStringT@D@@@stl@@U?$_HashMapTraitsT@U?$pair@$$CBV?$CryStringT@D@@I@stlpmtx_std@@@priv@2@U?$_Select1st@U?$pair@$$CBV?$CryStringT@D@@I@stlpmtx_std@@@72@U?$stlport_hash_equal@V?$CryStringT@D@@V?$hash_stricmp@V?$CryStringT@D@@@stl@@@5@V?$allocator@U?$pair@V?$CryStringT@D@@I@stlpmtx_std@@@2@@stlpmtx_std@@IAE?AU?$_Ht_iterator@V?$_Slist_iterator@U?$pair@$$CBV?$CryStringT@D@@I@stlpmtx_std@@U?$_Nonconst_traits@U?$pair@$$CBV?$CryStringT@D@@I@stlpmtx_std@@@2@@priv@stlpmtx_std@@U?$_NonLocalHashMapTraitsT@U?$pair@$$CBV?$CryStringT@D@@I@stlpmtx_std@@@23@@priv@2@IABU?$pair@$$CBV?$CryStringT@D@@I@2@@Z 3404e750 f i EntityNode.obj
 0001:0004d820       ?Reset@CAnimEntityNode@@UAEXXZ 3404e820 f   EntityNode.obj
 0001:0004d8b0       ?LoadFacialSequence@CAnimEntityNode@@IAEPAUIFacialAnimSequence@@PBD@Z 3404e8b0 f   EntityNode.obj
 0001:0004da20       ?AnimateFacialSequence@CAnimEntityNode@@IAEXPAVCFaceSeqTrack@@AAUSAnimContext@@@Z 3404ea20 f   EntityNode.obj
 0001:0004dbb0       ?RemoveFromCache@CAnimationCacher@@QAEXI@Z 3404ebb0 f   EntityNode.obj
 0001:0004dc30       ?ClearCache@CAnimationCacher@@QAEXXZ 3404ec30 f   EntityNode.obj
 0001:0004dc90       ?erase@?$_Impl_vector@USSoundInfo@@V?$allocator@USSoundInfo@@@stlpmtx_std@@@priv@stlpmtx_std@@QAEPAUSSoundInfo@@PAU4@0@Z 3404ec90 f i EntityNode.obj
 0001:0004dcf0       ??0?$hashtable@U?$pair@$$CBV?$CryStringT@D@@I@stlpmtx_std@@V?$CryStringT@D@@V?$hash_stricmp@V?$CryStringT@D@@@stl@@U?$_HashMapTraitsT@U?$pair@$$CBV?$CryStringT@D@@I@stlpmtx_std@@@priv@2@U?$_Select1st@U?$pair@$$CBV?$CryStringT@D@@I@stlpmtx_std@@@72@U?$stlport_hash_equal@V?$CryStringT@D@@V?$hash_stricmp@V?$CryStringT@D@@@stl@@@5@V?$allocator@U?$pair@V?$CryStringT@D@@I@stlpmtx_std@@@2@@stlpmtx_std@@QAE@IABV?$hash_stricmp@V?$CryStringT@D@@@stl@@ABU?$stlport_hash_equal@V?$CryStringT@D@@V?$hash_stricmp@V?$CryStringT@D@@@stl@@@3@ABV?$allocator@U?$pair@V?$CryStringT@D@@I@stlpmtx_std@@@1@@Z 3404ecf0 f i EntityNode.obj
 0001:0004dd90       ?insert_unique_noresize@?$hashtable@U?$pair@$$CBV?$CryStringT@D@@I@stlpmtx_std@@V?$CryStringT@D@@V?$hash_stricmp@V?$CryStringT@D@@@stl@@U?$_HashMapTraitsT@U?$pair@$$CBV?$CryStringT@D@@I@stlpmtx_std@@@priv@2@U?$_Select1st@U?$pair@$$CBV?$CryStringT@D@@I@stlpmtx_std@@@72@U?$stlport_hash_equal@V?$CryStringT@D@@V?$hash_stricmp@V?$CryStringT@D@@@stl@@@5@V?$allocator@U?$pair@V?$CryStringT@D@@I@stlpmtx_std@@@2@@stlpmtx_std@@QAE?AU?$pair@U?$_Ht_iterator@V?$_Slist_iterator@U?$pair@$$CBV?$CryStringT@D@@I@stlpmtx_std@@U?$_Nonconst_traits@U?$pair@$$CBV?$CryStringT@D@@I@stlpmtx_std@@@2@@priv@stlpmtx_std@@U?$_NonLocalHashMapTraitsT@U?$pair@$$CBV?$CryStringT@D@@I@stlpmtx_std@@@23@@priv@stlpmtx_std@@_N@2@ABU?$pair@$$CBV?$CryStringT@D@@I@2@@Z 3404ed90 f i EntityNode.obj
 0001:0004de90       ?Initialize@CAnimEntityNode@@SAXXZ 3404ee90 f   EntityNode.obj
 0001:0004e220       ?PrepareAnimations@CAnimEntityNode@@IAEXXZ 3404f220 f   EntityNode.obj
 0001:0004e480       ?Activate@CAnimEntityNode@@UAEX_N@Z 3404f480 f   EntityNode.obj
 0001:0004e4e0       ?PrecacheKeys@CAnimEntityNode@@QAEXM@Z 3404f4e0 f   EntityNode.obj
 0001:0004e6a0       ??1?$hashtable@U?$pair@$$CBV?$CryStringT@D@@I@stlpmtx_std@@V?$CryStringT@D@@V?$hash_stricmp@V?$CryStringT@D@@@stl@@U?$_HashMapTraitsT@U?$pair@$$CBV?$CryStringT@D@@I@stlpmtx_std@@@priv@2@U?$_Select1st@U?$pair@$$CBV?$CryStringT@D@@I@stlpmtx_std@@@72@U?$stlport_hash_equal@V?$CryStringT@D@@V?$hash_stricmp@V?$CryStringT@D@@@stl@@@5@V?$allocator@U?$pair@V?$CryStringT@D@@I@stlpmtx_std@@@2@@stlpmtx_std@@QAE@XZ 3404f6a0 f i EntityNode.obj
 0001:0004e710       ??1CAnimEntityNode@@UAE@XZ 3404f710 f   EntityNode.obj
 0001:0004e970       ??_ECAnimEntityNode@@$4PPPPPPPM@A@AEPAXI@Z 3404f970 f i EntityNode.obj
 0001:0004e980       ?Release@CAnimNode@@$4PPPPPPPM@BHA@AEXXZ 3404f980 f i EntityNode.obj
 0001:0004e990       ??$AddObject@V?$CryStringT@D@@U?$less@V?$CryStringT@D@@@stlpmtx_std@@V?$allocator@V?$CryStringT@D@@@3@@ICrySizer@@QAEXABV?$set@V?$CryStringT@D@@U?$less@V?$CryStringT@D@@@stlpmtx_std@@V?$allocator@V?$CryStringT@D@@@3@@stlpmtx_std@@@Z 3404f990 f i EntityNode.obj
 0001:0004ea20       ??$AddObject@USSoundInfo@@V?$allocator@USSoundInfo@@@stlpmtx_std@@@ICrySizer@@QAEXABV?$vector@USSoundInfo@@V?$allocator@USSoundInfo@@@stlpmtx_std@@@stlpmtx_std@@@Z 3404fa20 f i EntityNode.obj
 0001:0004eaa0       ?GetMemoryUsage@CAnimEntityNode@@UBEXPAVICrySizer@@@Z 3404faa0 f i EntityNode.obj
 0001:0004eb20       ?resize@?$_Impl_vector@USSoundInfo@@V?$allocator@USSoundInfo@@@stlpmtx_std@@@priv@stlpmtx_std@@QAEXIABUSSoundInfo@@@Z 3404fb20 f i EntityNode.obj
 0001:0004ebc0       ??0CAnimEntityNode@@QAE@XZ 3404fbc0 f   EntityNode.obj
 0001:0004ef20       ?_M_rehash@?$hashtable@U?$pair@$$CBV?$CryStringT@D@@I@stlpmtx_std@@V?$CryStringT@D@@V?$hash_stricmp@V?$CryStringT@D@@@stl@@U?$_HashMapTraitsT@U?$pair@$$CBV?$CryStringT@D@@I@stlpmtx_std@@@priv@2@U?$_Select1st@U?$pair@$$CBV?$CryStringT@D@@I@stlpmtx_std@@@72@U?$stlport_hash_equal@V?$CryStringT@D@@V?$hash_stricmp@V?$CryStringT@D@@@stl@@@5@V?$allocator@U?$pair@V?$CryStringT@D@@I@stlpmtx_std@@@2@@stlpmtx_std@@AAEXI@Z 3404ff20 f i EntityNode.obj
 0001:0004f1d0       ??_GCAnimEntityNode@@UAEPAXI@Z 340501d0 f i EntityNode.obj
 0001:0004f1d0       ??_ECAnimEntityNode@@UAEPAXI@Z 340501d0 f i EntityNode.obj
 0001:0004f210       ?Animate@CAnimEntityNode@@UAEXAAUSAnimContext@@@Z 34050210 f   EntityNode.obj
 0001:00050a80       ?_M_enlarge@?$hashtable@U?$pair@$$CBV?$CryStringT@D@@I@stlpmtx_std@@V?$CryStringT@D@@V?$hash_stricmp@V?$CryStringT@D@@@stl@@U?$_HashMapTraitsT@U?$pair@$$CBV?$CryStringT@D@@I@stlpmtx_std@@@priv@2@U?$_Select1st@U?$pair@$$CBV?$CryStringT@D@@I@stlpmtx_std@@@72@U?$stlport_hash_equal@V?$CryStringT@D@@V?$hash_stricmp@V?$CryStringT@D@@@stl@@@5@V?$allocator@U?$pair@V?$CryStringT@D@@I@stlpmtx_std@@@2@@stlpmtx_std@@AAEXI@Z 34051a80 f i EntityNode.obj
 0001:00050b20       ??$?AV?$CryStringT@D@@@?$hash_map@V?$CryStringT@D@@IV?$hash_stricmp@V?$CryStringT@D@@@stl@@U?$stlport_hash_equal@V?$CryStringT@D@@V?$hash_stricmp@V?$CryStringT@D@@@stl@@@3@V?$allocator@U?$pair@V?$CryStringT@D@@I@stlpmtx_std@@@stlpmtx_std@@@stlpmtx_std@@QAEAAIABV?$CryStringT@D@@@Z 34051b20 f i EntityNode.obj
 0001:00050bd0       ?FindDynamicPropertiesRec@CAnimEntityNode@@IAEXPAUIScriptTable@@ABV?$CryStringT@D@@I@Z 34051bd0 f   EntityNode.obj
 0001:000512a0       ?UpdateDynamicParams@CAnimEntityNode@@MAEXXZ 340522a0 f   EntityNode.obj
 0001:00051420       ?Reset@CAnimEventNode@@UAEXXZ 34052420 f   EventNode.obj
 0001:00051430       ??0CAnimEventNode@@QAE@XZ  34052430 f   EventNode.obj
 0001:000514a0       ?GetType@CAnimEventNode@@UBE?AW4EAnimNodeType@@XZ 340524a0 f i EventNode.obj
 0001:000514b0       ?GetParamInfo@CAnimEventNode@@UBE_NHAAUSParamInfo@IAnimNode@@@Z 340524b0 f   EventNode.obj
 0001:000514f0       ?GetParamInfoFromId@CAnimEventNode@@UBE_NABVAnimParamType@@AAUSParamInfo@IAnimNode@@@Z 340524f0 f   EventNode.obj
 0001:00051520       ?CreateDefaultTracks@CAnimEventNode@@UAEXXZ 34052520 f   EventNode.obj
 0001:00051570       ?Animate@CAnimEventNode@@UAEXAAUSAnimContext@@@Z 34052570 f   EventNode.obj
 0001:00051690       ?Reset@CLayerNode@@UAEXXZ  34052690 f   LayerNode.obj
 0001:000516a0       ?Activate@CCommentNode@@UAEX_N@Z 340526a0 f   CommentNode.obj
 0001:000516a0       ?Activate@CLayerNode@@UAEX_N@Z 340526a0 f   LayerNode.obj
 0001:000516b0       ?Serialize@CCommentNode@@UAEXAAVXmlNodeRef@@_N1@Z 340526b0 f   CommentNode.obj
 0001:000516b0       ?Serialize@CLayerNode@@UAEXAAVXmlNodeRef@@_N1@Z 340526b0 f   LayerNode.obj
 0001:000516c0       ?CreateDefaultTracks@CLayerNode@@UAEXXZ 340526c0 f   LayerNode.obj
 0001:00051710       ?GetParamCount@CLayerNode@@UBEHXZ 34052710 f   LayerNode.obj
 0001:00051730       ?Animate@CLayerNode@@UAEXAAUSAnimContext@@@Z 34052730 f   LayerNode.obj
 0001:000518a0       ?GetParamInfo@CLayerNode@@UBE_NHAAUSParamInfo@IAnimNode@@@Z 340528a0 f   LayerNode.obj
 0001:000518f0       ?GetParamInfoFromId@CLayerNode@@UBE_NABVAnimParamType@@AAUSParamInfo@IAnimNode@@@Z 340528f0 f   LayerNode.obj
 0001:000519b0       ?Initialize@CLayerNode@@SAXXZ 340529b0 f   LayerNode.obj
 0001:00051a30       ??0CLayerNode@@QAE@XZ      34052a30 f   LayerNode.obj
 0001:00051aa0       ?GetType@CLayerNode@@UBE?AW4EAnimNodeType@@XZ 34052aa0 f i LayerNode.obj
 0001:00051ab0       ?GetMaterialByName@CAnimMaterialNode@@AAEPAUIMaterial@@PBD@Z 34052ab0 f   MaterialNode.obj
 0001:00051ba0       ?GetParamName@CAnimMaterialNode@@UBEPBDVAnimParamType@@@Z 34052ba0 f   MaterialNode.obj
 0001:00051d30       ??$__copy@PAUSParamInfo@IAnimNode@@PAU12@H@priv@stlpmtx_std@@YAPAUSParamInfo@IAnimNode@@PAU23@00ABUrandom_access_iterator_tag@1@PAH@Z 34052d30 f i MaterialNode.obj
 0001:00051dd0       ?CreateTrack@CAnimMaterialNode@@UAEPAUIAnimTrack@@ABVAnimParamType@@@Z 34052dd0 f   MaterialNode.obj
 0001:00051e30       ?GetParamCount@CAnimMaterialNode@@UBEHXZ 34052e30 f   MaterialNode.obj
 0001:00051e70       ?GetParamInfo@CAnimMaterialNode@@UBE_NHAAUSParamInfo@IAnimNode@@@Z 34052e70 f   MaterialNode.obj
 0001:00051f20       ?GetParamInfoFromId@CAnimMaterialNode@@UBE_NABVAnimParamType@@AAUSParamInfo@IAnimNode@@@Z 34052f20 f   MaterialNode.obj
 0001:000520a0       ??$__destroy_range_aux@PAUSParamInfo@IAnimNode@@U12@@stlpmtx_std@@YAXPAUSParamInfo@IAnimNode@@00ABU__false_type@0@@Z 340530a0 f i MaterialNode.obj
 0001:000520e0       ?SetName@CAnimMaterialNode@@UAEXPBD@Z 340530e0 f   MaterialNode.obj
 0001:00052130       ??$_M_bkt_num_key@$$BY0CA@$$CBD@?$hashtable@U?$pair@$$CBV?$CryStringT@D@@I@stlpmtx_std@@V?$CryStringT@D@@V?$hash_stricmp@V?$CryStringT@D@@@stl@@U?$_HashMapTraitsT@U?$pair@$$CBV?$CryStringT@D@@I@stlpmtx_std@@@priv@2@U?$_Select1st@U?$pair@$$CBV?$CryStringT@D@@I@stlpmtx_std@@@72@U?$stlport_hash_equal@V?$CryStringT@D@@V?$hash_stricmp@V?$CryStringT@D@@@stl@@@5@V?$allocator@U?$pair@V?$CryStringT@D@@I@stlpmtx_std@@@2@@stlpmtx_std@@ABEIAAY0CA@$$CBDI@Z 34053130 f i MaterialNode.obj
 0001:000521b0       ??$_M_find@$$BY0CA@$$CBD@?$hashtable@U?$pair@$$CBV?$CryStringT@D@@I@stlpmtx_std@@V?$CryStringT@D@@V?$hash_stricmp@V?$CryStringT@D@@@stl@@U?$_HashMapTraitsT@U?$pair@$$CBV?$CryStringT@D@@I@stlpmtx_std@@@priv@2@U?$_Select1st@U?$pair@$$CBV?$CryStringT@D@@I@stlpmtx_std@@@72@U?$stlport_hash_equal@V?$CryStringT@D@@V?$hash_stricmp@V?$CryStringT@D@@@stl@@@5@V?$allocator@U?$pair@V?$CryStringT@D@@I@stlpmtx_std@@@2@@stlpmtx_std@@ABE?AV?$_Slist_iterator@U?$pair@$$CBV?$CryStringT@D@@I@stlpmtx_std@@U?$_Nonconst_traits@U?$pair@$$CBV?$CryStringT@D@@I@stlpmtx_std@@@2@@priv@1@AAY0CA@$$CBD@Z 340531b0 f i MaterialNode.obj
 0001:000522f0       ?AnimateNamedParameter@CAnimMaterialNode@@AAEXAAUSAnimContext@@PAUIRenderShaderResources@@PBDPAUIAnimTrack@@@Z 340532f0 f   MaterialNode.obj
 0001:00052460       ?Initialize@CAnimMaterialNode@@SAXXZ 34053460 f   MaterialNode.obj
 0001:00052650       ?Animate@CAnimMaterialNode@@UAEXAAUSAnimContext@@@Z 34053650 f   MaterialNode.obj
 0001:00052970       ??0CAnimMaterialNode@@QAE@XZ 34053970 f   MaterialNode.obj
 0001:00052a10       ?GetType@CAnimMaterialNode@@UBE?AW4EAnimNodeType@@XZ 34053a10 f i MaterialNode.obj
 0001:00052a20       ?GetKeyValueRange@CAnimMaterialNode@@UBEXAAM0@Z 34053a20 f i MaterialNode.obj
 0001:00052a20       ?GetKeyValueRange@?$TAnimTrack@UIBoolKey@@@@UBEXAAM0@Z 34053a20 f i AnimNode.obj
 0001:00052a20       ?GetKeyValueRange@?$TAnimTrack@UISelectKey@@@@UBEXAAM0@Z 34053a20 f i AnimNode.obj
 0001:00052a20       ?GetKeyValueRange@?$TAnimTrack@UIScreenFaderKey@@@@UBEXAAM0@Z 34053a20 f i ScreenFaderTrack.obj
 0001:00052a20       ?GetKeyValueRange@?$TAnimTrack@UISequenceKey@@@@UBEXAAM0@Z 34053a20 f i AnimNode.obj
 0001:00052a20       ?GetKeyValueRange@?$TAnimTrack@UILookAtKey@@@@UBEXAAM0@Z 34053a20 f i AnimNode.obj
 0001:00052a20       ?GetKeyValueRange@?$TAnimTrack@UIDiscreteFloatKey@@@@UBEXAAM0@Z 34053a20 f i GotoTrack.obj
 0001:00052a20       ?GetKeyValueRange@?$TAnimTrack@UIMusicKey@@@@UBEXAAM0@Z 34053a20 f i AnimNode.obj
 0001:00052a20       ?GetKeyValueRange@?$TAnimTrack@UICharacterKey@@@@UBEXAAM0@Z 34053a20 f i AnimNode.obj
 0001:00052a20       ?GetKeyValueRange@?$TAnimTrack@UIEventKey@@@@UBEXAAM0@Z 34053a20 f i AnimNode.obj
 0001:00052a20       ?GetKeyValueRange@?$TAnimTrack@UIFaceSeqKey@@@@UBEXAAM0@Z 34053a20 f i AnimNode.obj
 0001:00052a20       ?GetKeyValueRange@?$TAnimTrack@UIExprKey@@@@UBEXAAM0@Z 34053a20 f i AnimNode.obj
 0001:00052a20       ?GetKeyValueRange@?$TAnimTrack@UICaptureKey@@@@UBEXAAM0@Z 34053a20 f i AnimNode.obj
 0001:00052a20       ?GetKeyValueRange@?$TAnimTrack@UISoundKey@@@@UBEXAAM0@Z 34053a20 f i AnimNode.obj
 0001:00052a20       ?GetKeyValueRange@?$TAnimTrack@UIConsoleKey@@@@UBEXAAM0@Z 34053a20 f i AnimNode.obj
 0001:00052a20       ?GetKeyValueRange@?$TAnimTrack@UICommentKey@@@@UBEXAAM0@Z 34053a20 f i CommentTrack.obj
 0001:00052a40       ??_ECAnimMaterialNode@@$4PPPPPPPM@A@AEPAXI@Z 34053a40 f i MaterialNode.obj
 0001:00052a50       ?Release@CAnimNode@@$4PPPPPPPM@DA@AEXXZ 34053a50 f i MaterialNode.obj
 0001:00052a60       ?GetMemoryUsage@CAnimMaterialNode@@UBEXPAVICrySizer@@@Z 34053a60 f i MaterialNode.obj
 0001:00052aa0       ??_DCAnimMaterialNode@@QAEXXZ 34053aa0 f i MaterialNode.obj
 0001:00052b10       ??_GCAnimMaterialNode@@UAEPAXI@Z 34053b10 f i MaterialNode.obj
 0001:00052b10       ??_ECAnimMaterialNode@@UAEPAXI@Z 34053b10 f i MaterialNode.obj
 0001:00052b40       ??$?A$$BY0CA@D@?$hash_map@V?$CryStringT@D@@IV?$hash_stricmp@V?$CryStringT@D@@@stl@@U?$stlport_hash_equal@V?$CryStringT@D@@V?$hash_stricmp@V?$CryStringT@D@@@stl@@@3@V?$allocator@U?$pair@V?$CryStringT@D@@I@stlpmtx_std@@@stlpmtx_std@@@stlpmtx_std@@QAEAAIAAY0CA@$$CBD@Z 34053b40 f i MaterialNode.obj
 0001:00052c30       ?UpdateDynamicParams@CAnimMaterialNode@@UAEXXZ 34053c30 f   MaterialNode.obj
 0001:00052e30       ?Serialize@CAnimSceneNode@@UAEXAAVXmlNodeRef@@_N1@Z 34053e30 f   SceneNode.obj
 0001:00052e70       ??$?DMM@@YA?AU?$Vec3_tpl@M@@ABU?$QuatT_tpl@M@@ABU0@@Z 34053e70 f i SceneNode.obj
 0001:00052f70       ?ApplyEventKey@CAnimSceneNode@@AAEXAAUIEventKey@@AAUSAnimContext@@@Z 34053f70 f   SceneNode.obj
 0001:00052fd0       ?ApplySequenceKey@CAnimSceneNode@@AAEXPAUIAnimTrack@@HHAAUISequenceKey@@AAUSAnimContext@@@Z 34053fd0 f   SceneNode.obj
 0001:00053130       ?CreateDefaultTracks@CAnimSceneNode@@UAEXXZ 34054130 f   SceneNode.obj
 0001:00053180       ?GetParamCount@CAnimSceneNode@@UBEHXZ 34054180 f   SceneNode.obj
 0001:000531a0       ?GetActiveKey@?$TAnimTrack@UIConsoleKey@@@@QAEHMPAUIConsoleKey@@@Z 340541a0 f i SceneNode.obj
 0001:00053360       ?GetActiveKey@?$TAnimTrack@UIMusicKey@@@@QAEHMPAUIMusicKey@@@Z 34054360 f i SceneNode.obj
 0001:00053500       ?GetActiveKey@?$TAnimTrack@UISequenceKey@@@@QAEHMPAUISequenceKey@@@Z 34054500 f i SceneNode.obj
 0001:000536b0       ?GetActiveKey@?$TAnimTrack@UIDiscreteFloatKey@@@@QAEHMPAUIDiscreteFloatKey@@@Z 340546b0 f i SceneNode.obj
 0001:00053870       ?GetActiveKey@?$TAnimTrack@UICaptureKey@@@@QAEHMPAUICaptureKey@@@Z 34054870 f i SceneNode.obj
 0001:00053a20       ?GetParamInfo@CAnimSceneNode@@UBE_NHAAUSParamInfo@IAnimNode@@@Z 34054a20 f   SceneNode.obj
 0001:00053a70       ?GetParamInfoFromId@CAnimSceneNode@@UBE_NABVAnimParamType@@AAUSParamInfo@IAnimNode@@@Z 34054a70 f   SceneNode.obj
 0001:00053b30       ?Activate@CAnimSceneNode@@UAEX_N@Z 34054b30 f   SceneNode.obj
 0001:00053d10       ?ReleaseSounds@CAnimSceneNode@@AAEXXZ 34054d10 f   SceneNode.obj
 0001:00053dd0       ?Reset@CAnimSceneNode@@UAEXXZ 34054dd0 f   SceneNode.obj
 0001:00054080       ?Pause@CAnimSceneNode@@UAEXXZ 34055080 f   SceneNode.obj
 0001:00054090       ?ApplySoundKey@CAnimSceneNode@@AAEXPAUIAnimTrack@@HHAAUISoundKey@@AAUSAnimContext@@@Z 34055090 f   SceneNode.obj
 0001:000544d0       ?ApplyGotoKey@CAnimSceneNode@@AAEXPAVCGotoTrack@@AAUSAnimContext@@@Z 340554d0 f   SceneNode.obj
 0001:00054570       ??1CAnimSceneNode@@UAE@XZ  34055570 f   SceneNode.obj
 0001:00054600       ?Release@CAnimNode@@$4PPPPPPPM@IA@AEXXZ 34055600 f i SceneNode.obj
 0001:00054610       ??_ECAnimSceneNode@@$4PPPPPPPM@A@AEPAXI@Z 34055610 f i SceneNode.obj
 0001:00054620       ?GetMemoryUsage@CAnimSceneNode@@UBEXPAVICrySizer@@@Z 34055620 f i SceneNode.obj
 0001:00054690       ?GetCameraBoneLinkQuatT@CAnimSceneNode@@QAE_NPAUIEntity@@AAU?$QuatT_tpl@M@@_N@Z 34055690 f   SceneNode.obj
 0001:00054c10       ?ApplyCameraKey@CAnimSceneNode@@AAEXAAUISelectKey@@AAUSAnimContext@@@Z 34055c10 f   SceneNode.obj
 0001:00056d50       ?Animate@CAnimSceneNode@@UAEXAAUSAnimContext@@@Z 34057d50 f   SceneNode.obj
 0001:000577d0       ??_ECAnimSceneNode@@UAEPAXI@Z 340587d0 f i SceneNode.obj
 0001:000577d0       ??_GCAnimSceneNode@@UAEPAXI@Z 340587d0 f i SceneNode.obj
 0001:00057810       ?Initialize@CAnimSceneNode@@SAXXZ 34058810 f   SceneNode.obj
 0001:00057b10       ??0CAnimSceneNode@@QAE@XZ  34058b10 f   SceneNode.obj
 0001:00057c60       ??$SetGlobalValue@M@IScriptSystem@@QAEXPBDABM@Z 34058c60 f i ScriptVarNode.obj
 0001:00057cd0       ??0CAnimScriptVarNode@@QAE@XZ 34058cd0 f   ScriptVarNode.obj
 0001:00057d40       ?GetType@CAnimScriptVarNode@@UBE?AW4EAnimNodeType@@XZ 34058d40 f i ScriptVarNode.obj
 0001:00057d40       ?GetValueType@CSelectTrack@@UAE?AW4EAnimValue@@XZ 34058d40 f i AnimNode.obj
 0001:00057d50       ??_ECAnimEventNode@@$4PPPPPPPM@A@AEPAXI@Z 34058d50 f i EventNode.obj
 0001:00057d50       ??_ECAnimCVarNode@@$4PPPPPPPM@A@AEPAXI@Z 34058d50 f i CVarNode.obj
 0001:00057d50       ??_ECAnimPostFXNode@@$4PPPPPPPM@A@AEPAXI@Z 34058d50 f i AnimPostFXNode.obj
 0001:00057d50       ??_ECLayerNode@@$4PPPPPPPM@A@AEPAXI@Z 34058d50 f i LayerNode.obj
 0001:00057d50       ??_ECAnimScriptVarNode@@$4PPPPPPPM@A@AEPAXI@Z 34058d50 f i ScriptVarNode.obj
 0001:00057d60       ?GetParamInfo@CAnimCVarNode@@UBE_NHAAUSParamInfo@IAnimNode@@@Z 34058d60 f   CVarNode.obj
 0001:00057d60       ?GetParamInfo@CAnimScriptVarNode@@UBE_NHAAUSParamInfo@IAnimNode@@@Z 34058d60 f   ScriptVarNode.obj
 0001:00057d90       ??$GetGlobalValue@VSmartScriptTable@@@IScriptSystem@@QAE_NPBDAAVSmartScriptTable@@@Z 34058d90 f i ScriptVarNode.obj
 0001:00057e50       ??_GCLayerNode@@UAEPAXI@Z  34058e50 f i LayerNode.obj
 0001:00057e50       ??_ECAnimScriptVarNode@@UAEPAXI@Z 34058e50 f i ScriptVarNode.obj
 0001:00057e50       ??_GCAnimScriptVarNode@@UAEPAXI@Z 34058e50 f i ScriptVarNode.obj
 0001:00057e50       ??_GCAnimCVarNode@@UAEPAXI@Z 34058e50 f i CVarNode.obj
 0001:00057e50       ??_ECLayerNode@@UAEPAXI@Z  34058e50 f i LayerNode.obj
 0001:00057e50       ??_GCAnimPostFXNode@@UAEPAXI@Z 34058e50 f i AnimPostFXNode.obj
 0001:00057e50       ??_ECAnimPostFXNode@@UAEPAXI@Z 34058e50 f i AnimPostFXNode.obj
 0001:00057e50       ??_GCAnimEventNode@@UAEPAXI@Z 34058e50 f i EventNode.obj
 0001:00057e50       ??_ECAnimCVarNode@@UAEPAXI@Z 34058e50 f i CVarNode.obj
 0001:00057e50       ??_ECAnimEventNode@@UAEPAXI@Z 34058e50 f i EventNode.obj
 0001:00057e80       ?CreateDefaultTracks@CAnimCVarNode@@UAEXXZ 34058e80 f   CVarNode.obj
 0001:00057e80       ?CreateDefaultTracks@CAnimScriptVarNode@@UAEXXZ 34058e80 f   ScriptVarNode.obj
 0001:00057ed0       ?SetScriptValue@CAnimScriptVarNode@@AAEXXZ 34058ed0 f   ScriptVarNode.obj
 0001:00057fc0       ?Animate@CAnimScriptVarNode@@UAEXAAUSAnimContext@@@Z 34058fc0 f   ScriptVarNode.obj
 0001:00058070       ?GetMemoryUsage@CAnimScriptVarNode@@UBEXPAVICrySizer@@@Z 34059070 f i ScriptVarNode.obj
 0001:00058070       ?GetMemoryUsage@CAnimEventNode@@UBEXPAVICrySizer@@@Z 34059070 f i EventNode.obj
 0001:00058070       ?GetMemoryUsage@CAnimCVarNode@@UBEXPAVICrySizer@@@Z 34059070 f i CVarNode.obj
 0001:000580b0       __chkstk                   340590b0 f   MSVCRT:chkstk.obj
 0001:000580b0       __alloca_probe             340590b0     MSVCRT:chkstk.obj
 0001:000580dc       _memcpy                    340590dc f   MSVCRT:MSVCR100.dll
 0001:000580e2       __onexit                   340590e2 f   MSVCRT:atonexit.obj
 0001:00058183       _atexit                    34059183 f   MSVCRT:atonexit.obj
 0001:0005819a       __purecall                 3405919a f   MSVCRT:MSVCR100.dll
 0001:000581a0       _memset                    340591a0 f   MSVCRT:MSVCR100.dll
 0001:000581b0       __allmul                   340591b0 f   MSVCRT:llmul.obj
 0001:000581e4       ?what@exception@std@@UBEPBDXZ 340591e4 f   MSVCRT:MSVCR100.dll
 0001:000581f0       __allshl                   340591f0 f   MSVCRT:llshl.obj
 0001:00058210       __aullshr                  34059210 f   MSVCRT:ullshr.obj
 0001:00058230       __CIfmod                   34059230 f   MSVCRT:MSVCR100.dll
 0001:00058236       __CIasin                   34059236 f   MSVCRT:MSVCR100.dll
 0001:0005823c       _floor                     3405923c f   MSVCRT:MSVCR100.dll
 0001:00058250       __ftol2_sse                34059250 f   MSVCRT:ftol2.obj
 0001:00058259       __ftol2_pentium4           34059259 f   MSVCRT:ftol2.obj
 0001:0005826c       __ftol2_sse_excpt          3405926c f   MSVCRT:ftol2.obj
 0001:00058286       __ftol2                    34059286 f   MSVCRT:ftol2.obj
 0001:00058349       __CRT_INIT@12              34059349 f   MSVCRT:crtdll.obj
 0001:00058669       __DllMainCRTStartup@12     34059669 f   MSVCRT:crtdll.obj
 0001:0005868c       __unlock                   3405968c f   MSVCRT:MSVCR100.dll
 0001:00058692       ___dllonexit               34059692 f   MSVCRT:MSVCR100.dll
 0001:00058698       __lock                     34059698 f   MSVCRT:MSVCR100.dll
 0001:000586a0       __SEH_prolog4              340596a0 f   MSVCRT:sehprolg4.obj
 0001:000586e5       __SEH_epilog4              340596e5 f   MSVCRT:sehprolg4.obj
 0001:000586f9       __except_handler4          340596f9 f   MSVCRT:chandler4gs.obj
 0001:0005871e       ___sse2_available_init     3405971e f   MSVCRT:cpu_disp.obj
 0001:0005872e       ___clean_type_info_names   3405972e f   MSVCRT:tncleanup.obj
 0001:0005873a       __RTC_Initialize           3405973a f   MSVCRT:_initsect_.obj
 0001:00058760       __RTC_Terminate            34059760 f   MSVCRT:_initsect_.obj
 0001:00058790       __ValidateImageBase        34059790 f   MSVCRT:pesect.obj
 0001:000587d0       __FindPESection            340597d0 f   MSVCRT:pesect.obj
 0001:00058820       __IsNonwritableInCurrentImage 34059820 f   MSVCRT:pesect.obj
 0001:000588dc       __initterm                 340598dc f   MSVCRT:MSVCR100.dll
 0001:000588e2       __initterm_e               340598e2 f   MSVCRT:MSVCR100.dll
 0001:000588e8       __amsg_exit                340598e8 f   MSVCRT:MSVCR100.dll
 0001:000588ee       ___CppXcptFilter           340598ee f   MSVCRT:MSVCR100.dll
 0001:000588f4       _DllMain@12                340598f4 f   MSVCRT:dllmain.obj
 0001:00058918       ___security_init_cookie    34059918 f   MSVCRT:gs_support.obj
 0001:000589b3       @__security_check_cookie@4 340599b3 f   MSVCRT:secchk.obj
 0001:000589c2       __except_handler4_common   340599c2 f   MSVCRT:MSVCR100.dll
 0001:000589c8       ___clean_type_info_names_internal 340599c8 f   MSVCRT:MSVCR100.dll
 0001:000589ce       ___report_gsfailure        340599ce f   MSVCRT:gs_report.obj
 0001:00058ad4       __crt_debugger_hook        34059ad4 f   MSVCRT:MSVCR100.dll
 0001:00058e50       ??__Fs_dummyMemReplay@?1??CryGetIMemReplay@@YAPAUIMemReplay@@XZ@YAXXZ 34059e50 f i AnimSequence.obj
 0001:00058e90       ??__Fp@?1??CreateClassInstance@CFactory@CEngineModule_CryMovie@@UBE?AV?$shared_ptr@UICryUnknown@@@boost@@XZ@YAXXZ 34059e90 f i CryMovie.obj
 0002:00000000       __imp__InterlockedCompareExchange@12 3405b000     kernel32:KERNEL32.dll
 0002:00000004       __imp__InitializeCriticalSection@4 3405b004     kernel32:KERNEL32.dll
 0002:00000008       __imp__DeleteCriticalSection@4 3405b008     kernel32:KERNEL32.dll
 0002:0000000c       __imp__EnterCriticalSection@4 3405b00c     kernel32:KERNEL32.dll
 0002:00000010       __imp__LeaveCriticalSection@4 3405b010     kernel32:KERNEL32.dll
 0002:00000014       __imp__GetCurrentThreadId@0 3405b014     kernel32:KERNEL32.dll
 0002:00000018       __imp__LoadLibraryA@4      3405b018     kernel32:KERNEL32.dll
 0002:0000001c       __imp__GetProcAddress@8    3405b01c     kernel32:KERNEL32.dll
 0002:00000020       __imp__GetModuleHandleA@4  3405b020     kernel32:KERNEL32.dll
 0002:00000024       __imp__IsDebuggerPresent@0 3405b024     kernel32:KERNEL32.dll
 0002:00000028       __imp__Sleep@4             3405b028     kernel32:KERNEL32.dll
 0002:0000002c       __imp__InterlockedIncrement@4 3405b02c     kernel32:KERNEL32.dll
 0002:00000030       __imp__InterlockedDecrement@4 3405b030     kernel32:KERNEL32.dll
 0002:00000034       __imp__InterlockedExchangeAdd@8 3405b034     kernel32:KERNEL32.dll
 0002:00000038       __imp__UnhandledExceptionFilter@4 3405b038     kernel32:KERNEL32.dll
 0002:0000003c       __imp__GetCurrentProcess@0 3405b03c     kernel32:KERNEL32.dll
 0002:00000040       __imp__TerminateProcess@8  3405b040     kernel32:KERNEL32.dll
 0002:00000044       __imp__GetSystemTimeAsFileTime@4 3405b044     kernel32:KERNEL32.dll
 0002:00000048       __imp__GetCurrentProcessId@0 3405b048     kernel32:KERNEL32.dll
 0002:0000004c       __imp__GetTickCount@0      3405b04c     kernel32:KERNEL32.dll
 0002:00000050       __imp__QueryPerformanceCounter@4 3405b050     kernel32:KERNEL32.dll
 0002:00000054       __imp__DisableThreadLibraryCalls@4 3405b054     kernel32:KERNEL32.dll
 0002:00000058       __imp__IsProcessorFeaturePresent@4 3405b058     kernel32:KERNEL32.dll
 0002:0000005c       __imp__InterlockedExchange@8 3405b05c     kernel32:KERNEL32.dll
 0002:00000060       __imp__DecodePointer@4     3405b060     kernel32:KERNEL32.dll
 0002:00000064       __imp__EncodePointer@4     3405b064     kernel32:KERNEL32.dll
 0002:00000068       __imp__SetUnhandledExceptionFilter@4 3405b068     kernel32:KERNEL32.dll
 0002:0000006c       \177KERNEL32_NULL_THUNK_DATA 3405b06c     kernel32:KERNEL32.dll
 0002:00000070       __imp__strcspn             3405b070     MSVCRT:MSVCR100.dll
 0002:00000074       __imp__strchr              3405b074     MSVCRT:MSVCR100.dll
 0002:00000078       __imp__atof                3405b078     MSVCRT:MSVCR100.dll
 0002:0000007c       __imp__memset              3405b07c     MSVCRT:MSVCR100.dll
 0002:00000080       __imp___set_invalid_parameter_handler 3405b080     MSVCRT:MSVCR100.dll
 0002:00000084       __imp___set_purecall_handler 3405b084     MSVCRT:MSVCR100.dll
 0002:00000088       __imp_??0exception@std@@QAE@ABQBDH@Z 3405b088     MSVCRT:MSVCR100.dll
 0002:0000008c       __imp_?what@exception@std@@UBEPBDXZ 3405b08c     MSVCRT:MSVCR100.dll
 0002:00000090       __imp_??1exception@std@@UAE@XZ 3405b090     MSVCRT:MSVCR100.dll
 0002:00000094       __imp___vscprintf          3405b094     MSVCRT:MSVCR100.dll
 0002:00000098       __imp___vsnprintf          3405b098     MSVCRT:MSVCR100.dll
 0002:00000098       __imp__vsnprintf           3405b098     MSVCRT:MSVCR100.dll
 0002:0000009c       __imp__strcpy_s            3405b09c     MSVCRT:MSVCR100.dll
 0002:000000a0       __imp__strspn              3405b0a0     MSVCRT:MSVCR100.dll
 0002:000000a4       __imp___CIfmod             3405b0a4     MSVCRT:MSVCR100.dll
 0002:000000a8       __imp___CIasin             3405b0a8     MSVCRT:MSVCR100.dll
 0002:000000ac       __imp__vsprintf_s          3405b0ac     MSVCRT:MSVCR100.dll
 0002:000000b0       __imp__strncpy             3405b0b0     MSVCRT:MSVCR100.dll
 0002:000000b4       __imp__strncpy_s           3405b0b4     MSVCRT:MSVCR100.dll
 0002:000000b8       __imp__sprintf_s           3405b0b8     MSVCRT:MSVCR100.dll
 0002:000000bc       __imp__strcat_s            3405b0bc     MSVCRT:MSVCR100.dll
 0002:000000c0       __imp__strpbrk             3405b0c0     MSVCRT:MSVCR100.dll
 0002:000000c4       __imp__sscanf              3405b0c4     MSVCRT:MSVCR100.dll
 0002:000000c8       __imp__strstr              3405b0c8     MSVCRT:MSVCR100.dll
 0002:000000cc       __imp__floor               3405b0cc     MSVCRT:MSVCR100.dll
 0002:000000d0       __imp___localtime64        3405b0d0     MSVCRT:MSVCR100.dll
 0002:000000d4       __imp___time64             3405b0d4     MSVCRT:MSVCR100.dll
 0002:000000d8       __imp__strftime            3405b0d8     MSVCRT:MSVCR100.dll
 0002:000000dc       __imp__strncmp             3405b0dc     MSVCRT:MSVCR100.dll
 0002:000000e0       __imp__atoi                3405b0e0     MSVCRT:MSVCR100.dll
 0002:000000e4       __imp__tolower             3405b0e4     MSVCRT:MSVCR100.dll
 0002:000000e8       __imp___unlock             3405b0e8     MSVCRT:MSVCR100.dll
 0002:000000ec       __imp____dllonexit         3405b0ec     MSVCRT:MSVCR100.dll
 0002:000000f0       __imp___lock               3405b0f0     MSVCRT:MSVCR100.dll
 0002:000000f4       __imp___onexit             3405b0f4     MSVCRT:MSVCR100.dll
 0002:000000f8       __imp___malloc_crt         3405b0f8     MSVCRT:MSVCR100.dll
 0002:000000fc       __imp__free                3405b0fc     MSVCRT:MSVCR100.dll
 0002:00000100       __imp___encoded_null       3405b100     MSVCRT:MSVCR100.dll
 0002:00000104       __imp___initterm           3405b104     MSVCRT:MSVCR100.dll
 0002:00000108       __imp___initterm_e         3405b108     MSVCRT:MSVCR100.dll
 0002:0000010c       __imp___amsg_exit          3405b10c     MSVCRT:MSVCR100.dll
 0002:00000110       __imp____CppXcptFilter     3405b110     MSVCRT:MSVCR100.dll
 0002:00000114       __imp___except_handler4_common 3405b114     MSVCRT:MSVCR100.dll
 0002:00000118       __imp____clean_type_info_names_internal 3405b118     MSVCRT:MSVCR100.dll
 0002:0000011c       __imp___crt_debugger_hook  3405b11c     MSVCRT:MSVCR100.dll
 0002:00000120       __imp__memmove             3405b120     MSVCRT:MSVCR100.dll
 0002:00000124       __imp__exit                3405b124     MSVCRT:MSVCR100.dll
 0002:00000128       __imp__puts                3405b128     MSVCRT:MSVCR100.dll
 0002:0000012c       __imp__abort               3405b12c     MSVCRT:MSVCR100.dll
 0002:00000130       __imp__strrchr             3405b130     MSVCRT:MSVCR100.dll
 0002:00000134       __imp___purecall           3405b134     MSVCRT:MSVCR100.dll
 0002:00000138       __imp__memcpy              3405b138     MSVCRT:MSVCR100.dll
 0002:0000013c       __imp__stricmp             3405b13c     MSVCRT:MSVCR100.dll
 0002:0000013c       __imp___stricmp            3405b13c     MSVCRT:MSVCR100.dll
 0002:0000013c       __imp__strcmpi             3405b13c     MSVCRT:MSVCR100.dll
 0002:00000140       \177MSVCR100_NULL_THUNK_DATA 3405b140     MSVCRT:MSVCR100.dll
 0002:00000144       __imp__MessageBoxA@16      3405b144     user32:USER32.dll
 0002:00000148       \177USER32_NULL_THUNK_DATA 3405b148     user32:USER32.dll
 0002:0000014c       ___xc_a                    3405b14c     MSVCRT:cinitexe.obj
 0002:000001a0       ___xc_z                    3405b1a0     MSVCRT:cinitexe.obj
 0002:000001a4       ___xi_a                    3405b1a4     MSVCRT:cinitexe.obj
 0002:000001b0       ___xi_z                    3405b1b0     MSVCRT:cinitexe.obj
 0002:000001e0       ??_7CAnimLightNode@@6B?$_i_reference_target@H@@@ 3405b1e0     AnimLightNode.obj
 0002:000001f0       ??_7CAnimLightNode@@6BIAnimNode@@@ 3405b1f0     AnimLightNode.obj
 0002:00000300       ??_7?$_i_reference_target@H@@6B@ 3405b300     AnimLightNode.obj
 0002:0000030c       ??_C@_02DKCKIIND@?$CFs?$AA@ 3405b30c     AnimLightNode.obj
 0002:00000310       ??_C@_0CI@IOKCCNHB@Deleting?5Reference?5Counted?5Objec@ 3405b310     AnimLightNode.obj
 0002:00000338       __real@437f0000            3405b338     AnimLightNode.obj
 0002:0000033c       __real@42c80000            3405b33c     AnimLightNode.obj
 0002:00000340       __real@3f800000            3405b340     AnimLightNode.obj
 0002:00000344       __real@41200000            3405b344     AnimLightNode.obj
 0002:00000348       ??_8CAnimLightNode@@7B@    3405b348     AnimLightNode.obj
 0002:00000350       __real@00000000            3405b350     AnimLightNode.obj
 0002:00000354       ??_C@_0BD@PAENNAGK@SpecularPercentage?$AA@ 3405b354     AnimLightNode.obj
 0002:00000368       ??_C@_0BD@MNKCNEFE@SpecularMultiplier?$AA@ 3405b368     AnimLightNode.obj
 0002:0000037c       ??_C@_0L@LBBHPGLO@HDRDynamic?$AA@ 3405b37c     AnimLightNode.obj
 0002:00000388       ??_C@_0N@KAGFAILC@DiffuseColor?$AA@ 3405b388     AnimLightNode.obj
 0002:00000398       ??_C@_0BC@CLIBCEGM@DiffuseMultiplier?$AA@ 3405b398     AnimLightNode.obj
 0002:000003ac       ??_C@_06GJMFONGK@Radius?$AA@ 3405b3ac     AnimLightNode.obj
 0002:000003b4       ??_C@_0BE@IOLHOPEA@fSpecularPercentage?$AA@ 3405b3b4     AnimLightNode.obj
 0002:000003c8       ??_C@_0M@GGCKEINF@fHDRDynamic?$AA@ 3405b3c8     AnimLightNode.obj
 0002:000003d4       ??_C@_0BE@LDFIOLHO@fSpecularMultiplier?$AA@ 3405b3d4     AnimLightNode.obj
 0002:000003e8       ??_C@_0BD@GAMCLDGB@fDiffuseMultiplier?$AA@ 3405b3e8     AnimLightNode.obj
 0002:000003fc       ??_C@_0L@CBDKADEJ@clrDiffuse?$AA@ 3405b3fc     AnimLightNode.obj
 0002:00000408       ??_C@_08GCJNLIKG@Position?$AA@ 3405b408     AnimLightNode.obj
 0002:00000414       ??_C@_08GFJPCMMD@Rotation?$AA@ 3405b414     AnimLightNode.obj
 0002:00000420       ??_C@_0L@KLDABBOG@Visibility?$AA@ 3405b420     AnimLightNode.obj
 0002:0000042c       ??_C@_05GCNIINAF@Event?$AA@ 3405b42c     AnimLightNode.obj
 0002:00000438       ??_7IMemReplay@@6B@        3405b438     AnimSequence.obj
 0002:000004d0       ??_C@_0P@PCJPAHLM@out?5of?5memory?6?$AA@ 3405b4d0     AnimSequence.obj
 0002:000004e0       ??_C@_06NBFPPGEG@vector?$AA@ 3405b4e0     AnimSequence.obj
 0002:000004e8       ??_7CCommentNode@@6B?$_i_reference_target@H@@@ 3405b4e8     CommentNode.obj
 0002:000004e8       ??_7CAnimNode@@6B?$_i_reference_target@H@@@ 3405b4e8     AnimNode.obj
 0002:000004e8       ??_7CAnimNodeGroup@@6B?$_i_reference_target@H@@@ 3405b4e8     AnimSequence.obj
 0002:000004f8       ??_7CAnimNodeGroup@@6BIAnimNode@@@ 3405b4f8     AnimSequence.obj
 0002:00000600       ??_8CAnimNodeGroup@@7B@    3405b600     AnimSequence.obj
 0002:00000600       ??_8CAnimNode@@7B@         3405b600     AnimNode.obj
 0002:00000600       ??_8CCommentNode@@7B@      3405b600     CommentNode.obj
 0002:00000608       ??_7CDummyMemReplay@@6B@   3405b608     AnimSequence.obj
 0002:000006a0       ??_C@_04OKAPPFIB@Node?$AA@ 3405b6a0     AnimSequence.obj
 0002:000006a8       ??_C@_0BF@LIPFJOIM@CurrentCinematicName?$AA@ 3405b6a8     AnimSequence.obj
 0002:000006c0       ??_C@_0P@LBMFPPIC@anim_sequence_?$AA@ 3405b6c0     AnimSequence.obj
 0002:000006d0       __real@40800000            3405b6d0     AnimSequence.obj
 0002:000006d4       ??_C@_0DA@HJCMBEDE@?$DN?$DN?$DN?5Precaching?5render?5data?5for?5c@ 3405b6d4     AnimSequence.obj
 0002:00000704       ??_C@_00CNPNBAHC@?$AA@     3405b704     AnimSequence.obj
 0002:00000708       ??_C@_01KMDKNFGN@?1?$AA@   3405b708     AnimSequence.obj
 0002:0000070c       ??_C@_0L@MFFDMPJ@ParentNode?$AA@ 3405b70c     AnimSequence.obj
 0002:00000718       ??_C@_02HOGEDOAB@Id?$AA@   3405b718     AnimSequence.obj
 0002:0000071c       ??_C@_04KOACHJEN@Type?$AA@ 3405b71c     AnimSequence.obj
 0002:00000728       ??_7CAnimSequence@@6B@     3405b728     AnimSequence.obj
 0002:00000810       ??_C@_06HEBKAGDH@Events?$AA@ 3405b810     AnimSequence.obj
 0002:00000818       ??_C@_05JOEHJGHG@Nodes?$AA@ 3405b818     AnimSequence.obj
 0002:00000820       ??_C@_0EF@LCJCGODD@Loading?5sequence?5?8?$CFs?8?5?$CIstart?5tim@ 3405b820     AnimSequence.obj
 0002:00000868       ??_C@_07DLHCIBDH@default?$AA@ 3405b868     AnimSequence.obj
 0002:00000870       ??_C@_08PNBPAFID@override?$AA@ 3405b870     AnimSequence.obj
 0002:0000087c       ??_C@_02OLOABKKD@ID?$AA@   3405b87c     AnimSequence.obj
 0002:00000880       ??_C@_07GAHEIAPI@EndTime?$AA@ 3405b880     AnimSequence.obj
 0002:00000888       ??_C@_09MHCEAAPI@StartTime?$AA@ 3405b888     AnimSequence.obj
 0002:00000894       ??_C@_05BOOEKJH@Flags?$AA@ 3405b894     AnimSequence.obj
 0002:0000089c       ??_C@_04FABLJDN@Name?$AA@  3405b89c     AnimSequence.obj
 0002:000008a4       ??_C@_0BA@IBCEKOCF@SequenceVersion?$AA@ 3405b8a4     AnimSequence.obj
 0002:000008b4       ??_C@_08DOCONEG@Sequence?$AA@ 3405b8b4     AnimSequenceGroup.obj
 0002:000008c0       ??_C@_0O@PNOCNOGC@SequenceGroup?$AA@ 3405b8c0     AnimSequenceGroup.obj
 0002:000008d0       ??_C@_0P@IPMGNDHC@ChildSequences?$AA@ 3405b8d0     AnimSequenceGroup.obj
 0002:000008e0       ??_C@_0M@DKOCMNMM@ChildGroups?$AA@ 3405b8e0     AnimSequenceGroup.obj
 0002:000008f0       ??_7CAnimSequenceGroup@@6B@ 3405b8f0     AnimSequenceGroup.obj
 0002:00000948       ??_C@_04LOAJBDKD@true?$AA@ 3405b948     CryMovie.obj
 0002:00000950       __real@4f800000            3405b950     CryMovie.obj
 0002:00000954       ??_C@_0DJ@DLJMMMP@Could?5not?5access?5CrySystem?4dll?5?$CI@ 3405b954     CryMovie.obj
 0002:00000990       ??_C@_0P@NHEMOHAI@Memory?5Manager?$AA@ 3405b990     CryMovie.obj
 0002:000009a0       ??_C@_0O@FFDHMLKN@CrySystem?4dll?$AA@ 3405b9a0     CryMovie.obj
 0002:000009b0       ??_C@_0BO@JDKBDPNB@CryGetIMemoryManagerInterface?$AA@ 3405b9b0     CryMovie.obj
 0002:000009d0       ??_C@_0BB@PNKHDABP@CrySystemCrtFree?$AA@ 3405b9d0     CryMovie.obj
 0002:000009e4       ??_C@_0BB@MFMFBMDO@CrySystemCrtSize?$AA@ 3405b9e4     CryMovie.obj
 0002:000009f8       ??_C@_0BD@BBIFHONI@CrySystemCrtMalloc?$AA@ 3405b9f8     CryMovie.obj
 0002:00000a0c       ??_C@_0O@LCCIKADF@CryGetMemSize?$AA@ 3405ba0c     CryMovie.obj
 0002:00000a1c       ??_C@_07CKAGCLEE@CryFree?$AA@ 3405ba1c     CryMovie.obj
 0002:00000a24       ??_C@_0L@FICCDMFO@CryRealloc?$AA@ 3405ba24     CryMovie.obj
 0002:00000a30       ??_C@_09MCKPOEAK@CryMalloc?$AA@ 3405ba30     CryMovie.obj
 0002:00000a40       ?iid@?1??IID@IEngineModule@@CAABUCryGUID@@XZ@4U3@B 3405ba40     CryMovie.obj
 0002:00000a50       ??_7ICryFactory@@6B@       3405ba50     CryMovie.obj
 0002:00000a68       ??_7ISystemEventListener@@6B@ 3405ba68     CryMovie.obj
 0002:00000a70       ??_7ICryUnknown@@6B@       3405ba70     CryMovie.obj
 0002:00000a80       ?iid@?1??IID@ICryUnknown@@CAABUCryGUID@@XZ@4U3@B 3405ba80     CryMovie.obj
 0002:00000a90       ??_C@_0BD@PJOKHJBB@Pure?5function?5call?$AA@ 3405ba90     CryMovie.obj
 0002:00000aa4       ??_C@_0CL@LKHBOBAH@Invalid?5parameter?5detected?5in?5CR@ 3405baa4     CryMovie.obj
 0002:00000ad0       ??_C@_0BO@HAMEIFMK@Critical?5Section?5hanging?5lock?$AA@ 3405bad0     CryMovie.obj
 0002:00000af0       ??_7CSystemEventListner_Movie@@6B@ 3405baf0     CryMovie.obj
 0002:00000af8       ??_7CEngineModule_CryMovie@@6B@ 3405baf8     CryMovie.obj
 0002:00000b14       ??_C@_08NABALOKF@CryMovie?$AA@ 3405bb14     CryMovie.obj
 0002:00000b20       ??_C@_09BHIABECK@CryEngine?$AA@ 3405bb20     CryMovie.obj
 0002:00000b2c       ??_C@_05KNFBNCOH@float?$AA@ 3405bb2c     CryMovie.obj
 0002:00000b34       ??_7CFactory@CEngineModule_CryMovie@@6B@ 3405bb34     CryMovie.obj
 0002:00000b4c       ??_7bad_alloc@std@@6B@     3405bb4c     CryMovie.obj
 0002:00000b54       ??_C@_0P@GHFPNOJB@bad?5allocation?$AA@ 3405bb54     CryMovie.obj
 0002:00000b64       ??_C@_0BG@OKNPKAAP@EngineModule_CryMovie?$AA@ 3405bb64     CryMovie.obj
 0002:00000b80       ?cid@?1??GetClassID@CFactory@CEngineModule_CryMovie@@UBEABUCryGUID@@XZ@4U4@B 3405bb80     CryMovie.obj
 0002:00000b90       ??_7sp_counted_base@detail@boost@@6B@ 3405bb90     CryMovie.obj
 0002:00000ba0       ??_7?$sp_counted_impl_p@VCEngineModule_CryMovie@@@detail@boost@@6B@ 3405bba0     CryMovie.obj
 0002:00000bb0       ??_C@_0BN@FOKPCDPC@Boost?5threw?5an?5exception?3?5?$CFs?$AA@ 3405bbb0     CryMovie.obj
 0002:00000bd0       ??_C@_01IHBHIGKO@?0?$AA@   3405bbd0     CryMovie.obj
 0002:00000bd4       ??_C@_06HPGEIPLA@?$DMnull?$DO?$AA@ 3405bbd4     Movie.obj
 0002:00000bdc       ??_C@_07KAALEJHI@?$DMlocal?$DO?$AA@ 3405bbdc     Movie.obj
 0002:00000bf8       ??_7ISplineInterpolator@@6B@ 3405bbf8     Movie.obj
 0002:00000c50       ??_7IConsoleArgumentAutoComplete@@6B@ 3405bc50     Movie.obj
 0002:00000c60       ??_7IMovieSystem@@6B@      3405bc60     Movie.obj
 0002:00000d90       ??_C@_0DL@FNHKFACD@CMovieSystem?3?3PlaySequence?3?5Erro@ 3405bd90     Movie.obj
 0002:00000dd0       ??_C@_0FG@DBDANOMP@GoToFrame?5failed?$CB?5You?5should?5pro@ 3405bdd0     Movie.obj
 0002:00000e28       __real@ff7fffff            3405be28     Movie.obj
 0002:00000e2c       ??_C@_0P@FCFLEIGN@NextSequenceId?$AA@ 3405be2c     Movie.obj
 0002:00000e3c       ??_C@_03LJIJAGL@tga?$AA@   3405be3c     Movie.obj
 0002:00000e40       __real@bf800000            3405be40     Movie.obj
 0002:00000e44       __real@3e800000            3405be44     Movie.obj
 0002:00000e48       ??_7SMovieSequenceAutoComplete@@6B@ 3405be48     Movie.obj
 0002:00000e54       ??_C@_0BM@JEDFLJOI@capture_misc_render_buffers?$AA@ 3405be54     Movie.obj
 0002:00000e70       ??_C@_0BE@MHHODHHP@capture_file_prefix?$AA@ 3405be70     Movie.obj
 0002:00000e84       ??_C@_0P@JJKCHCIP@capture_frames?$AA@ 3405be84     Movie.obj
 0002:00000e94       ??_C@_0M@OENHLMCH@t_FixedStep?$AA@ 3405be94     Movie.obj
 0002:00000ea0       ??_C@_0P@LKGJNJLA@capture_folder?$AA@ 3405bea0     Movie.obj
 0002:00000eb0       ??_C@_0BD@BFEDKAKC@capture_frame_once?$AA@ 3405beb0     Movie.obj
 0002:00000ec4       ??_C@_0BE@NLFPFNOJ@capture_file_format?$AA@ 3405bec4     Movie.obj
 0002:00000ed8       __real@3d072b02            3405bed8     Movie.obj
 0002:00000edc       __real@3f000000            3405bedc     Movie.obj
 0002:00000ee0       ??_7ILightAnimWrapper@@6B@ 3405bee0     Movie.obj
 0002:00000ef0       ??_C@_0BD@FAMGONEB@CMovieSystem?3?3Load?$AA@ 3405bef0     Movie.obj
 0002:00000f04       ??_C@_0DF@NHHJKDFO@Movie?5system?5is?5loading?5the?5file@ 3405bf04     Movie.obj
 0002:00000f3c       ??_C@_0CH@OJMGPPDJ@SequenceData?5tag?5contains?5?$CFu?5seq@ 3405bf3c     Movie.obj
 0002:00000f64       ??_C@_0N@OLPDHAED@SequenceData?$AA@ 3405bf64     Movie.obj
 0002:00000f74       ??_C@_0BK@CIDFHAOL@mov_goToFrameEditor?5?$CFs?5?$CFf?$AA@ 3405bf74     Movie.obj
 0002:00000f90       ??_7CLightAnimWrapper@@6B@ 3405bf90     Movie.obj
 0002:00000fa0       __real@42000000            3405bfa0     Movie.obj
 0002:00000fa4       __real@41a80000            3405bfa4     Movie.obj
 0002:00000fa8       __real@41000000            3405bfa8     Movie.obj
 0002:00000fac       __real@41800000            3405bfac     Movie.obj
 0002:00000fb0       ??_C@_0BI@CCOIKCJG@Sequence?5?$CFs?5?3?5?$CFf?5?$CIx?5?$CFf?$CJ?$AA@ 3405bfb0     Movie.obj
 0002:00000fc8       __real@3fa66666            3405bfc8     Movie.obj
 0002:00000fcc       ??_7?$TSpline@U?$TCBSplineKey@U?$Quat_tpl@M@@@spline@@VHermitBasis@2@@spline@@6B@ 3405bfcc     Movie.obj
 0002:00000fdc       ??_7?$TSpline@U?$TCBSplineKeyEx@M@spline@@VHermitBasis@2@@spline@@6B@ 3405bfdc     Movie.obj
 0002:00000fec       ??_7?$TSpline@U?$TCBSplineKeyEx@U?$Vec3_tpl@M@@@spline@@VHermitBasis@2@@spline@@6B@ 3405bfec     Movie.obj
 0002:00000ffc       ??_C@_0BD@PACKHAKI@ca_eyes_procedural?$AA@ 3405bffc     Movie.obj
 0002:00001010       __real@42700000            3405c010     Movie.obj
 0002:00001014       ??_7?$TCBSpline@MU?$TCBSplineKeyEx@M@spline@@@spline@@6B@ 3405c014     Movie.obj
 0002:00001024       __real@40400000            3405c024     Movie.obj
 0002:00001028       __real@40000000            3405c028     Movie.obj
 0002:0000102c       __real@bf000000            3405c02c     Movie.obj
 0002:00001030       ??_7?$TCBSpline@U?$Vec3_tpl@M@@U?$TCBSplineKeyEx@U?$Vec3_tpl@M@@@spline@@@spline@@6B@ 3405c030     Movie.obj
 0002:00001040       __mask@@NegFloat@          3405c040     Movie.obj
 0002:00001050       ??_7ISplineBackup@@6B@     3405c050     Movie.obj
 0002:0000105c       __real@40490fdb            3405c05c     Movie.obj
 0002:00001060       ??_7TCBQuatSpline@spline@@6B@ 3405c060     Movie.obj
 0002:00001070       __real@3fc00000            3405c070     Movie.obj
 0002:00001074       __real@322bcc77            3405c074     Movie.obj
 0002:00001078       __real@3f7ff972            3405c078     Movie.obj
 0002:0000107c       ??_7?$SSplineBackup@V?$TCBSpline@MU?$TCBSplineKeyEx@M@spline@@@spline@@@spline@@6B?$TCBSpline@MU?$TCBSplineKeyEx@M@spline@@@1@@ 3405c07c     Movie.obj
 0002:0000108c       ??_7?$SSplineBackup@V?$TCBSpline@MU?$TCBSplineKeyEx@M@spline@@@spline@@@spline@@6BISplineBackup@@@ 3405c08c     Movie.obj
 0002:00001098       ??_7?$SSplineBackup@V?$TCBSpline@U?$Vec3_tpl@M@@U?$TCBSplineKeyEx@U?$Vec3_tpl@M@@@spline@@@spline@@@spline@@6B?$TCBSpline@U?$Vec3_tpl@M@@U?$TCBSplineKeyEx@U?$Vec3_tpl@M@@@spline@@@1@@ 3405c098     Movie.obj
 0002:000010a8       ??_7?$SSplineBackup@V?$TCBSpline@U?$Vec3_tpl@M@@U?$TCBSplineKeyEx@U?$Vec3_tpl@M@@@spline@@@spline@@@spline@@6BISplineBackup@@@ 3405c0a8     Movie.obj
 0002:000010b8       ??_7CMovieSystem@@6B@      3405c0b8     Movie.obj
 0002:000011e8       ??_7?$TrackSplineInterpolator@M@spline@@6B?$TCBSpline@MU?$TCBSplineKeyEx@M@spline@@@1@@ 3405c1e8     Movie.obj
 0002:000011f8       ??_7?$TrackSplineInterpolator@M@spline@@6BISplineInterpolator@@@ 3405c1f8     Movie.obj
 0002:00001250       ??_7?$TrackSplineInterpolator@U?$Vec3_tpl@M@@@spline@@6B?$TCBSpline@U?$Vec3_tpl@M@@U?$TCBSplineKeyEx@U?$Vec3_tpl@M@@@spline@@@1@@ 3405c250     Movie.obj
 0002:00001260       ??_7?$TrackSplineInterpolator@U?$Vec3_tpl@M@@@spline@@6BISplineInterpolator@@@ 3405c260     Movie.obj
 0002:000012b8       ??_C@_0BB@KDGHNNGG@mov_playSequence?$AA@ 3405c2b8     Movie.obj
 0002:000012cc       ??_C@_0BA@KOLGJNJO@Play?5a?5sequence?$AA@ 3405c2cc     Movie.obj
 0002:000012dc       ??_C@_0BC@NKLPKJLD@mov_listSequences?$AA@ 3405c2dc     Movie.obj
 0002:000012f0       ??_C@_0BH@GOMEJNPB@List?5current?5sequences?$AA@ 3405c2f0     Movie.obj
 0002:00001308       ??_C@_0BC@HMHKALIC@mov_debugCamShake?$AA@ 3405c308     Movie.obj
 0002:0000131c       ??_C@_0CF@CBLMJJLP@Enable?5debug?5log?5for?5camera?5shak@ 3405c31c     Movie.obj
 0002:00001344       ??_C@_0L@FCLIKKBE@mov_useCam?$AA@ 3405c344     Movie.obj
 0002:00001350       ??_C@_0O@IBKOOGLC@mov_goToFrame?$AA@ 3405c350     Movie.obj
 0002:00001360       ??_C@_0CM@MONLFHLP@Set?5specified?5sequence?5to?5given?5@ 3405c360     Movie.obj
 0002:0000138c       ??_C@_0BA@KAPIFHHD@mov_debugEvents?$AA@ 3405c38c     Movie.obj
 0002:0000139c       ??_C@_0CJ@NBPACGFN@Enable?5debug?5output?5for?5Cinemati@ 3405c39c     Movie.obj
 0002:000013c8       ??_C@_0BA@IOGPMBJH@mov_overrideCam?$AA@ 3405c3c8     Movie.obj
 0002:000013d8       ??_C@_0FM@IFGACBLE@Set?5the?5camera?5used?5for?5the?5sequ@ 3405c3d8     Movie.obj
 0002:00001434       ??_C@_0BA@GHLGKIEP@mov_NoCutscenes?$AA@ 3405c434     Movie.obj
 0002:00001444       ??_C@_0BO@GLPGILNG@Disable?5playing?5of?5Cut?9Scenes?$AA@ 3405c444     Movie.obj
 0002:00001464       ??_C@_04NBFCGMPH@root?$AA@ 3405c464     Movie.obj
 0002:0000146c       ??_7?$TrackSplineInterpolator@U?$Quat_tpl@M@@@spline@@6BTCBQuatSpline@1@@ 3405c46c     Movie.obj
 0002:00001480       ??_7?$TrackSplineInterpolator@U?$Quat_tpl@M@@@spline@@6BISplineInterpolator@@@ 3405c480     Movie.obj
 0002:000014d8       ??_7?$SSplineBackup@VTCBQuatSpline@spline@@@spline@@6BTCBQuatSpline@1@@ 3405c4d8     Movie.obj
 0002:000014e8       ??_7?$SSplineBackup@VTCBQuatSpline@spline@@@spline@@6BISplineBackup@@@ 3405c4e8     Movie.obj
 0002:000014f8       ??_7?$TAnimSplineTrack@M@@6B@ 3405c4f8     Movie.obj
 0002:000015e4       __real@42652ee1            3405c5e4     Movie.obj
 0002:000015e8       __real@3c8efa35            3405c5e8     Movie.obj
 0002:000015ec       __real@3c23d70a            3405c5ec     Movie.obj
 0002:000015f0       __real@3fc90fdb            3405c5f0     Movie.obj
 0002:000015f4       __real@c0000000            3405c5f4     Movie.obj
 0002:000015f8       ??_C@_03CCEPDEKL@Key?$AA@  3405c5f8     Movie.obj
 0002:000015fc       ??_C@_02EOPBOLLC@dd?$AA@   3405c5fc     Movie.obj
 0002:00001600       ??_C@_02ELHCGPCE@ds?$AA@   3405c600     Movie.obj
 0002:00001604       ??_C@_05GECEPKB@flags?$AA@ 3405c604     Movie.obj
 0002:0000160c       ??_C@_08NCGGKIMN@easefrom?$AA@ 3405c60c     Movie.obj
 0002:00001618       ??_C@_06HLKCLFPG@easeto?$AA@ 3405c618     Movie.obj
 0002:00001620       ??_C@_04NBAGBPGE@bias?$AA@ 3405c620     Movie.obj
 0002:00001628       ??_C@_04INBALIPC@cont?$AA@ 3405c628     Movie.obj
 0002:00001630       ??_C@_04HPCMIFMD@tens?$AA@ 3405c630     Movie.obj
 0002:00001638       ??_C@_05MFEJDJP@value?$AA@ 3405c638     Movie.obj
 0002:00001640       ??_C@_04CLCEDBPF@time?$AA@ 3405c640     Movie.obj
 0002:00001648       ??_C@_0M@KCOFNGNN@CustomColor?$AA@ 3405c648     Movie.obj
 0002:00001654       ??_C@_0P@BNHNNKLK@HasCustomColor?$AA@ 3405c654     Movie.obj
 0002:00001664       ??_C@_0N@GIOGCODL@defaultValue?$AA@ 3405c664     Movie.obj
 0002:00001674       ??_C@_09CBCMCCID@TrackType?$AA@ 3405c674     Movie.obj
 0002:00001680       ??_C@_04GEFJINEE@?$CF?42f?$AA@ 3405c680     Movie.obj
 0002:00001688       ??_C@_06JJLAMBGK@target?$AA@ 3405c688     Movie.obj
 0002:00001690       ??_C@_05FFMGLIAD@?1xfov?$AA@ 3405c690     Movie.obj
 0002:00001698       ??_C@_0P@DENFGKM@?1rotateZ?4ANGLE?$AA@ 3405c698     Movie.obj
 0002:000016a8       ??_C@_0P@INMCFBEP@?1rotateY?4ANGLE?$AA@ 3405c6a8     Movie.obj
 0002:000016b8       ??_C@_0P@EBGIFBNB@?1rotateX?4ANGLE?$AA@ 3405c6b8     Movie.obj
 0002:000016c8       ??_C@_0N@JAEPLAGL@?1translate?4Z?$AA@ 3405c6c8     Movie.obj
 0002:000016d8       ??_C@_0N@LLGCODKI@?1translate?4Y?$AA@ 3405c6d8     Movie.obj
 0002:000016e8       ??_C@_0N@KCHJNCOJ@?1translate?4X?$AA@ 3405c6e8     Movie.obj
 0002:000016f8       ??_C@_0M@BCMNDPAP@?$CD?$CFs?9sampler?$AA@ 3405c6f8     Movie.obj
 0002:00001704       ??_C@_07MFOHDNMP@channel?$AA@ 3405c704     Movie.obj
 0002:0000170c       ??_C@_0L@NNBPAECM@?$CD?$CFs?9interp?$AA@ 3405c70c     Movie.obj
 0002:00001718       ??_C@_0L@NBDKLHGC@?$CD?$CFs?9output?$AA@ 3405c718     Movie.obj
 0002:00001724       ??_C@_06DOKNKOPH@OUTPUT?$AA@ 3405c724     Movie.obj
 0002:0000172c       ??_C@_09IHGDAHPC@?$CD?$CFs?9input?$AA@ 3405c72c     Movie.obj
 0002:00001738       ??_C@_08KKJDHNGI@semantic?$AA@ 3405c738     Movie.obj
 0002:00001744       ??_C@_05POAEJIHJ@INPUT?$AA@ 3405c744     Movie.obj
 0002:0000174c       ??_C@_05DFJCHPDH@input?$AA@ 3405c74c     Movie.obj
 0002:00001754       ??_C@_0L@GNDAEBIE@?$CFs?9sampler?$AA@ 3405c754     Movie.obj
 0002:00001760       ??_C@_07PKJOFHPL@sampler?$AA@ 3405c760     Movie.obj
 0002:00001768       ??_C@_0O@FILABAAA@INTERPOLATION?$AA@ 3405c768     Movie.obj
 0002:00001778       ??_C@_0L@PILNCGCJ@Name_array?$AA@ 3405c778     Movie.obj
 0002:00001784       ??_C@_09EKGMDEGA@?$CFs?9interp?$AA@ 3405c784     Movie.obj
 0002:00001790       ??_C@_05MHMCHENB@VALUE?$AA@ 3405c790     Movie.obj
 0002:00001798       ??_C@_09EGEJIHCO@?$CFs?9output?$AA@ 3405c798     Movie.obj
 0002:000017a4       ??_C@_04GPMDFGEJ@type?$AA@ 3405c7a4     Movie.obj
 0002:000017ac       ??_C@_04MEMAJGDJ@name?$AA@ 3405c7ac     Movie.obj
 0002:000017b4       ??_C@_04OHBONDIN@TIME?$AA@ 3405c7b4     Movie.obj
 0002:000017bc       ??_C@_05LJDNNBIK@param?$AA@ 3405c7bc     Movie.obj
 0002:000017c4       ??_C@_06LNMIFCNI@stride?$AA@ 3405c7c4     Movie.obj
 0002:000017cc       ??_C@_08HHJHBDHL@accessor?$AA@ 3405c7cc     Movie.obj
 0002:000017d8       ??_C@_0BB@CJEENCBC@technique_common?$AA@ 3405c7d8     Movie.obj
 0002:000017ec       ??_C@_08GLEBIGHN@?$CFs?9array?$AA@ 3405c7ec     Movie.obj
 0002:000017f8       ??_C@_05IOMEMJEC@count?$AA@ 3405c7f8     Movie.obj
 0002:00001800       ??_C@_0M@LJJMFMEG@float_array?$AA@ 3405c800     Movie.obj
 0002:0000180c       ??_C@_08CGIKMDPJ@?$CFs?9input?$AA@ 3405c80c     Movie.obj
 0002:00001818       ??_C@_06OEKOLKIL@source?$AA@ 3405c818     Movie.obj
 0002:00001820       ??_C@_02EGCJHIOB@id?$AA@   3405c820     Movie.obj
 0002:00001824       ??_C@_09KCBFNMAJ@animation?$AA@ 3405c824     Movie.obj
 0002:00001830       ??_C@_06HLLDPCCO@LINEAR?$AA@ 3405c830     Movie.obj
 0002:00001838       ??_C@_02NJPGOMH@?$CFf?$AA@ 3405c838     Movie.obj
 0002:0000183c       ??_C@_01CLKCMJKC@?5?$AA@   3405c83c     Movie.obj
 0002:00001840       ??_7?$TAnimSplineTrack@U?$Vec3_tpl@M@@@@6B@ 3405c840     Movie.obj
 0002:0000192c       ??_C@_0BB@EFFIPBKC@?$CF?42f?5?5?$CF?42f?5?5?$CF?42f?$AA@ 3405c92c     Movie.obj
 0002:00001940       ??_7?$TAnimSplineTrack@U?$Quat_tpl@M@@@@6B@ 3405c940     Movie.obj
 0002:00001a30       ??_C@_0EE@IBOFGHHD@CMovieSystem?3?3AddMovieListener?3?5@ 3405ca30     Movie.obj
 0002:00001a88       ??_C@_03PEGNKCLE@jpg?$AA@  3405ca88     CaptureTrack.obj
 0002:00001a8c       ??_C@_03CAKEDOOO@bmp?$AA@  3405ca8c     CaptureTrack.obj
 0002:00001a90       ??_C@_03HCPOIHIH@hdr?$AA@  3405ca90     CaptureTrack.obj
 0002:00001a94       ??_C@_0BA@PJFAJLPL@bufferToCapture?$AA@ 3405ca94     CaptureTrack.obj
 0002:00001aa4       ??_C@_06CHGOAPND@prefix?$AA@ 3405caa4     CaptureTrack.obj
 0002:00001aac       ??_C@_04KLFNICNF@once?$AA@ 3405caac     CaptureTrack.obj
 0002:00001ab4       ??_C@_06MIMEAMHG@folder?$AA@ 3405cab4     CaptureTrack.obj
 0002:00001abc       ??_C@_06DLEPGFEF@format?$AA@ 3405cabc     CaptureTrack.obj
 0002:00001ac4       ??_C@_08DDIIIDDJ@timeStep?$AA@ 3405cac4     CaptureTrack.obj
 0002:00001ad0       ??_C@_08LGBPINEC@duration?$AA@ 3405cad0     CaptureTrack.obj
 0002:00001adc       ??_C@_0O@POMLKGIJ@?$FL?$CFs?$FN?5?$CFs?0?5?$CF?43f?$AA@ 3405cadc     CaptureTrack.obj
 0002:00001aec       ??_C@_0BC@KBDIMKPI@?$FL?$CFs?$FN?5?$CFs?0?5?$CF?43f?0?5?$CFs?$AA@ 3405caec     CaptureTrack.obj
 0002:00001b00       ??_C@_05MPDBFDHF@Frame?$AA@ 3405cb00     CaptureTrack.obj
 0002:00001b08       ??_C@_05FAGFPHJG@start?$AA@ 3405cb08     CharacterTrack.obj
 0002:00001b10       ??_C@_07IJBEBMO@inplace?$AA@ 3405cb10     CharacterTrack.obj
 0002:00001b18       ??_C@_06JJDOMDIK@unload?$AA@ 3405cb18     CharacterTrack.obj
 0002:00001b20       ??_C@_08LAMJDAH@blendGap?$AA@ 3405cb20     CharacterTrack.obj
 0002:00001b2c       ??_C@_04GKOOIABA@loop?$AA@ 3405cb2c     CharacterTrack.obj
 0002:00001b34       ??_C@_05HJCMGBKF@speed?$AA@ 3405cb34     CharacterTrack.obj
 0002:00001b3c       ??_C@_03JBJLGPFL@end?$AA@  3405cb3c     CharacterTrack.obj
 0002:00001b40       ??_C@_06IJDLPEM@length?$AA@ 3405cb40     CharacterTrack.obj
 0002:00001b48       ??_C@_04NBCDDDGK@anim?$AA@ 3405cb48     CharacterTrack.obj
 0002:00001b50       ??_C@_0P@PGGBIMHN@AnimationLayer?$AA@ 3405cb50     CharacterTrack.obj
 0002:00001b60       __real@3a83126f            3405cb60     CharacterTrack.obj
 0002:00001b64       ??_C@_05CBJPDLOK@align?$AA@ 3405cb64     CommentTrack.obj
 0002:00001b6c       ??_C@_04IAGNFIBA@size?$AA@ 3405cb6c     CommentTrack.obj
 0002:00001b74       ??_C@_05PEENBMOG@color?$AA@ 3405cb74     CommentTrack.obj
 0002:00001b7c       ??_C@_04EFPADHIC@font?$AA@ 3405cb7c     CommentTrack.obj
 0002:00001b84       ??_C@_07GJGNEJFD@comment?$AA@ 3405cb84     CommentTrack.obj
 0002:00001b90       ??_7?$TAnimTrack@UICommentKey@@@@6B@ 3405cb90     CommentTrack.obj
 0002:00001c80       ??_7CCommentTrack@@6B@     3405cc80     CommentTrack.obj
 0002:00001d78       __real@43b40000            3405cd78     CompoundSplineTrack.obj
 0002:00001d7c       __real@3b360b61            3405cd7c     CompoundSplineTrack.obj
 0002:00001d80       __real@4076800000000000    3405cd80     CompoundSplineTrack.obj
 0002:00001d88       __real@7f7fffff            3405cd88     CompoundSplineTrack.obj
 0002:00001d8c       ??_C@_05MPOCIJBL@?$CFs?9?$CFs?$AA@ 3405cd8c     CompoundSplineTrack.obj
 0002:00001d94       ??_7?$TSpline@U?$SplineKeyEx@U?$Vec2_tpl@M@@@spline@@VBezierBasis@2@@spline@@6B@ 3405cd94     CompoundSplineTrack.obj
 0002:00001da4       ??_7?$BezierSpline@U?$Vec2_tpl@M@@U?$SplineKeyEx@U?$Vec2_tpl@M@@@spline@@@spline@@6B@ 3405cda4     CompoundSplineTrack.obj
 0002:00001db4       __real@40c00000            3405cdb4     CompoundSplineTrack.obj
 0002:00001db8       __real@3eaaaaab            3405cdb8     CompoundSplineTrack.obj
 0002:00001dbc       ??_7?$SSplineBackup@V?$BezierSpline@U?$Vec2_tpl@M@@U?$SplineKeyEx@U?$Vec2_tpl@M@@@spline@@@spline@@@spline@@6B?$BezierSpline@U?$Vec2_tpl@M@@U?$SplineKeyEx@U?$Vec2_tpl@M@@@spline@@@1@@ 3405cdbc     CompoundSplineTrack.obj
 0002:00001dcc       ??_7?$SSplineBackup@V?$BezierSpline@U?$Vec2_tpl@M@@U?$SplineKeyEx@U?$Vec2_tpl@M@@@spline@@@spline@@@spline@@6BISplineBackup@@@ 3405cdcc     CompoundSplineTrack.obj
 0002:00001dd8       ??_7?$TrackSplineInterpolator@U?$Vec2_tpl@M@@@spline@@6B?$BezierSpline@U?$Vec2_tpl@M@@U?$SplineKeyEx@U?$Vec2_tpl@M@@@spline@@@1@@ 3405cdd8     CompoundSplineTrack.obj
 0002:00001de8       ??_7?$TrackSplineInterpolator@U?$Vec2_tpl@M@@@spline@@6BISplineInterpolator@@@ 3405cde8     CompoundSplineTrack.obj
 0002:00001e40       __real@00800000            3405ce40     CompoundSplineTrack.obj
 0002:00001e44       __real@bfc90fdb            3405ce44     CompoundSplineTrack.obj
 0002:00001e48       __real@358637bd            3405ce48     CompoundSplineTrack.obj
 0002:00001e4c       __real@41400000            3405ce4c     CompoundSplineTrack.obj
 0002:00001e50       __real@41100000            3405ce50     CompoundSplineTrack.obj
 0002:00001e58       ??_7?$TAnimSplineTrack@U?$Vec2_tpl@M@@@@6B@ 3405ce58     CompoundSplineTrack.obj
 0002:00001f48       ??_C@_0FL@IKMMBANA@?$FLCRYMOVIE?3TAnimSplineTrack?$DMVec2?$DO@ 3405cf48     CompoundSplineTrack.obj
 0002:00001fa8       ??_C@_0GD@IFENOGLH@?$FLCRYMOVIE?3TAnimSplineTrack?$DMVec2?$DO@ 3405cfa8     CompoundSplineTrack.obj
 0002:00002010       ??_C@_0FP@JCGKBLA@?$FLCRYMOVIE?3TAnimSplineTrack?$DMVec2?$DO@ 3405d010     CompoundSplineTrack.obj
 0002:00002070       ??_C@_0FO@KILGMLPP@?$FLCRYMOVIE?3TAnimSplineTrack?$DMVec2?$DO@ 3405d070     CompoundSplineTrack.obj
 0002:000020d0       ??_C@_03IMLOPEAE@?5?$AN?6?$AA@ 3405d0d0     CompoundSplineTrack.obj
 0002:000020d4       ??_C@_05BMMNJPJB@meter?$AA@ 3405d0d4     CompoundSplineTrack.obj
 0002:000020dc       ??_C@_04NPEDKLDA@unit?$AA@ 3405d0dc     CompoundSplineTrack.obj
 0002:000020e4       ??_C@_05EPCCKCPH@asset?$AA@ 3405d0e4     CompoundSplineTrack.obj
 0002:000020ec       ??_C@_0N@ICDJINAL@aspect_ratio?$AA@ 3405d0ec     CompoundSplineTrack.obj
 0002:000020fc       ??_C@_0M@EDEFNCAL@perspective?$AA@ 3405d0fc     CompoundSplineTrack.obj
 0002:00002108       ??_C@_06BALALAIG@optics?$AA@ 3405d108     CompoundSplineTrack.obj
 0002:00002110       ??_C@_06FNKMPIBD@camera?$AA@ 3405d110     CompoundSplineTrack.obj
 0002:00002118       ??_C@_0BA@KGFCDGAH@library_cameras?$AA@ 3405d118     CompoundSplineTrack.obj
 0002:00002128       __real@3fe38e3b            3405d128     CompoundSplineTrack.obj
 0002:0000212c       ??_C@_01ELNMCGJD@W?$AA@    3405d12c     CompoundSplineTrack.obj
 0002:00002130       ??_C@_01POHCFINO@Z?$AA@    3405d130     CompoundSplineTrack.obj
 0002:00002134       ??_C@_01NFFPALBN@Y?$AA@    3405d134     CompoundSplineTrack.obj
 0002:00002138       ??_C@_01MMEEDKFM@X?$AA@    3405d138     CompoundSplineTrack.obj
 0002:00002140       ??_7CCompoundSplineTrack@@6B@ 3405d140     CompoundSplineTrack.obj
 0002:00002228       ??_C@_0M@IACHOIFD@NewSubTrack?$AA@ 3405d228     CompoundSplineTrack.obj
 0002:00002234       ??_C@_08PBLPPKOH@SubTrack?$AA@ 3405d234     CompoundSplineTrack.obj
 0002:00002240       __real@3727c5ac            3405d240     CompoundSplineTrack.obj
 0002:00002244       ??_C@_07KMMNMMFF@command?$AA@ 3405d244     ConsoleTrack.obj
 0002:0000224c       ??_C@_0L@MANLMLBJ@eventValue?$AA@ 3405d24c     EventTrack.obj
 0002:00002258       ??_C@_05GFHEIIDD@event?$AA@ 3405d258     EventTrack.obj
 0002:00002260       ??_C@_02KEGNLNML@?0?5?$AA@ 3405d260     EventTrack.obj
 0002:00002264       ??_C@_08BBMJNKHO@blendout?$AA@ 3405d264     ExprTrack.obj
 0002:00002270       ??_C@_04LDIGEPNM@hold?$AA@ 3405d270     ExprTrack.obj
 0002:00002278       ??_C@_07DCACCANG@blendin?$AA@ 3405d278     ExprTrack.obj
 0002:00002280       ??_C@_03DCBBJBAA@amp?$AA@  3405d280     ExprTrack.obj
 0002:00002284       ??_C@_04CLMONKIF@node?$AA@ 3405d284     FaceSeqTrack.obj
 0002:00002290       ??_7?$TAnimTrack@UIDiscreteFloatKey@@@@6B@ 3405d290     GotoTrack.obj
 0002:00002380       ??_7CGotoTrack@@6B@        3405d380     GotoTrack.obj
 0002:0000246c       ??_C@_08KAMMIJBG@lookPose?$AA@ 3405d46c     LookAtTrack.obj
 0002:00002478       ??_C@_0L@HCAIGGFP@smoothTime?$AA@ 3405d478     LookAtTrack.obj
 0002:00002484       ??_C@_0N@BLJBMLJE@volramp_time?$AA@ 3405d484     MusicTrack.obj
 0002:00002494       ??_C@_04HJCAHOPF@mood?$AA@ 3405d494     MusicTrack.obj
 0002:0000249c       ??_C@_08NMKGCDEA@RampDown?$AA@ 3405d49c     MusicTrack.obj
 0002:000024a8       ??_C@_0M@KNEJBCAK@useCurColor?$AA@ 3405d4a8     ScreenFaderTrack.obj
 0002:000024b4       ??_C@_07JDHEGGGP@texture?$AA@ 3405d4b4     ScreenFaderTrack.obj
 0002:000024bc       ??_C@_0P@KFJFCJKP@fadeChangeType?$AA@ 3405d4bc     ScreenFaderTrack.obj
 0002:000024cc       ??_C@_08JKNBDEOK@fadeType?$AA@ 3405d4cc     ScreenFaderTrack.obj
 0002:000024d8       ??_C@_09LLGHPMNG@fadeColor?$AA@ 3405d4d8     ScreenFaderTrack.obj
 0002:000024e4       ??_C@_08NODGFDFG@fadeTime?$AA@ 3405d4e4     ScreenFaderTrack.obj
 0002:000024f0       ??_C@_03EKFHOMB@Out?$AA@   3405d4f0     ScreenFaderTrack.obj
 0002:000024f4       ??_C@_02IEILNGIL@In?$AA@   3405d4f4     ScreenFaderTrack.obj
 0002:000024f8       ??_7?$TAnimTrack@UIScreenFaderKey@@@@6B@ 3405d4f8     ScreenFaderTrack.obj
 0002:000025e8       ??_7CScreenFaderTrack@@6B@ 3405d5e8     ScreenFaderTrack.obj
 0002:000026d4       ??_C@_09DPLCPAJM@BlendTime?$AA@ 3405d6d4     SelectTrack.obj
 0002:000026e0       ??_C@_07FIMDMNKK@endtime?$AA@ 3405d6e0     SequenceTrack.obj
 0002:000026e8       ??_C@_09EJLICMCM@starttime?$AA@ 3405d6e8     SequenceTrack.obj
 0002:000026f4       ??_C@_09FJBEOEJL@donotstop?$AA@ 3405d6f4     SequenceTrack.obj
 0002:00002700       ??_C@_0O@PACDBHAG@overridetimes?$AA@ 3405d700     SequenceTrack.obj
 0002:00002710       ??_C@_0P@DGCPLGDP@UseCustomColor?$AA@ 3405d710     SoundTrack.obj
 0002:00002720       ??_C@_04EBPADADD@desc?$AA@ 3405d720     SoundTrack.obj
 0002:00002728       ??_C@_07JEPOHHIA@LipSync?$AA@ 3405d728     SoundTrack.obj
 0002:00002730       ??_C@_04KLCPKPBE@Loop?$AA@ 3405d730     SoundTrack.obj
 0002:00002738       ??_C@_04KHIMOMGA@Is3D?$AA@ 3405d738     SoundTrack.obj
 0002:00002740       ??_C@_06PGLBJMBP@Stream?$AA@ 3405d740     SoundTrack.obj
 0002:00002748       ??_C@_09OKLMBPLP@OutRadius?$AA@ 3405d748     SoundTrack.obj
 0002:00002754       ??_C@_08KFPACBGP@InRadius?$AA@ 3405d754     SoundTrack.obj
 0002:00002760       __real@447a0000            3405d760     SoundTrack.obj
 0002:00002764       ??_C@_0M@HJDOMPGI@SoundLength?$AA@ 3405d764     SoundTrack.obj
 0002:00002770       ??_C@_03HOPGHEB@pan?$AA@   3405d770     SoundTrack.obj
 0002:00002774       ??_C@_06EMCPHFGM@volume?$AA@ 3405d774     SoundTrack.obj
 0002:0000277c       ??_C@_08BABJIOEM@filename?$AA@ 3405d77c     SoundTrack.obj
 0002:00002788       ??_C@_05JLLNAHDI@Voice?$AA@ 3405d788     SoundTrack.obj
 0002:000027a0       ??_7CAnimCameraNode@@6B?$_i_reference_target@H@@@ 3405d7a0     AnimCameraNode.obj
 0002:000027b0       ??_7CAnimCameraNode@@6BIAnimNode@@@ 3405d7b0     AnimCameraNode.obj
 0002:000028c0       ??_C@_0L@BPOMBEHI@Dof_Active?$AA@ 3405d8c0     AnimCameraNode.obj
 0002:000028cc       ??_C@_0N@MCCJMDPA@DepthOfField?$AA@ 3405d8cc     AnimCameraNode.obj
 0002:000028dc       ??_C@_0M@EHGIIOIJ@TimeOffsetB?$AA@ 3405d8dc     AnimCameraNode.obj
 0002:000028e8       ??_C@_0P@BIICNJDM@NoiseBFreqMult?$AA@ 3405d8e8     AnimCameraNode.obj
 0002:000028f8       ??_C@_0O@GKBMANIL@NoiseBAmpMult?$AA@ 3405d8f8     AnimCameraNode.obj
 0002:00002908       ??_C@_0P@NIBNDADN@FrequencyBMult?$AA@ 3405d908     AnimCameraNode.obj
 0002:00002918       ??_C@_0L@FOKABDAD@FrequencyB?$AA@ 3405d918     AnimCameraNode.obj
 0002:00002924       ??_C@_0P@KAALNBLD@AmplitudeBMult?$AA@ 3405d924     AnimCameraNode.obj
 0002:00002934       ??_C@_0L@FHPIBMJL@AmplitudeB?$AA@ 3405d934     AnimCameraNode.obj
 0002:00002940       ??_C@_0M@GMEFNNEK@TimeOffsetA?$AA@ 3405d940     AnimCameraNode.obj
 0002:0000294c       ??_C@_0P@PDLFGCDP@NoiseAFreqMult?$AA@ 3405d94c     AnimCameraNode.obj
 0002:0000295c       ??_C@_0O@FDJBDBEO@NoiseAAmpMult?$AA@ 3405d95c     AnimCameraNode.obj
 0002:0000296c       ??_C@_0P@FOIJECJD@FrequencyAMult?$AA@ 3405d96c     AnimCameraNode.obj
 0002:0000297c       ??_C@_0L@HFINEAMA@FrequencyA?$AA@ 3405d97c     AnimCameraNode.obj
 0002:00002988       ??_C@_0P@CGJPKDBN@AmplitudeAMult?$AA@ 3405d988     AnimCameraNode.obj
 0002:00002998       ??_C@_0L@HMNFEPFI@AmplitudeA?$AA@ 3405d998     AnimCameraNode.obj
 0002:000029a4       ??_C@_05LOAGFEPL@NearZ?$AA@ 3405d9a4     AnimCameraNode.obj
 0002:000029ac       ??_C@_03PHODBHCN@FOV?$AA@  3405d9ac     AnimCameraNode.obj
 0002:000029b0       __real@3e2aaaab            3405d9b0     AnimCameraNode.obj
 0002:000029b4       __real@3e4ccccd            3405d9b4     AnimCameraNode.obj
 0002:000029b8       __real@41a00000            3405d9b8     AnimCameraNode.obj
 0002:000029bc       ??_C@_0BK@PDPNLALO@?$CD?$CFd?5shaking?5of?5?8?$CFs?8?5at?5?$CFf?$AA@ 3405d9bc     AnimCameraNode.obj
 0002:000029d8       ??_C@_03BMGHOINI@url?$AA@  3405d9d8     AnimCameraNode.obj
 0002:000029dc       ??_C@_07KFHLHGPD@?$CD?$CFs?9lib?$AA@ 3405d9dc     AnimCameraNode.obj
 0002:000029e4       ??_C@_0BA@JKDIDFNA@instance_camera?$AA@ 3405d9e4     AnimCameraNode.obj
 0002:000029f4       ??_C@_0L@PLMGKELA@1?50?50?590?40?$AA@ 3405d9f4     AnimCameraNode.obj
 0002:00002a00       ??_C@_07OFJEHCAB@rotateX?$AA@ 3405da00     AnimCameraNode.obj
 0002:00002a08       ??_C@_07MJGKDJMJ@0?51?50?50?$AA@ 3405da08     AnimCameraNode.obj
 0002:00002a10       ??_C@_07PMIPEDEA@rotateY?$AA@ 3405da10     AnimCameraNode.obj
 0002:00002a18       ??_C@_07LKIKINAJ@0?50?51?50?$AA@ 3405da18     AnimCameraNode.obj
 0002:00002a20       ??_C@_07NHKCBAID@rotateZ?$AA@ 3405da20     AnimCameraNode.obj
 0002:00002a28       ??_C@_06CEHMNFAL@rotate?$AA@ 3405da28     AnimCameraNode.obj
 0002:00002a30       ??_C@_05JMKGPOEH@0?50?50?$AA@ 3405da30     AnimCameraNode.obj
 0002:00002a38       ??_C@_03OBKGHBJN@sid?$AA@  3405da38     AnimCameraNode.obj
 0002:00002a3c       ??_C@_09ODNGOEIO@translate?$AA@ 3405da3c     AnimCameraNode.obj
 0002:00002a48       ??_C@_0BL@HBIGAAMP@AdjustDefaultCameraPose_?$CFd?$AA@ 3405da48     AnimCameraNode.obj
 0002:00002a64       ??_C@_0N@DEBPIDNF@visual_scene?$AA@ 3405da64     AnimCameraNode.obj
 0002:00002a74       ??_C@_0BG@HMJCKGDE@library_visual_scenes?$AA@ 3405da74     AnimCameraNode.obj
 0002:00002a8c       ??_C@_05ELCCFCFH@scene?$AA@ 3405da8c     AnimCameraNode.obj
 0002:00002a94       ??_C@_09PGIPFCHJ@?$CFs?9lib?9?$CFs?$AA@ 3405da94     AnimCameraNode.obj
 0002:00002aa0       ??_C@_0BD@CEDLKOGJ@library_animations?$AA@ 3405daa0     AnimCameraNode.obj
 0002:00002ab4       ??_C@_0M@IPMMALNC@1000?4000000?$AA@ 3405dab4     AnimCameraNode.obj
 0002:00002ac0       ??_C@_04MAOOOCDA@zfar?$AA@ 3405dac0     AnimCameraNode.obj
 0002:00002ac8       ??_C@_08BGFJLJPJ@0?4010000?$AA@ 3405dac8     AnimCameraNode.obj
 0002:00002ad4       ??_C@_05JKGCAEIF@znear?$AA@ 3405dad4     AnimCameraNode.obj
 0002:00002adc       ??_C@_04NENMFJFO@xfov?$AA@ 3405dadc     AnimCameraNode.obj
 0002:00002ae4       ??_C@_06CFKIOFLK@?$CFsMesh?$AA@ 3405dae4     AnimCameraNode.obj
 0002:00002aec       ??_C@_06CKMMBDFB@?$CFs?9lib?$AA@ 3405daec     AnimCameraNode.obj
 0002:00002af4       ??_C@_05GIKGJBLD@?1yfov?$AA@ 3405daf4     AnimCameraNode.obj
 0002:00002afc       ??_C@_01IPJKGB@?$CD?$AA@   3405dafc     AnimCameraNode.obj
 0002:00002b00       ??_C@_04GBLBFCGG@?9lib?$AA@ 3405db00     AnimCameraNode.obj
 0002:00002b08       ??_C@_09JHGACOGG@cryengine?$AA@ 3405db08     AnimCameraNode.obj
 0002:00002b14       ??_C@_0P@LLBKMAFH@authoring_tool?$AA@ 3405db14     AnimCameraNode.obj
 0002:00002b24       ??_C@_0M@EECBLNBL@contributor?$AA@ 3405db24     AnimCameraNode.obj
 0002:00002b30       ??_C@_06DDODHFJI@Near?5Z?$AA@ 3405db30     AnimCameraNode.obj
 0002:00002b38       ??_C@_0P@DEDAIKO@Depth?5of?5Field?$AA@ 3405db38     AnimCameraNode.obj
 0002:00002b48       ??_C@_05LCPHDDMM@Shake?$AA@ 3405db48     AnimCameraNode.obj
 0002:00002b50       ??_C@_0M@PJNHCOKF@FocusEntity?$AA@ 3405db50     AnimCameraNode.obj
 0002:00002b5c       ??_C@_03FKCKHFGP@Fov?$AA@  3405db5c     AnimCameraNode.obj
 0002:00002b60       ??_8CAnimCameraNode@@7B@   3405db60     AnimCameraNode.obj
 0002:00002b68       __real@41f40000            3405db68     AnimCameraNode.obj
 0002:00002b6c       __real@428c0000            3405db6c     AnimCameraNode.obj
 0002:00002b70       __real@42ca6666            3405db70     AnimCameraNode.obj
 0002:00002b74       __real@425c6666            3405db74     AnimCameraNode.obj
 0002:00002b78       __real@41700000            3405db78     AnimCameraNode.obj
 0002:00002b7c       __real@3bb60b61            3405db7c     AnimCameraNode.obj
 0002:00002b80       __real@3ea2f983            3405db80     AnimCameraNode.obj
 0002:00002b84       __real@43340000            3405db84     AnimCameraNode.obj
 0002:00002b88       ??_C@_0P@FLCKMFCD@Dof_BlurAmount?$AA@ 3405db88     AnimCameraNode.obj
 0002:00002b98       ??_C@_0P@HLCLEICD@Dof_FocusRange?$AA@ 3405db98     AnimCameraNode.obj
 0002:00002ba8       ??_C@_0BC@FNABKFJB@Dof_FocusDistance?$AA@ 3405dba8     AnimCameraNode.obj
 0002:00002bc8       ??_C@_07CGBANJHP@up_axis?$AA@ 3405dbc8     AnimNode.obj
 0002:00002bd0       ??_C@_07NHEMPLFH@COLLADA?$AA@ 3405dbd0     AnimNode.obj
 0002:00002bd8       ??_7IAnimNode@@6B?$_i_reference_target@H@@@ 3405dbd8     AnimNode.obj
 0002:00002be8       ??_7IAnimNode@@6B0@@       3405dbe8     AnimNode.obj
 0002:00002ce4       ??_C@_07NBCGADJA@Unknown?$AA@ 3405dce4     AnimNode.obj
 0002:00002cec       ??_C@_0M@BAELMDGA@Frequency?5B?$AA@ 3405dcec     AnimNode.obj
 0002:00002cf8       ??_C@_0M@DLGGJAKD@Frequency?5A?$AA@ 3405dcf8     AnimNode.obj
 0002:00002d04       ??_C@_0M@OOJGIABJ@Amplitude?5B?$AA@ 3405dd04     AnimNode.obj
 0002:00002d10       ??_C@_0M@MFLLNDNK@Amplitude?5A?$AA@ 3405dd10     AnimNode.obj
 0002:00002d1c       ??_C@_0P@HAFEHBOA@Rot?5Noise?5Freq?$AA@ 3405dd1c     AnimNode.obj
 0002:00002d2c       ??_C@_0O@KEJPBEEP@Rot?5Noise?5Amp?$AA@ 3405dd2c     AnimNode.obj
 0002:00002d3c       ??_C@_0P@KFKBMGCJ@Pos?5Noise?5Freq?$AA@ 3405dd3c     AnimNode.obj
 0002:00002d4c       ??_C@_0O@DBGJDJGN@Pos?5Noise?5Amp?$AA@ 3405dd4c     AnimNode.obj
 0002:00002d5c       ??_C@_0O@OBHBHCCK@ParamIdIsName?$AA@ 3405dd5c     AnimNode.obj
 0002:00002d6c       ??_C@_07LHBEFBAE@ParamId?$AA@ 3405dd6c     AnimNode.obj
 0002:00002d74       ??_C@_04INMHBHD@Z_UP?$AA@  3405dd74     AnimNode.obj
 0002:00002d7c       ??_C@_0M@KOAEBPJJ@Centimeters?$AA@ 3405dd7c     AnimNode.obj
 0002:00002d88       ??_C@_04DKCHIKEL@0?401?$AA@ 3405dd88     AnimNode.obj
 0002:00002d90       ??_C@_08LPECPNPM@revision?$AA@ 3405dd90     AnimNode.obj
 0002:00002d9c       ??_C@_08PCMCJENN@modified?$AA@ 3405dd9c     AnimNode.obj
 0002:00002da8       ??_C@_07OIPFBGHL@created?$AA@ 3405dda8     AnimNode.obj
 0002:00002db0       ??_C@_0BD@CNMAADNI@?$CFY?9?$CFm?9?$CFdT?$CFH?3?$CFM?3?$CFSZ?$AA@ 3405ddb0     AnimNode.obj
 0002:00002dc4       ??_C@_0M@GAODAIFM@source_data?$AA@ 3405ddc4     AnimNode.obj
 0002:00002dd0       ??_C@_04HDOCAJNK@?$CFs?$CFs?$AA@ 3405ddd0     AnimNode.obj
 0002:00002dd8       ??_C@_07CAIJGPF@file?3?1?1?$AA@ 3405ddd8     AnimNode.obj
 0002:00002de0       ??_C@_0BE@FCMFCFKC@CryENGINE?5TrackView?$AA@ 3405dde0     AnimNode.obj
 0002:00002df4       ??_C@_02HHCFIJHE@JJ?$AA@   3405ddf4     AnimNode.obj
 0002:00002df8       ??_C@_06LIPPPFCI@author?$AA@ 3405ddf8     AnimNode.obj
 0002:00002e00       ??_C@_07CPCPJPKL@version?$AA@ 3405de00     AnimNode.obj
 0002:00002e08       ??_C@_05HECNBIJP@1?44?41?$AA@ 3405de08     AnimNode.obj
 0002:00002e10       ??_C@_05PPEFOGKI@xmlns?$AA@ 3405de10     AnimNode.obj
 0002:00002e18       ??_C@_0CN@LBCAMMNI@http?3?1?1www?4collada?4org?12005?111?1C@ 3405de18     AnimNode.obj
 0002:00002e48       ??_7?$TAnimTrack@UICharacterKey@@@@6B@ 3405de48     AnimNode.obj
 0002:00002f38       ??_7?$TAnimTrack@UIBoolKey@@@@6B@ 3405df38     AnimNode.obj
 0002:00003028       ??_7?$TAnimTrack@UISelectKey@@@@6B@ 3405e028     AnimNode.obj
 0002:00003118       ??_7?$TAnimTrack@UIEventKey@@@@6B@ 3405e118     AnimNode.obj
 0002:00003208       ??_7?$TAnimTrack@UISoundKey@@@@6B@ 3405e208     AnimNode.obj
 0002:000032f8       ??_7?$TAnimTrack@UIExprKey@@@@6B@ 3405e2f8     AnimNode.obj
 0002:000033e8       ??_7?$TAnimTrack@UIConsoleKey@@@@6B@ 3405e3e8     AnimNode.obj
 0002:000034d8       ??_7?$TAnimTrack@UIMusicKey@@@@6B@ 3405e4d8     AnimNode.obj
 0002:000035c8       ??_7?$TAnimTrack@UIFaceSeqKey@@@@6B@ 3405e5c8     AnimNode.obj
 0002:000036b8       ??_7?$TAnimTrack@UILookAtKey@@@@6B@ 3405e6b8     AnimNode.obj
 0002:000037a8       ??_7?$TAnimTrack@UISequenceKey@@@@6B@ 3405e7a8     AnimNode.obj
 0002:00003898       ??_7?$TAnimTrack@UICaptureKey@@@@6B@ 3405e898     AnimNode.obj
 0002:00003988       ??_7CCharacterTrack@@6B@   3405e988     AnimNode.obj
 0002:00003a78       ??_7CLookAtTrack@@6B@      3405ea78     AnimNode.obj
 0002:00003b68       ??_7CEventTrack@@6B@       3405eb68     AnimNode.obj
 0002:00003c58       ??_7CSoundTrack@@6B@       3405ec58     AnimNode.obj
 0002:00003d48       ??_7CExprTrack@@6B@        3405ed48     AnimNode.obj
 0002:00003e38       ??_7CConsoleTrack@@6B@     3405ee38     AnimNode.obj
 0002:00003f28       ??_7CMusicTrack@@6B@       3405ef28     AnimNode.obj
 0002:00004018       ??_7CFaceSeqTrack@@6B@     3405f018     AnimNode.obj
 0002:00004108       ??_7CTrackEventTrack@@6B@  3405f108     AnimNode.obj
 0002:000041f8       ??_7CSequenceTrack@@6B@    3405f1f8     AnimNode.obj
 0002:000042e8       ??_7CCaptureTrack@@6B@     3405f2e8     AnimNode.obj
 0002:000043d8       ??_7CBoolTrack@@6B@        3405f3d8     AnimNode.obj
 0002:000044c8       ??_7CSelectTrack@@6B@      3405f4c8     AnimNode.obj
 0002:000045b8       ??_7CAnimNode@@6BIAnimNode@@@ 3405f5b8     AnimNode.obj
 0002:000046c0       ??_C@_04CAKOHOCJ@Blue?$AA@ 3405f6c0     AnimNode.obj
 0002:000046c8       ??_C@_05GGOIJPPE@Green?$AA@ 3405f6c8     AnimNode.obj
 0002:000046d0       ??_C@_03PADCEAKC@Red?$AA@  3405f6d0     AnimNode.obj
 0002:000046d4       ??_C@_0L@JNEJJCBH@BlurAmount?$AA@ 3405f6d4     AnimNode.obj
 0002:000046e0       ??_C@_0L@LNEIBPBH@FocusRange?$AA@ 3405f6e0     AnimNode.obj
 0002:000046ec       ??_C@_09JHDAKFFL@FocusDist?$AA@ 3405f6ec     AnimNode.obj
 0002:000046f8       ??_C@_05BFDCPAGB@Track?$AA@ 3405f6f8     AnimNode.obj
 0002:00004700       ??_C@_09BFJFFBFP@ValueType?$AA@ 3405f700     AnimNode.obj
 0002:0000470c       ??_C@_0DB@DLHGFFOC@ScriptTable?3Properties?1Color?1fSp@ 3405f70c     AnimNode.obj
 0002:00004740       ??_C@_0DB@GJJFBNM@ScriptTable?3Properties?1Color?1fSp@ 3405f740     AnimNode.obj
 0002:00004774       ??_C@_0CJ@IMIENLPN@ScriptTable?3Properties?1Color?1fHD@ 3405f774     AnimNode.obj
 0002:000047a0       ??_C@_0DA@HBLHCANM@ScriptTable?3Properties?1Color?1fDi@ 3405f7a0     AnimNode.obj
 0002:000047d0       ??_C@_0BO@CIMLNGDL@ScriptTable?3Properties?1Radius?$AA@ 3405f7d0     AnimNode.obj
 0002:000047f0       ??_C@_0CI@FKOOBCMN@ScriptTable?3Properties?1Color?1clr@ 3405f7f0     AnimNode.obj
 0002:00004818       ??_C@_0CA@DFHJLFOJ@ScriptTable?3Properties?1Strength?$AA@ 3405f818     AnimNode.obj
 0002:00004838       ??_C@_0CC@DIOJAGFG@ScriptTable?3Properties?1SpeedScal@ 3405f838     AnimNode.obj
 0002:0000485c       ??_C@_0BN@MKCJCFPD@ScriptTable?3Properties?1Scale?$AA@ 3405f85c     AnimNode.obj
 0002:0000487c       ??_C@_0CD@JALFLMEP@ScriptTable?3Properties?1PulsePeri@ 3405f87c     AnimNode.obj
 0002:000048a0       ??_C@_0CC@NGMONKBB@ScriptTable?3Properties?1CountScal@ 3405f8a0     AnimNode.obj
 0002:000048c4       ??_C@_0P@GKNMGFEL@ParamIdVersion?$AA@ 3405f8c4     AnimNode.obj
 0002:000048e0       ??_7CAnimEventNode@@6B?$_i_reference_target@H@@@ 3405f8e0     EventNode.obj
 0002:000048e0       ??_7CAnimPostFXNode@@6B?$_i_reference_target@H@@@ 3405f8e0     AnimPostFXNode.obj
 0002:000048e0       ??_7CAnimCVarNode@@6B?$_i_reference_target@H@@@ 3405f8e0     CVarNode.obj
 0002:000048e0       ??_7CAnimScriptVarNode@@6B?$_i_reference_target@H@@@ 3405f8e0     ScriptVarNode.obj
 0002:000048e0       ??_7CLayerNode@@6B?$_i_reference_target@H@@@ 3405f8e0     LayerNode.obj
 0002:000048f0       ??_7CAnimPostFXNode@@6BIAnimNode@@@ 3405f8f0     AnimPostFXNode.obj
 0002:000049f8       ??_7CControlParamBase@CFXNodeDescription@@6B@ 3405f9f8     AnimPostFXNode.obj
 0002:00004a14       ??_7?$TControlParam@M@CFXNodeDescription@@6B@ 3405fa14     AnimPostFXNode.obj
 0002:00004a30       ??_7?$TControlParam@_N@CFXNodeDescription@@6B@ 3405fa30     AnimPostFXNode.obj
 0002:00004a4c       ??_7CFXNodeDescription@@6B@ 3405fa4c     AnimPostFXNode.obj
 0002:00004a58       ??_C@_08HDDBOKL@GSMCache?$AA@ 3405fa58     AnimPostFXNode.obj
 0002:00004a64       ??_C@_0O@COPBMJMF@GSMCacheParam?$AA@ 3405fa64     AnimPostFXNode.obj
 0002:00004a74       ??_C@_0BD@BPKIOLCJ@HDRBrightThreshold?$AA@ 3405fa74     AnimPostFXNode.obj
 0002:00004a88       ??_C@_0BP@PHGDALPH@Global_User_HDRBrightThreshold?$AA@ 3405fa88     AnimPostFXNode.obj
 0002:00004aa8       ??_C@_0P@IIBKBPIE@HDRBrightLevel?$AA@ 3405faa8     AnimPostFXNode.obj
 0002:00004ab8       ??_C@_0BL@PBEHDCOM@Global_User_HDRBrightLevel?$AA@ 3405fab8     AnimPostFXNode.obj
 0002:00004ad4       ??_C@_0BE@PGCHAMBD@Dof_User_BlurAmount?$AA@ 3405fad4     AnimPostFXNode.obj
 0002:00004ae8       ??_C@_0BE@NGCGIBBD@Dof_User_FocusRange?$AA@ 3405fae8     AnimPostFXNode.obj
 0002:00004afc       __real@40a00000            3405fafc     AnimPostFXNode.obj
 0002:00004b00       ??_C@_0O@FPCCBDGK@FocusDistance?$AA@ 3405fb00     AnimPostFXNode.obj
 0002:00004b10       ??_C@_0BH@BNODFABG@Dof_User_FocusDistance?$AA@ 3405fb10     AnimPostFXNode.obj
 0002:00004b28       __real@40600000            3405fb28     AnimPostFXNode.obj
 0002:00004b2c       ??_C@_06CKGENIKG@Enable?$AA@ 3405fb2c     AnimPostFXNode.obj
 0002:00004b34       ??_C@_0BA@GNELAECO@Dof_User_Active?$AA@ 3405fb34     AnimPostFXNode.obj
 0002:00004b44       ??_C@_03MKKLGFGI@Hue?$AA@  3405fb44     AnimPostFXNode.obj
 0002:00004b48       ??_C@_0BF@JDKGAOBN@Global_User_ColorHue?$AA@ 3405fb48     AnimPostFXNode.obj
 0002:00004b60       ??_C@_0L@EICILOBK@Saturation?$AA@ 3405fb60     AnimPostFXNode.obj
 0002:00004b6c       ??_C@_0BH@LNGIODIN@Global_User_Saturation?$AA@ 3405fb6c     AnimPostFXNode.obj
 0002:00004b84       ??_C@_08KBHEFHNJ@Contrast?$AA@ 3405fb84     AnimPostFXNode.obj
 0002:00004b90       ??_C@_0BF@OHEGFCHK@Global_User_Contrast?$AA@ 3405fb90     AnimPostFXNode.obj
 0002:00004ba8       ??_C@_0L@JCLLFKLB@Brightness?$AA@ 3405fba8     AnimPostFXNode.obj
 0002:00004bb4       ??_C@_0BH@GHPLAHCG@Global_User_Brightness?$AA@ 3405fbb4     AnimPostFXNode.obj
 0002:00004bcc       ??_C@_09GIEJBABN@Luminance?$AA@ 3405fbcc     AnimPostFXNode.obj
 0002:00004bd8       ??_C@_0BD@PANJBHLM@Global_User_ColorK?$AA@ 3405fbd8     AnimPostFXNode.obj
 0002:00004bec       ??_C@_06ICCAKDNH@Yellow?$AA@ 3405fbec     AnimPostFXNode.obj
 0002:00004bf4       ??_C@_0BD@IICNGHGP@Global_User_ColorY?$AA@ 3405fbf4     AnimPostFXNode.obj
 0002:00004c08       ??_C@_07LFEAGNHO@Magenta?$AA@ 3405fc08     AnimPostFXNode.obj
 0002:00004c10       ??_C@_0BD@KGIDLADK@Global_User_ColorM?$AA@ 3405fc10     AnimPostFXNode.obj
 0002:00004c24       ??_C@_04ICNCCCFD@Cyan?$AA@ 3405fc24     AnimPostFXNode.obj
 0002:00004c2c       ??_C@_0BD@DIAAJNLE@Global_User_ColorC?$AA@ 3405fc2c     AnimPostFXNode.obj
 0002:00004c40       ??_C@_0P@ENLGACPL@BlurringRadius?$AA@ 3405fc40     AnimPostFXNode.obj
 0002:00004c50       ??_C@_0BM@OAEMOEOM@FilterRadialBlurring_Radius?$AA@ 3405fc50     AnimPostFXNode.obj
 0002:00004c6c       ??_C@_0L@IEECBKCL@ScreenPosY?$AA@ 3405fc6c     AnimPostFXNode.obj
 0002:00004c78       ??_C@_0CA@DNIENAMF@FilterRadialBlurring_ScreenPosY?$AA@ 3405fc78     AnimPostFXNode.obj
 0002:00004c98       ??_C@_0L@JNFJCLGK@ScreenPosX?$AA@ 3405fc98     AnimPostFXNode.obj
 0002:00004ca4       ??_C@_0CA@CEJPOBIE@FilterRadialBlurring_ScreenPosX?$AA@ 3405fca4     AnimPostFXNode.obj
 0002:00004cc4       ??_C@_06HKBMKICC@Amount?$AA@ 3405fcc4     AnimPostFXNode.obj
 0002:00004ccc       ??_C@_0BM@PDJFKBKE@FilterRadialBlurring_Amount?$AA@ 3405fccc     AnimPostFXNode.obj
 0002:00004ce8       ??_7CAnimScreenFaderNode@@6B?$_i_reference_target@H@@@ 3405fce8     AnimScreenFaderNode.obj
 0002:00004cf8       ??_7CAnimScreenFaderNode@@6BIAnimNode@@@ 3405fcf8     AnimScreenFaderNode.obj
 0002:00004e00       ??_C@_05NEDPJLDL@Fader?$AA@ 3405fe00     AnimScreenFaderNode.obj
 0002:00004e08       __real@44160000            3405fe08     AnimScreenFaderNode.obj
 0002:00004e0c       __real@44480000            3405fe0c     AnimScreenFaderNode.obj
 0002:00004e10       ??_8CAnimScreenFaderNode@@7B@ 3405fe10     AnimScreenFaderNode.obj
 0002:00004e20       __real@42480000            3405fe20     CommentNode.obj
 0002:00004e24       ??_C@_0L@HIIKNNFL@Unit?5Pos?5Y?$AA@ 3405fe24     CommentNode.obj
 0002:00004e30       ??_C@_0L@GBJBOMBK@Unit?5Pos?5X?$AA@ 3405fe30     CommentNode.obj
 0002:00004e3c       ??_C@_04OJAHODMC@Text?$AA@ 3405fe3c     CommentNode.obj
 0002:00004e48       ??_7CCommentNode@@6BIAnimNode@@@ 3405fe48     CommentNode.obj
 0002:00004f50       __real@9e3ce508            3405ff50     CVarNode.obj
 0002:00004f58       ??_7CAnimCVarNode@@6BIAnimNode@@@ 3405ff58     CVarNode.obj
 0002:00005060       ??_C@_05LPIJGKJ@Value?$AA@ 34060060     CVarNode.obj
 0002:00005068       ??_C@_0BA@PDOCIMMI@lightanimation_?$AA@ 34060068     EntityNode.obj
 0002:00005078       ??_C@_06BHELCHEP@seqid_?$AA@ 34060078     EntityNode.obj
 0002:00005080       ??_C@_08KDEFNGDD@mission_?$AA@ 34060080     EntityNode.obj
 0002:0000508c       ??_C@_04ODEHNGDA@seq_?$AA@ 3406008c     EntityNode.obj
 0002:00005094       ??_C@_09CEKCFLOE@gametoken?$AA@ 34060094     EntityNode.obj
 0002:000050a0       ??_C@_0N@POCFBNBB@customaction?$AA@ 340600a0     EntityNode.obj
 0002:000050b0       ??_C@_0L@JDHJGMLK@sotemplate?$AA@ 340600b0     EntityNode.obj
 0002:000050bc       ??_C@_07OOLFFMIG@soevent?$AA@ 340600bc     EntityNode.obj
 0002:000050c4       ??_C@_0N@MMKBBBOE@soanimhelper?$AA@ 340600c4     EntityNode.obj
 0002:000050d4       ??_C@_0M@HOFDIFFN@sonavhelper?$AA@ 340600d4     EntityNode.obj
 0002:000050e0       ??_C@_08FNJLBCFC@sohelper?$AA@ 340600e0     EntityNode.obj
 0002:000050ec       ??_C@_08IIDLKIEB@soaction?$AA@ 340600ec     EntityNode.obj
 0002:000050f8       ??_C@_0BC@OLGKKABB@sostatessopattern?$AA@ 340600f8     EntityNode.obj
 0002:0000510c       ??_C@_07IMPAHMIB@sostate?$AA@ 3406010c     EntityNode.obj
 0002:00005114       ??_C@_09NOPNAMMC@soclasses?$AA@ 34060114     EntityNode.obj
 0002:00005120       ??_C@_07MGGBABAL@soclass?$AA@ 34060120     EntityNode.obj
 0002:00005128       ??_C@_08PMPHKJEF@aianchor?$AA@ 34060128     EntityNode.obj
 0002:00005134       ??_C@_09JIIDHJOI@eaxpreset?$AA@ 34060134     EntityNode.obj
 0002:00005140       ??_C@_0N@HAIFEOCM@reverbpreset?$AA@ 34060140     EntityNode.obj
 0002:00005150       ??_C@_05OGGONADN@equip?$AA@ 34060150     EntityNode.obj
 0002:00005158       ??_C@_04CIMGMMMG@text?$AA@ 34060158     EntityNode.obj
 0002:00005160       ??_C@_06OADHBOPL@aiwave?$AA@ 34060160     EntityNode.obj
 0002:00005168       ??_C@_0M@IJPEIGOF@aiterritory?$AA@ 34060168     EntityNode.obj
 0002:00005174       ??_C@_0BA@LPBBGEGF@aientityclasses?$AA@ 34060174     EntityNode.obj
 0002:00005184       ??_C@_0BD@GKEFOHAH@aipfpropertieslist?$AA@ 34060184     EntityNode.obj
 0002:00005198       ??_C@_0M@MOLLILE@aicharacter?$AA@ 34060198     EntityNode.obj
 0002:000051a4       ??_C@_0L@NHIBMLFO@aibehavior?$AA@ 340601a4     EntityNode.obj
 0002:000051b0       ??_C@_04DAMGJPCA@file?$AA@ 340601b0     EntityNode.obj
 0002:000051b8       ??_C@_06IEOJBDIK@object?$AA@ 340601b8     EntityNode.obj
 0002:000051c0       ??_C@_03GJLPFLNF@obj?$AA@  340601c0     EntityNode.obj
 0002:000051c4       ??_C@_03JDBMONBN@tex?$AA@  340601c4     EntityNode.obj
 0002:000051c8       ??_C@_06IOAEHBNO@dialog?$AA@ 340601c8     EntityNode.obj
 0002:000051d0       ??_C@_05MHNANJII@sound?$AA@ 340601d0     EntityNode.obj
 0002:000051d8       ??_C@_03OEOJGHBI@snd?$AA@  340601d8     EntityNode.obj
 0002:000051dc       ??_C@_03KLOMFBDO@clr?$AA@  340601dc     EntityNode.obj
 0002:000051e0       ??_C@_06BILHELBG@shader?$AA@ 340601e0     EntityNode.obj
 0002:000051e8       ??_C@_02EKLAAFBD@es?$AA@   340601e8     EntityNode.obj
 0002:000051ec       ??_C@_02PKJNPPMI@ei?$AA@   340601ec     EntityNode.obj
 0002:000051f0       ??_C@_01LKDEMHDF@s?$AA@    340601f0     EntityNode.obj
 0002:000051f4       ??_C@_01INIBCBCB@f?$AA@    340601f4     EntityNode.obj
 0002:000051f8       ??_C@_01OJONOECF@b?$AA@    340601f8     EntityNode.obj
 0002:000051fc       ??_C@_01KBJDNOO@i?$AA@     340601fc     EntityNode.obj
 0002:00005200       ??_C@_01EFFIKLCJ@n?$AA@    34060200     EntityNode.obj
 0002:00005220       ??_C@_01EOFPKCAF@?$EA?$AA@ 34060220     EntityNode.obj
 0002:00005224       ??_C@_0BJ@DBLLCGAH@BoneLinkTransformEnabled?$AA@ 34060224     EntityNode.obj
 0002:00005240       ??_C@_0BB@NNBGAFHK@EntityGUIDSource?$AA@ 34060240     EntityNode.obj
 0002:00005254       ??_C@_0BB@KAAIHOJL@EntityGUIDTarget?$AA@ 34060254     EntityNode.obj
 0002:00005268       ??_C@_0L@FHPGAJIC@EntityGUID?$AA@ 34060268     EntityNode.obj
 0002:00005274       ??_C@_05MAGIBEFI@Scale?$AA@ 34060274     EntityNode.obj
 0002:0000527c       ??_C@_06OLMBOMJH@Rotate?$AA@ 3406027c     EntityNode.obj
 0002:00005284       ??_C@_03FCCPIJGJ@Pos?$AA@  34060284     EntityNode.obj
 0002:00005288       ?_list@?1??_S_primes@?$_Stl_prime@_N@priv@stlpmtx_std@@CAPBIAAI@Z@4QBIB 34060288     EntityNode.obj
 0002:00005300       ??_C@_08GJNPJIKN@?$CFf?0?$CFf?0?$CFf?$AA@ 34060300     EntityNode.obj
 0002:0000530c       __real@461c4000            3406030c     EntityNode.obj
 0002:00005310       ??_C@_09NDOPHKAF@?$CDRootNode?$AA@ 34060310     EntityNode.obj
 0002:0000531c       ??_C@_0BG@BECEDFJD@instance_visual_scene?$AA@ 3406031c     EntityNode.obj
 0002:00005334       ??_C@_07MOJMOKPC@1?50?50?50?$AA@ 34060334     EntityNode.obj
 0002:0000533c       ??_C@_08HCAGLOAO@RootNode?$AA@ 3406033c     EntityNode.obj
 0002:00005348       __real@34000000            34060348     EntityNode.obj
 0002:0000534c       ??_C@_0BI@FOOLGHCF@Unkown?5Entity?5Parameter?$AA@ 3406034c     EntityNode.obj
 0002:00005364       ??_C@_0O@LFGNNOCC@LUA?5call?5?$CI?$CFs?$CJ?$AA@ 34060364     EntityNode.obj
 0002:00005374       __real@3dcccccd            34060374     EntityNode.obj
 0002:00005378       ??_C@_0ED@BPALKBOA@?$DMSound?$DO?5In?5Trackview?5EntityNode?5@ 34060378     EntityNode.obj
 0002:000053bc       __real@40060a92            340603bc     EntityNode.obj
 0002:000053c0       ??_C@_0L@GHIHOBPC@Bip01?5Head?$AA@ 340603c0     EntityNode.obj
 0002:000053cc       ??_C@_0N@GDCLNJBE@_LocalPlayer?$AA@ 340603cc     EntityNode.obj
 0002:000053dc       ??_C@_01JOAMLHOP@?9?$AA@   340603dc     EntityNode.obj
 0002:000053e0       ??_C@_0O@NJGINBIP@rotateZ?4ANGLE?$AA@ 340603e0     EntityNode.obj
 0002:000053f0       ??_C@_0O@FHOHNGGM@rotateY?4ANGLE?$AA@ 340603f0     EntityNode.obj
 0002:00005400       ??_C@_0O@JLENNGPC@rotateX?4ANGLE?$AA@ 34060400     EntityNode.obj
 0002:00005410       ??_C@_0M@HAOAKOEG@translate?4Z?$AA@ 34060410     EntityNode.obj
 0002:0000541c       ??_C@_0M@FLMNPNIF@translate?4Y?$AA@ 3406041c     EntityNode.obj
 0002:00005428       ??_C@_0M@ECNGMMME@translate?4X?$AA@ 34060428     EntityNode.obj
 0002:00005434       ??_C@_0BI@JJMNGNII@OnSequenceAnimationStop?$AA@ 34060434     EntityNode.obj
 0002:0000544c       ??_C@_0BJ@ELPCNJNA@OnSequenceAnimationStart?$AA@ 3406044c     EntityNode.obj
 0002:00005468       ??_C@_01GLPGHMHM@z?$AA@    34060468     EntityNode.obj
 0002:0000546c       ??_C@_01EANLCPLP@y?$AA@    3406046c     EntityNode.obj
 0002:00005470       ??_C@_01FJMABOPO@x?$AA@    34060470     EntityNode.obj
 0002:00005474       __real@3b808081            34060474     EntityNode.obj
 0002:00005478       ??_C@_0CE@NGGHJNKA@movie_physicalentity_animation_l@ 34060478     EntityNode.obj
 0002:0000549c       ??_C@_0DC@FPENOFAD@Lerp?5value?5for?5animation?9driven?5@ 3406049c     EntityNode.obj
 0002:000054d0       __real@3f59999a            340604d0     EntityNode.obj
 0002:000054d4       ??_C@_05GIBOCELO@Noise?$AA@ 340604d4     EntityNode.obj
 0002:000054dc       ??_C@_06NFNEEJJI@LookAt?$AA@ 340604dc     EntityNode.obj
 0002:000054e4       ??_C@_0BA@FAMEOOKE@Facial?5Sequence?$AA@ 340604e4     EntityNode.obj
 0002:000054f4       ??_C@_0L@NMLOJPGF@Expression?$AA@ 340604f4     EntityNode.obj
 0002:00005500       ??_C@_09ONEINPNJ@Animation?$AA@ 34060500     EntityNode.obj
 0002:0000550c       ??_C@_05MAHMNMLO@Sound?$AA@ 3406050c     EntityNode.obj
 0002:00005514       ??_7CAnimEntityNode@@6B?$_i_reference_target@H@@@ 34060514     EntityNode.obj
 0002:00005520       ??_7CAnimEntityNode@@6BIAnimNode@@@ 34060520     EntityNode.obj
 0002:00005630       ??_8CAnimEntityNode@@7B@   34060630     EntityNode.obj
 0002:00005638       ??_C@_0BB@EKNEDHOO@OnPropertyChange?$AA@ 34060638     EntityNode.obj
 0002:0000564c       ??_C@_06FIHJNPKE@UnHide?$AA@ 3406064c     EntityNode.obj
 0002:00005654       ??_C@_04EACEFPPN@Hide?$AA@ 34060654     EntityNode.obj
 0002:0000565c       ??_C@_0L@LPOEKEBI@Ragdollize?$AA@ 3406065c     EntityNode.obj
 0002:00005668       ??_C@_0FI@HIDOMMED@An?5EntityNode?5?$DM?$CFs?$DO?5gets?5an?5inval@ 34060668     EntityNode.obj
 0002:000056c0       __real@3f847ae147ae147b    340606c0     EntityNode.obj
 0002:000056c8       ??_C@_0N@KFIHGOHC@ScriptTable?3?$AA@ 340606c8     EntityNode.obj
 0002:000056d8       ??_C@_0BE@EAPHPKOM@PropertiesInstance?1?$AA@ 340606d8     EntityNode.obj
 0002:000056ec       ??_C@_0BD@IDCALHLD@PropertiesInstance?$AA@ 340606ec     EntityNode.obj
 0002:00005700       ??_C@_0M@GBGOMIOF@Properties?1?$AA@ 34060700     EntityNode.obj
 0002:0000570c       ??_C@_0L@KOOGALIH@Properties?$AA@ 3406070c     EntityNode.obj
 0002:00005718       ??_7CAnimEventNode@@6BIAnimNode@@@ 34060718     EventNode.obj
 0002:00005820       ??_C@_0M@CIALDHNG@Track?5Event?$AA@ 34060820     EventNode.obj
 0002:00005830       ??_7CLayerNode@@6BIAnimNode@@@ 34060830     LayerNode.obj
 0002:00005938       ??_8CAnimEventNode@@7B@    34060938     EventNode.obj
 0002:00005938       ??_8CAnimScriptVarNode@@7B@ 34060938     ScriptVarNode.obj
 0002:00005938       ??_8CAnimPostFXNode@@7B@   34060938     AnimPostFXNode.obj
 0002:00005938       ??_8CAnimCVarNode@@7B@     34060938     CVarNode.obj
 0002:00005938       ??_8CLayerNode@@7B@        34060938     LayerNode.obj
 0002:00005948       ??_C@_02GLCCMJJI@?4?$FL?$AA@ 34060948     MaterialNode.obj
 0002:0000594c       ??_C@_0BF@GELFMFMH@Unknown?5Shader?5Param?$AA@ 3406094c     MaterialNode.obj
 0002:00005964       ??_C@_0P@MEGJPILI@Shader?5Param?59?$AA@ 34060964     MaterialNode.obj
 0002:00005974       ??_C@_0P@NNHCMJPJ@Shader?5Param?58?$AA@ 34060974     MaterialNode.obj
 0002:00005984       ??_C@_0P@FKOKNFDG@Shader?5Param?57?$AA@ 34060984     MaterialNode.obj
 0002:00005994       ??_C@_0P@EDPBOEHH@Shader?5Param?56?$AA@ 34060994     MaterialNode.obj
 0002:000059a4       ??_C@_0P@GINMLHLE@Shader?5Param?55?$AA@ 340609a4     MaterialNode.obj
 0002:000059b4       ??_C@_0P@HBMHIGPF@Shader?5Param?54?$AA@ 340609b4     MaterialNode.obj
 0002:000059c4       ??_C@_0P@DOIGBADC@Shader?5Param?53?$AA@ 340609c4     MaterialNode.obj
 0002:000059d4       ??_C@_0P@CHJNCBHD@Shader?5Param?52?$AA@ 340609d4     MaterialNode.obj
 0002:000059e4       ??_C@_0P@MLAHCLA@Shader?5Param?51?$AA@ 340609e4     MaterialNode.obj
 0002:000059f4       ??_C@_0L@ILPBNIIC@Glossiness?$AA@ 340609f4     MaterialNode.obj
 0002:00005a00       ??_C@_08BFCMIGII@Emission?$AA@ 34060a00     MaterialNode.obj
 0002:00005a0c       ??_C@_08LNEJIEKD@Specular?$AA@ 34060a0c     MaterialNode.obj
 0002:00005a18       ??_C@_07PDCHJCFI@Diffuse?$AA@ 34060a18     MaterialNode.obj
 0002:00005a20       ??_C@_07EBHHCJEE@Ambient?$AA@ 34060a20     MaterialNode.obj
 0002:00005a28       ??_C@_07HABJELCE@Opacity?$AA@ 34060a28     MaterialNode.obj
 0002:00005a30       ??_7CAnimMaterialNode@@6B?$_i_reference_target@H@@@ 34060a30     MaterialNode.obj
 0002:00005a40       ??_7CAnimMaterialNode@@6BIAnimNode@@@ 34060a40     MaterialNode.obj
 0002:00005b50       ??_8CAnimMaterialNode@@7B@ 34060b50     MaterialNode.obj
 0002:00005b68       ??_C@_06ENCLGNJJ@Event_?$AA@ 34060b68     SceneNode.obj
 0002:00005b70       ??_C@_0EC@FIGELDAF@?$DMSound?$DO?5In?5Trackview?5SceneNode?5?$DM@ 34060b70     SceneNode.obj
 0002:00005bb4       ??_7CAnimSceneNode@@6B?$_i_reference_target@H@@@ 34060bb4     SceneNode.obj
 0002:00005bc0       ??_7CAnimSceneNode@@6BIAnimNode@@@ 34060bc0     SceneNode.obj
 0002:00005cc8       ??_C@_0O@GNBPGJHI@FixedTimeStep?$AA@ 34060cc8     SceneNode.obj
 0002:00005cd8       ??_C@_08PLJGJKAG@Timewarp?$AA@ 34060cd8     SceneNode.obj
 0002:00005ce4       ??_C@_07EGAJKHF@Capture?$AA@ 34060ce4     SceneNode.obj
 0002:00005cec       ??_C@_04DJJLJKOK@GoTo?$AA@ 34060cec     SceneNode.obj
 0002:00005cf4       ??_C@_05LMJFOPOI@Music?$AA@ 34060cf4     SceneNode.obj
 0002:00005cfc       ??_C@_07PGLPGHFC@Console?$AA@ 34060cfc     SceneNode.obj
 0002:00005d04       ??_C@_06JCBBMBIP@Camera?$AA@ 34060d04     SceneNode.obj
 0002:00005d0c       ??_C@_05EMIOFHGB@Scene?$AA@ 34060d0c     SceneNode.obj
 0002:00005d14       ??_8CAnimSceneNode@@7B@    34060d14     SceneNode.obj
 0002:00005d20       ??_7CAnimScriptVarNode@@6BIAnimNode@@@ 34060d20     ScriptVarNode.obj
 0002:00005e28       __pDefaultRawDllMain       34060e28     MSVCRT:crtdll.obj
 0002:00005e28       __pRawDllMain              34060e28     MSVCRT:crtdll.obj
 0002:00005e38       __load_config_used         34060e38     MSVCRT:loadcfg.obj
 0002:00005ee0       ___safe_se_handler_table   34060ee0     <linker-defined>
 0002:00005ee4       ___rtc_iaa                 34060ee4     MSVCRT:_initsect_.obj
 0002:00005ee8       ___rtc_izz                 34060ee8     MSVCRT:_initsect_.obj
 0002:00005eec       ___rtc_taa                 34060eec     MSVCRT:_initsect_.obj
 0002:00005ef0       ___rtc_tzz                 34060ef0     MSVCRT:_initsect_.obj
 0002:00005f5c       __IMPORT_DESCRIPTOR_KERNEL32 34060f5c     kernel32:KERNEL32.dll
 0002:00005f70       __IMPORT_DESCRIPTOR_USER32 34060f70     user32:USER32.dll
 0002:00005f84       __IMPORT_DESCRIPTOR_MSVCR100 34060f84     MSVCRT:MSVCR100.dll
 0002:00005f98       __NULL_IMPORT_DESCRIPTOR   34060f98     kernel32:KERNEL32.dll
 0003:00000000       ?sEmptyStringBuffer@?1??_emptyHeader@?$CryStringT@D@@KAPAUStrHeader@2@XZ@4PAU32@A 34062000     AnimLightNode.obj
 0003:00000018       ?s_nodeParams@CAnimLightNode@@0PAUSParamInfo@IAnimNode@@A 34062018     AnimLightNode.obj
 0003:000000e0       ?m_seed@CLCGRndGen@@0_KA   340620e0     CryMovie.obj
 0003:00000110       ?fVec3_Zero@?$Vec3Constants@M@@2U?$Vec3_tpl@M@@B 34062110     StdAfx.obj
 0003:0000011c       ?fVec3_One@?$Vec3Constants@M@@2U?$Vec3_tpl@M@@B 3406211c     StdAfx.obj
 0003:00000128       ?fVec2_Zero@?$Vec2Constants@M@@2U?$Vec2_tpl@M@@A 34062128     StdAfx.obj
 0003:00000130       ?fVec2_OneX@?$Vec2Constants@M@@2U?$Vec2_tpl@M@@A 34062130     StdAfx.obj
 0003:00000138       ?fVec2_OneY@?$Vec2Constants@M@@2U?$Vec2_tpl@M@@A 34062138     StdAfx.obj
 0003:00000140       ?fVec2_One@?$Vec2Constants@M@@2U?$Vec2_tpl@M@@A 34062140     StdAfx.obj
 0003:00000148       ?kParamIdAttrName@?1??Serialize@AnimParamType@@QAEXAAVXmlNodeRef@@_N@Z@4PBDB 34062148     AnimNode.obj
 0003:0000014c       ?kByNameAttrName@?1??Serialize@AnimParamType@@QAEXAAVXmlNodeRef@@_N@Z@4PBDB 3406214c     AnimNode.obj
 0003:00000210       ___native_dllmain_reason   34062210     MSVCRT:natstart.obj
 0003:00000214       ___native_vcclrit_reason   34062214     MSVCRT:natstart.obj
 0003:00000218       ___security_cookie         34062218     MSVCRT:gs_cookie.obj
 0003:0000021c       ___security_cookie_complement 3406221c     MSVCRT:gs_cookie.obj
 0003:00000220       ?s_used_memory@?1??_usedMemory@?$CryStringT@D@@SAIH@Z@4IA 34062220     AnimLightNode.obj
 0003:00000224       ?s_used_memory@?1??_usedMemory@?$CryStackStringT@D$0CAA@@@SAII@Z@4IA 34062224     AnimSequence.obj
 0003:00000228       ?s_pMemReplay@?1??CryGetIMemReplay@@YAPAUIMemReplay@@XZ@4PAU2@A 34062228     AnimSequence.obj
 0003:0000022c       ?s_dummyMemReplay@?1??CryGetIMemReplay@@YAPAUIMemReplay@@XZ@4UCDummyMemReplay@@A 3406222c     AnimSequence.obj
 0003:00000230       ??_B?1??CryGetIMemReplay@@YAPAUIMemReplay@@XZ@51 34062230     AnimSequence.obj
 0003:00000234       ?numAllocations@_CryMemoryManagerPoolHelper@@2HC 34062234     CryMovie.obj
 0003:00000238       ?requestedMemory@_CryMemoryManagerPoolHelper@@2JC 34062238     CryMovie.obj
 0003:0000023c       ?freedMemory@_CryMemoryManagerPoolHelper@@2JC 3406223c     CryMovie.obj
 0003:00000240       ?allocatedMemory@_CryMemoryManagerPoolHelper@@2JC 34062240     CryMovie.obj
 0003:00000244       ?gEnv@@3PAUSSystemGlobalEnvironment@@A 34062244     CryMovie.obj
 0003:00000248       ?m_pFirst@Test@CryUnitTest@@2PAU12@A 34062248     CryMovie.obj
 0003:0000024c       ?m_pLast@Test@CryUnitTest@@2PAU12@A 3406224c     CryMovie.obj
 0003:00000250       ?g_pHeadToRegFactories@@3PAUSRegFactoryNode@@A 34062250     CryMovie.obj
 0003:00000254       ?g_bProfilerEnabled@@3_NA  34062254     CryMovie.obj
 0003:00000258       ?g_iTraceAllocations@@3HA  34062258     CryMovie.obj
 0003:0000025c       ?_CryMalloc@_CryMemoryManagerPoolHelper@@2P6APAXIAAII@ZA 3406225c     CryMovie.obj
 0003:00000260       ?_CryGetMemSize@_CryMemoryManagerPoolHelper@@2P6AIPAXI@ZA 34062260     CryMovie.obj
 0003:00000264       ?_CryRealloc@_CryMemoryManagerPoolHelper@@2P6APAXPAXIAAI1I@ZA 34062264     CryMovie.obj
 0003:00000268       ?_CryFree@_CryMemoryManagerPoolHelper@@2P6AIPAXI@ZA 34062268     CryMovie.obj
 0003:0000026c       ?_CryCrtMalloc@_CryMemoryManagerPoolHelper@@2P6APAXI@ZA 3406226c     CryMovie.obj
 0003:00000270       ?_CryCrtRealloc@_CryMemoryManagerPoolHelper@@2P6APAXPAXI@ZA 34062270     CryMovie.obj
 0003:00000274       ?_CryCrtFree@_CryMemoryManagerPoolHelper@@2P6AIPAX@ZA 34062274     CryMovie.obj
 0003:00000278       ?_CryCrtSize@_CryMemoryManagerPoolHelper@@2P6AIPAX@ZA 34062278     CryMovie.obj
 0003:0000027c       ?_CryGetIMemoryManagerInterface@_CryMemoryManagerPoolHelper@@2P6AXPAPAX@ZA 3406227c     CryMovie.obj
 0003:00000280       ?m_bInitialized@_CryMemoryManagerPoolHelper@@2HA 34062280     CryMovie.obj
 0003:00000284       ?g_random_generator@@3VCLCGRndGen@@A 34062284     CryMovie.obj
 0003:00000288       ?s_factory@CFactory@CEngineModule_CryMovie@@0V12@A 34062288     CryMovie.obj
 0003:000002b8       ?s_used_memory@?1??_usedMemory@?$CryStringT@_W@@SAIH@Z@4IA 340622b8     CryMovie.obj
 0003:000002c0       ?supportedIIDs@?1???0CFactory@CEngineModule_CryMovie@@AAE@XZ@4PAUCryGUID@@A 340622c0     CryMovie.obj
 0003:000002e0       ?p@?1??CreateClassInstance@CFactory@CEngineModule_CryMovie@@UBE?AV?$shared_ptr@UICryUnknown@@@boost@@XZ@4V?$shared_ptr@VCEngineModule_CryMovie@@@5@A 340622e0     CryMovie.obj
 0003:000002e8       ??_B?1??CreateClassInstance@CFactory@CEngineModule_CryMovie@@UBE?AV?$shared_ptr@UICryUnknown@@@boost@@XZ@51 340622e8     CryMovie.obj
 0003:000002f0       ?m_mov_NoCutscenes@CMovieSystem@@0HA 340622f0     Movie.obj
 0003:000002f4       ?m_mov_DebugEvents@CMovieSystem@@2HA 340622f4     Movie.obj
 0003:000002f8       ?m_mov_debugCamShake@CMovieSystem@@2HA 340622f8     Movie.obj
 0003:00000314       ?ms_lightAnimWrapperCache@CLightAnimWrapper@@0V?$map@V?$CryStringT@D@@PAVCLightAnimWrapper@@U?$less@V?$CryStringT@D@@@stlpmtx_std@@V?$allocator@U?$pair@$$CBV?$CryStringT@D@@PAVCLightAnimWrapper@@@stlpmtx_std@@@4@@stlpmtx_std@@A 34062314     Movie.obj
 0003:0000032c       ?ms_pLightAnimSet@CLightAnimWrapper@@0V?$_smart_ptr@UIAnimSequence@@@@A 3406232c     Movie.obj
 0003:00000330       ?s_EmptyElems@?1??set_null@?$SmallDynStorage@U?$TCBSplineKey@U?$Quat_tpl@M@@@spline@@HUStandardAlloc@NAlloc@@@NArray@@IAEXXZ@4PAU?$TCBSplineKey@U?$Quat_tpl@M@@@spline@@A 34062330     Movie.obj
 0003:00000334       ?s_EmptyHeader@?1??set_null@?$SmallDynStorage@U?$TCBSplineKey@U?$Quat_tpl@M@@@spline@@HUStandardAlloc@NAlloc@@@NArray@@IAEXXZ@4UEmptyHeader@23@A 34062334     Movie.obj
 0003:0000033c       ??_B?1??set_null@?$SmallDynStorage@U?$TCBSplineKey@U?$Quat_tpl@M@@@spline@@HUStandardAlloc@NAlloc@@@NArray@@IAEXXZ@51 3406233c     Movie.obj
 0003:00000340       ?s_EmptyElems@?1??set_null@?$SmallDynStorage@U?$TCBSplineKeyEx@M@spline@@HUStandardAlloc@NAlloc@@@NArray@@IAEXXZ@4PAU?$TCBSplineKeyEx@M@spline@@A 34062340     Movie.obj
 0003:00000344       ?s_EmptyHeader@?1??set_null@?$SmallDynStorage@U?$TCBSplineKeyEx@M@spline@@HUStandardAlloc@NAlloc@@@NArray@@IAEXXZ@4UEmptyHeader@23@A 34062344     Movie.obj
 0003:0000034c       ??_B?1??set_null@?$SmallDynStorage@U?$TCBSplineKeyEx@M@spline@@HUStandardAlloc@NAlloc@@@NArray@@IAEXXZ@51 3406234c     Movie.obj
 0003:00000350       ?s_EmptyElems@?1??set_null@?$SmallDynStorage@U?$TCBSplineKeyEx@U?$Vec3_tpl@M@@@spline@@HUStandardAlloc@NAlloc@@@NArray@@IAEXXZ@4PAU?$TCBSplineKeyEx@U?$Vec3_tpl@M@@@spline@@A 34062350     Movie.obj
 0003:00000354       ?s_EmptyHeader@?1??set_null@?$SmallDynStorage@U?$TCBSplineKeyEx@U?$Vec3_tpl@M@@@spline@@HUStandardAlloc@NAlloc@@@NArray@@IAEXXZ@4UEmptyHeader@23@A 34062354     Movie.obj
 0003:0000035c       ??_B?1??set_null@?$SmallDynStorage@U?$TCBSplineKeyEx@U?$Vec3_tpl@M@@@spline@@HUStandardAlloc@NAlloc@@@NArray@@IAEXXZ@51 3406235c     Movie.obj
 0003:00000360       ?str@?1??GetKeyInfo@?$TAnimSplineTrack@M@@UAEXHAAPBDAAM@Z@4PADA 34062360     Movie.obj
 0003:000003a0       ?str@?1??GetKeyInfo@?$TAnimSplineTrack@U?$Vec3_tpl@M@@@@UAEXHAAPBDAAM@Z@4PADA 340623a0     Movie.obj
 0003:000003e0       ?str@?1??GetKeyInfo@?$TAnimSplineTrack@U?$Quat_tpl@M@@@@UAEXHAAPBDAAM@Z@4PADA 340623e0     Movie.obj
 0003:00000420       ?g_globalSections@?$Node_Alloc_Lock@$00$00@@2PAUInternalCriticalSectionDummy@@A 34062420     StdAfx.obj
 0003:000024a0       ?m_bInitialized@?$Node_Alloc_Lock@$00$00@@2_NA 340644a0     StdAfx.obj
 0003:00002668       ?s_EmptyElems@?1??set_null@?$SmallDynStorage@U?$SplineKeyEx@U?$Vec2_tpl@M@@@spline@@HUStandardAlloc@NAlloc@@@NArray@@IAEXXZ@4PAU?$SplineKeyEx@U?$Vec2_tpl@M@@@spline@@A 34064668     CompoundSplineTrack.obj
 0003:0000266c       ?s_EmptyHeader@?1??set_null@?$SmallDynStorage@U?$SplineKeyEx@U?$Vec2_tpl@M@@@spline@@HUStandardAlloc@NAlloc@@@NArray@@IAEXXZ@4UEmptyHeader@23@A 3406466c     CompoundSplineTrack.obj
 0003:00002674       ??_B?1??set_null@?$SmallDynStorage@U?$SplineKeyEx@U?$Vec2_tpl@M@@@spline@@HUStandardAlloc@NAlloc@@@NArray@@IAEXXZ@51 34064674     CompoundSplineTrack.obj
 0003:00002678       ?str@?1??GetKeyInfo@?$TAnimSplineTrack@U?$Vec2_tpl@M@@@@UAEXHAAPBDAAM@Z@4PADA 34064678     CompoundSplineTrack.obj
 0003:00002818       ?s_nodeParamsInitializedCam@?A0x2c775c5d@@3_NA 34064818     AnimCameraNode.obj
 0003:0000281c       ?s_nodeParamsCam@?A0x2c775c5d@@3V?$vector@USParamInfo@IAnimNode@@V?$allocator@USParamInfo@IAnimNode@@@stlpmtx_std@@@stlpmtx_std@@A 3406481c     AnimCameraNode.obj
 0003:0000285c       ?s_initialized@CAnimPostFXNode@@1_NA 3406485c     AnimPostFXNode.obj
 0003:00002860       ?s_fxNodeDescriptions@CAnimPostFXNode@@1V?$map@W4EAnimNodeType@@V?$_smart_ptr@VCFXNodeDescription@@@@U?$less@W4EAnimNodeType@@@stlpmtx_std@@V?$allocator@U?$pair@$$CBW4EAnimNodeType@@V?$_smart_ptr@VCFXNodeDescription@@@@@stlpmtx_std@@@4@@stlpmtx_std@@A 34064860     AnimPostFXNode.obj
 0003:00002878       ?s_screenFaderNodeParamsInitialized@?A0x4f335370@@3_NA 34064878     AnimScreenFaderNode.obj
 0003:0000287c       ?s_screenFaderNodeParams@?A0x4f335370@@3V?$vector@USParamInfo@IAnimNode@@V?$allocator@USParamInfo@IAnimNode@@@stlpmtx_std@@@stlpmtx_std@@A 3406487c     AnimScreenFaderNode.obj
 0003:00002888       ?s_nodeParamsInit@?A0x68dd79ca@@3_NA 34064888     CommentNode.obj
 0003:0000288c       ?s_nodeParameters@?A0x68dd79ca@@3V?$vector@USParamInfo@IAnimNode@@V?$allocator@USParamInfo@IAnimNode@@@stlpmtx_std@@@stlpmtx_std@@A 3406488c     CommentNode.obj
 0003:0000289c       ?s_nodeParamsInitializedEnt@?A0x6681eb95@@3_NA 3406489c     EntityNode.obj
 0003:000028b8       ?s_nodeParamsEnt@?A0x6681eb95@@3V?$vector@USParamInfo@IAnimNode@@V?$allocator@USParamInfo@IAnimNode@@@stlpmtx_std@@@stlpmtx_std@@A 340648b8     EntityNode.obj
 0003:000028c4       ?s_nodeParamsInitialized@?A0x25328b82@@3_NA 340648c4     LayerNode.obj
 0003:000028c8       ?s_nodeParams@?A0x25328b82@@3V?$vector@USParamInfo@IAnimNode@@V?$allocator@USParamInfo@IAnimNode@@@stlpmtx_std@@@stlpmtx_std@@A 340648c8     LayerNode.obj
 0003:000028d4       ?s_nodeParamsInitializedMat@?A0x579b7ae3@@3_NA 340648d4     MaterialNode.obj
 0003:000028d8       ?s_nodeParamsMat@?A0x579b7ae3@@3V?$vector@USParamInfo@IAnimNode@@V?$allocator@USParamInfo@IAnimNode@@@stlpmtx_std@@@stlpmtx_std@@A 340648d8     MaterialNode.obj
 0003:000028e4       ?s_nodeParamsInitializedScene@?A0x9a090bfb@@3_NA 340648e4     SceneNode.obj
 0003:000028e8       ?s_nodeParamsSene@?A0x9a090bfb@@3V?$vector@USParamInfo@IAnimNode@@V?$allocator@USParamInfo@IAnimNode@@@stlpmtx_std@@@stlpmtx_std@@A 340648e8     SceneNode.obj
 0003:000028f8       ?__type_info_root_node@@3U__type_info_node@@A 340648f8     MSVCRT:tncleanup.obj
 0003:00002c24       ___native_startup_state    34064c24     <common>
 0003:00002c28       ___native_startup_lock     34064c28     <common>
 0003:00002c2c       ___sse2_available          34064c2c     <common>
 0003:00002c30       ___dyn_tls_init_callback   34064c30     <common>
 0003:00002c34       ___onexitend               34064c34     <common>
 0003:00002c38       ___onexitbegin             34064c38     <common>
 0004:00000000       ?m_Self@CrySimpleThreadSelf@@1PAV1@A 34065000     CryMovie.obj

 entry point at        0001:00058669

 Static symbols

 0001:000471b0       ?GetActiveKeys@@YAHQAHMPAVCCharacterTrack@@@Z 340481b0 f   EntityNode.obj
 0001:00047310       ?GetNearestKeys@@YA_NQAHMPAVCCharacterTrack@@AAH@Z 34048310 f   EntityNode.obj
 0001:000582fb       _pre_c_init                340592fb f   MSVCRT:crtdll.obj
 0001:00058553       ___DllMainCRTStartup       34059553 f   MSVCRT:crtdll.obj
 0001:00058ae0       ??__E?s_nodeParams@CAnimLightNode@@0PAUSParamInfo@IAnimNode@@A@@YAXXZ 34059ae0 f   AnimLightNode.obj
 0001:00058af0       ??__Eg_random_generator@@YAXXZ 34059af0 f   CryMovie.obj
 0001:00058b10       ??__Eg_system_event_listener_movie@@YAXXZ 34059b10 f   CryMovie.obj
 0001:00058b20       ??__E?s_factory@CFactory@CEngineModule_CryMovie@@0V12@A@@YAXXZ 34059b20 f   CryMovie.obj
 0001:00058b40       ??__ECryUserInvalidID@@YAXXZ 34059b40 f   Movie.obj
 0001:00058b50       ??__ECrySessionInvalidID@@YAXXZ 34059b50 f   Movie.obj
 0001:00058b60       ??__Es_movieSequenceAutoComplete@@YAXXZ 34059b60 f   Movie.obj
 0001:00058b70       ??__E?ms_lightAnimWrapperCache@CLightAnimWrapper@@0V?$map@V?$CryStringT@D@@PAVCLightAnimWrapper@@U?$less@V?$CryStringT@D@@@stlpmtx_std@@V?$allocator@U?$pair@$$CBV?$CryStringT@D@@PAVCLightAnimWrapper@@@stlpmtx_std@@@4@@stlpmtx_std@@A@@YAXXZ 34059b70 f   Movie.obj
 0001:00058be0       ??__E?ms_pLightAnimSet@CLightAnimWrapper@@0V?$_smart_ptr@UIAnimSequence@@@@A@@YAXXZ 34059be0 f   Movie.obj
 0001:00058bf0       ??__EautoInitializer@@YAXXZ 34059bf0 f   StdAfx.obj
 0001:00058c30       ??__Es_nodeParamsCam@?A0x2c775c5d@@YAXXZ 34059c30 f   AnimCameraNode.obj
 0001:00058c60       ??__E?s_fxNodeDescriptions@CAnimPostFXNode@@1V?$map@W4EAnimNodeType@@V?$_smart_ptr@VCFXNodeDescription@@@@U?$less@W4EAnimNodeType@@@stlpmtx_std@@V?$allocator@U?$pair@$$CBW4EAnimNodeType@@V?$_smart_ptr@VCFXNodeDescription@@@@@stlpmtx_std@@@4@@stlpmtx_std@@A@@YAXXZ 34059c60 f   AnimPostFXNode.obj
 0001:00058cd0       ??__Es_screenFaderNodeParams@?A0x4f335370@@YAXXZ 34059cd0 f   AnimScreenFaderNode.obj
 0001:00058d00       ??__Es_nodeParameters@?A0x68dd79ca@@YAXXZ 34059d00 f   CommentNode.obj
 0001:00058d30       ??__ECryUserInvalidID@@YAXXZ 34059d30 f   EntityNode.obj
 0001:00058d40       ??__ECrySessionInvalidID@@YAXXZ 34059d40 f   EntityNode.obj
 0001:00058d50       ??__Es_nodeParamsEnt@?A0x6681eb95@@YAXXZ 34059d50 f   EntityNode.obj
 0001:00058d80       ??__Es_nodeParams@?A0x25328b82@@YAXXZ 34059d80 f   LayerNode.obj
 0001:00058db0       ??__Es_nodeParamsMat@?A0x579b7ae3@@YAXXZ 34059db0 f   MaterialNode.obj
 0001:00058de0       ??__Es_nodeParamsSene@?A0x9a090bfb@@YAXXZ 34059de0 f   SceneNode.obj
 0001:00058e10       ??__F?s_nodeParams@CAnimLightNode@@0PAUSParamInfo@IAnimNode@@A@@YAXXZ 34059e10 f   AnimLightNode.obj
 0001:00058e60       ??__F?s_factory@CFactory@CEngineModule_CryMovie@@0V12@A@@YAXXZ 34059e60 f   CryMovie.obj
 0001:00058e80       ??__Fg_system_event_listener_movie@@YAXXZ 34059e80 f   CryMovie.obj
 0001:00058ed0       ??__F?ms_pLightAnimSet@CLightAnimWrapper@@0V?$_smart_ptr@UIAnimSequence@@@@A@@YAXXZ 34059ed0 f   Movie.obj
 0001:00058ef0       ??__FCrySessionInvalidID@@YAXXZ 34059ef0 f   Movie.obj
 0001:00058f30       ??__Fs_movieSequenceAutoComplete@@YAXXZ 34059f30 f   Movie.obj
 0001:00058f40       ??__FCryUserInvalidID@@YAXXZ 34059f40 f   Movie.obj
 0001:00058f80       ??__F?ms_lightAnimWrapperCache@CLightAnimWrapper@@0V?$map@V?$CryStringT@D@@PAVCLightAnimWrapper@@U?$less@V?$CryStringT@D@@@stlpmtx_std@@V?$allocator@U?$pair@$$CBV?$CryStringT@D@@PAVCLightAnimWrapper@@@stlpmtx_std@@@4@@stlpmtx_std@@A@@YAXXZ 34059f80 f   Movie.obj
 0001:00058fe0       ??__FautoInitializer@@YAXXZ 34059fe0 f   StdAfx.obj
 0001:00058ff0       ??__Fs_nodeParamsCam@?A0x2c775c5d@@YAXXZ 34059ff0 f   AnimCameraNode.obj
 0001:00059050       ??__F?s_fxNodeDescriptions@CAnimPostFXNode@@1V?$map@W4EAnimNodeType@@V?$_smart_ptr@VCFXNodeDescription@@@@U?$less@W4EAnimNodeType@@@stlpmtx_std@@V?$allocator@U?$pair@$$CBW4EAnimNodeType@@V?$_smart_ptr@VCFXNodeDescription@@@@@stlpmtx_std@@@4@@stlpmtx_std@@A@@YAXXZ 3405a050 f   AnimPostFXNode.obj
 0001:000590b0       ??__Fs_screenFaderNodeParams@?A0x4f335370@@YAXXZ 3405a0b0 f   AnimScreenFaderNode.obj
 0001:00059110       ??__Fs_nodeParameters@?A0x68dd79ca@@YAXXZ 3405a110 f   CommentNode.obj
 0001:00059170       ??__FCrySessionInvalidID@@YAXXZ 3405a170 f   EntityNode.obj
 0001:000591b0       ??__FCryUserInvalidID@@YAXXZ 3405a1b0 f   EntityNode.obj
 0001:000591f0       ??__Fs_nodeParamsEnt@?A0x6681eb95@@YAXXZ 3405a1f0 f   EntityNode.obj
 0001:00059250       ??__Fs_nodeParams@?A0x25328b82@@YAXXZ 3405a250 f   LayerNode.obj
 0001:000592b0       ??__Fs_nodeParamsMat@?A0x579b7ae3@@YAXXZ 3405a2b0 f   MaterialNode.obj
 0001:00059310       ??__Fs_nodeParamsSene@?A0x9a090bfb@@YAXXZ 3405a310 f   SceneNode.obj
